 windowsaccessbridge-64

 Timestamp is ada98626 (reproducible build file hash)

 Preferred load address is 0000000180000000

 Start         Length     Name                   Class
 0001:00000000 0001daa0H .text$mn                CODE
 0001:0001daa0 00000040H .text$mn$00             CODE
 0001:0001dae0 00000550H .text$x                 CODE
 0002:00000000 000002f0H .idata$5                DATA
 0002:000002f0 00000038H .00cfg                  DATA
 0002:00000328 00000008H .CRT$XCA                DATA
 0002:00000330 00000008H .CRT$XCZ                DATA
 0002:00000338 00000008H .CRT$XIA                DATA
 0002:00000340 00000020H .CRT$XIC                DATA
 0002:00000360 00000008H .CRT$XIZ                DATA
 0002:00000368 00000008H .CRT$XPA                DATA
 0002:00000370 00000010H .CRT$XPX                DATA
 0002:00000380 00000008H .CRT$XPXA               DATA
 0002:00000388 00000008H .CRT$XPZ                DATA
 0002:00000390 00000008H .CRT$XTA                DATA
 0002:00000398 00000008H .CRT$XTZ                DATA
 0002:000003a0 00000000H .gehcont$y              DATA
 0002:000003a0 00000000H .gfids$y                DATA
 0002:000003a0 0000b960H .rdata                  DATA
 0002:0000bd00 00000000H .rdata$CastGuardVftablesA DATA
 0002:0000bd00 00000000H .rdata$CastGuardVftablesC DATA
 0002:0000bd00 00000274H .rdata$r                DATA
 0002:0000bf74 000002c8H .rdata$voltmd           DATA
 0002:0000c23c 0000035cH .rdata$zzzdbg           DATA
 0002:0000c598 00000008H .rtc$IAA                DATA
 0002:0000c5a0 00000008H .rtc$IZZ                DATA
 0002:0000c5a8 00000008H .rtc$TAA                DATA
 0002:0000c5b0 00000008H .rtc$TZZ                DATA
 0002:0000c5b8 000016c0H .xdata                  DATA
 0002:0000dc78 00000158H .xdata$x                DATA
 0002:0000ddd0 00000e44H .edata                  DATA
 0002:0000ec14 00000028H .idata$2                DATA
 0002:0000ec3c 00000014H .idata$3                DATA
 0002:0000ec50 000002f0H .idata$4                DATA
 0002:0000ef40 000006b4H .idata$6                DATA
 0003:00000000 00000a40H .data                   DATA
 0003:00000a40 000000a8H .data$r                 DATA
 0003:00000ae8 00000028H .data$rs                DATA
 0003:00000b10 00001228H .bss                    DATA
 0004:00000000 00001dd0H .pdata                  DATA
 0005:00000000 0000015cH _RDATA                  DATA
 0006:00000000 00000120H .rsrc$01                DATA
 0006:00000120 00000638H .rsrc$02                DATA

  Address         Publics by Value              Rva+Base               Lib:Object

 0000:00000000       __AbsoluteZero             0000000000000000     <absolute>
 0000:00000000       ___safe_se_handler_count   0000000000000000     <absolute>
 0000:00000000       ___safe_se_handler_table   0000000000000000     <absolute>
 0000:00000000       __arm64x_extra_rfe_table   0000000000000000     <absolute>
 0000:00000000       __arm64x_extra_rfe_table_size 0000000000000000     <absolute>
 0000:00000000       __arm64x_native_entrypoint 0000000000000000     <absolute>
 0000:00000000       __arm64x_redirection_metadata 0000000000000000     <absolute>
 0000:00000000       __arm64x_redirection_metadata_count 0000000000000000     <absolute>
 0000:00000000       __dynamic_value_reloc_table 0000000000000000     <absolute>
 0000:00000000       __enclave_config           0000000000000000     <absolute>
 0000:00000000       __guard_check_icall_a64n_fptr 0000000000000000     <absolute>
 0000:00000000       __guard_eh_cont_count      0000000000000000     <absolute>
 0000:00000000       __guard_eh_cont_table      0000000000000000     <absolute>
 0000:00000000       __guard_fids_count         0000000000000000     <absolute>
 0000:00000000       __guard_fids_table         0000000000000000     <absolute>
 0000:00000000       __guard_iat_count          0000000000000000     <absolute>
 0000:00000000       __guard_iat_table          0000000000000000     <absolute>
 0000:00000000       __guard_longjmp_count      0000000000000000     <absolute>
 0000:00000000       __guard_longjmp_table      0000000000000000     <absolute>
 0000:00000000       __hybrid_auxiliary_delayload_iat 0000000000000000     <absolute>
 0000:00000000       __hybrid_auxiliary_delayload_iat_copy 0000000000000000     <absolute>
 0000:00000000       __hybrid_auxiliary_iat     0000000000000000     <absolute>
 0000:00000000       __hybrid_auxiliary_iat_copy 0000000000000000     <absolute>
 0000:00000000       __hybrid_code_map          0000000000000000     <absolute>
 0000:00000000       __hybrid_code_map_count    0000000000000000     <absolute>
 0000:00000000       __hybrid_image_info_bitfield 0000000000000000     <absolute>
 0000:00000000       __x64_code_ranges_to_entry_points 0000000000000000     <absolute>
 0000:00000000       __x64_code_ranges_to_entry_points_count 0000000000000000     <absolute>
 0000:00000100       __guard_flags              0000000000000100     <absolute>
 0000:00000000       __ImageBase                0000000180000000     <linker-defined>
 0001:00000000       PrintDebugString           0000000180001000 f   AccessBridgeDebug.obj
 0001:0000007c       __local_stdio_printf_options 000000018000107c f i AccessBridgeDebug.obj
 0001:00000084       finalizeFileLogger         0000000180001084 f   AccessBridgeDebug.obj
 0001:000000a8       fprintf                    00000001800010a8 f i AccessBridgeDebug.obj
 0001:000000ec       getTimeStamp               00000001800010ec f   AccessBridgeDebug.obj
 0001:00000124       initializeFileLogger       0000000180001124 f   AccessBridgeDebug.obj
 0001:00000230       printf                     0000000180001230 f i AccessBridgeDebug.obj
 0001:00000284       ??0AccessBridgeEventHandler@@QEAA@XZ 0000000180001284 f   AccessBridgeEventHandler.obj
 0001:00000320       ??1AccessBridgeEventHandler@@QEAA@XZ 0000000180001320 f   AccessBridgeEventHandler.obj
 0001:00000320       ??1AccessBridgeMessageQueue@@QEAA@XZ 0000000180001320 f   AccessBridgeMessageQueue.obj
 0001:00000320       _guard_check_icall_nop     0000000180001320 f   LIBCMT:guard_support.obj
 0001:00000324       ?fireCaretUpdate@AccessBridgeEventHandler@@QEAAXJ_J0@Z 0000000180001324 f   AccessBridgeEventHandler.obj
 0001:00000348       ?fireFocusGained@AccessBridgeEventHandler@@QEAAXJ_J0@Z 0000000180001348 f   AccessBridgeEventHandler.obj
 0001:0000036c       ?fireFocusLost@AccessBridgeEventHandler@@QEAAXJ_J0@Z 000000018000136c f   AccessBridgeEventHandler.obj
 0001:00000390       ?fireJavaShutdown@AccessBridgeEventHandler@@QEAAXJ@Z 0000000180001390 f   AccessBridgeEventHandler.obj
 0001:000003a8       ?fireMenuCanceled@AccessBridgeEventHandler@@QEAAXJ_J0@Z 00000001800013a8 f   AccessBridgeEventHandler.obj
 0001:000003cc       ?fireMenuDeselected@AccessBridgeEventHandler@@QEAAXJ_J0@Z 00000001800013cc f   AccessBridgeEventHandler.obj
 0001:000003f0       ?fireMenuSelected@AccessBridgeEventHandler@@QEAAXJ_J0@Z 00000001800013f0 f   AccessBridgeEventHandler.obj
 0001:00000414       ?fireMouseClicked@AccessBridgeEventHandler@@QEAAXJ_J0@Z 0000000180001414 f   AccessBridgeEventHandler.obj
 0001:00000438       ?fireMouseEntered@AccessBridgeEventHandler@@QEAAXJ_J0@Z 0000000180001438 f   AccessBridgeEventHandler.obj
 0001:0000045c       ?fireMouseExited@AccessBridgeEventHandler@@QEAAXJ_J0@Z 000000018000145c f   AccessBridgeEventHandler.obj
 0001:00000480       ?fireMousePressed@AccessBridgeEventHandler@@QEAAXJ_J0@Z 0000000180001480 f   AccessBridgeEventHandler.obj
 0001:000004a4       ?fireMouseReleased@AccessBridgeEventHandler@@QEAAXJ_J0@Z 00000001800014a4 f   AccessBridgeEventHandler.obj
 0001:000004c8       ?firePopupMenuCanceled@AccessBridgeEventHandler@@QEAAXJ_J0@Z 00000001800014c8 f   AccessBridgeEventHandler.obj
 0001:000004ec       ?firePopupMenuWillBecomeInvisible@AccessBridgeEventHandler@@QEAAXJ_J0@Z 00000001800014ec f   AccessBridgeEventHandler.obj
 0001:00000510       ?firePopupMenuWillBecomeVisible@AccessBridgeEventHandler@@QEAAXJ_J0@Z 0000000180001510 f   AccessBridgeEventHandler.obj
 0001:00000538       ?firePropertyActiveDescendentChange@AccessBridgeEventHandler@@QEAAXJ_J000@Z 0000000180001538 f   AccessBridgeEventHandler.obj
 0001:0000057c       ?firePropertyCaretChange@AccessBridgeEventHandler@@QEAAXJ_J0HH@Z 000000018000157c f   AccessBridgeEventHandler.obj
 0001:000005c0       ?firePropertyChildChange@AccessBridgeEventHandler@@QEAAXJ_J000@Z 00000001800015c0 f   AccessBridgeEventHandler.obj
 0001:00000604       ?firePropertyDescriptionChange@AccessBridgeEventHandler@@QEAAXJ_J0PEAG1@Z 0000000180001604 f   AccessBridgeEventHandler.obj
 0001:00000648       ?firePropertyNameChange@AccessBridgeEventHandler@@QEAAXJ_J0PEAG1@Z 0000000180001648 f   AccessBridgeEventHandler.obj
 0001:0000068c       ?firePropertySelectionChange@AccessBridgeEventHandler@@QEAAXJ_J0@Z 000000018000168c f   AccessBridgeEventHandler.obj
 0001:000006b4       ?firePropertyStateChange@AccessBridgeEventHandler@@QEAAXJ_J0PEAG1@Z 00000001800016b4 f   AccessBridgeEventHandler.obj
 0001:000006f8       ?firePropertyTableModelChange@AccessBridgeEventHandler@@QEAAXJ_J0PEAG1@Z 00000001800016f8 f   AccessBridgeEventHandler.obj
 0001:0000073c       ?firePropertyTextChange@AccessBridgeEventHandler@@QEAAXJ_J0@Z 000000018000173c f   AccessBridgeEventHandler.obj
 0001:00000764       ?firePropertyValueChange@AccessBridgeEventHandler@@QEAAXJ_J0PEAG1@Z 0000000180001764 f   AccessBridgeEventHandler.obj
 0001:000007a8       ?firePropertyVisibleDataChange@AccessBridgeEventHandler@@QEAAXJ_J0@Z 00000001800017a8 f   AccessBridgeEventHandler.obj
 0001:000007d0       ?setCaretUpdateFP@AccessBridgeEventHandler@@QEAAXP6AXJ_J0@ZPEAVWinAccessBridge@@@Z 00000001800017d0 f   AccessBridgeEventHandler.obj
 0001:000007fc       ?setFocusGainedFP@AccessBridgeEventHandler@@QEAAXP6AXJ_J0@ZPEAVWinAccessBridge@@@Z 00000001800017fc f   AccessBridgeEventHandler.obj
 0001:00000828       ?setFocusLostFP@AccessBridgeEventHandler@@QEAAXP6AXJ_J0@ZPEAVWinAccessBridge@@@Z 0000000180001828 f   AccessBridgeEventHandler.obj
 0001:00000854       ?setJavaShutdownFP@AccessBridgeEventHandler@@QEAAXP6AXJ@ZPEAVWinAccessBridge@@@Z 0000000180001854 f   AccessBridgeEventHandler.obj
 0001:00000880       ?setMenuCanceledFP@AccessBridgeEventHandler@@QEAAXP6AXJ_J0@ZPEAVWinAccessBridge@@@Z 0000000180001880 f   AccessBridgeEventHandler.obj
 0001:000008ac       ?setMenuDeselectedFP@AccessBridgeEventHandler@@QEAAXP6AXJ_J0@ZPEAVWinAccessBridge@@@Z 00000001800018ac f   AccessBridgeEventHandler.obj
 0001:000008d8       ?setMenuSelectedFP@AccessBridgeEventHandler@@QEAAXP6AXJ_J0@ZPEAVWinAccessBridge@@@Z 00000001800018d8 f   AccessBridgeEventHandler.obj
 0001:00000904       ?setMouseClickedFP@AccessBridgeEventHandler@@QEAAXP6AXJ_J0@ZPEAVWinAccessBridge@@@Z 0000000180001904 f   AccessBridgeEventHandler.obj
 0001:00000930       ?setMouseEnteredFP@AccessBridgeEventHandler@@QEAAXP6AXJ_J0@ZPEAVWinAccessBridge@@@Z 0000000180001930 f   AccessBridgeEventHandler.obj
 0001:0000095c       ?setMouseExitedFP@AccessBridgeEventHandler@@QEAAXP6AXJ_J0@ZPEAVWinAccessBridge@@@Z 000000018000195c f   AccessBridgeEventHandler.obj
 0001:00000988       ?setMousePressedFP@AccessBridgeEventHandler@@QEAAXP6AXJ_J0@ZPEAVWinAccessBridge@@@Z 0000000180001988 f   AccessBridgeEventHandler.obj
 0001:000009b4       ?setMouseReleasedFP@AccessBridgeEventHandler@@QEAAXP6AXJ_J0@ZPEAVWinAccessBridge@@@Z 00000001800019b4 f   AccessBridgeEventHandler.obj
 0001:000009e0       ?setPopupMenuCanceledFP@AccessBridgeEventHandler@@QEAAXP6AXJ_J0@ZPEAVWinAccessBridge@@@Z 00000001800019e0 f   AccessBridgeEventHandler.obj
 0001:00000a0c       ?setPopupMenuWillBecomeInvisibleFP@AccessBridgeEventHandler@@QEAAXP6AXJ_J0@ZPEAVWinAccessBridge@@@Z 0000000180001a0c f   AccessBridgeEventHandler.obj
 0001:00000a38       ?setPopupMenuWillBecomeVisibleFP@AccessBridgeEventHandler@@QEAAXP6AXJ_J0@ZPEAVWinAccessBridge@@@Z 0000000180001a38 f   AccessBridgeEventHandler.obj
 0001:00000a68       ?setPropertyActiveDescendentChangeFP@AccessBridgeEventHandler@@QEAAXP6AXJ_J000@ZPEAVWinAccessBridge@@@Z 0000000180001a68 f   AccessBridgeEventHandler.obj
 0001:00000a98       ?setPropertyCaretChangeFP@AccessBridgeEventHandler@@QEAAXP6AXJ_J0HH@ZPEAVWinAccessBridge@@@Z 0000000180001a98 f   AccessBridgeEventHandler.obj
 0001:00000ac8       ?setPropertyChangeFP@AccessBridgeEventHandler@@QEAAXP6AXJ_J0PEAG11@ZPEAVWinAccessBridge@@@Z 0000000180001ac8 f   AccessBridgeEventHandler.obj
 0001:00000af4       ?setPropertyChildChangeFP@AccessBridgeEventHandler@@QEAAXP6AXJ_J000@ZPEAVWinAccessBridge@@@Z 0000000180001af4 f   AccessBridgeEventHandler.obj
 0001:00000b24       ?setPropertyDescriptionChangeFP@AccessBridgeEventHandler@@QEAAXP6AXJ_J0PEAG1@ZPEAVWinAccessBridge@@@Z 0000000180001b24 f   AccessBridgeEventHandler.obj
 0001:00000b54       ?setPropertyNameChangeFP@AccessBridgeEventHandler@@QEAAXP6AXJ_J0PEAG1@ZPEAVWinAccessBridge@@@Z 0000000180001b54 f   AccessBridgeEventHandler.obj
 0001:00000b84       ?setPropertySelectionChangeFP@AccessBridgeEventHandler@@QEAAXP6AXJ_J0@ZPEAVWinAccessBridge@@@Z 0000000180001b84 f   AccessBridgeEventHandler.obj
 0001:00000bb4       ?setPropertyStateChangeFP@AccessBridgeEventHandler@@QEAAXP6AXJ_J0PEAG1@ZPEAVWinAccessBridge@@@Z 0000000180001bb4 f   AccessBridgeEventHandler.obj
 0001:00000be4       ?setPropertyTableModelChangeFP@AccessBridgeEventHandler@@QEAAXP6AXJ_J0PEAG1@ZPEAVWinAccessBridge@@@Z 0000000180001be4 f   AccessBridgeEventHandler.obj
 0001:00000c14       ?setPropertyTextChangeFP@AccessBridgeEventHandler@@QEAAXP6AXJ_J0@ZPEAVWinAccessBridge@@@Z 0000000180001c14 f   AccessBridgeEventHandler.obj
 0001:00000c44       ?setPropertyValueChangeFP@AccessBridgeEventHandler@@QEAAXP6AXJ_J0PEAG1@ZPEAVWinAccessBridge@@@Z 0000000180001c44 f   AccessBridgeEventHandler.obj
 0001:00000c74       ?setPropertyVisibleDataChangeFP@AccessBridgeEventHandler@@QEAAXP6AXJ_J0@ZPEAVWinAccessBridge@@@Z 0000000180001c74 f   AccessBridgeEventHandler.obj
 0001:00000ca4       ??0AccessBridgeJavaVMInstance@@QEAA@PEAUHWND__@@0JPEAV0@@Z 0000000180001ca4 f   AccessBridgeJavaVMInstance.obj
 0001:00000cf0       ??1AccessBridgeJavaVMInstance@@QEAA@XZ 0000000180001cf0 f   AccessBridgeJavaVMInstance.obj
 0001:00000d4c       ?findABJavaVMInstanceFromJavaHWND@AccessBridgeJavaVMInstance@@QEAAPEAV1@PEAUHWND__@@@Z 0000000180001d4c f   AccessBridgeJavaVMInstance.obj
 0001:00000da0       ?findAccessBridgeWindow@AccessBridgeJavaVMInstance@@QEAAPEAUHWND__@@J@Z 0000000180001da0 f   AccessBridgeJavaVMInstance.obj
 0001:00000e00       ?initiateIPC@AccessBridgeJavaVMInstance@@QEAA_JXZ 0000000180001e00 f   AccessBridgeJavaVMInstance.obj
 0001:00000ef8       ?sendMemoryPackage@AccessBridgeJavaVMInstance@@QEAAHPEADJ@Z 0000000180001ef8 f   AccessBridgeJavaVMInstance.obj
 0001:00000fec       ?sendPackage@AccessBridgeJavaVMInstance@@QEAA_JPEADJ@Z 0000000180001fec f   AccessBridgeJavaVMInstance.obj
 0001:0000105c       sprintf                    000000018000205c f i AccessBridgeJavaVMInstance.obj
 0001:000010b4       ??0AccessBridgeMessageQueue@@QEAA@XZ 00000001800020b4 f   AccessBridgeMessageQueue.obj
 0001:000010c8       ??0AccessBridgeQueueElement@@QEAA@PEADH@Z 00000001800020c8 f   AccessBridgeMessageQueue.obj
 0001:00001130       ??0bad_alloc@std@@QEAA@AEBV01@@Z 0000000180002130 f i AccessBridgeMessageQueue.obj
 0001:0000116c       ??0bad_alloc@std@@QEAA@XZ  000000018000216c f i AccessBridgeMessageQueue.obj
 0001:0000118c       ??0exception@std@@QEAA@AEBV01@@Z 000000018000218c f i AccessBridgeMessageQueue.obj
 0001:000011c0       ??1AccessBridgeQueueElement@@QEAA@XZ 00000001800021c0 f   AccessBridgeMessageQueue.obj
 0001:000011c8       ??1bad_alloc@std@@UEAA@XZ  00000001800021c8 f i AccessBridgeMessageQueue.obj
 0001:000011c8       ??1bad_array_new_length@std@@UEAA@XZ 00000001800021c8 f i LIBCMT:throw_bad_alloc.obj
 0001:000011c8       ??1bad_exception@std@@UEAA@XZ 00000001800021c8 f i libvcruntime:frame.obj
 0001:000011dc       ??_Ebad_alloc@std@@UEAAPEAXI@Z 00000001800021dc f i AccessBridgeMessageQueue.obj
 0001:000011dc       ??_Ebad_array_new_length@std@@UEAAPEAXI@Z 00000001800021dc f i LIBCMT:throw_bad_alloc.obj
 0001:000011dc       ??_Ebad_exception@std@@UEAAPEAXI@Z 00000001800021dc f i libvcruntime:frame.obj
 0001:000011dc       ??_Eexception@std@@UEAAPEAXI@Z 00000001800021dc f i AccessBridgeMessageQueue.obj
 0001:000011dc       ??_Gbad_alloc@std@@UEAAPEAXI@Z 00000001800021dc f i AccessBridgeMessageQueue.obj
 0001:000011dc       ??_Gbad_array_new_length@std@@UEAAPEAXI@Z 00000001800021dc f i LIBCMT:throw_bad_alloc.obj
 0001:000011dc       ??_Gbad_exception@std@@UEAAPEAXI@Z 00000001800021dc f i libvcruntime:frame.obj
 0001:000011dc       ??_Gexception@std@@UEAAPEAXI@Z 00000001800021dc f i AccessBridgeMessageQueue.obj
 0001:00001220       ?add@AccessBridgeMessageQueue@@QEAA?AW4QueueReturns@@PEAVAccessBridgeQueueElement@@@Z 0000000180002220 f   AccessBridgeMessageQueue.obj
 0001:000012e4       ?getEventsWaiting@AccessBridgeMessageQueue@@QEAAHXZ 00000001800022e4 f   AccessBridgeMessageQueue.obj
 0001:000012e8       ?getRemoveLockSetting@AccessBridgeMessageQueue@@QEAAHXZ 00000001800022e8 f   AccessBridgeMessageQueue.obj
 0001:000012ec       ?remove@AccessBridgeMessageQueue@@QEAA?AW4QueueReturns@@PEAPEAVAccessBridgeQueueElement@@@Z 00000001800022ec f   AccessBridgeMessageQueue.obj
 0001:000013b0       ?setRemoveLock@AccessBridgeMessageQueue@@QEAA?AW4QueueReturns@@H@Z 00000001800023b0 f   AccessBridgeMessageQueue.obj
 0001:000013c4       ?what@exception@std@@UEBAPEBDXZ 00000001800023c4 f i AccessBridgeMessageQueue.obj
 0001:000013d8       ?initBroadcastMessageIDs@@YAHXZ 00000001800023d8 f   AccessBridgeMessages.obj
 0001:00001418       Windows_run                0000000180002418 f   AccessBridgeWindowsEntryPoints.obj
 0001:00001434       activateAccessibleHyperlink 0000000180002434 f   AccessBridgeWindowsEntryPoints.obj
 0001:00001454       addAccessibleSelectionFromContext 0000000180002454 f   AccessBridgeWindowsEntryPoints.obj
 0001:00001478       clearAccessibleSelectionFromContext 0000000180002478 f   AccessBridgeWindowsEntryPoints.obj
 0001:0000149c       doAccessibleActions        000000018000249c f   AccessBridgeWindowsEntryPoints.obj
 0001:000014cc       getAccessibleActions       00000001800024cc f   AccessBridgeWindowsEntryPoints.obj
 0001:000014ec       getAccessibleChildFromContext 00000001800024ec f   AccessBridgeWindowsEntryPoints.obj
 0001:0000150c       getAccessibleContextAt     000000018000250c f   AccessBridgeWindowsEntryPoints.obj
 0001:00001548       getAccessibleContextFromHWND 0000000180002548 f   AccessBridgeWindowsEntryPoints.obj
 0001:00001568       getAccessibleContextInfo   0000000180002568 f   AccessBridgeWindowsEntryPoints.obj
 0001:00001588       getAccessibleContextWithFocus 0000000180002588 f   AccessBridgeWindowsEntryPoints.obj
 0001:000015a8       getAccessibleHyperlink     00000001800025a8 f   AccessBridgeWindowsEntryPoints.obj
 0001:000015d8       getAccessibleHyperlinkCount 00000001800025d8 f   AccessBridgeWindowsEntryPoints.obj
 0001:000015f4       getAccessibleHypertext     00000001800025f4 f   AccessBridgeWindowsEntryPoints.obj
 0001:00001614       getAccessibleHypertextExt  0000000180002614 f   AccessBridgeWindowsEntryPoints.obj
 0001:00001644       getAccessibleHypertextLinkIndex 0000000180002644 f   AccessBridgeWindowsEntryPoints.obj
 0001:00001664       getAccessibleIcons         0000000180002664 f   AccessBridgeWindowsEntryPoints.obj
 0001:00001684       getAccessibleKeyBindings   0000000180002684 f   AccessBridgeWindowsEntryPoints.obj
 0001:000016a4       getAccessibleParentFromContext 00000001800026a4 f   AccessBridgeWindowsEntryPoints.obj
 0001:000016c0       getAccessibleRelationSet   00000001800026c0 f   AccessBridgeWindowsEntryPoints.obj
 0001:000016e0       getAccessibleSelectionCountFromContext 00000001800026e0 f   AccessBridgeWindowsEntryPoints.obj
 0001:000016fc       getAccessibleSelectionFromContext 00000001800026fc f   AccessBridgeWindowsEntryPoints.obj
 0001:0000171c       getAccessibleTableCellInfo 000000018000271c f   AccessBridgeWindowsEntryPoints.obj
 0001:00001758       getAccessibleTableColumn   0000000180002758 f   AccessBridgeWindowsEntryPoints.obj
 0001:00001778       getAccessibleTableColumnDescription 0000000180002778 f   AccessBridgeWindowsEntryPoints.obj
 0001:00001798       getAccessibleTableColumnHeader 0000000180002798 f   AccessBridgeWindowsEntryPoints.obj
 0001:000017b8       getAccessibleTableColumnSelectionCount 00000001800027b8 f   AccessBridgeWindowsEntryPoints.obj
 0001:000017d4       getAccessibleTableColumnSelections 00000001800027d4 f   AccessBridgeWindowsEntryPoints.obj
 0001:00001804       getAccessibleTableIndex    0000000180002804 f   AccessBridgeWindowsEntryPoints.obj
 0001:00001834       getAccessibleTableInfo     0000000180002834 f   AccessBridgeWindowsEntryPoints.obj
 0001:00001854       getAccessibleTableRow      0000000180002854 f   AccessBridgeWindowsEntryPoints.obj
 0001:00001874       getAccessibleTableRowDescription 0000000180002874 f   AccessBridgeWindowsEntryPoints.obj
 0001:00001894       getAccessibleTableRowHeader 0000000180002894 f   AccessBridgeWindowsEntryPoints.obj
 0001:000018b4       getAccessibleTableRowSelectionCount 00000001800028b4 f   AccessBridgeWindowsEntryPoints.obj
 0001:000018d0       getAccessibleTableRowSelections 00000001800028d0 f   AccessBridgeWindowsEntryPoints.obj
 0001:00001900       getAccessibleTextAttributes 0000000180002900 f   AccessBridgeWindowsEntryPoints.obj
 0001:00001930       getAccessibleTextInfo      0000000180002930 f   AccessBridgeWindowsEntryPoints.obj
 0001:00001968       getAccessibleTextItems     0000000180002968 f   AccessBridgeWindowsEntryPoints.obj
 0001:00001998       getAccessibleTextLineBounds 0000000180002998 f   AccessBridgeWindowsEntryPoints.obj
 0001:000019d4       getAccessibleTextRange     00000001800029d4 f   AccessBridgeWindowsEntryPoints.obj
 0001:00001a18       getAccessibleTextRect      0000000180002a18 f   AccessBridgeWindowsEntryPoints.obj
 0001:00001a48       getAccessibleTextSelectionInfo 0000000180002a48 f   AccessBridgeWindowsEntryPoints.obj
 0001:00001a68       getActiveDescendent        0000000180002a68 f   AccessBridgeWindowsEntryPoints.obj
 0001:00001a84       getCaretLocation           0000000180002a84 f   AccessBridgeWindowsEntryPoints.obj
 0001:00001ab4       getCurrentAccessibleValueFromContext 0000000180002ab4 f   AccessBridgeWindowsEntryPoints.obj
 0001:00001ae4       getEventsWaiting           0000000180002ae4 f   AccessBridgeWindowsEntryPoints.obj
 0001:00001af8       getHWNDFromAccessibleContext 0000000180002af8 f   AccessBridgeWindowsEntryPoints.obj
 0001:00001b14       getMaximumAccessibleValueFromContext 0000000180002b14 f   AccessBridgeWindowsEntryPoints.obj
 0001:00001b44       getMinimumAccessibleValueFromContext 0000000180002b44 f   AccessBridgeWindowsEntryPoints.obj
 0001:00001b74       getObjectDepth             0000000180002b74 f   AccessBridgeWindowsEntryPoints.obj
 0001:00001b90       getParentWithRole          0000000180002b90 f   AccessBridgeWindowsEntryPoints.obj
 0001:00001bb0       getParentWithRoleElseRoot  0000000180002bb0 f   AccessBridgeWindowsEntryPoints.obj
 0001:00001bd0       getTextAttributesInRange   0000000180002bd0 f   AccessBridgeWindowsEntryPoints.obj
 0001:00001c14       getTopLevelHWND            0000000180002c14 f   AccessBridgeWindowsEntryPoints.obj
 0001:00001c60       getTopLevelObject          0000000180002c60 f   AccessBridgeWindowsEntryPoints.obj
 0001:00001c7c       getVersionInfo             0000000180002c7c f   AccessBridgeWindowsEntryPoints.obj
 0001:00001ca0       getVirtualAccessibleName   0000000180002ca0 f   AccessBridgeWindowsEntryPoints.obj
 0001:00001cd0       getVisibleChildren         0000000180002cd0 f   AccessBridgeWindowsEntryPoints.obj
 0001:00001d00       getVisibleChildrenCount    0000000180002d00 f   AccessBridgeWindowsEntryPoints.obj
 0001:00001d1c       isAccessibleChildSelectedFromContext 0000000180002d1c f   AccessBridgeWindowsEntryPoints.obj
 0001:00001d3c       isAccessibleTableColumnSelected 0000000180002d3c f   AccessBridgeWindowsEntryPoints.obj
 0001:00001d5c       isAccessibleTableRowSelected 0000000180002d5c f   AccessBridgeWindowsEntryPoints.obj
 0001:00001d7c       isJavaWindow               0000000180002d7c f   AccessBridgeWindowsEntryPoints.obj
 0001:00001d94       isSameObject               0000000180002d94 f   AccessBridgeWindowsEntryPoints.obj
 0001:00001de4       releaseJavaObject          0000000180002de4 f   AccessBridgeWindowsEntryPoints.obj
 0001:00001e08       removeAccessibleSelectionFromContext 0000000180002e08 f   AccessBridgeWindowsEntryPoints.obj
 0001:00001e2c       requestFocus               0000000180002e2c f   AccessBridgeWindowsEntryPoints.obj
 0001:00001e48       selectAllAccessibleSelectionFromContext 0000000180002e48 f   AccessBridgeWindowsEntryPoints.obj
 0001:00001e6c       selectTextRange            0000000180002e6c f   AccessBridgeWindowsEntryPoints.obj
 0001:00001e9c       setCaretPosition           0000000180002e9c f   AccessBridgeWindowsEntryPoints.obj
 0001:00001ebc       setCaretUpdateFP           0000000180002ebc f   AccessBridgeWindowsEntryPoints.obj
 0001:00001edc       setFocusGainedFP           0000000180002edc f   AccessBridgeWindowsEntryPoints.obj
 0001:00001efc       setFocusLostFP             0000000180002efc f   AccessBridgeWindowsEntryPoints.obj
 0001:00001f1c       setJavaShutdownFP          0000000180002f1c f   AccessBridgeWindowsEntryPoints.obj
 0001:00001f3c       setMenuCanceledFP          0000000180002f3c f   AccessBridgeWindowsEntryPoints.obj
 0001:00001f5c       setMenuDeselectedFP        0000000180002f5c f   AccessBridgeWindowsEntryPoints.obj
 0001:00001f7c       setMenuSelectedFP          0000000180002f7c f   AccessBridgeWindowsEntryPoints.obj
 0001:00001f9c       setMouseClickedFP          0000000180002f9c f   AccessBridgeWindowsEntryPoints.obj
 0001:00001fbc       setMouseEnteredFP          0000000180002fbc f   AccessBridgeWindowsEntryPoints.obj
 0001:00001fdc       setMouseExitedFP           0000000180002fdc f   AccessBridgeWindowsEntryPoints.obj
 0001:00001ffc       setMousePressedFP          0000000180002ffc f   AccessBridgeWindowsEntryPoints.obj
 0001:0000201c       setMouseReleasedFP         000000018000301c f   AccessBridgeWindowsEntryPoints.obj
 0001:0000203c       setPopupMenuCanceledFP     000000018000303c f   AccessBridgeWindowsEntryPoints.obj
 0001:0000205c       setPopupMenuWillBecomeInvisibleFP 000000018000305c f   AccessBridgeWindowsEntryPoints.obj
 0001:0000207c       setPopupMenuWillBecomeVisibleFP 000000018000307c f   AccessBridgeWindowsEntryPoints.obj
 0001:0000209c       setPropertyActiveDescendentChangeFP 000000018000309c f   AccessBridgeWindowsEntryPoints.obj
 0001:000020bc       setPropertyCaretChangeFP   00000001800030bc f   AccessBridgeWindowsEntryPoints.obj
 0001:000020dc       setPropertyChangeFP        00000001800030dc f   AccessBridgeWindowsEntryPoints.obj
 0001:000020fc       setPropertyChildChangeFP   00000001800030fc f   AccessBridgeWindowsEntryPoints.obj
 0001:0000211c       setPropertyDescriptionChangeFP 000000018000311c f   AccessBridgeWindowsEntryPoints.obj
 0001:0000213c       setPropertyNameChangeFP    000000018000313c f   AccessBridgeWindowsEntryPoints.obj
 0001:0000215c       setPropertySelectionChangeFP 000000018000315c f   AccessBridgeWindowsEntryPoints.obj
 0001:0000217c       setPropertyStateChangeFP   000000018000317c f   AccessBridgeWindowsEntryPoints.obj
 0001:0000219c       setPropertyTableModelChangeFP 000000018000319c f   AccessBridgeWindowsEntryPoints.obj
 0001:000021bc       setPropertyTextChangeFP    00000001800031bc f   AccessBridgeWindowsEntryPoints.obj
 0001:000021dc       setPropertyValueChangeFP   00000001800031dc f   AccessBridgeWindowsEntryPoints.obj
 0001:000021fc       setPropertyVisibleDataChangeFP 00000001800031fc f   AccessBridgeWindowsEntryPoints.obj
 0001:0000221c       setTextContents            000000018000321c f   AccessBridgeWindowsEntryPoints.obj
 0001:0000223c       ??0WinAccessBridge@@QEAA@PEAUHINSTANCE__@@@Z 000000018000323c f   WinAccessBridge.obj
 0001:000022d8       ??1WinAccessBridge@@QEAA@XZ 00000001800032d8 f   WinAccessBridge.obj
 0001:000023c0       ?JavaVMDestroyed@WinAccessBridge@@QEAAXPEAUHWND__@@@Z 00000001800033c0 f   WinAccessBridge.obj
 0001:00002468       ?activateAccessibleHyperlink@WinAccessBridge@@QEAAHJ_J0@Z 0000000180003468 f   WinAccessBridge.obj
 0001:00002510       ?addAccessibilityEventNotification@WinAccessBridge@@QEAAX_J@Z 0000000180003510 f   WinAccessBridge.obj
 0001:000025b0       ?addAccessibleSelectionFromContext@WinAccessBridge@@QEAAXJ_JH@Z 00000001800035b0 f   WinAccessBridge.obj
 0001:0000261c       ?addJavaEventNotification@WinAccessBridge@@QEAAX_J@Z 000000018000361c f   WinAccessBridge.obj
 0001:000026bc       ?clearAccessibleSelectionFromContext@WinAccessBridge@@QEAAXJ_J@Z 00000001800036bc f   WinAccessBridge.obj
 0001:00002724       ?doAccessibleActions@WinAccessBridge@@QEAAHJ_JPEAUAccessibleActionsToDoTag@@PEAJ@Z 0000000180003724 f   WinAccessBridge.obj
 0001:00002810       ?getAccessibleActions@WinAccessBridge@@QEAAHJ_JPEAUAccessibleActionsTag@@@Z 0000000180003810 f   WinAccessBridge.obj
 0001:000028ec       ?getAccessibleChildFromContext@WinAccessBridge@@QEAA_JJ_JJ@Z 00000001800038ec f   WinAccessBridge.obj
 0001:00002978       ?getAccessibleContextAt@WinAccessBridge@@QEAAHJ_JJJPEA_J@Z 0000000180003978 f   WinAccessBridge.obj
 0001:00002a1c       ?getAccessibleContextFromHWND@WinAccessBridge@@QEAAHPEAUHWND__@@PEAJPEA_J@Z 0000000180003a1c f   WinAccessBridge.obj
 0001:00002b20       ?getAccessibleContextInfo@WinAccessBridge@@QEAAHJ_JPEAUAccessibleContextInfoTag@@@Z 0000000180003b20 f   WinAccessBridge.obj
 0001:00002c18       ?getAccessibleContextWithFocus@WinAccessBridge@@QEAAHPEAUHWND__@@PEAJPEA_J@Z 0000000180003c18 f   WinAccessBridge.obj
 0001:00002cc4       ?getAccessibleHyperlink@WinAccessBridge@@QEAAHJ_JJPEAUAccessibleHyperlinkInfoTag@@@Z 0000000180003cc4 f   WinAccessBridge.obj
 0001:00002da0       ?getAccessibleHyperlinkCount@WinAccessBridge@@QEAAJJ_J@Z 0000000180003da0 f   WinAccessBridge.obj
 0001:00002e58       ?getAccessibleHypertext@WinAccessBridge@@QEAAHJ_JPEAUAccessibleHypertextInfoTag@@@Z 0000000180003e58 f   WinAccessBridge.obj
 0001:00002f34       ?getAccessibleHypertextExt@WinAccessBridge@@QEAAHJ_JJPEAUAccessibleHypertextInfoTag@@@Z 0000000180003f34 f   WinAccessBridge.obj
 0001:00003048       ?getAccessibleHypertextLinkIndex@WinAccessBridge@@QEAAJJ_JJ@Z 0000000180004048 f   WinAccessBridge.obj
 0001:00003114       ?getAccessibleIcons@WinAccessBridge@@QEAAHJ_JPEAUAccessibleIconsTag@@@Z 0000000180004114 f   WinAccessBridge.obj
 0001:000031f0       ?getAccessibleKeyBindings@WinAccessBridge@@QEAAHJ_JPEAUAccessibleKeyBindingsTag@@@Z 00000001800041f0 f   WinAccessBridge.obj
 0001:000032f8       ?getAccessibleParentFromContext@WinAccessBridge@@QEAA_JJ_J@Z 00000001800042f8 f   WinAccessBridge.obj
 0001:00003388       ?getAccessibleRelationSet@WinAccessBridge@@QEAAHJ_JPEAUAccessibleRelationSetInfoTag@@@Z 0000000180004388 f   WinAccessBridge.obj
 0001:00003460       ?getAccessibleSelectionCountFromContext@WinAccessBridge@@QEAAHJ_J@Z 0000000180004460 f   WinAccessBridge.obj
 0001:000034d4       ?getAccessibleSelectionFromContext@WinAccessBridge@@QEAA_JJ_JH@Z 00000001800044d4 f   WinAccessBridge.obj
 0001:0000354c       ?getAccessibleTableCellInfo@WinAccessBridge@@QEAAHJ_JJJPEAUAccessibleTableCellInfoTag@@@Z 000000018000454c f   WinAccessBridge.obj
 0001:00003650       ?getAccessibleTableColumn@WinAccessBridge@@QEAAJJ_JJ@Z 0000000180004650 f   WinAccessBridge.obj
 0001:000036fc       ?getAccessibleTableColumnDescription@WinAccessBridge@@QEAA_JJ_JJ@Z 00000001800046fc f   WinAccessBridge.obj
 0001:000037a8       ?getAccessibleTableColumnHeader@WinAccessBridge@@QEAAHJ_JPEAUAccessibleTableInfoTag@@@Z 00000001800047a8 f   WinAccessBridge.obj
 0001:00003864       ?getAccessibleTableColumnSelectionCount@WinAccessBridge@@QEAAJJ_J@Z 0000000180004864 f   WinAccessBridge.obj
 0001:00003908       ?getAccessibleTableColumnSelections@WinAccessBridge@@QEAAHJ_JJPEAJ@Z 0000000180004908 f   WinAccessBridge.obj
 0001:000039e0       ?getAccessibleTableIndex@WinAccessBridge@@QEAAJJ_JJJ@Z 00000001800049e0 f   WinAccessBridge.obj
 0001:00003aa0       ?getAccessibleTableInfo@WinAccessBridge@@QEAAHJ_JPEAUAccessibleTableInfoTag@@@Z 0000000180004aa0 f   WinAccessBridge.obj
 0001:00003b60       ?getAccessibleTableRow@WinAccessBridge@@QEAAJJ_JJ@Z 0000000180004b60 f   WinAccessBridge.obj
 0001:00003c0c       ?getAccessibleTableRowDescription@WinAccessBridge@@QEAA_JJ_JJ@Z 0000000180004c0c f   WinAccessBridge.obj
 0001:00003cb8       ?getAccessibleTableRowHeader@WinAccessBridge@@QEAAHJ_JPEAUAccessibleTableInfoTag@@@Z 0000000180004cb8 f   WinAccessBridge.obj
 0001:00003d74       ?getAccessibleTableRowSelectionCount@WinAccessBridge@@QEAAJJ_J@Z 0000000180004d74 f   WinAccessBridge.obj
 0001:00003e18       ?getAccessibleTableRowSelections@WinAccessBridge@@QEAAHJ_JJPEAJ@Z 0000000180004e18 f   WinAccessBridge.obj
 0001:00003ef0       ?getAccessibleTextAttributes@WinAccessBridge@@QEAAHJ_JJPEAUAccessibleTextAttributesInfoTag@@@Z 0000000180004ef0 f   WinAccessBridge.obj
 0001:00003fac       ?getAccessibleTextInfo@WinAccessBridge@@QEAAHJ_JPEAUAccessibleTextInfoTag@@JJ@Z 0000000180004fac f   WinAccessBridge.obj
 0001:00004088       ?getAccessibleTextItems@WinAccessBridge@@QEAAHJ_JPEAUAccessibleTextItemsInfoTag@@J@Z 0000000180005088 f   WinAccessBridge.obj
 0001:00004160       ?getAccessibleTextLineBounds@WinAccessBridge@@QEAAHJ_JJPEAJ1@Z 0000000180005160 f   WinAccessBridge.obj
 0001:00004208       ?getAccessibleTextRange@WinAccessBridge@@QEAAHJ_JJJPEAGF@Z 0000000180005208 f   WinAccessBridge.obj
 0001:000042d8       ?getAccessibleTextRect@WinAccessBridge@@QEAAHJ_JPEAUAccessibleTextRectInfoTag@@J@Z 00000001800052d8 f   WinAccessBridge.obj
 0001:00004384       ?getAccessibleTextSelectionInfo@WinAccessBridge@@QEAAHJ_JPEAUAccessibleTextSelectionInfoTag@@@Z 0000000180005384 f   WinAccessBridge.obj
 0001:00004430       ?getActiveDescendent@WinAccessBridge@@QEAA_JJ_J@Z 0000000180005430 f   WinAccessBridge.obj
 0001:000044c0       ?getCaretLocation@WinAccessBridge@@QEAAHJ_JPEAUAccessibleTextRectInfoTag@@J@Z 00000001800054c0 f   WinAccessBridge.obj
 0001:0000456c       ?getCurrentAccessibleValueFromContext@WinAccessBridge@@QEAAHJ_JPEAGF@Z 000000018000556c f   WinAccessBridge.obj
 0001:00004610       ?getEventsWaiting@WinAccessBridge@@QEAAHXZ 0000000180005610 f   WinAccessBridge.obj
 0001:00004620       ?getHWNDFromAccessibleContext@WinAccessBridge@@QEAAPEAUHWND__@@J_J@Z 0000000180005620 f   WinAccessBridge.obj
 0001:000046b8       ?getMaximumAccessibleValueFromContext@WinAccessBridge@@QEAAHJ_JPEAGF@Z 00000001800056b8 f   WinAccessBridge.obj
 0001:0000475c       ?getMinimumAccessibleValueFromContext@WinAccessBridge@@QEAAHJ_JPEAGF@Z 000000018000575c f   WinAccessBridge.obj
 0001:00004800       ?getObjectDepth@WinAccessBridge@@QEAAHJ_J@Z 0000000180005800 f   WinAccessBridge.obj
 0001:00004890       ?getParentWithRole@WinAccessBridge@@QEAA_JJ_JPEBG@Z 0000000180005890 f   WinAccessBridge.obj
 0001:00004978       ?getParentWithRoleElseRoot@WinAccessBridge@@QEAA_JJ_JPEBG@Z 0000000180005978 f   WinAccessBridge.obj
 0001:00004a2c       ?getTextAttributesInRange@WinAccessBridge@@QEAAHJ_JHHPEAUAccessibleTextAttributesInfoTag@@PEAF@Z 0000000180005a2c f   WinAccessBridge.obj
 0001:00004b38       ?getTopLevelObject@WinAccessBridge@@QEAA_JJ_J@Z 0000000180005b38 f   WinAccessBridge.obj
 0001:00004bc8       ?getVersionInfo@WinAccessBridge@@QEAAHJPEAUAccessBridgeVersionInfoTag@@@Z 0000000180005bc8 f   WinAccessBridge.obj
 0001:00004c9c       ?getVirtualAccessibleName@WinAccessBridge@@QEAAHJ_JPEAGH@Z 0000000180005c9c f   WinAccessBridge.obj
 0001:00004d74       ?getVisibleChildren@WinAccessBridge@@QEAAHJ_JHPEAUVisibleChildenInfoTag@@@Z 0000000180005d74 f   WinAccessBridge.obj
 0001:00004e2c       ?getVisibleChildrenCount@WinAccessBridge@@QEAAHJ_J@Z 0000000180005e2c f   WinAccessBridge.obj
 0001:00004ebc       ?initWindow@WinAccessBridge@@QEAAHXZ 0000000180005ebc f   WinAccessBridge.obj
 0001:00004f1c       ?isAccessibleChildSelectedFromContext@WinAccessBridge@@QEAAHJ_JH@Z 0000000180005f1c f   WinAccessBridge.obj
 0001:00004fa4       ?isAccessibleTableColumnSelected@WinAccessBridge@@QEAAHJ_JJ@Z 0000000180005fa4 f   WinAccessBridge.obj
 0001:0000505c       ?isAccessibleTableRowSelected@WinAccessBridge@@QEAAHJ_JJ@Z 000000018000605c f   WinAccessBridge.obj
 0001:00005114       ?isJavaWindow@WinAccessBridge@@QEAAHPEAUHWND__@@@Z 0000000180006114 f   WinAccessBridge.obj
 0001:000051dc       ?isSameObject@WinAccessBridge@@QEAAHJ_J0@Z 00000001800061dc f   WinAccessBridge.obj
 0001:000052a0       ?preProcessPackage@WinAccessBridge@@QEAAXPEADJ@Z 00000001800062a0 f   WinAccessBridge.obj
 0001:000053ac       ?processPackage@WinAccessBridge@@QEAAXPEADJ@Z 00000001800063ac f   WinAccessBridge.obj
 0001:00005b48       ?queuePackage@WinAccessBridge@@QEAAHPEADJ@Z 0000000180006b48 f   WinAccessBridge.obj
 0001:00005bc4       ?receiveAQueuedPackage@WinAccessBridge@@QEAAHXZ 0000000180006bc4 f   WinAccessBridge.obj
 0001:00005cfc       ?releaseJavaObject@WinAccessBridge@@QEAAXJ_J@Z 0000000180006cfc f   WinAccessBridge.obj
 0001:00005d78       ?removeAccessibilityEventNotification@WinAccessBridge@@QEAAX_J@Z 0000000180006d78 f   WinAccessBridge.obj
 0001:00005e18       ?removeAccessibleSelectionFromContext@WinAccessBridge@@QEAAXJ_JH@Z 0000000180006e18 f   WinAccessBridge.obj
 0001:00005e84       ?removeJavaEventNotification@WinAccessBridge@@QEAAX_J@Z 0000000180006e84 f   WinAccessBridge.obj
 0001:00005f24       ?rendezvousWithNewJavaDLL@WinAccessBridge@@QEAA_JPEAUHWND__@@J@Z 0000000180006f24 f   WinAccessBridge.obj
 0001:00006000       ?requestFocus@WinAccessBridge@@QEAAHJ_J@Z 0000000180007000 f   WinAccessBridge.obj
 0001:00006088       ?selectAllAccessibleSelectionFromContext@WinAccessBridge@@QEAAXJ_J@Z 0000000180007088 f   WinAccessBridge.obj
 0001:000060f0       ?selectTextRange@WinAccessBridge@@QEAAHJ_JHH@Z 00000001800070f0 f   WinAccessBridge.obj
 0001:0000618c       ?sendMemoryPackage@WinAccessBridge@@QEAAHPEADJPEAUHWND__@@@Z 000000018000718c f   WinAccessBridge.obj
 0001:000061f4       ?sendPackage@WinAccessBridge@@QEAAXPEADJPEAUHWND__@@@Z 00000001800071f4 f   WinAccessBridge.obj
 0001:00006228       ?setCaretPosition@WinAccessBridge@@QEAAHJ_JH@Z 0000000180007228 f   WinAccessBridge.obj
 0001:000062b4       ?setCaretUpdateFP@WinAccessBridge@@QEAAXP6AXJ_J0@Z@Z 00000001800072b4 f   WinAccessBridge.obj
 0001:000062c0       ?setFocusGainedFP@WinAccessBridge@@QEAAXP6AXJ_J0@Z@Z 00000001800072c0 f   WinAccessBridge.obj
 0001:000062cc       ?setFocusLostFP@WinAccessBridge@@QEAAXP6AXJ_J0@Z@Z 00000001800072cc f   WinAccessBridge.obj
 0001:000062d8       ?setJavaShutdownFP@WinAccessBridge@@QEAAXP6AXJ@Z@Z 00000001800072d8 f   WinAccessBridge.obj
 0001:000062e4       ?setMenuCanceledFP@WinAccessBridge@@QEAAXP6AXJ_J0@Z@Z 00000001800072e4 f   WinAccessBridge.obj
 0001:000062f0       ?setMenuDeselectedFP@WinAccessBridge@@QEAAXP6AXJ_J0@Z@Z 00000001800072f0 f   WinAccessBridge.obj
 0001:000062fc       ?setMenuSelectedFP@WinAccessBridge@@QEAAXP6AXJ_J0@Z@Z 00000001800072fc f   WinAccessBridge.obj
 0001:00006308       ?setMouseClickedFP@WinAccessBridge@@QEAAXP6AXJ_J0@Z@Z 0000000180007308 f   WinAccessBridge.obj
 0001:00006314       ?setMouseEnteredFP@WinAccessBridge@@QEAAXP6AXJ_J0@Z@Z 0000000180007314 f   WinAccessBridge.obj
 0001:00006320       ?setMouseExitedFP@WinAccessBridge@@QEAAXP6AXJ_J0@Z@Z 0000000180007320 f   WinAccessBridge.obj
 0001:0000632c       ?setMousePressedFP@WinAccessBridge@@QEAAXP6AXJ_J0@Z@Z 000000018000732c f   WinAccessBridge.obj
 0001:00006338       ?setMouseReleasedFP@WinAccessBridge@@QEAAXP6AXJ_J0@Z@Z 0000000180007338 f   WinAccessBridge.obj
 0001:00006344       ?setPopupMenuCanceledFP@WinAccessBridge@@QEAAXP6AXJ_J0@Z@Z 0000000180007344 f   WinAccessBridge.obj
 0001:00006350       ?setPopupMenuWillBecomeInvisibleFP@WinAccessBridge@@QEAAXP6AXJ_J0@Z@Z 0000000180007350 f   WinAccessBridge.obj
 0001:0000635c       ?setPopupMenuWillBecomeVisibleFP@WinAccessBridge@@QEAAXP6AXJ_J0@Z@Z 000000018000735c f   WinAccessBridge.obj
 0001:00006368       ?setPropertyActiveDescendentChangeFP@WinAccessBridge@@QEAAXP6AXJ_J000@Z@Z 0000000180007368 f   WinAccessBridge.obj
 0001:00006374       ?setPropertyCaretChangeFP@WinAccessBridge@@QEAAXP6AXJ_J0HH@Z@Z 0000000180007374 f   WinAccessBridge.obj
 0001:00006380       ?setPropertyChangeFP@WinAccessBridge@@QEAAXP6AXJ_J0PEAG11@Z@Z 0000000180007380 f   WinAccessBridge.obj
 0001:0000638c       ?setPropertyChildChangeFP@WinAccessBridge@@QEAAXP6AXJ_J000@Z@Z 000000018000738c f   WinAccessBridge.obj
 0001:00006398       ?setPropertyDescriptionChangeFP@WinAccessBridge@@QEAAXP6AXJ_J0PEAG1@Z@Z 0000000180007398 f   WinAccessBridge.obj
 0001:000063a4       ?setPropertyNameChangeFP@WinAccessBridge@@QEAAXP6AXJ_J0PEAG1@Z@Z 00000001800073a4 f   WinAccessBridge.obj
 0001:000063b0       ?setPropertySelectionChangeFP@WinAccessBridge@@QEAAXP6AXJ_J0@Z@Z 00000001800073b0 f   WinAccessBridge.obj
 0001:000063bc       ?setPropertyStateChangeFP@WinAccessBridge@@QEAAXP6AXJ_J0PEAG1@Z@Z 00000001800073bc f   WinAccessBridge.obj
 0001:000063c8       ?setPropertyTableModelChangeFP@WinAccessBridge@@QEAAXP6AXJ_J0PEAG1@Z@Z 00000001800073c8 f   WinAccessBridge.obj
 0001:000063d4       ?setPropertyTextChangeFP@WinAccessBridge@@QEAAXP6AXJ_J0@Z@Z 00000001800073d4 f   WinAccessBridge.obj
 0001:000063e0       ?setPropertyValueChangeFP@WinAccessBridge@@QEAAXP6AXJ_J0PEAG1@Z@Z 00000001800073e0 f   WinAccessBridge.obj
 0001:000063ec       ?setPropertyVisibleDataChangeFP@WinAccessBridge@@QEAAXP6AXJ_J0@Z@Z 00000001800073ec f   WinAccessBridge.obj
 0001:000063f8       ?setTextContents@WinAccessBridge@@QEAAHJ_JPEBG@Z 00000001800073f8 f   WinAccessBridge.obj
 0001:000064b4       AccessBridgeDialogProc     00000001800074b4 f   WinAccessBridge.obj
 0001:000065ec       DllMain                    00000001800075ec f   WinAccessBridge.obj
 0001:00006688       ??_U@YAPEAX_K@Z            0000000180007688 f   LIBCMT:new_array.obj
 0001:00006690       ??3@YAXPEAX_K@Z            0000000180007690 f   LIBCMT:delete_scalar_size.obj
 0001:00006690       ??_V@YAXPEAX@Z             0000000180007690 f   LIBCMT:delete_array.obj
 0001:00006698       __GSHandlerCheck           0000000180007698 f   LIBCMT:gshandler.obj
 0001:000066b8       __GSHandlerCheckCommon     00000001800076b8 f   LIBCMT:gshandler.obj
 0001:00006730       __security_check_cookie    0000000180007730 f   LIBCMT:amdsecgs.obj
 0001:00006750       ??_Etype_info@@UEAAPEAXI@Z 0000000180007750 f i LIBCMT:std_type_info_static.obj
 0001:00006750       ??_Gtype_info@@UEAAPEAXI@Z 0000000180007750 f i LIBCMT:std_type_info_static.obj
 0001:0000677c       ??2@YAPEAX_K@Z             000000018000777c f   LIBCMT:new_scalar.obj
 0001:000067d0       __chkstk                   00000001800077d0 f   LIBCMT:chkstk.obj
 0001:000067d0       _alloca_probe              00000001800077d0 f   LIBCMT:chkstk.obj
 0001:00006b40       _DllMainCRTStartup         0000000180007b40 f   LIBCMT:dll_dllmain.obj
 0001:00006b80       ??3@YAXPEAX@Z              0000000180007b80 f   LIBCMT:delete_scalar.obj
 0001:00006b88       __raise_securityfailure    0000000180007b88 f   LIBCMT:gs_report.obj
 0001:00006bbc       __report_gsfailure         0000000180007bbc f   LIBCMT:gs_report.obj
 0001:00006c90       __report_rangecheckfailure 0000000180007c90 f   LIBCMT:gs_report.obj
 0001:00006ca4       __report_securityfailure   0000000180007ca4 f   LIBCMT:gs_report.obj
 0001:00006e24       ??0bad_array_new_length@std@@QEAA@AEBV01@@Z 0000000180007e24 f i LIBCMT:throw_bad_alloc.obj
 0001:00006e60       ??0bad_array_new_length@std@@QEAA@XZ 0000000180007e60 f i LIBCMT:throw_bad_alloc.obj
 0001:00006e80       ?__scrt_throw_std_bad_alloc@@YAXXZ 0000000180007e80 f   LIBCMT:throw_bad_alloc.obj
 0001:00006ea0       ?__scrt_throw_std_bad_array_new_length@@YAXXZ 0000000180007ea0 f   LIBCMT:throw_bad_alloc.obj
 0001:00006ec0       __security_init_cookie     0000000180007ec0 f   LIBCMT:gs_support.obj
 0001:00006f6c       ?__scrt_initialize_type_info@@YAXXZ 0000000180007f6c f   LIBCMT:tncleanup.obj
 0001:00006f7c       ?__scrt_uninitialize_type_info@@YAXXZ 0000000180007f7c f   LIBCMT:tncleanup.obj
 0001:00006f88       __local_stdio_scanf_options 0000000180007f88 f i LIBCMT:default_local_stdio_options.obj
 0001:00006f90       __scrt_initialize_default_local_stdio_options 0000000180007f90 f   LIBCMT:default_local_stdio_options.obj
 0001:00006fac       __scrt_acquire_startup_lock 0000000180007fac f   LIBCMT:utility.obj
 0001:00006fe8       __scrt_dllmain_after_initialize_c 0000000180007fe8 f   LIBCMT:utility.obj
 0001:0000701c       __scrt_dllmain_before_initialize_c 000000018000801c f   LIBCMT:utility.obj
 0001:00007034       __scrt_dllmain_crt_thread_attach 0000000180008034 f   LIBCMT:utility.obj
 0001:0000705c       __scrt_dllmain_crt_thread_detach 000000018000805c f   LIBCMT:utility.obj
 0001:00007074       __scrt_dllmain_exception_filter 0000000180008074 f   LIBCMT:utility.obj
 0001:000070d4       __scrt_dllmain_uninitialize_c 00000001800080d4 f   LIBCMT:utility.obj
 0001:00007104       __scrt_dllmain_uninitialize_critical 0000000180008104 f   LIBCMT:utility.obj
 0001:00007118       __scrt_initialize_crt      0000000180008118 f   LIBCMT:utility.obj
 0001:00007164       __scrt_initialize_onexit_tables 0000000180008164 f   LIBCMT:utility.obj
 0001:000071f0       __scrt_is_nonwritable_in_current_image 00000001800081f0 f   LIBCMT:utility.obj
 0001:00007288       __scrt_release_startup_lock 0000000180008288 f   LIBCMT:utility.obj
 0001:000072ac       __scrt_uninitialize_crt    00000001800082ac f   LIBCMT:utility.obj
 0001:000072d8       __scrt_get_dyn_tls_init_callback 00000001800082d8 f   LIBCMT:dyn_tls_init.obj
 0001:000072e0       __crt_debugger_hook        00000001800082e0 f   LIBCMT:utility_desktop.obj
 0001:000072e8       __scrt_fastfail            00000001800082e8 f   LIBCMT:utility_desktop.obj
 0001:00007434       _RTC_Initialize            0000000180008434 f   LIBCMT:initsect.obj
 0001:00007470       _RTC_Terminate             0000000180008470 f   LIBCMT:initsect.obj
 0001:000074ac       __isa_available_init       00000001800084ac f   LIBCMT:cpu_disp.obj
 0001:00007658       _get_startup_argv_mode     0000000180008658 f   LIBCMT:argv_mode.obj
 0001:00007660       __scrt_is_ucrt_dll_in_use  0000000180008660 f   LIBCMT:ucrt_detection.obj
 0001:00007680       memcpy_repmovs             0000000180008680 f   libvcruntime:memcpy.obj
 0001:000076a0       memcpy                     00000001800086a0 f   libvcruntime:memcpy.obj
 0001:000076a0       memmove                    00000001800086a0 f   libvcruntime:memcpy.obj
 0001:00007d20       memset_repstos             0000000180008d20 f   libvcruntime:memset.obj
 0001:00007d40       memset                     0000000180008d40 f   libvcruntime:memset.obj
 0001:000080c8       __std_exception_copy       00000001800090c8 f   libvcruntime:std_exception.obj
 0001:00008158       __std_exception_destroy    0000000180009158 f   libvcruntime:std_exception.obj
 0001:00008180       _CxxThrowException         0000000180009180 f   libvcruntime:throw.obj
 0001:00008228       __C_specific_handler       0000000180009228 f   libvcruntime:riscchandler.obj
 0001:00008420       __std_type_info_compare    0000000180009420 f   libvcruntime:std_type_info.obj
 0001:00008448       __std_type_info_destroy_list 0000000180009448 f   libvcruntime:std_type_info.obj
 0001:00008474       __vcrt_initialize          0000000180009474 f   libvcruntime:initialization.obj
 0001:0000849c       __vcrt_thread_attach       000000018000949c f   libvcruntime:initialization.obj
 0001:000084b0       __vcrt_thread_detach       00000001800094b0 f   libvcruntime:initialization.obj
 0001:000084c0       __vcrt_uninitialize        00000001800094c0 f   libvcruntime:initialization.obj
 0001:000084dc       __vcrt_uninitialize_critical 00000001800094dc f   libvcruntime:initialization.obj
 0001:000084ec       __DestructExceptionObject  00000001800094ec f   libvcruntime:ehhelpers.obj
 0001:0000855c       ?_CallMemberFunction0@@YAXQEAX0@Z 000000018000955c f i libvcruntime:ehhelpers.obj
 0001:00008560       _IsExceptionObjectToBeDestroyed 0000000180009560 f   libvcruntime:ehhelpers.obj
 0001:00008590       __AdjustPointer            0000000180009590 f   libvcruntime:ehhelpers.obj
 0001:000085b4       __FrameUnwindFilter        00000001800095b4 f   libvcruntime:ehhelpers.obj
 0001:0000861c       __std_terminate            000000018000961c f   libvcruntime:ehhelpers.obj
 0001:00008640       _NLG_Notify                0000000180009640 f   libvcruntime:notify.obj
 0001:00008660       __NLG_Dispatch2            0000000180009660 f   libvcruntime:notify.obj
 0001:00008670       __NLG_Return2              0000000180009670 f   libvcruntime:notify.obj
 0001:00008674       __except_validate_context_record 0000000180009674 f   libvcruntime:jbcxrval.obj
 0001:000086ac       __vcrt_freefls             00000001800096ac f   libvcruntime:per_thread_data.obj
 0001:000086cc       __vcrt_freeptd_for_this_thread 00000001800096cc f   libvcruntime:per_thread_data.obj
 0001:00008714       __vcrt_getptd              0000000180009714 f   libvcruntime:per_thread_data.obj
 0001:00008730       __vcrt_getptd_noexit       0000000180009730 f   libvcruntime:per_thread_data.obj
 0001:000087f0       __vcrt_initialize_ptd      00000001800097f0 f   libvcruntime:per_thread_data.obj
 0001:00008838       __vcrt_uninitialize_ptd    0000000180009838 f   libvcruntime:per_thread_data.obj
 0001:0000885c       __vcrt_initialize_locks    000000018000985c f   libvcruntime:locks.obj
 0001:000088a4       __vcrt_uninitialize_locks  00000001800098a4 f   libvcruntime:locks.obj
 0001:000088dc       ??$_CallSETranslator@V__FrameHandler3@@@@YAHPEAUEHExceptionRecord@@PEA_KPEAU_CONTEXT@@PEAU_xDISPATCHER_CONTEXT@@PEBU_s_FuncInfo@@K1H@Z 00000001800098dc f i libvcruntime:risctrnsctrl.obj
 0001:00008930       ?CatchTryBlock@__FrameHandler3@@SAPEBU_s_TryBlockMapEntry@@PEBU_s_FuncInfo@@H@Z 0000000180009930 f   libvcruntime:risctrnsctrl.obj
 0001:00008994       ?ExecutionInCatch@__FrameHandler3@@SA_NPEAU_xDISPATCHER_CONTEXT@@PEBU_s_FuncInfo@@@Z 0000000180009994 f   libvcruntime:risctrnsctrl.obj
 0001:000089c0       ?FrameUnwindToEmptyState@__FrameHandler3@@SAXPEA_KPEAU_xDISPATCHER_CONTEXT@@PEBU_s_FuncInfo@@@Z 00000001800099c0 f   libvcruntime:risctrnsctrl.obj
 0001:00008a24       ?GetEstablisherFrame@__FrameHandler3@@SAPEA_KPEA_KPEAU_xDISPATCHER_CONTEXT@@PEBU_s_FuncInfo@@0@Z 0000000180009a24 f   libvcruntime:risctrnsctrl.obj
 0001:00008af0       ?GetRangeOfTrysToCheck@__FrameHandler3@@SA?AU?$pair@Viterator@TryBlockMap@__FrameHandler3@@V123@@std@@AEAVTryBlockMap@1@HPEAU_xDISPATCHER_CONTEXT@@PEBU_s_FuncInfo@@H@Z 0000000180009af0 f   libvcruntime:risctrnsctrl.obj
 0001:00008c30       ?UnwindNestedFrames@__FrameHandler3@@SAXPEA_KPEAUEHExceptionRecord@@PEAU_CONTEXT@@0PEAXPEBU_s_FuncInfo@@HHPEBU_s_HandlerType@@PEAU_xDISPATCHER_CONTEXT@@E@Z 0000000180009c30 f   libvcruntime:risctrnsctrl.obj
 0001:00008d34       _CreateFrameInfo           0000000180009d34 f   libvcruntime:risctrnsctrl.obj
 0001:00008d70       _FindAndUnlinkFrame        0000000180009d70 f   libvcruntime:risctrnsctrl.obj
 0001:00008dc4       _GetImageBase              0000000180009dc4 f   libvcruntime:risctrnsctrl.obj
 0001:00008dd8       _GetThrowImageBase         0000000180009dd8 f   libvcruntime:risctrnsctrl.obj
 0001:00008dec       _SetImageBase              0000000180009dec f   libvcruntime:risctrnsctrl.obj
 0001:00008e04       _SetThrowImageBase         0000000180009e04 f   libvcruntime:risctrnsctrl.obj
 0001:00008e1c       __CxxFrameHandler3         0000000180009e1c f   libvcruntime:risctrnsctrl.obj
 0001:00008ff4       __vcrt_FlsAlloc            0000000180009ff4 f   libvcruntime:winapi_downlevel.obj
 0001:0000903c       __vcrt_FlsFree             000000018000a03c f   libvcruntime:winapi_downlevel.obj
 0001:00009084       __vcrt_FlsGetValue         000000018000a084 f   libvcruntime:winapi_downlevel.obj
 0001:000090cc       __vcrt_FlsSetValue         000000018000a0cc f   libvcruntime:winapi_downlevel.obj
 0001:00009120       __vcrt_InitializeCriticalSectionEx 000000018000a120 f   libvcruntime:winapi_downlevel.obj
 0001:00009184       ?GetCurrentState@__FrameHandler3@@SAHPEA_KPEAU_xDISPATCHER_CONTEXT@@PEBU_s_FuncInfo@@@Z 000000018000a184 f   libvcruntime:ehstate.obj
 0001:000091ac       ?GetUnwindTryBlock@__FrameHandler3@@SAHPEA_KPEAU_xDISPATCHER_CONTEXT@@PEBU_s_FuncInfo@@@Z 000000018000a1ac f   libvcruntime:ehstate.obj
 0001:000091d8       ?SetState@__FrameHandler3@@SAXPEA_KPEBU_s_FuncInfo@@H@Z 000000018000a1d8 f   libvcruntime:ehstate.obj
 0001:000091e4       ?SetUnwindTryBlock@__FrameHandler3@@SAXPEA_KPEAU_xDISPATCHER_CONTEXT@@PEBU_s_FuncInfo@@H@Z 000000018000a1e4 f   libvcruntime:ehstate.obj
 0001:00009220       ?StateFromControlPc@__FrameHandler3@@SAHPEBU_s_FuncInfo@@PEAU_xDISPATCHER_CONTEXT@@@Z 000000018000a220 f   libvcruntime:ehstate.obj
 0001:00009228       ?StateFromIp@__FrameHandler3@@SAHPEBU_s_FuncInfo@@PEAU_xDISPATCHER_CONTEXT@@_K@Z 000000018000a228 f   libvcruntime:ehstate.obj
 0001:00009d18       ??$TypeMatchHelper@V__FrameHandler3@@@@YAHPEBU_s_HandlerType@@PEBU_s_CatchableType@@PEBU_s_ThrowInfo@@@Z 000000018000ad18 f i libvcruntime:frame.obj
 0001:00009e58       ??$__InternalCxxFrameHandler@V__FrameHandler3@@@@YA?AW4_EXCEPTION_DISPOSITION@@PEAUEHExceptionRecord@@PEA_KPEAU_CONTEXT@@PEAU_xDISPATCHER_CONTEXT@@PEBU_s_FuncInfo@@H1E@Z 000000018000ae58 f i libvcruntime:frame.obj
 0001:0000a090       ??$__InternalCxxFrameHandlerWrapper@V__FrameHandler3@@@@YA?AW4_EXCEPTION_DISPOSITION@@PEAUEHExceptionRecord@@PEA_KPEAU_CONTEXT@@PEAU_xDISPATCHER_CONTEXT@@PEBU_s_FuncInfo@@H1E@Z 000000018000b090 f i libvcruntime:frame.obj
 0001:0000a098       ??0bad_exception@std@@QEAA@AEBV01@@Z 000000018000b098 f i libvcruntime:frame.obj
 0001:0000a0d4       ??0bad_exception@std@@QEAA@XZ 000000018000b0d4 f i libvcruntime:frame.obj
 0001:0000a0f4       ?CxxCallCatchBlock@__FrameHandler3@@SAPEAXPEAU_EXCEPTION_RECORD@@@Z 000000018000b0f4 f   libvcruntime:frame.obj
 0001:0000a368       ?FrameUnwindToState@__FrameHandler3@@SAXPEA_KPEAU_xDISPATCHER_CONTEXT@@PEBU_s_FuncInfo@@H@Z 000000018000b368 f   libvcruntime:frame.obj
 0001:0000a4f4       ?GetHandlerSearchState@__FrameHandler3@@SAHPEA_KPEAU_xDISPATCHER_CONTEXT@@PEBU_s_FuncInfo@@@Z 000000018000b4f4 f i libvcruntime:frame.obj
 0001:0000a704       ?_CallMemberFunction1@@YAXQEAX00@Z 000000018000b704 f i libvcruntime:frame.obj
 0001:0000a710       ?_CallMemberFunction2@@YAXQEAX00H@Z 000000018000b710 f i libvcruntime:frame.obj
 0001:0000a730       _CallSettingFrame          000000018000b730 f   libvcruntime:handlers.obj
 0001:0000a780       _CallSettingFrame_LookupContinuationIndex 000000018000b780 f   libvcruntime:handlers.obj
 0001:0000a7b0       _CallSettingFrame_NotifyContinuationAddr 000000018000b7b0 f   libvcruntime:handlers.obj
 0001:0000a7e0       _CallSettingFrameEncoded   000000018000b7e0 f   libvcruntime:handlers.obj
 0001:0000a840       strlen                     000000018000b840 f   libucrt:strlen.obj
 0001:0000a900       strncat                    000000018000b900 f   libucrt:strncat.obj
 0001:0000aab0       strncpy                    000000018000bab0 f   libucrt:strncpy.obj
 0001:0000ac14       __acrt_initialize_stdio    000000018000bc14 f   libucrt:_file.obj
 0001:0000ad34       __acrt_iob_func            000000018000bd34 f   libucrt:_file.obj
 0001:0000ad48       __acrt_uninitialize_stdio  000000018000bd48 f   libucrt:_file.obj
 0001:0000ada4       _lock_file                 000000018000bda4 f   libucrt:_file.obj
 0001:0000adb0       _unlock_file               000000018000bdb0 f   libucrt:_file.obj
 0001:0000adfc       ??$ensure_buffer_is_big_enough@D@formatting_buffer@__crt_stdio_output@@QEAA_N_KAEAV__crt_cached_ptd_host@@@Z 000000018000bdfc f i libucrt:output.obj
 0001:0000aea4       ??$parse_integer@KV?$c_string_character_source@D@__crt_strtox@@$0A@@__crt_strtox@@YAKAEAV__crt_cached_ptd_host@@V?$c_string_character_source@D@0@H_N@Z 000000018000bea4 f i libucrt:output.obj
 0001:0000b158       ??$type_case_integer@$07@?$output_processor@DV?$stream_output_adapter@D@__crt_stdio_output@@V?$standard_base@DV?$stream_output_adapter@D@__crt_stdio_output@@@2@@__crt_stdio_output@@AEAA_N_N@Z 000000018000c158 f i libucrt:output.obj
 0001:0000b158       ??$type_case_integer@$07@?$output_processor@DV?$string_output_adapter@D@__crt_stdio_output@@V?$standard_base@DV?$string_output_adapter@D@__crt_stdio_output@@@2@@__crt_stdio_output@@AEAA_N_N@Z 000000018000c158 f i libucrt:output.obj
 0001:0000b35c       ??$type_case_integer@$09@?$output_processor@DV?$stream_output_adapter@D@__crt_stdio_output@@V?$standard_base@DV?$stream_output_adapter@D@__crt_stdio_output@@@2@@__crt_stdio_output@@AEAA_N_N@Z 000000018000c35c f i libucrt:output.obj
 0001:0000b35c       ??$type_case_integer@$09@?$output_processor@DV?$string_output_adapter@D@__crt_stdio_output@@V?$standard_base@DV?$string_output_adapter@D@__crt_stdio_output@@@2@@__crt_stdio_output@@AEAA_N_N@Z 000000018000c35c f i libucrt:output.obj
 0001:0000b560       ??$type_case_integer@$0BA@@?$output_processor@DV?$stream_output_adapter@D@__crt_stdio_output@@V?$standard_base@DV?$stream_output_adapter@D@__crt_stdio_output@@@2@@__crt_stdio_output@@AEAA_N_N@Z 000000018000c560 f i libucrt:output.obj
 0001:0000b560       ??$type_case_integer@$0BA@@?$output_processor@DV?$string_output_adapter@D@__crt_stdio_output@@V?$standard_base@DV?$string_output_adapter@D@__crt_stdio_output@@@2@@__crt_stdio_output@@AEAA_N_N@Z 000000018000c560 f i libucrt:output.obj
 0001:0000b764       ??$type_case_integer_parse_into_buffer@I$07@?$output_processor@DV?$stream_output_adapter@D@__crt_stdio_output@@V?$standard_base@DV?$stream_output_adapter@D@__crt_stdio_output@@@2@@__crt_stdio_output@@AEAAXI_N@Z 000000018000c764 f i libucrt:output.obj
 0001:0000b764       ??$type_case_integer_parse_into_buffer@I$07@?$output_processor@DV?$string_output_adapter@D@__crt_stdio_output@@V?$standard_base@DV?$string_output_adapter@D@__crt_stdio_output@@@2@@__crt_stdio_output@@AEAAXI_N@Z 000000018000c764 f i libucrt:output.obj
 0001:0000b7d4       ??$type_case_integer_parse_into_buffer@I$09@?$output_processor@DV?$stream_output_adapter@D@__crt_stdio_output@@V?$standard_base@DV?$stream_output_adapter@D@__crt_stdio_output@@@2@@__crt_stdio_output@@AEAAXI_N@Z 000000018000c7d4 f i libucrt:output.obj
 0001:0000b7d4       ??$type_case_integer_parse_into_buffer@I$09@?$output_processor@DV?$string_output_adapter@D@__crt_stdio_output@@V?$standard_base@DV?$string_output_adapter@D@__crt_stdio_output@@@2@@__crt_stdio_output@@AEAAXI_N@Z 000000018000c7d4 f i libucrt:output.obj
 0001:0000b880       ??$type_case_integer_parse_into_buffer@I$0BA@@?$output_processor@DV?$stream_output_adapter@D@__crt_stdio_output@@V?$standard_base@DV?$stream_output_adapter@D@__crt_stdio_output@@@2@@__crt_stdio_output@@AEAAXI_N@Z 000000018000c880 f i libucrt:output.obj
 0001:0000b880       ??$type_case_integer_parse_into_buffer@I$0BA@@?$output_processor@DV?$string_output_adapter@D@__crt_stdio_output@@V?$standard_base@DV?$string_output_adapter@D@__crt_stdio_output@@@2@@__crt_stdio_output@@AEAAXI_N@Z 000000018000c880 f i libucrt:output.obj
 0001:0000b904       ??$type_case_integer_parse_into_buffer@_K$07@?$output_processor@DV?$stream_output_adapter@D@__crt_stdio_output@@V?$standard_base@DV?$stream_output_adapter@D@__crt_stdio_output@@@2@@__crt_stdio_output@@AEAAX_K_N@Z 000000018000c904 f i libucrt:output.obj
 0001:0000b904       ??$type_case_integer_parse_into_buffer@_K$07@?$output_processor@DV?$string_output_adapter@D@__crt_stdio_output@@V?$standard_base@DV?$string_output_adapter@D@__crt_stdio_output@@@2@@__crt_stdio_output@@AEAAX_K_N@Z 000000018000c904 f i libucrt:output.obj
 0001:0000b974       ??$type_case_integer_parse_into_buffer@_K$09@?$output_processor@DV?$stream_output_adapter@D@__crt_stdio_output@@V?$standard_base@DV?$stream_output_adapter@D@__crt_stdio_output@@@2@@__crt_stdio_output@@AEAAX_K_N@Z 000000018000c974 f i libucrt:output.obj
 0001:0000b974       ??$type_case_integer_parse_into_buffer@_K$09@?$output_processor@DV?$string_output_adapter@D@__crt_stdio_output@@V?$standard_base@DV?$string_output_adapter@D@__crt_stdio_output@@@2@@__crt_stdio_output@@AEAAX_K_N@Z 000000018000c974 f i libucrt:output.obj
 0001:0000ba24       ??$type_case_integer_parse_into_buffer@_K$0BA@@?$output_processor@DV?$stream_output_adapter@D@__crt_stdio_output@@V?$standard_base@DV?$stream_output_adapter@D@__crt_stdio_output@@@2@@__crt_stdio_output@@AEAAX_K_N@Z 000000018000ca24 f i libucrt:output.obj
 0001:0000ba24       ??$type_case_integer_parse_into_buffer@_K$0BA@@?$output_processor@DV?$string_output_adapter@D@__crt_stdio_output@@V?$standard_base@DV?$string_output_adapter@D@__crt_stdio_output@@@2@@__crt_stdio_output@@AEAAX_K_N@Z 000000018000ca24 f i libucrt:output.obj
 0001:0000bbc4       ?crop_zeroes@__crt_stdio_output@@YAXPEADQEAU__crt_locale_pointers@@@Z 000000018000cbc4 f i libucrt:output.obj
 0001:0000bc30       ?get_raw_ptd@__crt_cached_ptd_host@@QEAAPEAU__acrt_ptd@@XZ 000000018000cc30 f i libucrt:output.obj
 0001:0000bc98       ?parse_int_from_format_string@?$output_processor@DV?$stream_output_adapter@D@__crt_stdio_output@@V?$standard_base@DV?$stream_output_adapter@D@__crt_stdio_output@@@2@@__crt_stdio_output@@AEAA_NQEAH@Z 000000018000cc98 f i libucrt:output.obj
 0001:0000bc98       ?parse_int_from_format_string@?$output_processor@DV?$string_output_adapter@D@__crt_stdio_output@@V?$standard_base@DV?$string_output_adapter@D@__crt_stdio_output@@@2@@__crt_stdio_output@@AEAA_NQEAH@Z 000000018000cc98 f i libucrt:output.obj
 0001:0000bd28       ?process@?$output_processor@DV?$stream_output_adapter@D@__crt_stdio_output@@V?$standard_base@DV?$stream_output_adapter@D@__crt_stdio_output@@@2@@__crt_stdio_output@@QEAAHXZ 000000018000cd28 f i libucrt:output.obj
 0001:0000c0c0       ?process@?$output_processor@DV?$string_output_adapter@D@__crt_stdio_output@@V?$standard_base@DV?$string_output_adapter@D@__crt_stdio_output@@@2@@__crt_stdio_output@@QEAAHXZ 000000018000d0c0 f i libucrt:output.obj
 0001:0000c440       ?state_case_size@?$output_processor@DV?$stream_output_adapter@D@__crt_stdio_output@@V?$standard_base@DV?$stream_output_adapter@D@__crt_stdio_output@@@2@@__crt_stdio_output@@AEAA_NXZ 000000018000d440 f i libucrt:output.obj
 0001:0000c5c8       ?state_case_size@?$output_processor@DV?$string_output_adapter@D@__crt_stdio_output@@V?$standard_base@DV?$string_output_adapter@D@__crt_stdio_output@@@2@@__crt_stdio_output@@AEAA_NXZ 000000018000d5c8 f i libucrt:output.obj
 0001:0000c750       ?state_case_type@?$output_processor@DV?$stream_output_adapter@D@__crt_stdio_output@@V?$standard_base@DV?$stream_output_adapter@D@__crt_stdio_output@@@2@@__crt_stdio_output@@AEAA_NXZ 000000018000d750 f i libucrt:output.obj
 0001:0000cb88       ?state_case_type@?$output_processor@DV?$string_output_adapter@D@__crt_stdio_output@@V?$standard_base@DV?$string_output_adapter@D@__crt_stdio_output@@@2@@__crt_stdio_output@@AEAA_NXZ 000000018000db88 f i libucrt:output.obj
 0001:0000cf8c       ?type_case_Z@?$output_processor@DV?$stream_output_adapter@D@__crt_stdio_output@@V?$standard_base@DV?$stream_output_adapter@D@__crt_stdio_output@@@2@@__crt_stdio_output@@AEAA_NXZ 000000018000df8c f i libucrt:output.obj
 0001:0000cf8c       ?type_case_Z@?$output_processor@DV?$string_output_adapter@D@__crt_stdio_output@@V?$standard_base@DV?$string_output_adapter@D@__crt_stdio_output@@@2@@__crt_stdio_output@@AEAA_NXZ 000000018000df8c f i libucrt:output.obj
 0001:0000d008       ?type_case_a@?$output_processor@DV?$stream_output_adapter@D@__crt_stdio_output@@V?$standard_base@DV?$stream_output_adapter@D@__crt_stdio_output@@@2@@__crt_stdio_output@@AEAA_NXZ 000000018000e008 f i libucrt:output.obj
 0001:0000d008       ?type_case_a@?$output_processor@DV?$string_output_adapter@D@__crt_stdio_output@@V?$standard_base@DV?$string_output_adapter@D@__crt_stdio_output@@@2@@__crt_stdio_output@@AEAA_NXZ 000000018000e008 f i libucrt:output.obj
 0001:0000d25c       ?type_case_c_tchar@?$output_processor@DV?$stream_output_adapter@D@__crt_stdio_output@@V?$standard_base@DV?$stream_output_adapter@D@__crt_stdio_output@@@2@@__crt_stdio_output@@AEAA_ND@Z 000000018000e25c f i libucrt:output.obj
 0001:0000d25c       ?type_case_c_tchar@?$output_processor@DV?$string_output_adapter@D@__crt_stdio_output@@V?$standard_base@DV?$string_output_adapter@D@__crt_stdio_output@@@2@@__crt_stdio_output@@AEAA_ND@Z 000000018000e25c f i libucrt:output.obj
 0001:0000d330       ?type_case_n@?$output_processor@DV?$stream_output_adapter@D@__crt_stdio_output@@V?$standard_base@DV?$stream_output_adapter@D@__crt_stdio_output@@@2@@__crt_stdio_output@@AEAA_NXZ 000000018000e330 f i libucrt:output.obj
 0001:0000d330       ?type_case_n@?$output_processor@DV?$string_output_adapter@D@__crt_stdio_output@@V?$standard_base@DV?$string_output_adapter@D@__crt_stdio_output@@@2@@__crt_stdio_output@@AEAA_NXZ 000000018000e330 f i libucrt:output.obj
 0001:0000d3e8       ?type_case_s@?$output_processor@DV?$stream_output_adapter@D@__crt_stdio_output@@V?$standard_base@DV?$stream_output_adapter@D@__crt_stdio_output@@@2@@__crt_stdio_output@@AEAA_NXZ 000000018000e3e8 f i libucrt:output.obj
 0001:0000d3e8       ?type_case_s@?$output_processor@DV?$string_output_adapter@D@__crt_stdio_output@@V?$standard_base@DV?$string_output_adapter@D@__crt_stdio_output@@@2@@__crt_stdio_output@@AEAA_NXZ 000000018000e3e8 f i libucrt:output.obj
 0001:0000d490       ?update_locale_slow@__crt_cached_ptd_host@@AEAAXXZ 000000018000e490 f i libucrt:output.obj
 0001:0000d508       ?validate_stream_is_ansi_if_required@?$__acrt_stdio_char_traits@D@@SA_NQEAU_iobuf@@@Z 000000018000e508 f i libucrt:output.obj
 0001:0000d5a4       ?write_string@?$string_output_adapter@D@__crt_stdio_output@@QEBAXQEBDHQEAHAEAV__crt_cached_ptd_host@@@Z 000000018000e5a4 f i libucrt:output.obj
 0001:0000d648       ?write_string_impl@?$output_adapter_common@DV?$stream_output_adapter@D@__crt_stdio_output@@@__crt_stdio_output@@IEBAXQEBDHQEAHAEAV__crt_cached_ptd_host@@@Z 000000018000e648 f i libucrt:output.obj
 0001:0000d714       __stdio_common_vfprintf    000000018000e714 f   libucrt:output.obj
 0001:0000d838       __stdio_common_vsprintf    000000018000e838 f   libucrt:output.obj
 0001:0000dbb0       fclose                     000000018000ebb0 f   libucrt:fclose.obj
 0001:0000dd04       fopen                      000000018000ed04 f   libucrt:fopen.obj
 0001:0000ddfc       getenv                     000000018000edfc f   libucrt:getenv.obj
 0001:0000de20       strcmp                     000000018000ee20 f   libucrt:strcmp.obj
 0001:0000dea0       strcat                     000000018000eea0 f   libucrt:strcat.obj
 0001:0000df40       strcpy                     000000018000ef40 f   libucrt:strcat.obj
 0001:0000df43       ___entry_from_strcat_in_strcpy 000000018000ef43     libucrt:strcat.obj
 0001:0000dff8       free                       000000018000eff8 f   libucrt:free.obj
 0001:0000e00c       malloc                     000000018000f00c f   libucrt:malloc.obj
 0001:0000e014       wcsncpy                    000000018000f014 f   libucrt:wcsncpy.obj
 0001:0000e05c       __acrt_initialize_new_handler 000000018000f05c f   libucrt:new_handler.obj
 0001:0000e064       _callnewh                  000000018000f064 f   libucrt:new_handler.obj
 0001:0000e0a4       _query_new_handler         000000018000f0a4 f   libucrt:new_handler.obj
 0001:0000e0dc       _initterm                  000000018000f0dc f   libucrt:initterm.obj
 0001:0000e120       _initterm_e                000000018000f120 f   libucrt:initterm.obj
 0001:0000e168       _seh_filter_dll            000000018000f168 f   libucrt:exception_filter.obj
 0001:0000e17c       _seh_filter_exe            000000018000f17c f   libucrt:exception_filter.obj
 0001:0000e594       __acrt_initialize_thread_local_exit_callback 000000018000f594 f   libucrt:exit.obj
 0001:0000e59c       _cexit                     000000018000f59c f   libucrt:exit.obj
 0001:0000e5ac       _exit                      000000018000f5ac f   libucrt:exit.obj
 0001:0000e5b8       _is_c_termination_complete 000000018000f5b8 f   libucrt:exit.obj
 0001:0000e788       __acrt_allocate_buffer_for_argv 000000018000f788 f   libucrt:argv_parsing.obj
 0001:0000e7e8       _configure_narrow_argv     000000018000f7e8 f   libucrt:argv_parsing.obj
 0001:0000ec50       __dcrt_get_or_create_narrow_environment_nolock 000000018000fc50 f   libucrt:environment_initialization.obj
 0001:0000ec8c       __dcrt_uninitialize_environments_nolock 000000018000fc8c f   libucrt:environment_initialization.obj
 0001:0000ecd0       _initialize_narrow_environment 000000018000fcd0 f   libucrt:environment_initialization.obj
 0001:0000ee34       _execute_onexit_table      000000018000fe34 f   libucrt:onexit.obj
 0001:0000ee78       _initialize_onexit_table   000000018000fe78 f   libucrt:onexit.obj
 0001:0000eed8       __acrt_uninitialize_command_line 000000018000fed8 f   libucrt:argv_data.obj
 0001:0000efd0       __acrt_initialize          000000018000ffd0 f   libucrt:initialization.obj
 0001:0000efe4       __acrt_thread_attach       000000018000ffe4 f   libucrt:initialization.obj
 0001:0000eff8       __acrt_thread_detach       000000018000fff8 f   libucrt:initialization.obj
 0001:0000f008       __acrt_uninitialize        0000000180010008 f   libucrt:initialization.obj
 0001:0000f040       __acrt_uninitialize_critical 0000000180010040 f   libucrt:initialization.obj
 0001:0000f050       terminate                  0000000180010050 f   libucrt:terminate.obj
 0001:0000f07c       strcpy_s                   000000018001007c f   libucrt:strcpy_s.obj
 0001:0000f0dc       abort                      00000001800100dc f   libucrt:abort.obj
 0001:0000f150       strncmp                    0000000180010150 f   libucrt:strncmp.obj
 0001:0000f1d0       calloc                     00000001800101d0 f   libucrt:calloc.obj
 0001:0000f1d8       wcsncmp                    00000001800101d8 f   libucrt:wcsncmp.obj
 0001:0000f204       ?get_raw_ptd_noexit@__crt_cached_ptd_host@@QEAAPEAU__acrt_ptd@@XZ 0000000180010204 f i libucrt:invalid_parameter.obj
 0001:0000f270       ?value@?$dual_state_global@P6AXPEB_W00I_K@Z@__crt_state_management@@QEAAAEAP6AXPEB_W00I_K@ZAEAV__crt_cached_ptd_host@@@Z 0000000180010270 f i libucrt:invalid_parameter.obj
 0001:0000f2bc       __acrt_call_reportfault    00000001800102bc f   libucrt:invalid_parameter.obj
 0001:0000f418       __acrt_initialize_invalid_parameter_handler 0000000180010418 f   libucrt:invalid_parameter.obj
 0001:0000f420       _invalid_parameter         0000000180010420 f   libucrt:invalid_parameter.obj
 0001:0000f4bc       _invalid_parameter_internal 00000001800104bc f   libucrt:invalid_parameter.obj
 0001:0000f588       _invalid_parameter_noinfo  0000000180010588 f   libucrt:invalid_parameter.obj
 0001:0000f5a8       _invoke_watson             00000001800105a8 f   libucrt:invalid_parameter.obj
 0001:0000f5f0       __acrt_errno_from_os_error 00000001800105f0 f   libucrt:errno.obj
 0001:0000f638       __acrt_errno_map_os_error  0000000180010638 f   libucrt:errno.obj
 0001:0000f680       __acrt_errno_map_os_error_ptd 0000000180010680 f   libucrt:errno.obj
 0001:0000f6a4       __doserrno                 00000001800106a4 f   libucrt:errno.obj
 0001:0000f6c4       _errno                     00000001800106c4 f   libucrt:errno.obj
 0001:0000f6e4       _calloc_base               00000001800106e4 f   libucrt:calloc_base.obj
 0001:0000f75c       _free_base                 000000018001075c f   libucrt:free_base.obj
 0001:0000f954       __acrt_AppPolicyGetProcessTerminationMethodInternal 0000000180010954 f   libucrt:winapi_thunks.obj
 0001:0000f9ac       __acrt_AreFileApisANSI     00000001800109ac f   libucrt:winapi_thunks.obj
 0001:0000f9f0       __acrt_CompareStringEx     00000001800109f0 f   libucrt:winapi_thunks.obj
 0001:0000fadc       __acrt_FlsAlloc            0000000180010adc f   libucrt:winapi_thunks.obj
 0001:0000fae4       __acrt_FlsFree             0000000180010ae4 f   libucrt:winapi_thunks.obj
 0001:0000faec       __acrt_FlsGetValue         0000000180010aec f   libucrt:winapi_thunks.obj
 0001:0000faf4       __acrt_FlsSetValue         0000000180010af4 f   libucrt:winapi_thunks.obj
 0001:0000fafc       __acrt_InitializeCriticalSectionEx 0000000180010afc f   libucrt:winapi_thunks.obj
 0001:0000fb6c       __acrt_LCMapStringEx       0000000180010b6c f   libucrt:winapi_thunks.obj
 0001:0000fc58       __acrt_LocaleNameToLCID    0000000180010c58 f   libucrt:winapi_thunks.obj
 0001:0000fcb8       __acrt_initialize_winapi_thunks 0000000180010cb8 f   libucrt:winapi_thunks.obj
 0001:0000fcdc       __acrt_uninitialize_winapi_thunks 0000000180010cdc f   libucrt:winapi_thunks.obj
 0001:0000fd20       _fcloseall                 0000000180010d20 f   libucrt:closeall.obj
 0001:0000ffb4       __acrt_stdio_flush_nolock  0000000180010fb4 f   libucrt:fflush.obj
 0001:00010040       _fflush_nolock             0000000180011040 f   libucrt:fflush.obj
 0001:00010114       _flushall                  0000000180011114 f   libucrt:fflush.obj
 0001:0001011c       __acrt_stdio_free_buffer_nolock 000000018001111c f   libucrt:_freebuf.obj
 0001:00010358       __acrt_initialize_lowio    0000000180011358 f   libucrt:ioinit.obj
 0001:00010394       __acrt_uninitialize_lowio  0000000180011394 f   libucrt:ioinit.obj
 0001:000103d4       _malloc_base               00000001800113d4 f   libucrt:malloc_base.obj
 0001:00010434       strnlen                    0000000180011434 f   libucrt:strnlen.obj
 0001:00010584       wcsnlen                    0000000180011584 f   libucrt:strnlen.obj
 0001:0001075c       __acrt_update_locale_info  000000018001175c f   libucrt:locale_update.obj
 0001:00010790       __acrt_update_locale_info_explicit 0000000180011790 f   libucrt:locale_update.obj
 0001:000107c8       __acrt_update_multibyte_info 00000001800117c8 f   libucrt:locale_update.obj
 0001:000107fc       __acrt_update_multibyte_info_explicit 00000001800117fc f   libucrt:locale_update.obj
 0001:00011348       __acrt_fp_format           0000000180012348 f   libucrt:cvt.obj
 0001:00011630       _wctomb_internal           0000000180012630 f   libucrt:wctomb.obj
 0001:000117e0       _mbtowc_internal           00000001800127e0 f   libucrt:mbtowc.obj
 0001:00011958       _fileno                    0000000180012958 f   libucrt:fileno.obj
 0001:00011980       _get_printf_count_output   0000000180012980 f   libucrt:printf_count_output.obj
 0001:00011998       _fputc_nolock_internal     0000000180012998 f   libucrt:fputc.obj
 0001:000119b0       __acrt_should_use_temporary_buffer 00000001800129b0 f   libucrt:_sftbuf.obj
 0001:000119fc       __acrt_stdio_begin_temporary_buffering_nolock 00000001800129fc f   libucrt:_sftbuf.obj
 0001:00011ac4       __acrt_stdio_end_temporary_buffering_nolock 0000000180012ac4 f   libucrt:_sftbuf.obj
 0001:00011e7c       __acrt_freeptd             0000000180012e7c f   libucrt:per_thread_data.obj
 0001:00011ec0       __acrt_getptd              0000000180012ec0 f   libucrt:per_thread_data.obj
 0001:00011f94       __acrt_getptd_head         0000000180012f94 f   libucrt:per_thread_data.obj
 0001:00012038       __acrt_getptd_noexit       0000000180013038 f   libucrt:per_thread_data.obj
 0001:00012100       __acrt_getptd_noexit_explicit 0000000180013100 f   libucrt:per_thread_data.obj
 0001:000121c0       __acrt_initialize_ptd      00000001800131c0 f   libucrt:per_thread_data.obj
 0001:000121fc       __acrt_uninitialize_ptd    00000001800131fc f   libucrt:per_thread_data.obj
 0001:00012290       __acrt_set_locale_changed  0000000180013290 f   libucrt:wsetlocale.obj
 0001:0001229c       __acrt_uninitialize_locale 000000018001329c f   libucrt:wsetlocale.obj
 0001:00012344       _close_internal            0000000180013344 f   libucrt:close.obj
 0001:00012408       _close_nolock              0000000180013408 f   libucrt:close.obj
 0001:000124a0       _close_nolock_internal     00000001800134a0 f   libucrt:close.obj
 0001:00012570       ?__acrt_stdio_allocate_stream@@YA?AV__crt_stdio_stream@@XZ 0000000180013570 f   libucrt:stream.obj
 0001:000125c8       ?__acrt_stdio_free_stream@@YAXV__crt_stdio_stream@@@Z 00000001800135c8 f   libucrt:stream.obj
 0001:000126d0       ??$__acrt_stdio_parse_mode@D@@YA?AU__acrt_stdio_stream_mode@@QEBD@Z 00000001800136d0 f i libucrt:openfile.obj
 0001:00012994       _openfile                  0000000180013994 f   libucrt:openfile.obj
 0001:00012a30       ??0_LocaleUpdate@@QEAA@QEAU__crt_locale_pointers@@@Z 0000000180013a30 f i libucrt:wcsnicol.obj
 0001:00012acc       _strnicoll                 0000000180013acc f   libucrt:strnicol.obj
 0001:00012ae4       _strnicoll_l               0000000180013ae4 f   libucrt:strnicol.obj
 0001:00012be4       __acrt_initialize_locks    0000000180013be4 f   libucrt:locks.obj
 0001:00012c2c       __acrt_lock                0000000180013c2c f   libucrt:locks.obj
 0001:00012c48       __acrt_uninitialize_locks  0000000180013c48 f   libucrt:locks.obj
 0001:00012c80       __acrt_unlock              0000000180013c80 f   libucrt:locks.obj
 0001:00012c9c       __acrt_app_verifier_enabled 0000000180013c9c f   libucrt:peb_access.obj
 0001:00012cb8       __acrt_is_secure_process   0000000180013cb8 f   libucrt:peb_access.obj
 0001:00012cd0       __acrt_get_process_end_policy 0000000180013cd0 f   libucrt:win_policies.obj
 0001:00012d14       ??$__acrt_convert_wcs_mbs_cp@D_WV<lambda_7c9dea7b4ca7285d2cdb541a38da6275>@@U__crt_win32_buffer_internal_dynamic_resizing@@@@YAHQEBDAEAV?$__crt_win32_buffer@_WU__crt_win32_buffer_internal_dynamic_resizing@@@@AEBV<lambda_7c9dea7b4ca7285d2cdb541a38da6275>@@I@Z 0000000180013d14 f i libucrt:argv_wildcards.obj
 0001:00012e90       ??$__acrt_convert_wcs_mbs_cp@_WDV<lambda_d8593a27d1aa8c02be35c86a17d324c4>@@U__crt_win32_buffer_internal_dynamic_resizing@@@@YAHQEB_WAEAV?$__crt_win32_buffer@DU__crt_win32_buffer_internal_dynamic_resizing@@@@AEBV<lambda_d8593a27d1aa8c02be35c86a17d324c4>@@I@Z 0000000180013e90 f i libucrt:argv_wildcards.obj
 0001:00013734       __acrt_expand_narrow_argv_wildcards 0000000180014734 f   libucrt:argv_wildcards.obj
 0001:0001373c       ??$__acrt_convert_wcs_mbs_cp@_WDV<lambda_f788ae46380686e8b737efdd8c720d07>@@U__crt_win32_buffer_no_resizing@@@@YAHQEB_WAEAV?$__crt_win32_buffer@DU__crt_win32_buffer_no_resizing@@@@AEBV<lambda_f788ae46380686e8b737efdd8c720d07>@@I@Z 000000018001473c f i libucrt:getmodulefilenamea.obj
 0001:00013858       __acrt_GetModuleFileNameA  0000000180014858 f   libucrt:getmodulefilenamea.obj
 0001:00014174       __acrt_initialize_multibyte 0000000180015174 f   libucrt:mbctype.obj
 0001:000141d4       __acrt_update_thread_multibyte_data 00000001800151d4 f   libucrt:mbctype.obj
 0001:000141f0       _setmbcp_nolock            00000001800151f0 f   libucrt:mbctype.obj
 0001:00014524       _ismbblead                 0000000180015524 f   libucrt:ismbbyte.obj
 0001:00014538       __acrt_initialize_command_line 0000000180015538 f   libucrt:argv_data.obj
 0001:00014560       __acrt_MultiByteToWideChar 0000000180015560 f   libucrt:multibytetowidechar.obj
 0001:000145f0       __acrt_WideCharToMultiByte 00000001800155f0 f   libucrt:widechartomultibyte.obj
 0001:000146d0       __dcrt_get_narrow_environment_from_os 00000001800156d0 f   libucrt:get_environment_from_os.obj
 0001:00014c20       __dcrt_set_variable_in_narrow_environment_nolock 0000000180015c20 f   libucrt:setenv.obj
 0001:00014c28       _recalloc_base             0000000180015c28 f   libucrt:recalloc.obj
 0001:00014cc0       __acrt_initialize_heap     0000000180015cc0 f   libucrt:heap_handle.obj
 0001:00014cdc       __acrt_uninitialize_heap   0000000180015cdc f   libucrt:heap_handle.obj
 0001:00014ce8       __acrt_execute_initializers 0000000180015ce8 f   libucrt:shared_initialization.obj
 0001:00014d7c       __acrt_execute_uninitializers 0000000180015d7c f   libucrt:shared_initialization.obj
 0001:00014e0c       __acrt_get_sigabrt_handler 0000000180015e0c f   libucrt:signal.obj
 0001:00014e3c       __acrt_initialize_signal_handlers 0000000180015e3c f   libucrt:signal.obj
 0001:00014e5c       raise                      0000000180015e5c f   libucrt:signal.obj
 0001:000150d8       __acrt_has_user_matherr    00000001800160d8 f   libucrt:matherr.obj
 0001:000150f8       __acrt_initialize_user_matherr 00000001800160f8 f   libucrt:matherr.obj
 0001:00015100       __acrt_invoke_user_matherr 0000000180016100 f   libucrt:matherr.obj
 0001:0001513c       _query_new_mode            000000018001613c f   libucrt:new_mode.obj
 0001:00015144       __acrt_DownlevelLocaleNameToLCID 0000000180016144 f   libucrt:lcidtoname_downlevel.obj
 0001:00015274       _commit                    0000000180016274 f   libucrt:commit.obj
 0001:00015b10       _write                     0000000180016b10 f   libucrt:write.obj
 0001:00015ba8       _write_internal            0000000180016ba8 f   libucrt:write.obj
 0001:00015cc8       _write_nolock              0000000180016cc8 f   libucrt:write.obj
 0001:00015fd0       __acrt_lowio_create_handle_array 0000000180016fd0 f   libucrt:osfinfo.obj
 0001:00016078       __acrt_lowio_destroy_handle_array 0000000180017078 f   libucrt:osfinfo.obj
 0001:000160c8       __acrt_lowio_ensure_fh_exists 00000001800170c8 f   libucrt:osfinfo.obj
 0001:00016170       __acrt_lowio_lock_fh       0000000180017170 f   libucrt:osfinfo.obj
 0001:00016198       __acrt_lowio_set_os_handle 0000000180017198 f   libucrt:osfinfo.obj
 0001:00016258       __acrt_lowio_unlock_fh     0000000180017258 f   libucrt:osfinfo.obj
 0001:00016280       _alloc_osfhnd              0000000180017280 f   libucrt:osfinfo.obj
 0001:000163c0       _free_osfhnd               00000001800173c0 f   libucrt:osfinfo.obj
 0001:0001647c       _get_osfhandle             000000018001747c f   libucrt:osfinfo.obj
 0001:000164f4       __acrt_add_locale_ref      00000001800174f4 f   libucrt:locale_refcounting.obj
 0001:00016580       __acrt_free_locale         0000000180017580 f   libucrt:locale_refcounting.obj
 0001:000166f8       __acrt_locale_add_lc_time_reference 00000001800176f8 f   libucrt:locale_refcounting.obj
 0001:00016720       __acrt_locale_free_lc_time_if_unreferenced 0000000180017720 f   libucrt:locale_refcounting.obj
 0001:00016758       __acrt_locale_release_lc_time_reference 0000000180017758 f   libucrt:locale_refcounting.obj
 0001:00016780       __acrt_release_locale_ref  0000000180017780 f   libucrt:locale_refcounting.obj
 0001:00016828       __acrt_update_thread_locale_data 0000000180017828 f   libucrt:locale_refcounting.obj
 0001:00016898       _updatetlocinfoEx_nolock   0000000180017898 f   libucrt:locale_refcounting.obj
 0001:000169d0       __acrt_fp_strflt_to_string 00000001800179d0 f   libucrt:_fptostr.obj
 0001:00016ae0       ?divide@__crt_strtox@@YA_KAEAUbig_integer@1@AEBU21@@Z 0000000180017ae0 f i libucrt:cfout.obj
 0001:00016f7c       __acrt_fltout              0000000180017f7c f   libucrt:cfout.obj
 0001:00018294       fegetround                 0000000180019294 f   libucrt:fegetround.obj
 0001:000182a8       ?__c32rtomb_utf8@__crt_mbstring@@YA_KPEAD_UPEAU_Mbstatet@@AEAV__crt_cached_ptd_host@@@Z 00000001800192a8 f   libucrt:c32rtomb.obj
 0001:0001834c       ?__mbrtowc_utf8@__crt_mbstring@@YA_KPEA_WPEBD_KPEAU_Mbstatet@@AEAV__crt_cached_ptd_host@@@Z 000000018001934c f   libucrt:mbrtowc.obj
 0001:00018390       ?__mbsrtowcs_utf8@__crt_mbstring@@YA_KPEA_WPEAPEBD_KPEAU_Mbstatet@@AEAV__crt_cached_ptd_host@@@Z 0000000180019390 f   libucrt:mbrtowc.obj
 0001:000186a8       __acrt_stdio_flush_and_write_narrow_nolock 00000001800196a8 f   libucrt:_flsbuf.obj
 0001:00018774       _isatty                    0000000180019774 f   libucrt:isatty.obj
 0001:000187d4       __acrt_locale_free_monetary 00000001800197d4 f   libucrt:initmon.obj
 0001:000188e0       __acrt_locale_free_numeric 00000001800198e0 f   libucrt:initnum.obj
 0001:00018980       __acrt_locale_free_time    0000000180019980 f   libucrt:inittime.obj
 0001:00018a88       __acrt_GetStringTypeA      0000000180019a88 f   libucrt:getstringtypea.obj
 0001:00018c18       __ascii_wcsnicmp           0000000180019c18 f   libucrt:wcsnicmp.obj
 0001:00018c64       __ascii_strnicmp           0000000180019c64 f   libucrt:strnicmp.obj
 0001:00018cb0       _strnicmp                  0000000180019cb0 f   libucrt:strnicmp.obj
 0001:00018d00       _strnicmp_l                0000000180019d00 f   libucrt:strnicmp.obj
 0001:000193c0       _sopen_nolock              000000018001a3c0 f   libucrt:open.obj
 0001:000194dc       _sopen_s                   000000018001a4dc f   libucrt:open.obj
 0001:00019510       _wsopen_nolock             000000018001a510 f   libucrt:open.obj
 0001:00019c84       __acrt_CompareStringA      000000018001ac84 f   libucrt:comparestringa.obj
 0001:00019d10       qsort                      000000018001ad10 f   libucrt:qsort.obj
 0001:0001a120       strncpy_s                  000000018001b120 f   libucrt:strncpy_s.obj
 0001:0001a2b0       strpbrk                    000000018001b2b0 f   libucrt:strpbrk.obj
 0001:0001a678       _mbsdec                    000000018001b678 f   libucrt:mbsdec.obj
 0001:0001a680       _mbsdec_l                  000000018001b680 f   libucrt:mbsdec.obj
 0001:0001aa48       __acrt_LCMapStringA        000000018001ba48 f   libucrt:lcmapstringa.obj
 0001:0001aaf8       __acrt_SetEnvironmentVariableA 000000018001baf8 f   libucrt:setenvironmentvariablea.obj
 0001:0001ac98       _msize_base                000000018001bc98 f   libucrt:msize.obj
 0001:0001acd4       _realloc_base              000000018001bcd4 f   libucrt:realloc_base.obj
 0001:0001af1c       _lseeki64                  000000018001bf1c f   libucrt:lseek.obj
 0001:0001afb8       _lseeki64_nolock           000000018001bfb8 f   libucrt:lseek.obj
 0001:0001b054       _lseeki64_nolock_internal  000000018001c054 f   libucrt:lseek.obj
 0001:0001b05c       _putwch_nolock             000000018001c05c f   libucrt:putwch.obj
 0001:0001b520       _read_nolock               000000018001c520 f   libucrt:read.obj
 0001:0001b970       _query_app_type            000000018001c970 f   libucrt:report_runtime_error.obj
 0001:0001b978       _controlfp_s               000000018001c978 f   libucrt:contrlfp.obj
 0001:0001b9dc       fegetenv                   000000018001c9dc f   libucrt:fegetenv.obj
 0001:0001b9fc       fesetenv                   000000018001c9fc f   libucrt:fesetenv.obj
 0001:0001ba54       feholdexcept               000000018001ca54 f   libucrt:feholdexcept.obj
 0001:0001baa4       ceil                       000000018001caa4 f   libucrt:ceil.obj
 0001:0001bb70       log10                      000000018001cb70 f   libucrt:log10.obj
 0001:0001c11c       __acrt_fenv_get_common_round_control 000000018001d11c f   libucrt:_fenvutils.obj
 0001:0001c128       __acrt_fenv_get_control    000000018001d128 f   libucrt:_fenvutils.obj
 0001:0001c20c       __acrt_fenv_get_status     000000018001d20c f   libucrt:_fenvutils.obj
 0001:0001c264       __acrt_fenv_set_control    000000018001d264 f   libucrt:_fenvutils.obj
 0001:0001c39c       __acrt_fenv_set_status     000000018001d39c f   libucrt:_fenvutils.obj
 0001:0001c410       ?reset_and_return@__crt_mbstring@@YA_K_KPEAU_Mbstatet@@@Z 000000018001d410 f   libucrt:common_utf8.obj
 0001:0001c418       ?return_illegal_sequence@__crt_mbstring@@YA_KPEAU_Mbstatet@@AEAV__crt_cached_ptd_host@@@Z 000000018001d418 f   libucrt:common_utf8.obj
 0001:0001c42c       ?__mbrtoc32_utf8@__crt_mbstring@@YA_KPEA_UPEBD_KPEAU_Mbstatet@@AEAV__crt_cached_ptd_host@@@Z 000000018001d42c f   libucrt:mbrtoc32.obj
 0001:0001c608       __acrt_stdio_allocate_buffer_nolock 000000018001d608 f   libucrt:_getbuf.obj
 0001:0001c674       _get_fmode                 000000018001d674 f   libucrt:setmode.obj
 0001:0001c6a4       _setmode_nolock            000000018001d6a4 f   libucrt:setmode.obj
 0001:0001c788       _chsize_nolock             000000018001d788 f   libucrt:chsize.obj
 0001:0001c820       _chsize_nolock_internal    000000018001d820 f   libucrt:chsize.obj
 0001:0001c9b4       __strncnt                  000000018001d9b4 f   libucrt:strncnt.obj
 0001:0001c9cc       __dcrt_lowio_ensure_console_output_initialized 000000018001d9cc f   libucrt:initcon.obj
 0001:0001ca20       __dcrt_terminate_console_output 000000018001da20 f   libucrt:initcon.obj
 0001:0001ca3c       __dcrt_write_console       000000018001da3c f   libucrt:initcon.obj
 0001:0001cafc       _clearfp                   000000018001dafc f   libucrt:ieee.obj
 0001:0001cb68       _control87                 000000018001db68 f   libucrt:ieee.obj
 0001:0001cf30       _handle_error              000000018001df30 f   libucrt:libm_error.obj
 0001:0001d058       _handle_nan                000000018001e058 f   libucrt:libm_error.obj
 0001:0001d080       __acrt_initialize_fma3     000000018001e080 f   libucrt:fma3_available.obj
 0001:0001d0f0       _log10_special             000000018001e0f0 f   libucrt:log_special.obj
 0001:0001d1a8       __acrt_initialize_fmode    000000018001e1a8 f   libucrt:txtmode.obj
 0001:0001d1e0       _get_fpsr                  000000018001e1e0 f   libucrt:fpsr.obj
 0001:0001d1f0       _set_fpsr                  000000018001e1f0 f   libucrt:fpsr.obj
 0001:0001d1fa       _fclrf                     000000018001e1fa f   libucrt:fpsr.obj
 0001:0001d20e       _frnd                      000000018001e20e f   libucrt:fpsr.obj
 0001:0001d230       _raise_exc                 000000018001e230 f   libucrt:fpexcept.obj
 0001:0001d258       _raise_exc_ex              000000018001e258 f   libucrt:fpexcept.obj
 0001:0001d560       _set_errno_from_matherr    000000018001e560 f   libucrt:fpexcept.obj
 0001:0001d590       _clrfp                     000000018001e590 f   libucrt:fpctrl.obj
 0001:0001d5b0       _ctrlfp                    000000018001e5b0 f   libucrt:fpctrl.obj
 0001:0001d62c       _set_statfp                000000018001e62c f   libucrt:fpctrl.obj
 0001:0001d64c       _statfp                    000000018001e64c f   libucrt:fpctrl.obj
 0001:0001d660       _FindPESection             000000018001e660 f   LIBCMT:pesect.obj
 0001:0001d6b0       _IsNonwritableInCurrentImage 000000018001e6b0 f   LIBCMT:pesect.obj
 0001:0001d700       _ValidateImageBase         000000018001e700 f   LIBCMT:pesect.obj
 0001:0001d72c       __GSHandlerCheck_EH        000000018001e72c f   LIBCMT:gshandlereh.obj
 0001:0001d7ac       __C_specific_handler_noexcept 000000018001e7ac f   libvcruntime:chandler_noexcept.obj
 0001:0001d7f8       strrchr                    000000018001e7f8 f   libvcruntime:strrchr.obj
 0001:0001d950       memcmp                     000000018001e950 f   libvcruntime:memcmp.obj
 0001:0001da18       strchr                     000000018001ea18 f   libvcruntime:strchr.obj
 0001:0001dab0       _guard_dispatch_icall_nop  000000018001eab0 f   LIBCMT:guard_dispatch.obj
 0001:0001dad0       _guard_xfg_dispatch_icall_nop 000000018001ead0 f   LIBCMT:guard_xfg_dispatch.obj
 0002:00000000       __imp_GetLastError         0000000180020000     kernel32:KERNEL32.dll
 0002:00000008       __imp_GetSystemTimeAsFileTime 0000000180020008     kernel32:KERNEL32.dll
 0002:00000010       __imp_CloseHandle          0000000180020010     kernel32:KERNEL32.dll
 0002:00000018       __imp_EnterCriticalSection 0000000180020018     kernel32:KERNEL32.dll
 0002:00000020       __imp_LeaveCriticalSection 0000000180020020     kernel32:KERNEL32.dll
 0002:00000028       __imp_MapViewOfFile        0000000180020028     kernel32:KERNEL32.dll
 0002:00000030       __imp_UnmapViewOfFile      0000000180020030     kernel32:KERNEL32.dll
 0002:00000038       __imp_CreateFileMappingA   0000000180020038     kernel32:KERNEL32.dll
 0002:00000040       __imp_InitializeCriticalSection 0000000180020040     kernel32:KERNEL32.dll
 0002:00000048       __imp_WriteConsoleW        0000000180020048     kernel32:KERNEL32.dll
 0002:00000050       __imp_SetEndOfFile         0000000180020050     kernel32:KERNEL32.dll
 0002:00000058       __imp_ReadConsoleW         0000000180020058     kernel32:KERNEL32.dll
 0002:00000060       __imp_ReadFile             0000000180020060     kernel32:KERNEL32.dll
 0002:00000068       __imp_HeapReAlloc          0000000180020068     kernel32:KERNEL32.dll
 0002:00000070       __imp_HeapSize             0000000180020070     kernel32:KERNEL32.dll
 0002:00000078       __imp_CreateFileW          0000000180020078     kernel32:KERNEL32.dll
 0002:00000080       __imp_GetStringTypeW       0000000180020080     kernel32:KERNEL32.dll
 0002:00000088       __imp_SetFilePointerEx     0000000180020088     kernel32:KERNEL32.dll
 0002:00000090       __imp_GetFileSizeEx        0000000180020090     kernel32:KERNEL32.dll
 0002:00000098       __imp_SetStdHandle         0000000180020098     kernel32:KERNEL32.dll
 0002:000000a0       __imp_GetConsoleMode       00000001800200a0     kernel32:KERNEL32.dll
 0002:000000a8       __imp_GetConsoleOutputCP   00000001800200a8     kernel32:KERNEL32.dll
 0002:000000b0       __imp_WriteFile            00000001800200b0     kernel32:KERNEL32.dll
 0002:000000b8       __imp_RtlCaptureContext    00000001800200b8     kernel32:KERNEL32.dll
 0002:000000c0       __imp_RtlLookupFunctionEntry 00000001800200c0     kernel32:KERNEL32.dll
 0002:000000c8       __imp_RtlVirtualUnwind     00000001800200c8     kernel32:KERNEL32.dll
 0002:000000d0       __imp_UnhandledExceptionFilter 00000001800200d0     kernel32:KERNEL32.dll
 0002:000000d8       __imp_SetUnhandledExceptionFilter 00000001800200d8     kernel32:KERNEL32.dll
 0002:000000e0       __imp_GetCurrentProcess    00000001800200e0     kernel32:KERNEL32.dll
 0002:000000e8       __imp_TerminateProcess     00000001800200e8     kernel32:KERNEL32.dll
 0002:000000f0       __imp_IsProcessorFeaturePresent 00000001800200f0     kernel32:KERNEL32.dll
 0002:000000f8       __imp_QueryPerformanceCounter 00000001800200f8     kernel32:KERNEL32.dll
 0002:00000100       __imp_GetCurrentProcessId  0000000180020100     kernel32:KERNEL32.dll
 0002:00000108       __imp_GetCurrentThreadId   0000000180020108     kernel32:KERNEL32.dll
 0002:00000110       __imp_InitializeSListHead  0000000180020110     kernel32:KERNEL32.dll
 0002:00000118       __imp_IsDebuggerPresent    0000000180020118     kernel32:KERNEL32.dll
 0002:00000120       __imp_GetStartupInfoW      0000000180020120     kernel32:KERNEL32.dll
 0002:00000128       __imp_GetModuleHandleW     0000000180020128     kernel32:KERNEL32.dll
 0002:00000130       __imp_RtlPcToFileHeader    0000000180020130     kernel32:KERNEL32.dll
 0002:00000138       __imp_RaiseException       0000000180020138     kernel32:KERNEL32.dll
 0002:00000140       __imp_RtlUnwindEx          0000000180020140     kernel32:KERNEL32.dll
 0002:00000148       __imp_InterlockedFlushSList 0000000180020148     kernel32:KERNEL32.dll
 0002:00000150       __imp_SetLastError         0000000180020150     kernel32:KERNEL32.dll
 0002:00000158       __imp_DeleteCriticalSection 0000000180020158     kernel32:KERNEL32.dll
 0002:00000160       __imp_InitializeCriticalSectionAndSpinCount 0000000180020160     kernel32:KERNEL32.dll
 0002:00000168       __imp_TlsAlloc             0000000180020168     kernel32:KERNEL32.dll
 0002:00000170       __imp_TlsGetValue          0000000180020170     kernel32:KERNEL32.dll
 0002:00000178       __imp_TlsSetValue          0000000180020178     kernel32:KERNEL32.dll
 0002:00000180       __imp_TlsFree              0000000180020180     kernel32:KERNEL32.dll
 0002:00000188       __imp_FreeLibrary          0000000180020188     kernel32:KERNEL32.dll
 0002:00000190       __imp_GetProcAddress       0000000180020190     kernel32:KERNEL32.dll
 0002:00000198       __imp_LoadLibraryExW       0000000180020198     kernel32:KERNEL32.dll
 0002:000001a0       __imp_EncodePointer        00000001800201a0     kernel32:KERNEL32.dll
 0002:000001a8       __imp_ExitProcess          00000001800201a8     kernel32:KERNEL32.dll
 0002:000001b0       __imp_GetModuleHandleExW   00000001800201b0     kernel32:KERNEL32.dll
 0002:000001b8       __imp_GetModuleFileNameW   00000001800201b8     kernel32:KERNEL32.dll
 0002:000001c0       __imp_HeapAlloc            00000001800201c0     kernel32:KERNEL32.dll
 0002:000001c8       __imp_HeapFree             00000001800201c8     kernel32:KERNEL32.dll
 0002:000001d0       __imp_FlsAlloc             00000001800201d0     kernel32:KERNEL32.dll
 0002:000001d8       __imp_FlsGetValue          00000001800201d8     kernel32:KERNEL32.dll
 0002:000001e0       __imp_FlsSetValue          00000001800201e0     kernel32:KERNEL32.dll
 0002:000001e8       __imp_FlsFree              00000001800201e8     kernel32:KERNEL32.dll
 0002:000001f0       __imp_CompareStringW       00000001800201f0     kernel32:KERNEL32.dll
 0002:000001f8       __imp_LCMapStringW         00000001800201f8     kernel32:KERNEL32.dll
 0002:00000200       __imp_GetStdHandle         0000000180020200     kernel32:KERNEL32.dll
 0002:00000208       __imp_GetFileType          0000000180020208     kernel32:KERNEL32.dll
 0002:00000210       __imp_FindClose            0000000180020210     kernel32:KERNEL32.dll
 0002:00000218       __imp_FindFirstFileExW     0000000180020218     kernel32:KERNEL32.dll
 0002:00000220       __imp_FindNextFileW        0000000180020220     kernel32:KERNEL32.dll
 0002:00000228       __imp_IsValidCodePage      0000000180020228     kernel32:KERNEL32.dll
 0002:00000230       __imp_GetACP               0000000180020230     kernel32:KERNEL32.dll
 0002:00000238       __imp_GetOEMCP             0000000180020238     kernel32:KERNEL32.dll
 0002:00000240       __imp_GetCPInfo            0000000180020240     kernel32:KERNEL32.dll
 0002:00000248       __imp_GetCommandLineA      0000000180020248     kernel32:KERNEL32.dll
 0002:00000250       __imp_GetCommandLineW      0000000180020250     kernel32:KERNEL32.dll
 0002:00000258       __imp_MultiByteToWideChar  0000000180020258     kernel32:KERNEL32.dll
 0002:00000260       __imp_WideCharToMultiByte  0000000180020260     kernel32:KERNEL32.dll
 0002:00000268       __imp_GetEnvironmentStringsW 0000000180020268     kernel32:KERNEL32.dll
 0002:00000270       __imp_FreeEnvironmentStringsW 0000000180020270     kernel32:KERNEL32.dll
 0002:00000278       __imp_SetEnvironmentVariableW 0000000180020278     kernel32:KERNEL32.dll
 0002:00000280       __imp_GetProcessHeap       0000000180020280     kernel32:KERNEL32.dll
 0002:00000288       __imp_FlushFileBuffers     0000000180020288     kernel32:KERNEL32.dll
 0002:00000290       \177KERNEL32_NULL_THUNK_DATA 0000000180020290     kernel32:KERNEL32.dll
 0002:00000298       __imp_CreateDialogParamA   0000000180020298     user32:USER32.dll
 0002:000002a0       __imp_ShowWindow           00000001800202a0     user32:USER32.dll
 0002:000002a8       __imp_DestroyWindow        00000001800202a8     user32:USER32.dll
 0002:000002b0       __imp_SendMessageA         00000001800202b0     user32:USER32.dll
 0002:000002b8       __imp_GetParent            00000001800202b8     user32:USER32.dll
 0002:000002c0       __imp_GetWindowLongA       00000001800202c0     user32:USER32.dll
 0002:000002c8       __imp_IsWindow             00000001800202c8     user32:USER32.dll
 0002:000002d0       __imp_RegisterWindowMessageA 00000001800202d0     user32:USER32.dll
 0002:000002d8       __imp_SendMessageTimeoutA  00000001800202d8     user32:USER32.dll
 0002:000002e0       __imp_PostMessageA         00000001800202e0     user32:USER32.dll
 0002:000002e8       \177USER32_NULL_THUNK_DATA 00000001800202e8     user32:USER32.dll
 0002:000002f0       __guard_check_icall_fptr   00000001800202f0     LIBCMT:guard_support.obj
 0002:000002f8       __guard_xfg_check_icall_fptr 00000001800202f8     LIBCMT:guard_support.obj
 0002:00000300       __guard_dispatch_icall_fptr 0000000180020300     LIBCMT:guard_support.obj
 0002:00000308       __guard_xfg_dispatch_icall_fptr 0000000180020308     LIBCMT:guard_support.obj
 0002:00000310       __guard_xfg_table_dispatch_icall_fptr 0000000180020310     LIBCMT:guard_support.obj
 0002:00000318       __castguard_check_failure_os_handled_fptr 0000000180020318     LIBCMT:guard_support.obj
 0002:00000320       __guard_memcpy_fptr        0000000180020320     libvcruntime:softmemtag.obj
 0002:00000328       __xc_a                     0000000180020328     LIBCMT:initializers.obj
 0002:00000330       __xc_z                     0000000180020330     LIBCMT:initializers.obj
 0002:00000338       __xi_a                     0000000180020338     LIBCMT:initializers.obj
 0002:00000340       __acrt_stdio_initializer   0000000180020340     libucrt:stdio_initializer.obj
 0002:00000348       __acrt_multibyte_initializer 0000000180020348     libucrt:multibyte_initializer.obj
 0002:00000350       __acrt_tran_fma3_initializer 0000000180020350     libucrt:fma3_initializer.obj
 0002:00000358       __acrt_fmode_initializer   0000000180020358     libucrt:fmode_initializer.obj
 0002:00000360       __xi_z                     0000000180020360     LIBCMT:initializers.obj
 0002:00000368       __xp_a                     0000000180020368     LIBCMT:initializers.obj
 0002:00000370       __acrt_locale_terminator   0000000180020370     libucrt:locale_initializer.obj
 0002:00000378       __dcrt_console_output_terminator 0000000180020378     libucrt:console_output_initializer.obj
 0002:00000380       __acrt_stdio_terminator    0000000180020380     libucrt:stdio_initializer.obj
 0002:00000388       __xp_z                     0000000180020388     LIBCMT:initializers.obj
 0002:00000390       __xt_a                     0000000180020390     LIBCMT:initializers.obj
 0002:00000398       __xt_z                     0000000180020398     LIBCMT:initializers.obj
 0002:000003a0       ??_C@_0BJ@FKCDJFDK@JAVA_ACCESSBRIDGE_LOGDIR@ 00000001800203a0     AccessBridgeDebug.obj
 0002:000003bc       ??_C@_04FPOLKAEB@?4log@    00000001800203bc     AccessBridgeDebug.obj
 0002:000003c4       ??_C@_01NOFIACDB@w@        00000001800203c4     AccessBridgeDebug.obj
 0002:000003c8       ??_C@_04EINJHBMM@?6?$CFs?6@ 00000001800203c8     AccessBridgeDebug.obj
 0002:000003d0       ??_C@_0BH@PPBGFLKL@Could?5not?5open?5file?5?$CFs@ 00000001800203d0     AccessBridgeDebug.obj
 0002:000003e8       ??_C@_07IBOBEFLP@?$FL?$CFllu?$FN?5@ 00000001800203e8     AccessBridgeDebug.obj
 0002:000003f0       ??_C@_02PCIJFNDE@?$AN?6@   00000001800203f0     AccessBridgeDebug.obj
 0002:000003f8       ??_C@_0BH@BLGOOJIK@AccessBridge?9?$CFp?9?$CFp?4mmf@ 00000001800203f8     AccessBridgeJavaVMInstance.obj
 0002:00000410       ??_C@_03DJNNCAJF@OK?$DP@   0000000180020410     AccessBridgeJavaVMInstance.obj
 0002:00000414       ??_C@_03ONJMBPEK@OK?$CB@   0000000180020414     AccessBridgeJavaVMInstance.obj
 0002:00000418       ??_C@_0CP@JIGBIHFH@?$FLINFO?$FN?3?5In?5AccessBridgeVMInstan@ 0000000180020418     AccessBridgeJavaVMInstance.obj
 0002:00000448       ??_C@_0CH@KAGNBCII@?$FLINFO?$FN?3?5?5?5?5?5javaAccessBridgeWin@ 0000000180020448     AccessBridgeJavaVMInstance.obj
 0002:00000470       ??_C@_0CC@NKGMANMJ@?$FLINFO?$FN?3?5In?5findAccessBridgeWind@ 0000000180020470     AccessBridgeJavaVMInstance.obj
 0002:00000498       ??_C@_0CK@NBPNOPCH@?$FLINFO?$FN?3?5In?5findABJavaInstanceFr@ 0000000180020498     AccessBridgeJavaVMInstance.obj
 0002:000004d0       ??_7exception@std@@6B@     00000001800204d0     AccessBridgeMessageQueue.obj
 0002:000004e0       ??_C@_0BC@EOODALEL@Unknown?5exception@ 00000001800204e0     AccessBridgeMessageQueue.obj
 0002:00000500       ??_7bad_alloc@std@@6B@     0000000180020500     AccessBridgeMessageQueue.obj
 0002:00000510       ??_C@_0P@GHFPNOJB@bad?5allocation@ 0000000180020510     AccessBridgeMessageQueue.obj
 0002:00000520       ??_C@_0CN@EPCNBBKD@?$FLINFO?$FN?3?5?5?5in?5AccessBridgeMessag@ 0000000180020520     AccessBridgeMessageQueue.obj
 0002:00000550       ??_C@_0BM@FHOEMINC@?$FLINFO?$FN?3?5?5?5?5?5queue?5size?5?$DN?5?$CFd@ 0000000180020550     AccessBridgeMessageQueue.obj
 0002:00000570       ??_C@_0DF@PKPPNDEN@?$FLWARN?$FN?3?5?5?5?5?5queue?5was?5locked?$DL?5r@ 0000000180020570     AccessBridgeMessageQueue.obj
 0002:000005a8       ??_C@_0CF@CAPEOLCL@?$FLINFO?$FN?3?5?5?5?5?5adding?5element?5to?5q@ 00000001800205a8     AccessBridgeMessageQueue.obj
 0002:000005d0       ??_C@_0DL@IILCMNMG@?$FLINFO?$FN?3?5?5?5?5?5returning?5from?5Acce@ 00000001800205d0     AccessBridgeMessageQueue.obj
 0002:00000610       ??_C@_0DA@NHLJEKKG@?$FLINFO?$FN?3?5?5?5in?5AccessBridgeMessag@ 0000000180020610     AccessBridgeMessageQueue.obj
 0002:00000640       ??_C@_0CJ@FBOCEMKO@?$FLINFO?$FN?3?5?5?5?5?5removing?5element?5fr@ 0000000180020640     AccessBridgeMessageQueue.obj
 0002:00000670       ??_C@_0DO@NEJIEHGM@?$FLINFO?$FN?3?5?5?5?5?5returning?5from?5Acce@ 0000000180020670     AccessBridgeMessageQueue.obj
 0002:000006b0       ??_C@_0BM@BIAOFPJG@AccessBridge?9FromJava?9Hello@ 00000001800206b0     AccessBridgeMessages.obj
 0002:000006d0       ??_C@_0BP@OELHMMDF@AccessBridge?9FromWindows?9Hello@ 00000001800206d0     AccessBridgeMessages.obj
 0002:000006f0       ??_C@_0EC@DLPGLEGA@?$AN?6AccessBridgeWindowsEntryPoint@ 00000001800206f0     AccessBridgeWindowsEntryPoints.obj
 0002:00000738       ??_C@_0BG@GGFIABLO@windows_access_bridge@ 0000000180020738     WinAccessBridge.obj
 0002:00000750       ??_C@_0BL@GLCNGDJJ@?$FLINFO?$FN?3?5DLL_PROCESS_ATTACH@ 0000000180020750     WinAccessBridge.obj
 0002:00000770       ??_C@_0EG@HHOMJPNP@?$FLINFO?$FN?3?5?$CK?$CK?$CK?5AccessBridgeDialogP@ 0000000180020770     WinAccessBridge.obj
 0002:000007b8       ??_C@_0CP@LHINEKAP@?$FLINFO?$FN?3?5AccessBridgeDialogProc?5@ 00000001800207b8     WinAccessBridge.obj
 0002:000007f0       ??_C@_0EH@MDELPMEJ@?$FLINFO?$FN?3?5AccessBridgeDialogProc?5@ 00000001800207f0     WinAccessBridge.obj
 0002:00000838       ??_C@_0DP@HBEMDAPF@?$FLINFO?$FN?3?5AccessBridgeDialogProc?5@ 0000000180020838     WinAccessBridge.obj
 0002:00000880       ??_C@_0EH@MPLEACPJ@?$FLINFO?$FN?3?5AccessBridgeDialogProc?5@ 0000000180020880     WinAccessBridge.obj
 0002:000008d0       ??_C@_0EG@GGGHDKAD@?$FLINFO?$FN?3?5?$CK?$CK?$CK?$CK?$CK?5AccessBridgeDialo@ 00000001800208d0     WinAccessBridge.obj
 0002:00000918       ??_C@_0DE@BGNNIIOB@?$FLINFO?$FN?3?5?5?5javaVMs?5chain?5in?5use?0@ 0000000180020918     WinAccessBridge.obj
 0002:00000950       ??_C@_0CC@NEJJLLGC@?$FLINFO?$FN?3?5?5?5calling?5javaVMDestroy@ 0000000180020950     WinAccessBridge.obj
 0002:00000980       ??_C@_0FG@BHPCMIAO@?$FLINFO?$FN?3?5AccessBridgeDialogProc?5@ 0000000180020980     WinAccessBridge.obj
 0002:000009d8       ??_C@_0BN@FIPGEIKI@?$FLINFO?$FN?3?5WinAccessBridge?5ctor@ 00000001800209d8     WinAccessBridge.obj
 0002:000009f8       ??_C@_0DE@JFKNENGC@?$FLINFO?$FN?3?5?$CK?$CK?$CK?$CK?$CKin?5WinAccessBridge@ 00000001800209f8     WinAccessBridge.obj
 0002:00000a30       ??_C@_0CG@EDMKMONP@?$FLINFO?$FN?3?5?5?5telling?5?$CFp?5we?8re?5goin@ 0000000180020a30     WinAccessBridge.obj
 0002:00000a58       ??_C@_0DB@CFPLAPDG@?$FLINFO?$FN?3?5?5?5finished?5telling?5JVMs@ 0000000180020a58     WinAccessBridge.obj
 0002:00000a90       ??_C@_0EE@GBJFCFOA@?$FLINFO?$FN?3?5?5?5finished?5deleting?5eve@ 0000000180020a90     WinAccessBridge.obj
 0002:00000ad8       ??_C@_0BP@EBFMIPOK@?$FLINFO?$FN?3?5GOODBYE?5CRUEL?5WORLD?4?4?4@ 0000000180020ad8     WinAccessBridge.obj
 0002:00000af8       ??_C@_0BJ@LMONFDOG@ACCESSBRIDGESTATUSWINDOW@ 0000000180020af8     WinAccessBridge.obj
 0002:00000b18       ??_C@_0DN@NNELAOKC@?$FLINFO?$FN?3?5in?5WinAccessBridge?3?3ren@ 0000000180020b18     WinAccessBridge.obj
 0002:00000b58       ??_C@_0CJ@LMLGKPGD@?$FLINFO?$FN?3?5?5?5Setting?5Java?5event?5ma@ 0000000180020b58     WinAccessBridge.obj
 0002:00000b88       ??_C@_0DC@IJKHOBEO@?$FLINFO?$FN?3?5?5?5Setting?5Accessibility@ 0000000180020b88     WinAccessBridge.obj
 0002:00000bc0       ??_C@_0DN@ECLBFGAO@?$FLERROR?$FN?3?5Failed?5to?5initiate?5IPC@ 0000000180020bc0     WinAccessBridge.obj
 0002:00000c00       ??_C@_0DG@OEMNKFJP@?$FLINFO?$FN?3?5?5?5Success?$CB?$CB?5?5We?5rendezv@ 0000000180020c00     WinAccessBridge.obj
 0002:00000c38       ??_C@_0DK@BLMJEFJH@?$FLERROR?$FN?3?5sending?5memory?5package@ 0000000180020c38     WinAccessBridge.obj
 0002:00000c78       ??_C@_0DC@BABNPCOM@?$FLINFO?$FN?3?5?5in?5WinAccessBridge?3?3qu@ 0000000180020c78     WinAccessBridge.obj
 0002:00000cb0       ??_C@_0DE@NOAFOCML@?$FLINFO?$FN?3?5in?5WinAccessBridge?3?3rec@ 0000000180020cb0     WinAccessBridge.obj
 0002:00000ce8       ??_C@_0BM@KNOOFOHJ@?$FLINFO?$FN?3?5?5dequeueing?5message@ 0000000180020ce8     WinAccessBridge.obj
 0002:00000d08       ??_C@_0CD@GBHFIMOB@?$FLERROR?$FN?3?5Queue?5seems?5to?5be?5brok@ 0000000180020d08     WinAccessBridge.obj
 0002:00000d30       ??_C@_0CA@LFELFFDM@?$FLINFO?$FN?3?5?5found?5one?$DL?5sending?5it?$CB@ 0000000180020d30     WinAccessBridge.obj
 0002:00000d50       ??_C@_0BP@ENBFDBDP@?$FLWARN?$FN?3?5?5?5ODD?4?4?4?5element?5?$DN?$DN?50?$CB@ 0000000180020d50     WinAccessBridge.obj
 0002:00000d70       ??_C@_0CP@OIAJKCPF@?$FLWARN?$FN?3?5?5Queue?5in?5use?0?5will?5try@ 0000000180020d70     WinAccessBridge.obj
 0002:00000da0       ??_C@_0DH@KAJCMPPF@?$FLWARN?$FN?3?5?5unable?5to?5dequeue?5mess@ 0000000180020da0     WinAccessBridge.obj
 0002:00000dd8       ??_C@_0CO@KCIANNAF@?$FLINFO?$FN?3?5PreProcessing?5package?5s@ 0000000180020dd8     WinAccessBridge.obj
 0002:00000e10       ??_C@_0EF@DFMGOCJF@?$FLERROR?$FN?3?5?5?5processing?5FAILED?$CB?$CB?5@ 0000000180020e10     WinAccessBridge.obj
 0002:00000e58       ??_C@_0CL@HBCKEPEE@?$FLINFO?$FN?3?5?5?5?5package?5preprocessin@ 0000000180020e58     WinAccessBridge.obj
 0002:00000e88       ??_C@_0DM@CCADHAH@?$FLINFO?$FN?3?5WinAccessBridge?3?3Proces@ 0000000180020e88     WinAccessBridge.obj
 0002:00000ec8       ??_C@_0CI@KAACKIJC@?$FLINFO?$FN?3?5?5?5?5type?5?$DN?$DN?5cJavaShutdow@ 0000000180020ec8     WinAccessBridge.obj
 0002:00000ef0       ??_C@_0CE@KGDIDFJM@?$FLINFO?$FN?3?5?5?5?5event?5callback?5compl@ 0000000180020ef0     WinAccessBridge.obj
 0002:00000f18       ??_C@_0BI@MGOIGNJM@?$FLINFO?$FN?3?5?5?5?5event?5fired?$CB@ 0000000180020f18     WinAccessBridge.obj
 0002:00000f30       ??_C@_0EC@JELBKKLB@?$FLERROR?$FN?3?5?5?5?5processing?5FAILED?$CB?$CB@ 0000000180020f30     WinAccessBridge.obj
 0002:00000f78       ??_C@_0CM@OIHFPHBP@?$FLINFO?$FN?3?5?5?5?5begin?5callback?5to?5AT@ 0000000180020f78     WinAccessBridge.obj
 0002:00000fb0       ??_C@_0EB@PCOLNIOI@?$FLERROR?$FN?3?5?5?5processing?5FAILED?$CB?$CB?5@ 0000000180020fb0     WinAccessBridge.obj
 0002:00001000       ??_C@_0EG@DADDGPDA@?$FLERROR?$FN?3?5?5?5?5processing?5FAILED?$CB?$CB@ 0000000180021000     WinAccessBridge.obj
 0002:00001048       ??_C@_0CI@PMGDCMNI@?$FLINFO?$FN?3?5?5?5?5package?5processing?5c@ 0000000180021048     WinAccessBridge.obj
 0002:00001070       ??_C@_0DD@EDMANGOO@?$FLINFO?$FN?3?5?$CK?$CK?$CK?$CK?$CK?5WinAccessBridge?3?3@ 0000000180021070     WinAccessBridge.obj
 0002:000010a8       ??_C@_0CP@IIHJFGGB@?$FLINFO?$FN?3?5?5?5data?5structures?5succe@ 00000001800210a8     WinAccessBridge.obj
 0002:000010d8       ??_C@_0DB@JABMCGEJ@?$FLERROR?$FN?3?5couldn?8t?5find?5matching@ 00000001800210d8     WinAccessBridge.obj
 0002:00001110       ??_C@_0DJ@EFGAHBMH@?$FLINFO?$FN?3?5WinAccessBridge?3?3releas@ 0000000180021110     WinAccessBridge.obj
 0002:00001150       ??_C@_0CO@GDCOMIDN@?$FLINFO?$FN?3?5WinAccessBridge?3?3getVer@ 0000000180021150     WinAccessBridge.obj
 0002:00001180       ??_C@_0IH@JNMBAFNI@?$FLINFO?$FN?3?5?5?5VMversion?3?5?$CFls?6?5?5?5?5?5?5@ 0000000180021180     WinAccessBridge.obj
 0002:00001208       ??_C@_0CJ@MFBANPLF@?$FLINFO?$FN?3?5In?5WinAccessBridge?3?3isJ@ 0000000180021208     WinAccessBridge.obj
 0002:00001238       ??_C@_0CK@OIADIKJK@?$FLINFO?$FN?3?5WinAccessBridge?3?3isJava@ 0000000180021238     WinAccessBridge.obj
 0002:00001268       ??_C@_0DJ@GDIICFAI@?$FLINFO?$FN?3?5WinAccessBridge?3?3isSame@ 0000000180021268     WinAccessBridge.obj
 0002:000012b0       ??_C@_0EF@JHJAECO@?$FLINFO?$FN?3?5?5?5WinAccessBridge?3?3isSa@ 00000001800212b0     WinAccessBridge.obj
 0002:00001300       ??_C@_0EL@EGCPHNBB@?$FLINFO?$FN?3?5?5?5WinAccessBridge?3?3isSa@ 0000000180021300     WinAccessBridge.obj
 0002:00001350       ??_C@_0FE@JNIGOBOL@?$FLERROR?$FN?3?5?5?5WinAccessBridge?3?3isS@ 0000000180021350     WinAccessBridge.obj
 0002:000013a8       ??_C@_0DM@KHCMPGEG@?$FLINFO?$FN?3?5WinAccessBridge?3?3getAcc@ 00000001800213a8     WinAccessBridge.obj
 0002:000013e8       ??_C@_0DA@KDJKNLAN@?$FLINFO?$FN?3?5?5?5?5?5current?9?$DOvmID?5?$DN?5?$CFX?0@ 00000001800213e8     WinAccessBridge.obj
 0002:00001418       ??_C@_0CP@IJNFIHAG@?$FLINFO?$FN?3?5?5?5?5?5pkg?9?$DOrAccessibleCon@ 0000000180021418     WinAccessBridge.obj
 0002:00001448       ??_C@_0DJ@FFBPMFOM@?$FLERROR?$FN?3?5getAccessibleContextFr@ 0000000180021448     WinAccessBridge.obj
 0002:00001488       ??_C@_0DO@IIGOCPCC@?$FLERROR?$FN?3?5getAccessibleContextFr@ 0000000180021488     WinAccessBridge.obj
 0002:000014c8       ??_C@_0DL@KEEIEGBJ@?$FLINFO?$FN?3?5?5?5in?5WinAccessBridge?3?3g@ 00000001800214c8     WinAccessBridge.obj
 0002:00001510       ??_C@_0EA@HDGDGEMM@?$FLINFO?$FN?3?5WinAccessBridge?3?3getHWN@ 0000000180021510     WinAccessBridge.obj
 0002:00001550       ??_C@_0EA@FHJPOEHJ@?$FLINFO?$FN?3?5WinAccessBridge?3?3getAcc@ 0000000180021550     WinAccessBridge.obj
 0002:00001590       ??_C@_0EB@HKEAOAKG@?$FLINFO?$FN?3?5WinAccessBridge?3?3getAcc@ 0000000180021590     WinAccessBridge.obj
 0002:000015e0       ??_C@_0EC@OFBFCAEJ@?$FLINFO?$FN?3?5WinAccessBridge?3?3getAcc@ 00000001800215e0     WinAccessBridge.obj
 0002:00001630       ??_C@_0JA@MODCAACP@?$FLINFO?$FN?3?5?5?5name?3?5?$CFls?6?5?5?5?5?5?5?5?5?5?5d@ 0000000180021630     WinAccessBridge.obj
 0002:000016c0       ??_C@_0EJ@HLHMECO@?$FLINFO?$FN?3?5WinAccessBridge?3?3getAcc@ 00000001800216c0     WinAccessBridge.obj
 0002:00001710       ??_C@_0EA@MDGJLODH@?$FLINFO?$FN?3?5WinAccessBridge?3?3getAcc@ 0000000180021710     WinAccessBridge.obj
 0002:00001750       ??_C@_0EI@IEEMIFOJ@?$FLINFO?$FN?3?5?$CD?$CD?$CD?$CD?$CD?5WinAccessBridge?3?3@ 0000000180021750     WinAccessBridge.obj
 0002:000017a0       ??_C@_0EC@FNKONEFN@?$FLINFO?$FN?3?5?5?5?$CD?$CD?$CD?$CD?$CD?5WinAccessBridge@ 00000001800217a0     WinAccessBridge.obj
 0002:000017f0       ??_C@_0EA@GPGOILHN@?$FLERROR?$FN?3?5?5?5?$CD?$CD?$CD?$CD?$CD?5WinAccessBridg@ 00000001800217f0     WinAccessBridge.obj
 0002:00001830       ??_C@_0EO@GIFIOBJO@?$FLINFO?$FN?3?5?$CD?$CD?$CD?$CD?$CD?5WinAccessBridge?3?3@ 0000000180021830     WinAccessBridge.obj
 0002:00001880       ??_C@_0DK@FPHEFKPF@?$FLINFO?$FN?3?5?5?5XXXX?5pkg?9?$DOrTableCellI@ 0000000180021880     WinAccessBridge.obj
 0002:000018c0       ??_C@_0EG@CFNEHAJF@?$FLINFO?$FN?3?5?5?5?$CD?$CD?$CD?$CD?$CD?5WinAccessBridge@ 00000001800218c0     WinAccessBridge.obj
 0002:00001910       ??_C@_0EE@DMEKGPAL@?$FLERROR?$FN?3?5?5?5?$CD?$CD?$CD?$CD?$CD?5WinAccessBridg@ 0000000180021910     WinAccessBridge.obj
 0002:00001960       ??_C@_0EJ@GHNOCBA@?$FLINFO?$FN?3?5?$CD?$CD?$CD?$CD?$CD?5WinAccessBridge?3?3@ 0000000180021960     WinAccessBridge.obj
 0002:000019b0       ??_C@_0EH@MMAIEADN@?$FLINFO?$FN?3?5?5?5?$CD?$CD?$CD?$CD?$CD?5WinAccessBridge@ 00000001800219b0     WinAccessBridge.obj
 0002:00001a00       ??_C@_0EF@IGPDOLOH@?$FLERROR?$FN?3?5?5?5?$CD?$CD?$CD?$CD?$CD?5WinAccessBridg@ 0000000180021a00     WinAccessBridge.obj
 0002:00001a50       ??_C@_0EM@KLDOANDG@?$FLINFO?$FN?3?5?$CD?$CD?$CD?$CD?$CD?5WinAccessBridge?3?3@ 0000000180021a50     WinAccessBridge.obj
 0002:00001aa0       ??_C@_0EK@DJMDCCLK@?$FLINFO?$FN?3?5?5?5?$CD?$CD?$CD?$CD?$CD?5WinAccessBridge@ 0000000180021aa0     WinAccessBridge.obj
 0002:00001af0       ??_C@_0EI@CELDDCKP@?$FLERROR?$FN?3?5?5?5?$CD?$CD?$CD?$CD?$CD?5WinAccessBridg@ 0000000180021af0     WinAccessBridge.obj
 0002:00001b40       ??_C@_0FC@BPONCABC@?$FLINFO?$FN?3?5?$CD?$CD?$CD?$CD?$CD?5WinAccessBridge?3?3@ 0000000180021b40     WinAccessBridge.obj
 0002:00001ba0       ??_C@_0EM@JPIPIDPC@?$FLINFO?$FN?3?5?5?5?$CD?$CD?$CD?$CD?$CD?5WinAccessBridge@ 0000000180021ba0     WinAccessBridge.obj
 0002:00001bf0       ??_C@_0EK@IGPCFPOI@?$FLERROR?$FN?3?5?5?5?$CD?$CD?$CD?$CD?$CD?5WinAccessBridg@ 0000000180021bf0     WinAccessBridge.obj
 0002:00001c40       ??_C@_0FF@GEJHIBCC@?$FLINFO?$FN?3?5?$CD?$CD?$CD?$CD?$CD?5WinAccessBridge?3?3@ 0000000180021c40     WinAccessBridge.obj
 0002:00001ca0       ??_C@_0EP@PJFHLMKB@?$FLINFO?$FN?3?5?5?5?$CD?$CD?$CD?$CD?$CD?5WinAccessBridge@ 0000000180021ca0     WinAccessBridge.obj
 0002:00001cf0       ??_C@_0EN@FJIGOJNI@?$FLERROR?$FN?3?5?5?5?$CD?$CD?$CD?$CD?$CD?5WinAccessBridg@ 0000000180021cf0     WinAccessBridge.obj
 0002:00001d40       ??_C@_0FB@IPIFJJKK@?$FLINFO?$FN?3?5?$CD?$CD?$CD?$CD?$CD?5WinAccessBridge?3?3@ 0000000180021d40     WinAccessBridge.obj
 0002:00001da0       ??_C@_0EP@DHAGNOBO@?$FLINFO?$FN?3?5?5?5?$CD?$CD?$CD?$CD?$CD?5WinAccessBridge@ 0000000180021da0     WinAccessBridge.obj
 0002:00001df0       ??_C@_0EN@IFAFODLF@?$FLERROR?$FN?3?5?5?5?$CD?$CD?$CD?$CD?$CD?5WinAccessBridg@ 0000000180021df0     WinAccessBridge.obj
 0002:00001e40       ??_C@_0EK@FCAMCNJB@?$FLINFO?$FN?3?5?$CD?$CD?$CD?$CD?$CD?5WinAccessBridge?3?3@ 0000000180021e40     WinAccessBridge.obj
 0002:00001e90       ??_C@_0EI@LCHMKLCB@?$FLINFO?$FN?3?5?5?5?$CD?$CD?$CD?$CD?$CD?5WinAccessBridge@ 0000000180021e90     WinAccessBridge.obj
 0002:00001ee0       ??_C@_0EG@PCFFNJPM@?$FLERROR?$FN?3?5?5?5?$CD?$CD?$CD?$CD?$CD?5WinAccessBridg@ 0000000180021ee0     WinAccessBridge.obj
 0002:00001f30       ??_C@_0EN@MHFLCDEG@?$FLINFO?$FN?3?5?$CD?$CD?$CD?$CD?$CD?5WinAccessBridge?3?3@ 0000000180021f30     WinAccessBridge.obj
 0002:00001f80       ??_C@_0EL@HPJEOBAF@?$FLINFO?$FN?3?5?5?5?$CD?$CD?$CD?$CD?$CD?5WinAccessBridge@ 0000000180021f80     WinAccessBridge.obj
 0002:00001fd0       ??_C@_0EJ@EFJNHGOC@?$FLERROR?$FN?3?5?5?5?$CD?$CD?$CD?$CD?$CD?5WinAccessBridg@ 0000000180021fd0     WinAccessBridge.obj
 0002:00002020       ??_C@_0FE@EEAPAHGA@?$FLINFO?$FN?3?5?$CD?$CD?$CD?$CD?$CD?5WinAccessBridge?3?3@ 0000000180022020     WinAccessBridge.obj
 0002:00002080       ??_C@_0FC@IJCKDOEL@?$FLINFO?$FN?3?5?5?5?$CD?$CD?$CD?$CD?$CD?5WinAccessBridge@ 0000000180022080     WinAccessBridge.obj
 0002:000020e0       ??_C@_0FA@EEJJLKOB@?$FLERROR?$FN?3?5?5?5?$CD?$CD?$CD?$CD?$CD?5WinAccessBridg@ 00000001800220e0     WinAccessBridge.obj
 0002:00002130       ??_C@_0EN@IKMAMDCJ@?$FLINFO?$FN?3?5?$CD?$CD?$CD?$CD?$CD?5WinAccessBridge?3?3@ 0000000180022130     WinAccessBridge.obj
 0002:00002180       ??_C@_0EL@MCFEFCEP@?$FLINFO?$FN?3?5?5?5?$CD?$CD?$CD?$CD?$CD?5WinAccessBridge@ 0000000180022180     WinAccessBridge.obj
 0002:000021d0       ??_C@_0EJ@OEGCIAEN@?$FLERROR?$FN?3?5?5?5?$CD?$CD?$CD?$CD?$CD?5WinAccessBridg@ 00000001800221d0     WinAccessBridge.obj
 0002:00002220       ??_C@_0FB@FBDIFIGA@?$FLERROR?$FN?3?5?$CD?$CD?$CD?$CD?$CD?5WinAccessBridge?3@ 0000000180022220     WinAccessBridge.obj
 0002:00002280       ??_C@_0EO@KBJAHINP@?$FLINFO?$FN?3?5?5?5?$CD?$CD?$CD?$CD?$CD?5WinAccessBridge@ 0000000180022280     WinAccessBridge.obj
 0002:000022d0       ??_C@_0EM@FBMEIFEO@?$FLERROR?$FN?3?5?5?5?$CD?$CD?$CD?$CD?$CD?5WinAccessBridg@ 00000001800222d0     WinAccessBridge.obj
 0002:00002320       ??_C@_0EN@EJPIGDNI@?$FLINFO?$FN?3?5?$CD?$CD?$CD?$CD?$CD?5WinAccessBridge?3?3@ 0000000180022320     WinAccessBridge.obj
 0002:00002370       ??_C@_0EB@EHNAMLGG@?$FLINFO?$FN?3?5?5?5?$CD?$CD?$CD?$CD?$CD?5WinAccessBridge@ 0000000180022370     WinAccessBridge.obj
 0002:000023b8       ??_C@_0DP@JGIKFGJD@?$FLERROR?$FN?3?5?5?5?$CD?$CD?$CD?$CD?$CD?5WinAccessBridg@ 00000001800223b8     WinAccessBridge.obj
 0002:00002400       ??_C@_0FA@BNCMMHDE@?$FLINFO?$FN?3?5?$CD?$CD?$CD?$CD?$CD?5WinAccessBridge?3?3@ 0000000180022400     WinAccessBridge.obj
 0002:00002450       ??_C@_0EE@HJIACDJB@?$FLINFO?$FN?3?5?5?5?$CD?$CD?$CD?$CD?$CD?5WinAccessBridge@ 0000000180022450     WinAccessBridge.obj
 0002:000024a0       ??_C@_0EC@HJIAKIIH@?$FLERROR?$FN?3?5?5?5?$CD?$CD?$CD?$CD?$CD?5WinAccessBridg@ 00000001800224a0     WinAccessBridge.obj
 0002:000024f0       ??_C@_0FF@NCBHFIIB@?$FLINFO?$FN?3?5?$CD?$CD?$CD?$CD?$CD?5WinAccessBridge?3?3@ 00000001800224f0     WinAccessBridge.obj
 0002:00002550       ??_C@_0ED@CBAGECAG@?$FLINFO?$FN?3?5?5?5?$CD?$CD?$CD?$CD?$CD?5WinAccessBridge@ 0000000180022550     WinAccessBridge.obj
 0002:000025a0       ??_C@_0EB@NLKCNKIL@?$FLERROR?$FN?3?5?5?5?$CD?$CD?$CD?$CD?$CD?5WinAccessBridg@ 00000001800225a0     WinAccessBridge.obj
 0002:000025f0       ??_C@_0EK@KPCBMLHL@?$FLINFO?$FN?3?5?$CD?$CD?$CD?$CD?$CD?5WinAccessBridge?3?3@ 00000001800225f0     WinAccessBridge.obj
 0002:00002640       ??_C@_0ED@KBOKJBJ@?$FLINFO?$FN?3?5?5?5?$CD?$CD?$CD?$CD?$CD?5pkg?9?$DOrAccessibl@ 0000000180022640     WinAccessBridge.obj
 0002:00002690       ??_C@_0EE@MLCJPFKH@?$FLINFO?$FN?3?5?5?5?$CD?$CD?$CD?$CD?$CD?5WinAccessBridge@ 0000000180022690     WinAccessBridge.obj
 0002:000026e0       ??_C@_0EC@ONHLHLKJ@?$FLERROR?$FN?3?5?5?5?$CD?$CD?$CD?$CD?$CD?5WinAccessBridg@ 00000001800226e0     WinAccessBridge.obj
 0002:00002730       ??_C@_0EI@BEINFODC@?$FLINFO?$FN?3?5?$CD?$CD?$CD?$CD?$CD?5WinAccessBridge?3?3@ 0000000180022730     WinAccessBridge.obj
 0002:00002778       ??_C@_0CN@CIJKLIHC@?$FLINFO?$FN?3?5?5?5?$CD?$CD?$CD?$CD?$CD?5hypertextInfo?4l@ 0000000180022778     WinAccessBridge.obj
 0002:000027b0       ??_C@_0EC@GJFIBKBJ@?$FLINFO?$FN?3?5?5?5?$CD?$CD?$CD?$CD?$CD?5WinAccessBridge@ 00000001800227b0     WinAccessBridge.obj
 0002:00002800       ??_C@_0EA@ENIAHHMF@?$FLERROR?$FN?3?5?5?5?$CD?$CD?$CD?$CD?$CD?5WinAccessBridg@ 0000000180022800     WinAccessBridge.obj
 0002:00002840       ??_C@_0EI@MFFNFMHA@?$FLINFO?$FN?3?5WinAccessBridge?3?3activa@ 0000000180022840     WinAccessBridge.obj
 0002:00002890       ??_C@_0GC@OOPIFCLD@?$FLERROR?$FN?3?5?5WinAccessBridge?3?3acti@ 0000000180022890     WinAccessBridge.obj
 0002:00002900       ??_C@_0EJ@KNECEC@?$FLINFO?$FN?3?5?$CD?$CD?$CD?$CD?$CD?5WinAccessBridge?3?3@ 0000000180022900     WinAccessBridge.obj
 0002:00002950       ??_C@_0CJ@CHHBPBDA@?$FLINFO?$FN?3?5?5?5?$CD?$CD?$CD?$CD?$CD?5hypetext?5link?5c@ 0000000180022950     WinAccessBridge.obj
 0002:00002980       ??_C@_0EG@OFFPNIFM@?$FLINFO?$FN?3?5?5?$CD?$CD?$CD?$CD?$CD?5WinAccessBridge?3@ 0000000180022980     WinAccessBridge.obj
 0002:000029d0       ??_C@_0EF@CJEMCIKC@?$FLERROR?$FN?3?5?5?5?$CD?$CD?$CD?$CD?$CD?5WinAccessBridg@ 00000001800229d0     WinAccessBridge.obj
 0002:00002a20       ??_C@_0EK@KALHBKDC@?$FLINFO?$FN?3?5?$CD?$CD?$CD?$CD?$CD?5WinAccessBridge?3?3@ 0000000180022a20     WinAccessBridge.obj
 0002:00002a70       ??_C@_0CD@FAKLHPNN@?$FLINFO?$FN?3?5?5?5?$CD?$CD?$CD?$CD?$CD?5pkg?9?$DOrSuccess?5?$DN@ 0000000180022a70     WinAccessBridge.obj
 0002:00002aa0       ??_C@_0ED@CLMPFLBE@?$FLERROR?$FN?3?5?5?5?$CD?$CD?$CD?$CD?$CD?5WinAccessBridg@ 0000000180022aa0     WinAccessBridge.obj
 0002:00002af0       ??_C@_0EC@DJBOOIDG@?$FLERROR?$FN?3?5?5?$CD?$CD?$CD?$CD?$CD?5WinAccessBridge@ 0000000180022af0     WinAccessBridge.obj
 0002:00002b40       ??_C@_0EN@IMDNGAME@?$FLINFO?$FN?3?5?$CD?$CD?$CD?$CD?$CD?5WinAccessBridge?3?3@ 0000000180022b40     WinAccessBridge.obj
 0002:00002b90       ??_C@_0CJ@LGNOCJK@?$FLINFO?$FN?3?5?5?5?$CD?$CD?$CD?$CD?$CD?5hypetext?5link?5i@ 0000000180022b90     WinAccessBridge.obj
 0002:00002bc0       ??_C@_0EM@KCINDCOI@?$FLINFO?$FN?3?5?5?5?$CD?$CD?$CD?$CD?$CD?5WinAccessBridge@ 0000000180022bc0     WinAccessBridge.obj
 0002:00002c10       ??_C@_0EI@IEJDJKBK@?$FLERROR?$FN?5?5?$CD?$CD?$CD?$CD?$CD?5WinAccessBridge?3@ 0000000180022c10     WinAccessBridge.obj
 0002:00002c60       ??_C@_0EI@OHHKPFCO@?$FLINFO?$FN?3?5?$CD?$CD?$CD?$CD?$CD?5WinAccessBridge?3?3@ 0000000180022c60     WinAccessBridge.obj
 0002:00002cb0       ??_C@_0EK@CIOPKHEJ@?$FLINFO?$FN?3?5?$CD?$CD?$CD?$CD?$CD?5WinAccessBridge?3?3@ 0000000180022cb0     WinAccessBridge.obj
 0002:00002d00       ??_C@_0DC@GOKFJHHA@?$FLINFO?$FN?3?5?5?5?$CD?$CD?$CD?$CD?$CD?5keyBindings?4key@ 0000000180022d00     WinAccessBridge.obj
 0002:00002d40       ??_C@_0KM@PICKCJIM@?$FLINFO?$FN?3?5?5?5Key?5Binding?5?$CD?5?$CFd?5?5?5?5?5@ 0000000180022d40     WinAccessBridge.obj
 0002:00002df0       ??_C@_0EE@LGIDNFJF@?$FLINFO?$FN?3?5?5?5?$CD?$CD?$CD?$CD?$CD?5WinAccessBridge@ 0000000180022df0     WinAccessBridge.obj
 0002:00002e40       ??_C@_0EB@PIGLELIJ@?$FLINFO?$FN?3?5?5?5?$CD?$CD?$CD?$CD?$CD?5WinAccessBridge@ 0000000180022e40     WinAccessBridge.obj
 0002:00002e90       ??_C@_0EE@KBJHDGDB@?$FLINFO?$FN?3?5?$CD?$CD?$CD?$CD?$CD?5WinAccessBridge?3?3@ 0000000180022e90     WinAccessBridge.obj
 0002:00002ed8       ??_C@_0CG@JNBKIMJN@?$FLINFO?$FN?3?5?5?5?$CD?$CD?$CD?$CD?$CD?5icons?4iconsCoun@ 0000000180022ed8     WinAccessBridge.obj
 0002:00002f00       ??_C@_0DO@JGGAAEEG@?$FLINFO?$FN?3?5?5?5?$CD?$CD?$CD?$CD?$CD?5WinAccessBridge@ 0000000180022f00     WinAccessBridge.obj
 0002:00002f40       ??_C@_0DM@PHFGBDGG@?$FLERROR?$FN?3?5?5?5?$CD?$CD?$CD?$CD?$CD?5WinAccessBridg@ 0000000180022f40     WinAccessBridge.obj
 0002:00002f80       ??_C@_0EG@EKEEJFO@?$FLINFO?$FN?3?5?$CD?$CD?$CD?$CD?$CD?5WinAccessBridge?3?3@ 0000000180022f80     WinAccessBridge.obj
 0002:00002fc8       ??_C@_0CK@COBILBN@?$FLINFO?$FN?3?5?5?5?$CD?$CD?$CD?$CD?$CD?5actions?4actions@ 0000000180022fc8     WinAccessBridge.obj
 0002:00003000       ??_C@_0EA@EKDNLNJA@?$FLINFO?$FN?3?5?5?5?$CD?$CD?$CD?$CD?$CD?5WinAccessBridge@ 0000000180023000     WinAccessBridge.obj
 0002:00003040       ??_C@_0DO@HNCGODDL@?$FLERROR?$FN?3?5?5?5?$CD?$CD?$CD?$CD?$CD?5WinAccessBridg@ 0000000180023040     WinAccessBridge.obj
 0002:00003080       ??_C@_0EH@IJHNMJPE@?$FLINFO?$FN?3?5WinAccessBridge?3?3doAcce@ 0000000180023080     WinAccessBridge.obj
 0002:000030d0       ??_C@_0FL@LJNDNJAB@?$FLERROR?$FN?3?5?5?5WinAccessBridge?3?3doA@ 00000001800230d0     WinAccessBridge.obj
 0002:00003130       ??_C@_0DF@LBCGPHPD@?$FLINFO?$FN?3?5WinAccessBridge?3?3setTex@ 0000000180023130     WinAccessBridge.obj
 0002:00003168       ??_C@_0DJ@BDMKEGCI@?$FLINFO?$FN?3?5WinAccessBridge?3?3getPar@ 0000000180023168     WinAccessBridge.obj
 0002:000031b0       ??_C@_0FE@FILBCBC@?$FLINFO?$FN?3?5?5?5pkg?9?$DOvmID?3?5?$CFX?5?5?5?5?5?5?5?5@ 00000001800231b0     WinAccessBridge.obj
 0002:00003208       ??_C@_0CG@EPJKPFNH@?$FLINFO?$FN?3?5?5?5pkg?9?$DOrAccessibleConte@ 0000000180023208     WinAccessBridge.obj
 0002:00003230       ??_C@_0DJ@LMOBJNAA@?$FLINFO?$FN?3?5WinAccessBridge?3?3getTop@ 0000000180023230     WinAccessBridge.obj
 0002:00003270       ??_C@_0EB@EGNBJNPN@?$FLINFO?$FN?3?5WinAccessBridge?3?3getPar@ 0000000180023270     WinAccessBridge.obj
 0002:000032b8       ??_C@_0DG@HMAMEAHE@?$FLINFO?$FN?3?5WinAccessBridge?3?3getObj@ 00000001800232b8     WinAccessBridge.obj
 0002:000032f0       ??_C@_0DL@DIELJEEF@?$FLINFO?$FN?3?5WinAccessBridge?3?3getAct@ 00000001800232f0     WinAccessBridge.obj
 0002:00003330       ??_C@_0EA@KKNJCPIF@?$FLINFO?$FN?3?5WinAccessBridge?3?3getVir@ 0000000180023330     WinAccessBridge.obj
 0002:00003370       ??_C@_0EK@LJJEDFEG@?$FLINFO?$FN?3?5?5?5?5?5WinAccessBridge?3?3ge@ 0000000180023370     WinAccessBridge.obj
 0002:000033c0       ??_C@_0DE@NGCOAPLI@?$FLINFO?$FN?3?5WinAccessBridge?3?3reques@ 00000001800233c0     WinAccessBridge.obj
 0002:00003400       ??_C@_0EB@LDKGCIL@?$FLINFO?$FN?3?5?5?5?5?5WinAccessBridge?3?3se@ 0000000180023400     WinAccessBridge.obj
 0002:00003450       ??_C@_0EK@FKPJFOFL@?$FLINFO?$FN?3?5?5?5?5?5WinAccessBridge?3?3ge@ 0000000180023450     WinAccessBridge.obj
 0002:000034a0       ??_C@_0DP@PHLAPJAH@?$FLINFO?$FN?3?5WinAccessBridge?3?3getVis@ 00000001800234a0     WinAccessBridge.obj
 0002:000034e0       ??_C@_0DK@FFJLHNNJ@?$FLINFO?$FN?3?5WinAccessBridge?3?3getVis@ 00000001800234e0     WinAccessBridge.obj
 0002:00003520       ??_C@_0DM@MCJMMMCP@?$FLINFO?$FN?3?5WinAccessBridge?3?3setCar@ 0000000180023520     WinAccessBridge.obj
 0002:00003560       ??_C@_0EJ@FBPIKPOJ@?$FLINFO?$FN?3?5WinAccessBridge?3?3getAcc@ 0000000180023560     WinAccessBridge.obj
 0002:000035b0       ??_C@_0EK@DNDDFNHD@?$FLINFO?$FN?3?5?5?5charCount?3?5?$CFd?5?5?5?5?5?5?5?5@ 00000001800235b0     WinAccessBridge.obj
 0002:00003600       ??_C@_0EG@BGFOEIHE@?$FLINFO?$FN?3?5WinAccessBridge?3?3getAcc@ 0000000180023600     WinAccessBridge.obj
 0002:00003650       ??_C@_0EK@KLCBPNFL@?$FLINFO?$FN?3?5WinAccessBridge?3?3getAcc@ 0000000180023650     WinAccessBridge.obj
 0002:000036a0       ??_C@_0EL@MJHEEFIF@?$FLINFO?$FN?3?5WinAccessBridge?3?3getAcc@ 00000001800236a0     WinAccessBridge.obj
 0002:000036f0       ??_C@_0EF@MMEINAI@?$FLINFO?$FN?3?5WinAccessBridge?3?3getAcc@ 00000001800236f0     WinAccessBridge.obj
 0002:00003740       ??_C@_0EA@GJMJEHDC@?$FLINFO?$FN?3?5WinAccessBridge?3?3getCar@ 0000000180023740     WinAccessBridge.obj
 0002:00003780       ??_C@_0EJ@BCHIKCEF@?$FLINFO?$FN?3?5WinAccessBridge?3?3getAcc@ 0000000180023780     WinAccessBridge.obj
 0002:000037d0       ??_C@_0EI@LCFAOBKP@?$FLINFO?$FN?3?5WinAccessBridge?3?3getAcc@ 00000001800237d0     WinAccessBridge.obj
 0002:00003818       ??_C@_0DM@NFGOCJPM@?$FLINFO?$FN?3?5WinAccessBridge?3?3addJav@ 0000000180023818     WinAccessBridge.obj
 0002:00003858       ??_C@_0DP@PIGNLFHB@?$FLINFO?$FN?3?5?5?5?9?$DOpkgType?5?$DN?5?$CFX?0?5event@ 0000000180023858     WinAccessBridge.obj
 0002:000038a0       ??_C@_0EC@OKCIJGM@?$FLINFO?$FN?3?5in?5WinAccessBridge?3?3rem@ 00000001800238a0     WinAccessBridge.obj
 0002:000038f0       ??_C@_0EI@HMKIAPB@?$FLINFO?$FN?3?5in?5WinAccessBridge?3?3add@ 00000001800238f0     WinAccessBridge.obj
 0002:00003938       ??_C@_0DP@KFDABLNL@?$FLINFO?$FN?3?5?5?5?9?$DOpkgType?5?$DN?5?$CFX?0?5event@ 0000000180023938     WinAccessBridge.obj
 0002:00003980       ??_C@_0EL@BFCCGHFN@?$FLINFO?$FN?3?5in?5WinAccessBridge?3?3rem@ 0000000180023980     WinAccessBridge.obj
 0002:000039d8       ??_7type_info@@6B@         00000001800239d8     LIBCMT:std_type_info_static.obj
 0002:000039e0       _pDefaultRawDllMain        00000001800239e0     LIBCMT:dll_dllmain.obj
 0002:000039e0       _pRawDllMain               00000001800239e0     LIBCMT:dll_dllmain.obj
 0002:00003a00       ??_7bad_array_new_length@std@@6B@ 0000000180023a00     LIBCMT:throw_bad_alloc.obj
 0002:00003a10       ??_C@_0BF@KINCDENJ@bad?5array?5new?5length@ 0000000180023a10     LIBCMT:throw_bad_alloc.obj
 0002:00003a30       __xmm@ffffffffffffffffffffffffffffffff 0000000180023a30     LIBCMT:utility.obj
 0002:00003a40       _pDestructExceptionObject  0000000180023a40     libvcruntime:ehhelpers.obj
 0002:00004160       ??_C@_08EHJDFFNH@__based?$CI@ 0000000180024160     libvcruntime:undname.obj
 0002:00004170       ??_C@_07KOLFKCDI@__cdecl@  0000000180024170     libvcruntime:undname.obj
 0002:00004178       ??_C@_08GHMPAG@__pascal@   0000000180024178     libvcruntime:undname.obj
 0002:00004188       ??_C@_09IFJBGAPI@__stdcall@ 0000000180024188     libvcruntime:undname.obj
 0002:00004198       ??_C@_0L@NPHFGOKO@__thiscall@ 0000000180024198     libvcruntime:undname.obj
 0002:000041a8       ??_C@_0L@JMKHOMEK@__fastcall@ 00000001800241a8     libvcruntime:undname.obj
 0002:000041b8       ??_C@_0N@BCKKPABJ@__vectorcall@ 00000001800241b8     libvcruntime:undname.obj
 0002:000041c8       ??_C@_09HIJEGCPM@__clrcall@ 00000001800241c8     libvcruntime:undname.obj
 0002:000041d4       ??_C@_06GHPCKEAG@__eabi@   00000001800241d4     libvcruntime:undname.obj
 0002:000041e0       ??_C@_09IOPIDJLG@__swift_1@ 00000001800241e0     libvcruntime:undname.obj
 0002:000041f0       ??_C@_09KFNFGKHF@__swift_2@ 00000001800241f0     libvcruntime:undname.obj
 0002:00004200       ??_C@_09LMMOFLDE@__swift_3@ 0000000180024200     libvcruntime:undname.obj
 0002:00004210       ??_C@_07JOMMBBKO@__ptr64@  0000000180024210     libvcruntime:undname.obj
 0002:00004218       ??_C@_0L@PILCLIHE@__restrict@ 0000000180024218     libvcruntime:undname.obj
 0002:00004228       ??_C@_0M@GFIIJFMG@__unaligned@ 0000000180024228     libvcruntime:undname.obj
 0002:00004238       ??_C@_09DHDLOLLB@restrict?$CI@ 0000000180024238     libvcruntime:undname.obj
 0002:00004242       ??_C@_00CNPNBAHC@@         0000000180024242     libvcruntime:undname.obj
 0002:00004244       ??_C@_04NIHEBCM@?5new@     0000000180024244     libvcruntime:undname.obj
 0002:00004250       ??_C@_07FPCDHGMM@?5delete@ 0000000180024250     libvcruntime:undname.obj
 0002:00004258       ??_C@_01NEMOKFLO@?$DN@     0000000180024258     libvcruntime:undname.obj
 0002:0000425c       ??_C@_02GPIOPFAK@?$DO?$DO@ 000000018002425c     libvcruntime:undname.obj
 0002:00004260       ??_C@_02FODMEDOG@?$DM?$DM@ 0000000180024260     libvcruntime:undname.obj
 0002:00004264       ??_C@_01DCLJPIOD@?$CB@     0000000180024264     libvcruntime:undname.obj
 0002:00004268       ??_C@_02EGOFBIJA@?$DN?$DN@ 0000000180024268     libvcruntime:undname.obj
 0002:0000426c       ??_C@_02FDNJECIE@?$CB?$DN@ 000000018002426c     libvcruntime:undname.obj
 0002:00004270       ??_C@_02GPECMEKF@?$FL?$FN@ 0000000180024270     libvcruntime:undname.obj
 0002:00004278       ??_C@_08LHJFAFGD@operator@ 0000000180024278     libvcruntime:undname.obj
 0002:00004284       ??_C@_02HBOOOICD@?9?$DO@   0000000180024284     libvcruntime:undname.obj
 0002:00004288       ??_C@_01NBENCBCI@?$CK@     0000000180024288     libvcruntime:undname.obj
 0002:0000428c       ??_C@_02ECNGHCIF@?$CL?$CL@ 000000018002428c     libvcruntime:undname.obj
 0002:00004290       ??_C@_02BAABKJLB@?9?9@     0000000180024290     libvcruntime:undname.obj
 0002:00004294       ??_C@_01JOAMLHOP@?9@       0000000180024294     libvcruntime:undname.obj
 0002:00004298       ??_C@_01MIFGBAGJ@?$CL@     0000000180024298     libvcruntime:undname.obj
 0002:0000429c       ??_C@_01HNPIGOCE@?$CG@     000000018002429c     libvcruntime:undname.obj
 0002:000042a0       ??_C@_03MNHNFDLC@?9?$DO?$CK@ 00000001800242a0     libvcruntime:undname.obj
 0002:000042a4       ??_C@_01KMDKNFGN@?1@       00000001800242a4     libvcruntime:undname.obj
 0002:000042a8       ??_C@_01FGNFDNOH@?$CF@     00000001800242a8     libvcruntime:undname.obj
 0002:000042ac       ??_C@_01MNNFJEPP@?$DM@     00000001800242ac     libvcruntime:undname.obj
 0002:000042b0       ??_C@_02EHCHHCKH@?$DM?$DN@ 00000001800242b0     libvcruntime:undname.obj
 0002:000042b4       ??_C@_01PPODPGHN@?$DO@     00000001800242b4     libvcruntime:undname.obj
 0002:000042b8       ??_C@_02EEKDKGMJ@?$DO?$DN@ 00000001800242b8     libvcruntime:undname.obj
 0002:000042bc       ??_C@_01IHBHIGKO@?0@       00000001800242bc     libvcruntime:undname.obj
 0002:000042c0       ??_C@_02HCKGKOFO@?$CI?$CJ@ 00000001800242c0     libvcruntime:undname.obj
 0002:000042c4       ??_C@_01PJKLJHI@?$HO@      00000001800242c4     libvcruntime:undname.obj
 0002:000042c8       ??_C@_01JKBOJNNK@?$FO@     00000001800242c8     libvcruntime:undname.obj
 0002:000042cc       ??_C@_01DNKMNLPK@?$HM@     00000001800242cc     libvcruntime:undname.obj
 0002:000042d0       ??_C@_02PPKAJPJL@?$CG?$CG@ 00000001800242d0     libvcruntime:undname.obj
 0002:000042d4       ??_C@_02NONPIBCD@?$HM?$HM@ 00000001800242d4     libvcruntime:undname.obj
 0002:000042d8       ??_C@_02FPIMKNGF@?$CK?$DN@ 00000001800242d8     libvcruntime:undname.obj
 0002:000042dc       ??_C@_02FOEOMHFC@?$CL?$DN@ 00000001800242dc     libvcruntime:undname.obj
 0002:000042e0       ??_C@_02FKMDLLOA@?9?$DN@   00000001800242e0     libvcruntime:undname.obj
 0002:000042e4       ??_C@_02FJEHGPIO@?1?$DN@   00000001800242e4     libvcruntime:undname.obj
 0002:000042e8       ??_C@_02FENAOKFI@?$CF?$DN@ 00000001800242e8     libvcruntime:undname.obj
 0002:000042ec       ??_C@_03IKFCCPFF@?$DO?$DO?$DN@ 00000001800242ec     libvcruntime:undname.obj
 0002:000042f0       ??_C@_03CDNPDDLA@?$DM?$DM?$DN@ 00000001800242f0     libvcruntime:undname.obj
 0002:000042f4       ??_C@_02FGJGFEAB@?$CG?$DN@ 00000001800242f4     libvcruntime:undname.obj
 0002:000042f8       ??_C@_02DHLNPPGH@?$HM?$DN@ 00000001800242f8     libvcruntime:undname.obj
 0002:000042fc       ??_C@_02MHEGNOJ@?$FO?$DN@  00000001800242fc     libvcruntime:undname.obj
 0002:00004300       ??_C@_09IFPLHPGF@?$GAvftable?8@ 0000000180024300     libvcruntime:undname.obj
 0002:00004310       ??_C@_09BLBHBJP@?$GAvbtable?8@ 0000000180024310     libvcruntime:undname.obj
 0002:00004320       ??_C@_07FEEIOKP@?$GAvcall?8@ 0000000180024320     libvcruntime:undname.obj
 0002:00004328       ??_C@_08LLFFHHDJ@?$GAtypeof?8@ 0000000180024328     libvcruntime:undname.obj
 0002:00004338       ??_C@_0BF@KDPPACIK@?$GAlocal?5static?5guard?8@ 0000000180024338     libvcruntime:undname.obj
 0002:00004350       ??_C@_08OBABFOLI@?$GAstring?8@ 0000000180024350     libvcruntime:undname.obj
 0002:00004360       ??_C@_0BD@JDLKDPAB@?$GAvbase?5destructor?8@ 0000000180024360     libvcruntime:undname.obj
 0002:00004378       ??_C@_0BN@DEGPLNFK@?$GAvector?5deleting?5destructor?8@ 0000000180024378     libvcruntime:undname.obj
 0002:00004398       ??_C@_0BO@OBMKPJIG@?$GAdefault?5constructor?5closure?8@ 0000000180024398     libvcruntime:undname.obj
 0002:000043b8       ??_C@_0BN@IMDCHIKM@?$GAscalar?5deleting?5destructor?8@ 00000001800243b8     libvcruntime:undname.obj
 0002:000043d8       ??_C@_0BO@PFGOCPJJ@?$GAvector?5constructor?5iterator?8@ 00000001800243d8     libvcruntime:undname.obj
 0002:000043f8       ??_C@_0BN@LFPFMEDL@?$GAvector?5destructor?5iterator?8@ 00000001800243f8     libvcruntime:undname.obj
 0002:00004418       ??_C@_0CE@IKBNEHA@?$GAvector?5vbase?5constructor?5itera@ 0000000180024418     libvcruntime:undname.obj
 0002:00004440       ??_C@_0BL@NILFHHPC@?$GAvirtual?5displacement?5map?8@ 0000000180024440     libvcruntime:undname.obj
 0002:00004460       ??_C@_0CB@JONCMFFK@?$GAeh?5vector?5constructor?5iterator@ 0000000180024460     libvcruntime:undname.obj
 0002:00004488       ??_C@_0CA@GCEOPDGL@?$GAeh?5vector?5destructor?5iterator?8@ 0000000180024488     libvcruntime:undname.obj
 0002:000044a8       ??_C@_0CH@OOJPLCPH@?$GAeh?5vector?5vbase?5constructor?5it@ 00000001800244a8     libvcruntime:undname.obj
 0002:000044d0       ??_C@_0BL@LLKPOHJI@?$GAcopy?5constructor?5closure?8@ 00000001800244d0     libvcruntime:undname.obj
 0002:000044f0       ??_C@_0BA@KBCDOMBN@?$GAudt?5returning?8@ 00000001800244f0     libvcruntime:undname.obj
 0002:00004500       ??_C@_03KLGMFNMG@?$GAEH@   0000000180024500     libvcruntime:undname.obj
 0002:00004504       ??_C@_05KHLCHHI@?$GARTTI@  0000000180024504     libvcruntime:undname.obj
 0002:00004510       ??_C@_0BA@KKLDJDLB@?$GAlocal?5vftable?8@ 0000000180024510     libvcruntime:undname.obj
 0002:00004520       ??_C@_0CE@IIHCMGGL@?$GAlocal?5vftable?5constructor?5clos@ 0000000180024520     libvcruntime:undname.obj
 0002:00004544       ??_C@_06FHBGPFGH@?5new?$FL?$FN@ 0000000180024544     libvcruntime:undname.obj
 0002:00004550       ??_C@_09LBNFPBCA@?5delete?$FL?$FN@ 0000000180024550     libvcruntime:undname.obj
 0002:00004560       ??_C@_0P@HJKNJFNN@?$GAomni?5callsig?8@ 0000000180024560     libvcruntime:undname.obj
 0002:00004570       ??_C@_0BL@CNOONJFP@?$GAplacement?5delete?5closure?8@ 0000000180024570     libvcruntime:undname.obj
 0002:00004590       ??_C@_0BN@CKNJLHMB@?$GAplacement?5delete?$FL?$FN?5closure?8@ 0000000180024590     libvcruntime:undname.obj
 0002:000045b0       ??_C@_0CG@CFDHKGGD@?$GAmanaged?5vector?5constructor?5ite@ 00000001800245b0     libvcruntime:undname.obj
 0002:000045d8       ??_C@_0CF@IMGKMJNO@?$GAmanaged?5vector?5destructor?5iter@ 00000001800245d8     libvcruntime:undname.obj
 0002:00004600       ??_C@_0CG@HLDDJMAG@?$GAeh?5vector?5copy?5constructor?5ite@ 0000000180024600     libvcruntime:undname.obj
 0002:00004628       ??_C@_0CM@FCBBDIGB@?$GAeh?5vector?5vbase?5copy?5construct@ 0000000180024628     libvcruntime:undname.obj
 0002:00004658       ??_C@_0BL@CLIPGLGB@?$GAdynamic?5initializer?5for?5?8@ 0000000180024658     libvcruntime:undname.obj
 0002:00004678       ??_C@_0CB@PDBIFEP@?$GAdynamic?5atexit?5destructor?5for?5@ 0000000180024678     libvcruntime:undname.obj
 0002:000046a0       ??_C@_0CD@CGAJBKEJ@?$GAvector?5copy?5constructor?5iterat@ 00000001800246a0     libvcruntime:undname.obj
 0002:000046c8       ??_C@_0CJ@GJELGAMM@?$GAvector?5vbase?5copy?5constructor?5@ 00000001800246c8     libvcruntime:undname.obj
 0002:000046f8       ??_C@_0CL@FGIJHLCE@?$GAmanaged?5vector?5copy?5constructo@ 00000001800246f8     libvcruntime:undname.obj
 0002:00004728       ??_C@_0BM@PMGGMLDN@?$GAlocal?5static?5thread?5guard?8@ 0000000180024728     libvcruntime:undname.obj
 0002:00004748       ??_C@_0N@BDNMDMOL@operator?5?$CC?$CC?5@ 0000000180024748     libvcruntime:undname.obj
 0002:00004758       ??_C@_0BC@GGEBGALA@operator?5co_await@ 0000000180024758     libvcruntime:undname.obj
 0002:00004770       ??_C@_0M@GAAIMMOH@operator?$DM?$DN?$DO@ 0000000180024770     libvcruntime:undname.obj
 0002:00004780       ??_C@_0BC@DAFEJGAK@?5Type?5Descriptor?8@ 0000000180024780     libvcruntime:undname.obj
 0002:00004798       ??_C@_0BM@LDKODKLH@?5Base?5Class?5Descriptor?5at?5?$CI@ 0000000180024798     libvcruntime:undname.obj
 0002:000047b8       ??_C@_0BD@LGICGFMM@?5Base?5Class?5Array?8@ 00000001800247b8     libvcruntime:undname.obj
 0002:000047d0       ??_C@_0BN@MECKDCOJ@?5Class?5Hierarchy?5Descriptor?8@ 00000001800247d0     libvcruntime:undname.obj
 0002:000047f0       ??_C@_0BK@CFCOFLF@?5Complete?5Object?5Locator?8@ 00000001800247f0     libvcruntime:undname.obj
 0002:00004810       ??_C@_0BG@JNJLAMPM@?$GAanonymous?5namespace?8@ 0000000180024810     libvcruntime:undname.obj
 0002:000048e0       ??_C@_1DM@KHCHBNEB@?$AAa?$AAp?$AAi?$AA?9?$AAm?$AAs?$AA?9?$AAw?$AAi?$AAn?$AA?9?$AAc?$AAo?$AAr?$AAe@ 00000001800248e0     libvcruntime:winapi_downlevel.obj
 0002:00004920       ??_C@_1DK@LPPGFMPP@?$AAa?$AAp?$AAi?$AA?9?$AAm?$AAs?$AA?9?$AAw?$AAi?$AAn?$AA?9?$AAc?$AAo?$AAr?$AAe@ 0000000180024920     libvcruntime:winapi_downlevel.obj
 0002:00004960       ??_C@_1BC@GDMECMAK@?$AAk?$AAe?$AAr?$AAn?$AAe?$AAl?$AA3?$AA2@ 0000000180024960     libvcruntime:winapi_downlevel.obj
 0002:00004978       ??_C@_1BA@PFFKHIOG@?$AAa?$AAp?$AAi?$AA?9?$AAm?$AAs?$AA?9@ 0000000180024978     libvcruntime:winapi_downlevel.obj
 0002:00004990       ??_C@_08KNHFBNJ@FlsAlloc@  0000000180024990     libvcruntime:winapi_downlevel.obj
 0002:000049a8       ??_C@_07PEJMOBNF@FlsFree@  00000001800249a8     libvcruntime:winapi_downlevel.obj
 0002:000049b8       ??_C@_0M@GDNOONDI@FlsGetValue@ 00000001800249b8     libvcruntime:winapi_downlevel.obj
 0002:000049d0       ??_C@_0M@JCPCPOEF@FlsSetValue@ 00000001800249d0     libvcruntime:winapi_downlevel.obj
 0002:000049e8       ??_C@_0BM@HCFOFFN@InitializeCriticalSectionEx@ 00000001800249e8     libvcruntime:winapi_downlevel.obj
 0002:00004a10       ??_7bad_exception@std@@6B@ 0000000180024a10     libvcruntime:frame.obj
 0002:00004a20       ??_C@_0O@DPKOEFFH@bad?5exception@ 0000000180024a20     libvcruntime:frame.obj
 0002:00004a30       ?standard_lookup_table_spectre@__crt_stdio_output@@3V?$spectre_mitigated_lookup_table@Ustate_transition_pair@__crt_stdio_output@@$0IA@@1@B 0000000180024a30     libucrt:output.obj
 0002:00004b30       ??_C@_1O@CEDCILHN@?$AA?$CI?$AAn?$AAu?$AAl?$AAl?$AA?$CJ@ 0000000180024b30     libucrt:output.obj
 0002:00004b40       ??_C@_06OJHGLDPL@?$CInull?$CJ@ 0000000180024b40     libucrt:output.obj
 0002:00004b50       __acrt_exception_action_table 0000000180024b50     libucrt:exception_filter.obj
 0002:00004c10       __acrt_signal_action_table_count 0000000180024c10     libucrt:exception_filter.obj
 0002:00004c18       __acrt_signal_action_first_fpe_index 0000000180024c18     libucrt:exception_filter.obj
 0002:00004c20       __acrt_signal_action_fpe_count 0000000180024c20     libucrt:exception_filter.obj
 0002:00004c78       ??_C@_1BI@BGOHAHKC@?$AAm?$AAs?$AAc?$AAo?$AAr?$AAe?$AAe?$AA?4?$AAd?$AAl?$AAl@ 0000000180024c78     libucrt:exit.obj
 0002:00004c90       ??_C@_0P@MIGLKIOC@CorExitProcess@ 0000000180024c90     libucrt:exit.obj
 0002:00005010       ??_C@_1EA@JGEFHKEI@?$AAa?$AAp?$AAi?$AA?9?$AAm?$AAs?$AA?9?$AAw?$AAi?$AAn?$AA?9?$AAc?$AAo?$AAr?$AAe@ 0000000180025010     libucrt:winapi_thunks.obj
 0002:00005050       ??_C@_1DI@KMEPCBPN@?$AAa?$AAp?$AAi?$AA?9?$AAm?$AAs?$AA?9?$AAw?$AAi?$AAn?$AA?9?$AAc?$AAo?$AAr?$AAe@ 0000000180025050     libucrt:winapi_thunks.obj
 0002:00005088       ??_C@_1DI@IJCEHOCB@?$AAa?$AAp?$AAi?$AA?9?$AAm?$AAs?$AA?9?$AAw?$AAi?$AAn?$AA?9?$AAc?$AAo?$AAr?$AAe@ 0000000180025088     libucrt:winapi_thunks.obj
 0002:000050c0       ??_C@_1EI@MPIAOHOC@?$AAa?$AAp?$AAi?$AA?9?$AAm?$AAs?$AA?9?$AAw?$AAi?$AAn?$AA?9?$AAc?$AAo?$AAr?$AAe@ 00000001800250c0     libucrt:winapi_thunks.obj
 0002:00005110       ??_C@_1FK@FPHCKFIE@?$AAa?$AAp?$AAi?$AA?9?$AAm?$AAs?$AA?9?$AAw?$AAi?$AAn?$AA?9?$AAc?$AAo?$AAr?$AAe@ 0000000180025110     libucrt:winapi_thunks.obj
 0002:00005170       ??_C@_1EM@DILCGIIO@?$AAa?$AAp?$AAi?$AA?9?$AAm?$AAs?$AA?9?$AAw?$AAi?$AAn?$AA?9?$AAc?$AAo?$AAr?$AAe@ 0000000180025170     libucrt:winapi_thunks.obj
 0002:000051c0       ??_C@_1DM@LNCGDDPN@?$AAa?$AAp?$AAi?$AA?9?$AAm?$AAs?$AA?9?$AAw?$AAi?$AAn?$AA?9?$AAc?$AAo?$AAr?$AAe@ 00000001800251c0     libucrt:winapi_thunks.obj
 0002:00005200       ??_C@_1DO@FPAPJEMD@?$AAa?$AAp?$AAi?$AA?9?$AAm?$AAs?$AA?9?$AAw?$AAi?$AAn?$AA?9?$AAc?$AAo?$AAr?$AAe@ 0000000180025200     libucrt:winapi_thunks.obj
 0002:00005240       ??_C@_1DK@NDHNAHIO@?$AAa?$AAp?$AAi?$AA?9?$AAm?$AAs?$AA?9?$AAw?$AAi?$AAn?$AA?9?$AAc?$AAo?$AAr?$AAe@ 0000000180025240     libucrt:winapi_thunks.obj
 0002:00005280       ??_C@_1DM@KGHDGBCM@?$AAa?$AAp?$AAi?$AA?9?$AAm?$AAs?$AA?9?$AAw?$AAi?$AAn?$AA?9?$AAc?$AAo?$AAr?$AAe@ 0000000180025280     libucrt:winapi_thunks.obj
 0002:000052c0       ??_C@_1EO@IJIOEFOH@?$AAa?$AAp?$AAi?$AA?9?$AAm?$AAs?$AA?9?$AAw?$AAi?$AAn?$AA?9?$AAr?$AAt?$AAc?$AAo@ 00000001800252c0     libucrt:winapi_thunks.obj
 0002:00005310       ??_C@_1FG@HHGEKANL@?$AAa?$AAp?$AAi?$AA?9?$AAm?$AAs?$AA?9?$AAw?$AAi?$AAn?$AA?9?$AAs?$AAe?$AAc?$AAu@ 0000000180025310     libucrt:winapi_thunks.obj
 0002:00005370       ??_C@_1EG@DBIOJECG@?$AAe?$AAx?$AAt?$AA?9?$AAm?$AAs?$AA?9?$AAw?$AAi?$AAn?$AA?9?$AAn?$AAt?$AAu?$AAs@ 0000000180025370     libucrt:winapi_thunks.obj
 0002:000053c0       ??_C@_1EO@FIHMJCLF@?$AAe?$AAx?$AAt?$AA?9?$AAm?$AAs?$AA?9?$AAw?$AAi?$AAn?$AA?9?$AAn?$AAt?$AAu?$AAs@ 00000001800253c0     libucrt:winapi_thunks.obj
 0002:00005410       ??_C@_1BC@DNHGCMLG@?$AAa?$AAd?$AAv?$AAa?$AAp?$AAi?$AA3?$AA2@ 0000000180025410     libucrt:winapi_thunks.obj
 0002:00005428       ??_C@_1BG@CJPGBMEF@?$AAk?$AAe?$AAr?$AAn?$AAe?$AAl?$AAb?$AAa?$AAs?$AAe@ 0000000180025428     libucrt:winapi_thunks.obj
 0002:00005440       ??_C@_1M@OAIMIKLP@?$AAn?$AAt?$AAd?$AAl?$AAl@ 0000000180025440     libucrt:winapi_thunks.obj
 0002:00005450       ??_C@_1EG@DPGNFKGC@?$AAa?$AAp?$AAi?$AA?9?$AAm?$AAs?$AA?9?$AAw?$AAi?$AAn?$AA?9?$AAa?$AAp?$AAp?$AAm@ 0000000180025450     libucrt:winapi_thunks.obj
 0002:00005498       ??_C@_1O@BCCLBEOE@?$AAu?$AAs?$AAe?$AAr?$AA3?$AA2@ 0000000180025498     libucrt:winapi_thunks.obj
 0002:000054a8       ??_C@_1BA@IAIFMGEF@?$AAe?$AAx?$AAt?$AA?9?$AAm?$AAs?$AA?9@ 00000001800254a8     libucrt:winapi_thunks.obj
 0002:000054c0       ??_C@_0BA@FHFNEAED@AreFileApisANSI@ 00000001800254c0     libucrt:winapi_thunks.obj
 0002:000054d8       ??_C@_0BA@IHGNDAEB@CompareStringEx@ 00000001800254d8     libucrt:winapi_thunks.obj
 0002:000054f8       ??_C@_0O@KKBNKAPF@LCMapStringEx@ 00000001800254f8     libucrt:winapi_thunks.obj
 0002:00005510       ??_C@_0BB@HBDEELFH@LocaleNameToLCID@ 0000000180025510     libucrt:winapi_thunks.obj
 0002:00005528       ??_C@_0CF@OJOFEIGO@AppPolicyGetProcessTerminationM@ 0000000180025528     libucrt:winapi_thunks.obj
 0002:000055d0       ??_C@_03OEIAHPBN@INF@      00000001800255d0     libucrt:cvt.obj
 0002:000055d4       ??_C@_03OJHLLCGB@inf@      00000001800255d4     libucrt:cvt.obj
 0002:000055d8       ??_C@_03LKNCIKJB@NAN@      00000001800255d8     libucrt:cvt.obj
 0002:000055dc       ??_C@_03LHCJEHON@nan@      00000001800255dc     libucrt:cvt.obj
 0002:000055e0       ??_C@_09OFJJIMPC@NAN?$CISNAN?$CJ@ 00000001800255e0     libucrt:cvt.obj
 0002:000055f0       ??_C@_09IPFBKMDL@nan?$CIsnan?$CJ@ 00000001800255f0     libucrt:cvt.obj
 0002:00005600       ??_C@_08IKHNHAJ@NAN?$CIIND?$CJ@ 0000000180025600     libucrt:cvt.obj
 0002:00005610       ??_C@_08OFCDMILK@nan?$CIind?$CJ@ 0000000180025610     libucrt:cvt.obj
 0002:0000561c       ??_C@_05KLBDPFGC@e?$CL000@ 000000018002561c     libucrt:cvt.obj
 0002:00005630       __lc_time_c                0000000180025630     libucrt:nlsdata.obj
 0002:000058f0       ??_C@_03KOEHGMDN@Sun@      00000001800258f0     libucrt:nlsdata.obj
 0002:000058f4       ??_C@_03PDAGKDH@Mon@       00000001800258f4     libucrt:nlsdata.obj
 0002:000058f8       ??_C@_03NAGEINEP@Tue@      00000001800258f8     libucrt:nlsdata.obj
 0002:000058fc       ??_C@_03MHOMLAJA@Wed@      00000001800258fc     libucrt:nlsdata.obj
 0002:00005900       ??_C@_03IOFIKPDN@Thu@      0000000180025900     libucrt:nlsdata.obj
 0002:00005904       ??_C@_03IDIOELNC@Fri@      0000000180025904     libucrt:nlsdata.obj
 0002:00005908       ??_C@_03FEFJNEK@Sat@       0000000180025908     libucrt:nlsdata.obj
 0002:0000590c       ??_C@_06OOPIFAJ@Sunday@    000000018002590c     libucrt:nlsdata.obj
 0002:00005914       ??_C@_06JLEDEDGH@Monday@   0000000180025914     libucrt:nlsdata.obj
 0002:00005920       ??_C@_07BAAGCFCM@Tuesday@  0000000180025920     libucrt:nlsdata.obj
 0002:00005928       ??_C@_09DLIGFAKA@Wednesday@ 0000000180025928     libucrt:nlsdata.obj
 0002:00005938       ??_C@_08HACCIKIA@Thursday@ 0000000180025938     libucrt:nlsdata.obj
 0002:00005944       ??_C@_06JECMNKMI@Friday@   0000000180025944     libucrt:nlsdata.obj
 0002:00005950       ??_C@_08INBOOONO@Saturday@ 0000000180025950     libucrt:nlsdata.obj
 0002:0000595c       ??_C@_03JIHJHPIE@Jan@      000000018002595c     libucrt:nlsdata.obj
 0002:00005960       ??_C@_03HJBDCHOM@Feb@      0000000180025960     libucrt:nlsdata.obj
 0002:00005964       ??_C@_03ODNJBKGA@Mar@      0000000180025964     libucrt:nlsdata.obj
 0002:00005968       ??_C@_03LEOLGMJP@Apr@      0000000180025968     libucrt:nlsdata.obj
 0002:0000596c       ??_C@_03CNMDKL@May@        000000018002596c     libucrt:nlsdata.obj
 0002:00005970       ??_C@_03IDFGHECI@Jun@      0000000180025970     libucrt:nlsdata.obj
 0002:00005974       ??_C@_03LBGABGKK@Jul@      0000000180025974     libucrt:nlsdata.obj
 0002:00005978       ??_C@_03IFJFEIGA@Aug@      0000000180025978     libucrt:nlsdata.obj
 0002:0000597c       ??_C@_03GGCAPAJC@Sep@      000000018002597c     libucrt:nlsdata.obj
 0002:00005980       ??_C@_03BMAOKBAD@Oct@      0000000180025980     libucrt:nlsdata.obj
 0002:00005984       ??_C@_03JPJOFNIA@Nov@      0000000180025984     libucrt:nlsdata.obj
 0002:00005988       ??_C@_03MKABNOCG@Dec@      0000000180025988     libucrt:nlsdata.obj
 0002:00005990       ??_C@_07CGJPFGJA@January@  0000000180025990     libucrt:nlsdata.obj
 0002:00005998       ??_C@_08GNJGEPFN@February@ 0000000180025998     libucrt:nlsdata.obj
 0002:000059a4       ??_C@_05HPCKOFNC@March@    00000001800259a4     libucrt:nlsdata.obj
 0002:000059ac       ??_C@_05DMJDNLEJ@April@    00000001800259ac     libucrt:nlsdata.obj
 0002:000059b4       ??_C@_04CNLMGBGM@June@     00000001800259b4     libucrt:nlsdata.obj
 0002:000059bc       ??_C@_04MIEPOIFP@July@     00000001800259bc     libucrt:nlsdata.obj
 0002:000059c4       ??_C@_06LBBHFDDG@August@   00000001800259c4     libucrt:nlsdata.obj
 0002:000059d0       ??_C@_09BHHEALKD@September@ 00000001800259d0     libucrt:nlsdata.obj
 0002:000059e0       ??_C@_07JJNFCEND@October@  00000001800259e0     libucrt:nlsdata.obj
 0002:000059e8       ??_C@_08HCHEGEOA@November@ 00000001800259e8     libucrt:nlsdata.obj
 0002:000059f8       ??_C@_08EDHMEBNP@December@ 00000001800259f8     libucrt:nlsdata.obj
 0002:00005a04       ??_C@_02DEDBPAFC@AM@       0000000180025a04     libucrt:nlsdata.obj
 0002:00005a08       ??_C@_02CJNFDJBF@PM@       0000000180025a08     libucrt:nlsdata.obj
 0002:00005a10       ??_C@_08BPBNCDIB@MM?1dd?1yy@ 0000000180025a10     libucrt:nlsdata.obj
 0002:00005a20       ??_C@_0BE@CKGJFCPC@dddd?0?5MMMM?5dd?0?5yyyy@ 0000000180025a20     libucrt:nlsdata.obj
 0002:00005a38       ??_C@_08JCCMCCIL@HH?3mm?3ss@ 0000000180025a38     libucrt:nlsdata.obj
 0002:00005a48       ??_C@_17MBGCMIPB@?$AAS?$AAu?$AAn@ 0000000180025a48     libucrt:nlsdata.obj
 0002:00005a50       ??_C@_17KBOMKBF@?$AAM?$AAo?$AAn@ 0000000180025a50     libucrt:nlsdata.obj
 0002:00005a58       ??_C@_17BMKGEGOJ@?$AAT?$AAu?$AAe@ 0000000180025a58     libucrt:nlsdata.obj
 0002:00005a60       ??_C@_17CJEDCEPE@?$AAW?$AAe?$AAd@ 0000000180025a60     libucrt:nlsdata.obj
 0002:00005a68       ??_C@_17PDPHAADD@?$AAT?$AAh?$AAu@ 0000000180025a68     libucrt:nlsdata.obj
 0002:00005a70       ??_C@_17HFOLPPLP@?$AAF?$AAr?$AAi@ 0000000180025a70     libucrt:nlsdata.obj
 0002:00005a78       ??_C@_17GGIBDPIH@?$AAS?$AAa?$AAt@ 0000000180025a78     libucrt:nlsdata.obj
 0002:00005a80       ??_C@_1O@IHNHDHPB@?$AAS?$AAu?$AAn?$AAd?$AAa?$AAy@ 0000000180025a80     libucrt:nlsdata.obj
 0002:00005a90       ??_C@_1O@MMNBFLIA@?$AAM?$AAo?$AAn?$AAd?$AAa?$AAy@ 0000000180025a90     libucrt:nlsdata.obj
 0002:00005aa0       ??_C@_1BA@ENFBFFEK@?$AAT?$AAu?$AAe?$AAs?$AAd?$AAa?$AAy@ 0000000180025aa0     libucrt:nlsdata.obj
 0002:00005ab0       ??_C@_1BE@EBOGMDOH@?$AAW?$AAe?$AAd?$AAn?$AAe?$AAs?$AAd?$AAa?$AAy@ 0000000180025ab0     libucrt:nlsdata.obj
 0002:00005ac8       ??_C@_1BC@HHMNLIHE@?$AAT?$AAh?$AAu?$AAr?$AAs?$AAd?$AAa?$AAy@ 0000000180025ac8     libucrt:nlsdata.obj
 0002:00005ae0       ??_C@_1O@PDICJHAG@?$AAF?$AAr?$AAi?$AAd?$AAa?$AAy@ 0000000180025ae0     libucrt:nlsdata.obj
 0002:00005af0       ??_C@_1BC@ENMNNPAJ@?$AAS?$AAa?$AAt?$AAu?$AAr?$AAd?$AAa?$AAy@ 0000000180025af0     libucrt:nlsdata.obj
 0002:00005b08       ??_C@_17DKNBKCHM@?$AAJ?$AAa?$AAn@ 0000000180025b08     libucrt:nlsdata.obj
 0002:00005b10       ??_C@_17LMDJEKJN@?$AAF?$AAe?$AAb@ 0000000180025b10     libucrt:nlsdata.obj
 0002:00005b18       ??_C@_17CKNLEDEC@?$AAM?$AAa?$AAr@ 0000000180025b18     libucrt:nlsdata.obj
 0002:00005b20       ??_C@_17LFPOIHDD@?$AAA?$AAp?$AAr@ 0000000180025b20     libucrt:nlsdata.obj
 0002:00005b28       ??_C@_17PNNKMEED@?$AAM?$AAa?$AAy@ 0000000180025b28     libucrt:nlsdata.obj
 0002:00005b30       ??_C@_17KCJGOCPB@?$AAJ?$AAu?$AAn@ 0000000180025b30     libucrt:nlsdata.obj
 0002:00005b38       ??_C@_17IJPCKHK@?$AAJ?$AAu?$AAl@ 0000000180025b38     libucrt:nlsdata.obj
 0002:00005b40       ??_C@_17ICPELBCN@?$AAA?$AAu?$AAg@ 0000000180025b40     libucrt:nlsdata.obj
 0002:00005b48       ??_C@_17HCHCOKMG@?$AAS?$AAe?$AAp@ 0000000180025b48     libucrt:nlsdata.obj
 0002:00005b50       ??_C@_17FNLKOI@?$AAO?$AAc?$AAt@ 0000000180025b50     libucrt:nlsdata.obj
 0002:00005b58       ??_C@_17BBDMLCIG@?$AAN?$AAo?$AAv@ 0000000180025b58     libucrt:nlsdata.obj
 0002:00005b60       ??_C@_17EGKACKIF@?$AAD?$AAe?$AAc@ 0000000180025b60     libucrt:nlsdata.obj
 0002:00005b68       ??_C@_1BA@EFMEIEBA@?$AAJ?$AAa?$AAn?$AAu?$AAa?$AAr?$AAy@ 0000000180025b68     libucrt:nlsdata.obj
 0002:00005b78       ??_C@_1BC@JGDDFFAM@?$AAF?$AAe?$AAb?$AAr?$AAu?$AAa?$AAr?$AAy@ 0000000180025b78     libucrt:nlsdata.obj
 0002:00005b90       ??_C@_1M@IKEENEDF@?$AAM?$AAa?$AAr?$AAc?$AAh@ 0000000180025b90     libucrt:nlsdata.obj
 0002:00005ba0       ??_C@_1M@GJNLMHFD@?$AAA?$AAp?$AAr?$AAi?$AAl@ 0000000180025ba0     libucrt:nlsdata.obj
 0002:00005bb0       ??_C@_19EPFLPGAP@?$AAJ?$AAu?$AAn?$AAe@ 0000000180025bb0     libucrt:nlsdata.obj
 0002:00005bc0       ??_C@_19BIFMLPCD@?$AAJ?$AAu?$AAl?$AAy@ 0000000180025bc0     libucrt:nlsdata.obj
 0002:00005bd0       ??_C@_1O@PAHLKOAC@?$AAA?$AAu?$AAg?$AAu?$AAs?$AAt@ 0000000180025bd0     libucrt:nlsdata.obj
 0002:00005be0       ??_C@_1BE@DKAAMBJL@?$AAS?$AAe?$AAp?$AAt?$AAe?$AAm?$AAb?$AAe?$AAr@ 0000000180025be0     libucrt:nlsdata.obj
 0002:00005bf8       ??_C@_1BA@EPANDLNG@?$AAO?$AAc?$AAt?$AAo?$AAb?$AAe?$AAr@ 0000000180025bf8     libucrt:nlsdata.obj
 0002:00005c08       ??_C@_1BC@BGLIFPF@?$AAN?$AAo?$AAv?$AAe?$AAm?$AAb?$AAe?$AAr@ 0000000180025c08     libucrt:nlsdata.obj
 0002:00005c20       ??_C@_1BC@FEMKIFH@?$AAD?$AAe?$AAc?$AAe?$AAm?$AAb?$AAe?$AAr@ 0000000180025c20     libucrt:nlsdata.obj
 0002:00005c34       ??_C@_15ODEHAHHF@?$AAA?$AAM@ 0000000180025c34     libucrt:nlsdata.obj
 0002:00005c3c       ??_C@_15CLMNNGEL@?$AAP?$AAM@ 0000000180025c3c     libucrt:nlsdata.obj
 0002:00005c48       ??_C@_1BC@IEBCMHCM@?$AAM?$AAM?$AA?1?$AAd?$AAd?$AA?1?$AAy?$AAy@ 0000000180025c48     libucrt:nlsdata.obj
 0002:00005c60       ??_C@_1CI@KNAKOEBC@?$AAd?$AAd?$AAd?$AAd?$AA?0?$AA?5?$AAM?$AAM?$AAM?$AAM?$AA?5?$AAd?$AAd?$AA?0?$AA?5@ 0000000180025c60     libucrt:nlsdata.obj
 0002:00005c88       ??_C@_1BC@GDGBMEMK@?$AAH?$AAH?$AA?3?$AAm?$AAm?$AA?3?$AAs?$AAs@ 0000000180025c88     libucrt:nlsdata.obj
 0002:00005ca0       ??_C@_1M@BMHNFIME@?$AAe?$AAn?$AA?9?$AAU?$AAS@ 0000000180025ca0     libucrt:nlsdata.obj
 0002:00005cac       ?ccs@?1???$__acrt_stdio_parse_mode@D@@YA?AU__acrt_stdio_stream_mode@@QEBD@Z@4QBDB 0000000180025cac     libucrt:openfile.obj
 0002:00005cb0       ?utf8_encoding@?1???$__acrt_stdio_parse_mode@D@@YA?AU__acrt_stdio_stream_mode@@QEBD@Z@4QBDB 0000000180025cb0     libucrt:openfile.obj
 0002:00005cb8       ?utf16_encoding@?1???$__acrt_stdio_parse_mode@D@@YA?AU__acrt_stdio_stream_mode@@QEBD@Z@4QBDB 0000000180025cb8     libucrt:openfile.obj
 0002:00005cc0       ?unicode_encoding@?1???$__acrt_stdio_parse_mode@D@@YA?AU__acrt_stdio_stream_mode@@QEBD@Z@4QBDB 0000000180025cc0     libucrt:openfile.obj
 0002:00005ce8       ??_C@_1M@HPNHIDJI@?$AAj?$AAa?$AA?9?$AAJ?$AAP@ 0000000180025ce8     libucrt:mbctype.obj
 0002:00005cf8       ??_C@_1M@BIBDDEMK@?$AAz?$AAh?$AA?9?$AAC?$AAN@ 0000000180025cf8     libucrt:mbctype.obj
 0002:00005d08       ??_C@_1M@JLOOOEGK@?$AAk?$AAo?$AA?9?$AAK?$AAR@ 0000000180025d08     libucrt:mbctype.obj
 0002:00005d18       ??_C@_1M@CLNBBOPM@?$AAz?$AAh?$AA?9?$AAT?$AAW@ 0000000180025d18     libucrt:mbctype.obj
 0002:00005d30       __newctype                 0000000180025d30     libucrt:ctype.obj
 0002:00006030       __newclmap                 0000000180026030     libucrt:ctype.obj
 0002:000061b0       __newcumap                 00000001800261b0     libucrt:ctype.obj
 0002:00007170       ??_C@_15EMKDOKLE@?$AAa?$AAr@ 0000000180027170     libucrt:lcidtoname_downlevel.obj
 0002:00007178       ??_C@_15KNPADPLH@?$AAb?$AAg@ 0000000180027178     libucrt:lcidtoname_downlevel.obj
 0002:00007180       ??_C@_15EDMHLDMO@?$AAc?$AAa@ 0000000180027180     libucrt:lcidtoname_downlevel.obj
 0002:00007188       ??_C@_1O@BPEAJADD@?$AAz?$AAh?$AA?9?$AAC?$AAH?$AAS@ 0000000180027188     libucrt:lcidtoname_downlevel.obj
 0002:00007198       ??_C@_15LJNHCMNK@?$AAc?$AAs@ 0000000180027198     libucrt:lcidtoname_downlevel.obj
 0002:000071a0       ??_C@_15FOMCIDHG@?$AAd?$AAa@ 00000001800271a0     libucrt:lcidtoname_downlevel.obj
 0002:000071a8       ??_C@_15NBKABECB@?$AAd?$AAe@ 00000001800271a8     libucrt:lcidtoname_downlevel.obj
 0002:000071b0       ??_C@_15GHPEIIAO@?$AAe?$AAl@ 00000001800271b0     libucrt:lcidtoname_downlevel.obj
 0002:000071b8       ??_C@_15MNPNEAIF@?$AAe?$AAn@ 00000001800271b8     libucrt:lcidtoname_downlevel.obj
 0002:000071c0       ??_C@_15GPIOMPMH@?$AAe?$AAs@ 00000001800271c0     libucrt:lcidtoname_downlevel.obj
 0002:000071c8       ??_C@_15NGLOAKJC@?$AAf?$AAi@ 00000001800271c8     libucrt:lcidtoname_downlevel.obj
 0002:000071d0       ??_C@_15FBKGNKAM@?$AAf?$AAr@ 00000001800271d0     libucrt:lcidtoname_downlevel.obj
 0002:000071d8       ??_C@_15KGGCNEFK@?$AAh?$AAe@ 00000001800271d8     libucrt:lcidtoname_downlevel.obj
 0002:000071e0       ??_C@_15PGHLIDMF@?$AAh?$AAu@ 00000001800271e0     libucrt:lcidtoname_downlevel.obj
 0002:000071e8       ??_C@_15BIEMAPLM@?$AAi?$AAs@ 00000001800271e8     libucrt:lcidtoname_downlevel.obj
 0002:000071f0       ??_C@_15IFJLDHAF@?$AAi?$AAt@ 00000001800271f0     libucrt:lcidtoname_downlevel.obj
 0002:000071f8       ??_C@_15GEMIOCAG@?$AAj?$AAa@ 00000001800271f8     libucrt:lcidtoname_downlevel.obj
 0002:00007200       ??_C@_15EPELEGJA@?$AAk?$AAo@ 0000000180027200     libucrt:lcidtoname_downlevel.obj
 0002:00007208       ??_C@_15NDDHIMN@?$AAn?$AAl@ 0000000180027208     libucrt:lcidtoname_downlevel.obj
 0002:00007210       ??_C@_15BPIGNHCD@?$AAn?$AAo@ 0000000180027210     libucrt:lcidtoname_downlevel.obj
 0002:00007218       ??_C@_15DEOPBLCG@?$AAp?$AAl@ 0000000180027218     libucrt:lcidtoname_downlevel.obj
 0002:00007220       ??_C@_15KBECGEFG@?$AAp?$AAt@ 0000000180027220     libucrt:lcidtoname_downlevel.obj
 0002:00007228       ??_C@_15GLJCBFMD@?$AAr?$AAo@ 0000000180027228     libucrt:lcidtoname_downlevel.obj
 0002:00007230       ??_C@_15FEDGKCDI@?$AAr?$AAu@ 0000000180027230     libucrt:lcidtoname_downlevel.obj
 0002:00007238       ??_C@_15GLKMLLHM@?$AAh?$AAr@ 0000000180027238     libucrt:lcidtoname_downlevel.obj
 0002:00007240       ??_C@_15CPKMFBDB@?$AAs?$AAk@ 0000000180027240     libucrt:lcidtoname_downlevel.obj
 0002:00007248       ??_C@_15BAAIOGMK@?$AAs?$AAq@ 0000000180027248     libucrt:lcidtoname_downlevel.obj
 0002:00007250       ??_C@_15INNPNOHD@?$AAs?$AAv@ 0000000180027250     libucrt:lcidtoname_downlevel.obj
 0002:00007258       ??_C@_15CABMMOGH@?$AAt?$AAh@ 0000000180027258     libucrt:lcidtoname_downlevel.obj
 0002:00007260       ??_C@_15BPLIHJJM@?$AAt?$AAr@ 0000000180027260     libucrt:lcidtoname_downlevel.obj
 0002:00007268       ??_C@_15NEOEKKDJ@?$AAu?$AAr@ 0000000180027268     libucrt:lcidtoname_downlevel.obj
 0002:00007270       ??_C@_15NFICGAJK@?$AAi?$AAd@ 0000000180027270     libucrt:lcidtoname_downlevel.obj
 0002:00007278       ??_C@_15PJPFLCCM@?$AAu?$AAk@ 0000000180027278     libucrt:lcidtoname_downlevel.obj
 0002:00007280       ??_C@_15HPJPHDM@?$AAb?$AAe@ 0000000180027280     libucrt:lcidtoname_downlevel.obj
 0002:00007288       ??_C@_15LCHLGJII@?$AAs?$AAl@ 0000000180027288     libucrt:lcidtoname_downlevel.obj
 0002:00007290       ??_C@_15PCFJPHHO@?$AAe?$AAt@ 0000000180027290     libucrt:lcidtoname_downlevel.obj
 0002:00007298       ??_C@_15HPFPGODN@?$AAl?$AAv@ 0000000180027298     libucrt:lcidtoname_downlevel.obj
 0002:000072a0       ??_C@_15NFFGKGLG@?$AAl?$AAt@ 00000001800272a0     libucrt:lcidtoname_downlevel.obj
 0002:000072a8       ??_C@_15BDAKCCHN@?$AAf?$AAa@ 00000001800272a8     libucrt:lcidtoname_downlevel.obj
 0002:000072b0       ??_C@_15NFGIAIAJ@?$AAv?$AAi@ 00000001800272b0     libucrt:lcidtoname_downlevel.obj
 0002:000072b8       ??_C@_15LMKNDMHN@?$AAh?$AAy@ 00000001800272b8     libucrt:lcidtoname_downlevel.obj
 0002:000072c0       ??_C@_15IJBHMCFL@?$AAa?$AAz@ 00000001800272c0     libucrt:lcidtoname_downlevel.obj
 0002:000072c8       ??_C@_15EKOFJABL@?$AAe?$AAu@ 00000001800272c8     libucrt:lcidtoname_downlevel.obj
 0002:000072d0       ??_C@_15BGHADCNK@?$AAm?$AAk@ 00000001800272d0     libucrt:lcidtoname_downlevel.obj
 0002:000072d8       ??_C@_15JDNICKHM@?$AAa?$AAf@ 00000001800272d8     libucrt:lcidtoname_downlevel.obj
 0002:000072e0       ??_C@_15KPJEDBKD@?$AAk?$AAa@ 00000001800272e0     libucrt:lcidtoname_downlevel.obj
 0002:000072e8       ??_C@_15PDNFFFEO@?$AAf?$AAo@ 00000001800272e8     libucrt:lcidtoname_downlevel.obj
 0002:000072f0       ??_C@_15OMLEGLOC@?$AAh?$AAi@ 00000001800272f0     libucrt:lcidtoname_downlevel.obj
 0002:000072f8       ??_C@_15IDNNENKK@?$AAm?$AAs@ 00000001800272f8     libucrt:lcidtoname_downlevel.obj
 0002:00007300       ??_C@_15MACJNBMH@?$AAk?$AAk@ 0000000180027300     libucrt:lcidtoname_downlevel.obj
 0002:00007308       ??_C@_15DKDJEOND@?$AAk?$AAy@ 0000000180027308     libucrt:lcidtoname_downlevel.obj
 0002:00007310       ??_C@_15DFGDLJBG@?$AAs?$AAw@ 0000000180027310     libucrt:lcidtoname_downlevel.obj
 0002:00007318       ??_C@_15BBFAICNG@?$AAu?$AAz@ 0000000180027318     libucrt:lcidtoname_downlevel.obj
 0002:00007320       ??_C@_15DKNDCGEA@?$AAt?$AAt@ 0000000180027320     libucrt:lcidtoname_downlevel.obj
 0002:00007328       ??_C@_15MGIFMDPL@?$AAp?$AAa@ 0000000180027328     libucrt:lcidtoname_downlevel.obj
 0002:00007330       ??_C@_15HCNDBBA@?$AAg?$AAu@ 0000000180027330     libucrt:lcidtoname_downlevel.obj
 0002:00007338       ??_C@_15FNBEIBON@?$AAt?$AAa@ 0000000180027338     libucrt:lcidtoname_downlevel.obj
 0002:00007340       ??_C@_15NCHGBGLK@?$AAt?$AAe@ 0000000180027340     libucrt:lcidtoname_downlevel.obj
 0002:00007348       ??_C@_15PHPHCBPF@?$AAk?$AAn@ 0000000180027348     libucrt:lcidtoname_downlevel.obj
 0002:00007350       ??_C@_15DLGBCKMP@?$AAm?$AAr@ 0000000180027350     libucrt:lcidtoname_downlevel.obj
 0002:00007358       ??_C@_15EABBLBFF@?$AAs?$AAa@ 0000000180027358     libucrt:lcidtoname_downlevel.obj
 0002:00007360       ??_C@_15CBKOMCOI@?$AAm?$AAn@ 0000000180027360     libucrt:lcidtoname_downlevel.obj
 0002:00007368       ??_C@_15CKDMCJAF@?$AAg?$AAl@ 0000000180027368     libucrt:lcidtoname_downlevel.obj
 0002:00007370       ??_C@_17CNJFBPG@?$AAk?$AAo?$AAk@ 0000000180027370     libucrt:lcidtoname_downlevel.obj
 0002:00007378       ??_C@_17FFBJICPL@?$AAs?$AAy?$AAr@ 0000000180027378     libucrt:lcidtoname_downlevel.obj
 0002:00007380       ??_C@_17KPNDCPAF@?$AAd?$AAi?$AAv@ 0000000180027380     libucrt:lcidtoname_downlevel.obj
 0002:00007388       ??_C@_11LOCGONAA@@         0000000180027388     libucrt:lcidtoname_downlevel.obj
 0002:00007390       ??_C@_1M@OKAHONE@?$AAa?$AAr?$AA?9?$AAS?$AAA@ 0000000180027390     libucrt:lcidtoname_downlevel.obj
 0002:000073a0       ??_C@_1M@FFFIGIGK@?$AAb?$AAg?$AA?9?$AAB?$AAG@ 00000001800273a0     libucrt:lcidtoname_downlevel.obj
 0002:000073b0       ??_C@_1M@BJNKEDC@?$AAc?$AAa?$AA?9?$AAE?$AAS@ 00000001800273b0     libucrt:lcidtoname_downlevel.obj
 0002:000073c0       ??_C@_1M@IJJHFJHA@?$AAc?$AAs?$AA?9?$AAC?$AAZ@ 00000001800273c0     libucrt:lcidtoname_downlevel.obj
 0002:000073d0       ??_C@_1M@CLPEOBGI@?$AAd?$AAa?$AA?9?$AAD?$AAK@ 00000001800273d0     libucrt:lcidtoname_downlevel.obj
 0002:000073e0       ??_C@_1M@MCMADGCB@?$AAd?$AAe?$AA?9?$AAD?$AAE@ 00000001800273e0     libucrt:lcidtoname_downlevel.obj
 0002:000073f0       ??_C@_1M@OOCKEMAM@?$AAe?$AAl?$AA?9?$AAG?$AAR@ 00000001800273f0     libucrt:lcidtoname_downlevel.obj
 0002:00007400       ??_C@_1M@DDNJFGID@?$AAf?$AAi?$AA?9?$AAF?$AAI@ 0000000180027400     libucrt:lcidtoname_downlevel.obj
 0002:00007410       ??_C@_1M@GLIPPMAC@?$AAf?$AAr?$AA?9?$AAF?$AAR@ 0000000180027410     libucrt:lcidtoname_downlevel.obj
 0002:00007420       ??_C@_1M@GFMCHPE@?$AAh?$AAe?$AA?9?$AAI?$AAL@ 0000000180027420     libucrt:lcidtoname_downlevel.obj
 0002:00007430       ??_C@_1M@MHLPGNKM@?$AAh?$AAu?$AA?9?$AAH?$AAU@ 0000000180027430     libucrt:lcidtoname_downlevel.obj
 0002:00007440       ??_C@_1M@LPDDNNPN@?$AAi?$AAs?$AA?9?$AAI?$AAS@ 0000000180027440     libucrt:lcidtoname_downlevel.obj
 0002:00007450       ??_C@_1M@MADIPODN@?$AAi?$AAt?$AA?9?$AAI?$AAT@ 0000000180027450     libucrt:lcidtoname_downlevel.obj
 0002:00007460       ??_C@_1M@IHBJJGG@?$AAn?$AAl?$AA?9?$AAN?$AAL@ 0000000180027460     libucrt:lcidtoname_downlevel.obj
 0002:00007470       ??_C@_1M@EANAGDL@?$AAn?$AAb?$AA?9?$AAN?$AAO@ 0000000180027470     libucrt:lcidtoname_downlevel.obj
 0002:00007480       ??_C@_1M@NEIEMEGP@?$AAp?$AAl?$AA?9?$AAP?$AAL@ 0000000180027480     libucrt:lcidtoname_downlevel.obj
 0002:00007490       ??_C@_1M@BOCFIGEP@?$AAp?$AAt?$AA?9?$AAB?$AAR@ 0000000180027490     libucrt:lcidtoname_downlevel.obj
 0002:000074a0       ??_C@_1M@IMPFOPBG@?$AAr?$AAo?$AA?9?$AAR?$AAO@ 00000001800274a0     libucrt:lcidtoname_downlevel.obj
 0002:000074b0       ??_C@_1M@IDNNEJMM@?$AAr?$AAu?$AA?9?$AAR?$AAU@ 00000001800274b0     libucrt:lcidtoname_downlevel.obj
 0002:000074c0       ??_C@_1M@LILEEOGM@?$AAh?$AAr?$AA?9?$AAH?$AAR@ 00000001800274c0     libucrt:lcidtoname_downlevel.obj
 0002:000074d0       ??_C@_1M@FKIFEHPB@?$AAs?$AAk?$AA?9?$AAS?$AAK@ 00000001800274d0     libucrt:lcidtoname_downlevel.obj
 0002:000074e0       ??_C@_1M@LJMAMNPJ@?$AAs?$AAq?$AA?9?$AAA?$AAL@ 00000001800274e0     libucrt:lcidtoname_downlevel.obj
 0002:000074f0       ??_C@_1M@GIAKDKJK@?$AAs?$AAv?$AA?9?$AAS?$AAE@ 00000001800274f0     libucrt:lcidtoname_downlevel.obj
 0002:00007500       ??_C@_1M@MKJKIKCL@?$AAt?$AAh?$AA?9?$AAT?$AAH@ 0000000180027500     libucrt:lcidtoname_downlevel.obj
 0002:00007510       ??_C@_1M@MFLCCMPB@?$AAt?$AAr?$AA?9?$AAT?$AAR@ 0000000180027510     libucrt:lcidtoname_downlevel.obj
 0002:00007520       ??_C@_1M@OIJHDKJN@?$AAu?$AAr?$AA?9?$AAP?$AAK@ 0000000180027520     libucrt:lcidtoname_downlevel.obj
 0002:00007530       ??_C@_1M@LHIPCIEK@?$AAi?$AAd?$AA?9?$AAI?$AAD@ 0000000180027530     libucrt:lcidtoname_downlevel.obj
 0002:00007540       ??_C@_1M@MFMOBGI@?$AAu?$AAk?$AA?9?$AAU?$AAA@ 0000000180027540     libucrt:lcidtoname_downlevel.obj
 0002:00007550       ??_C@_1M@OBGLJIPL@?$AAb?$AAe?$AA?9?$AAB?$AAY@ 0000000180027550     libucrt:lcidtoname_downlevel.obj
 0002:00007560       ??_C@_1M@BCFAJEAD@?$AAs?$AAl?$AA?9?$AAS?$AAI@ 0000000180027560     libucrt:lcidtoname_downlevel.obj
 0002:00007570       ??_C@_1M@FKFFEDDN@?$AAe?$AAt?$AA?9?$AAE?$AAE@ 0000000180027570     libucrt:lcidtoname_downlevel.obj
 0002:00007580       ??_C@_1M@KGKKAACI@?$AAl?$AAv?$AA?9?$AAL?$AAV@ 0000000180027580     libucrt:lcidtoname_downlevel.obj
 0002:00007590       ??_C@_1M@IFGBIJO@?$AAl?$AAt?$AA?9?$AAL?$AAT@ 0000000180027590     libucrt:lcidtoname_downlevel.obj
 0002:000075a0       ??_C@_1M@FGEAHEDM@?$AAf?$AAa?$AA?9?$AAI?$AAR@ 00000001800275a0     libucrt:lcidtoname_downlevel.obj
 0002:000075b0       ??_C@_1M@KBMAIBFN@?$AAv?$AAi?$AA?9?$AAV?$AAN@ 00000001800275b0     libucrt:lcidtoname_downlevel.obj
 0002:000075c0       ??_C@_1M@GPCBKDJK@?$AAh?$AAy?$AA?9?$AAA?$AAM@ 00000001800275c0     libucrt:lcidtoname_downlevel.obj
 0002:000075d0       ??_C@_1BG@BECMDDJB@?$AAa?$AAz?$AA?9?$AAA?$AAZ?$AA?9?$AAL?$AAa?$AAt?$AAn@ 00000001800275d0     libucrt:lcidtoname_downlevel.obj
 0002:000075e8       ??_C@_1M@MAOFCAEA@?$AAe?$AAu?$AA?9?$AAE?$AAS@ 00000001800275e8     libucrt:lcidtoname_downlevel.obj
 0002:000075f8       ??_C@_1M@IGHABKPI@?$AAm?$AAk?$AA?9?$AAM?$AAK@ 00000001800275f8     libucrt:lcidtoname_downlevel.obj
 0002:00007608       ??_C@_1M@IAIGNEJG@?$AAt?$AAn?$AA?9?$AAZ?$AAA@ 0000000180027608     libucrt:lcidtoname_downlevel.obj
 0002:00007618       ??_C@_1M@IIJCOJFA@?$AAx?$AAh?$AA?9?$AAZ?$AAA@ 0000000180027618     libucrt:lcidtoname_downlevel.obj
 0002:00007628       ??_C@_1M@LGPJHNJH@?$AAz?$AAu?$AA?9?$AAZ?$AAA@ 0000000180027628     libucrt:lcidtoname_downlevel.obj
 0002:00007638       ??_C@_1M@HOKAOIO@?$AAa?$AAf?$AA?9?$AAZ?$AAA@ 0000000180027638     libucrt:lcidtoname_downlevel.obj
 0002:00007648       ??_C@_1M@DPCLHLIE@?$AAk?$AAa?$AA?9?$AAG?$AAE@ 0000000180027648     libucrt:lcidtoname_downlevel.obj
 0002:00007658       ??_C@_1M@BLKMHJBI@?$AAf?$AAo?$AA?9?$AAF?$AAO@ 0000000180027658     libucrt:lcidtoname_downlevel.obj
 0002:00007668       ??_C@_1M@LGGJAPPB@?$AAh?$AAi?$AA?9?$AAI?$AAN@ 0000000180027668     libucrt:lcidtoname_downlevel.obj
 0002:00007678       ??_C@_1M@FIKPIHFE@?$AAm?$AAt?$AA?9?$AAM?$AAT@ 0000000180027678     libucrt:lcidtoname_downlevel.obj
 0002:00007688       ??_C@_1M@HEGGPBFA@?$AAs?$AAe?$AA?9?$AAN?$AAO@ 0000000180027688     libucrt:lcidtoname_downlevel.obj
 0002:00007698       ??_C@_1M@EIBJEEPA@?$AAm?$AAs?$AA?9?$AAM?$AAY@ 0000000180027698     libucrt:lcidtoname_downlevel.obj
 0002:000076a8       ??_C@_1M@FHLBGMPP@?$AAk?$AAk?$AA?9?$AAK?$AAZ@ 00000001800276a8     libucrt:lcidtoname_downlevel.obj
 0002:000076b8       ??_C@_1M@NGJJLCGI@?$AAk?$AAy?$AA?9?$AAK?$AAG@ 00000001800276b8     libucrt:lcidtoname_downlevel.obj
 0002:000076c8       ??_C@_1M@GIENNBFC@?$AAs?$AAw?$AA?9?$AAK?$AAE@ 00000001800276c8     libucrt:lcidtoname_downlevel.obj
 0002:000076d8       ??_C@_1BG@NDGMJIMJ@?$AAu?$AAz?$AA?9?$AAU?$AAZ?$AA?9?$AAL?$AAa?$AAt?$AAn@ 00000001800276d8     libucrt:lcidtoname_downlevel.obj
 0002:000076f0       ??_C@_1M@IDCCIHBC@?$AAt?$AAt?$AA?9?$AAR?$AAU@ 00000001800276f0     libucrt:lcidtoname_downlevel.obj
 0002:00007700       ??_C@_1M@LOICPMOJ@?$AAb?$AAn?$AA?9?$AAI?$AAN@ 0000000180027700     libucrt:lcidtoname_downlevel.obj
 0002:00007710       ??_C@_1M@KPKKNEAH@?$AAp?$AAa?$AA?9?$AAI?$AAN@ 0000000180027710     libucrt:lcidtoname_downlevel.obj
 0002:00007720       ??_C@_1M@PJGPPBOG@?$AAg?$AAu?$AA?9?$AAI?$AAN@ 0000000180027720     libucrt:lcidtoname_downlevel.obj
 0002:00007730       ??_C@_1M@KMKMOPHI@?$AAt?$AAa?$AA?9?$AAI?$AAN@ 0000000180027730     libucrt:lcidtoname_downlevel.obj
 0002:00007740       ??_C@_1M@KFEHEPAC@?$AAt?$AAe?$AA?9?$AAI?$AAN@ 0000000180027740     libucrt:lcidtoname_downlevel.obj
 0002:00007750       ??_C@_1M@CDCLMGHI@?$AAk?$AAn?$AA?9?$AAI?$AAN@ 0000000180027750     libucrt:lcidtoname_downlevel.obj
 0002:00007760       ??_C@_1M@MIODLDKF@?$AAm?$AAl?$AA?9?$AAI?$AAN@ 0000000180027760     libucrt:lcidtoname_downlevel.obj
 0002:00007770       ??_C@_1M@PBIEACPO@?$AAm?$AAr?$AA?9?$AAI?$AAN@ 0000000180027770     libucrt:lcidtoname_downlevel.obj
 0002:00007780       ??_C@_1M@NIDEAGPH@?$AAs?$AAa?$AA?9?$AAI?$AAN@ 0000000180027780     libucrt:lcidtoname_downlevel.obj
 0002:00007790       ??_C@_1M@FHIHCBIO@?$AAm?$AAn?$AA?9?$AAM?$AAN@ 0000000180027790     libucrt:lcidtoname_downlevel.obj
 0002:000077a0       ??_C@_1M@JAIJPENP@?$AAc?$AAy?$AA?9?$AAG?$AAB@ 00000001800277a0     libucrt:lcidtoname_downlevel.obj
 0002:000077b0       ??_C@_1M@PHGFBEPN@?$AAg?$AAl?$AA?9?$AAE?$AAS@ 00000001800277b0     libucrt:lcidtoname_downlevel.obj
 0002:000077c0       ??_C@_1O@KPIPDNCP@?$AAk?$AAo?$AAk?$AA?9?$AAI?$AAN@ 00000001800277c0     libucrt:lcidtoname_downlevel.obj
 0002:000077d0       ??_C@_1O@KNHJLDJA@?$AAs?$AAy?$AAr?$AA?9?$AAS?$AAY@ 00000001800277d0     libucrt:lcidtoname_downlevel.obj
 0002:000077e0       ??_C@_1O@MKEKBLAH@?$AAd?$AAi?$AAv?$AA?9?$AAM?$AAV@ 00000001800277e0     libucrt:lcidtoname_downlevel.obj
 0002:000077f0       ??_C@_1O@OHDCKDDF@?$AAq?$AAu?$AAz?$AA?9?$AAB?$AAO@ 00000001800277f0     libucrt:lcidtoname_downlevel.obj
 0002:00007800       ??_C@_1M@LEPJNLFD@?$AAn?$AAs?$AA?9?$AAZ?$AAA@ 0000000180027800     libucrt:lcidtoname_downlevel.obj
 0002:00007810       ??_C@_1M@OMLEIIJB@?$AAm?$AAi?$AA?9?$AAN?$AAZ@ 0000000180027810     libucrt:lcidtoname_downlevel.obj
 0002:00007820       ??_C@_1M@PMPEAILG@?$AAa?$AAr?$AA?9?$AAI?$AAQ@ 0000000180027820     libucrt:lcidtoname_downlevel.obj
 0002:00007830       ??_C@_1M@CNKPNOEE@?$AAd?$AAe?$AA?9?$AAC?$AAH@ 0000000180027830     libucrt:lcidtoname_downlevel.obj
 0002:00007840       ??_C@_1M@LKMGMLKO@?$AAe?$AAn?$AA?9?$AAG?$AAB@ 0000000180027840     libucrt:lcidtoname_downlevel.obj
 0002:00007850       ??_C@_1M@PGKJFFGL@?$AAe?$AAs?$AA?9?$AAM?$AAX@ 0000000180027850     libucrt:lcidtoname_downlevel.obj
 0002:00007860       ??_C@_1M@DNNANBDC@?$AAf?$AAr?$AA?9?$AAB?$AAE@ 0000000180027860     libucrt:lcidtoname_downlevel.obj
 0002:00007870       ??_C@_1M@HLGMDFHM@?$AAi?$AAt?$AA?9?$AAC?$AAH@ 0000000180027870     libucrt:lcidtoname_downlevel.obj
 0002:00007880       ??_C@_1M@CLLBGJH@?$AAn?$AAl?$AA?9?$AAB?$AAE@ 0000000180027880     libucrt:lcidtoname_downlevel.obj
 0002:00007890       ??_C@_1M@BODBOGLF@?$AAn?$AAn?$AA?9?$AAN?$AAO@ 0000000180027890     libucrt:lcidtoname_downlevel.obj
 0002:000078a0       ??_C@_1M@HFFAHKAD@?$AAp?$AAt?$AA?9?$AAP?$AAT@ 00000001800278a0     libucrt:lcidtoname_downlevel.obj
 0002:000078b0       ??_C@_1BG@LNOAKHIE@?$AAs?$AAr?$AA?9?$AAS?$AAP?$AA?9?$AAL?$AAa?$AAt?$AAn@ 00000001800278b0     libucrt:lcidtoname_downlevel.obj
 0002:000078c8       ??_C@_1M@HBMHBGAK@?$AAs?$AAv?$AA?9?$AAF?$AAI@ 00000001800278c8     libucrt:lcidtoname_downlevel.obj
 0002:000078d8       ??_C@_1BG@DGCJGJBE@?$AAa?$AAz?$AA?9?$AAA?$AAZ?$AA?9?$AAC?$AAy?$AAr?$AAl@ 00000001800278d8     libucrt:lcidtoname_downlevel.obj
 0002:000078f0       ??_C@_1M@KEJDAAHB@?$AAs?$AAe?$AA?9?$AAS?$AAE@ 00000001800278f0     libucrt:lcidtoname_downlevel.obj
 0002:00007900       ??_C@_1M@HEIBJJAD@?$AAm?$AAs?$AA?9?$AAB?$AAN@ 0000000180027900     libucrt:lcidtoname_downlevel.obj
 0002:00007910       ??_C@_1BG@PBGJMCEM@?$AAu?$AAz?$AA?9?$AAU?$AAZ?$AA?9?$AAC?$AAy?$AAr?$AAl@ 0000000180027910     libucrt:lcidtoname_downlevel.obj
 0002:00007928       ??_C@_1O@LAOBCMDF@?$AAq?$AAu?$AAz?$AA?9?$AAE?$AAC@ 0000000180027928     libucrt:lcidtoname_downlevel.obj
 0002:00007938       ??_C@_1M@POEEMAIO@?$AAa?$AAr?$AA?9?$AAE?$AAG@ 0000000180027938     libucrt:lcidtoname_downlevel.obj
 0002:00007948       ??_C@_1M@EFAKDEDL@?$AAz?$AAh?$AA?9?$AAH?$AAK@ 0000000180027948     libucrt:lcidtoname_downlevel.obj
 0002:00007958       ??_C@_1M@HKKIJHGI@?$AAd?$AAe?$AA?9?$AAA?$AAT@ 0000000180027958     libucrt:lcidtoname_downlevel.obj
 0002:00007968       ??_C@_1M@KBFBEHJF@?$AAe?$AAn?$AA?9?$AAA?$AAU@ 0000000180027968     libucrt:lcidtoname_downlevel.obj
 0002:00007978       ??_C@_1M@MNPLFAAH@?$AAe?$AAs?$AA?9?$AAE?$AAS@ 0000000180027978     libucrt:lcidtoname_downlevel.obj
 0002:00007988       ??_C@_1M@HJOOJFMA@?$AAf?$AAr?$AA?9?$AAC?$AAA@ 0000000180027988     libucrt:lcidtoname_downlevel.obj
 0002:00007998       ??_C@_1BG@JPOFPNAB@?$AAs?$AAr?$AA?9?$AAS?$AAP?$AA?9?$AAC?$AAy?$AAr?$AAl@ 0000000180027998     libucrt:lcidtoname_downlevel.obj
 0002:000079b0       ??_C@_1M@LNFOCMOB@?$AAs?$AAe?$AA?9?$AAF?$AAI@ 00000001800279b0     libucrt:lcidtoname_downlevel.obj
 0002:000079c0       ??_C@_1O@MGJBOAMB@?$AAq?$AAu?$AAz?$AA?9?$AAP?$AAE@ 00000001800279c0     libucrt:lcidtoname_downlevel.obj
 0002:000079d0       ??_C@_1M@GJINLBOK@?$AAa?$AAr?$AA?9?$AAL?$AAY@ 00000001800279d0     libucrt:lcidtoname_downlevel.obj
 0002:000079e0       ??_C@_1M@GGMNHJNL@?$AAz?$AAh?$AA?9?$AAS?$AAG@ 00000001800279e0     libucrt:lcidtoname_downlevel.obj
 0002:000079f0       ??_C@_1M@HOIKODND@?$AAd?$AAe?$AA?9?$AAL?$AAU@ 00000001800279f0     libucrt:lcidtoname_downlevel.obj
 0002:00007a00       ??_C@_1M@DDOCCGFG@?$AAe?$AAn?$AA?9?$AAC?$AAA@ 0000000180027a00     libucrt:lcidtoname_downlevel.obj
 0002:00007a10       ??_C@_1M@BNOEMJLF@?$AAe?$AAs?$AA?9?$AAG?$AAT@ 0000000180027a10     libucrt:lcidtoname_downlevel.obj
 0002:00007a20       ??_C@_1M@EOGNKEK@?$AAf?$AAr?$AA?9?$AAC?$AAH@ 0000000180027a20     libucrt:lcidtoname_downlevel.obj
 0002:00007a30       ??_C@_1M@FLIDJFHL@?$AAh?$AAr?$AA?9?$AAB?$AAA@ 0000000180027a30     libucrt:lcidtoname_downlevel.obj
 0002:00007a40       ??_C@_1O@FMCELNAJ@?$AAs?$AAm?$AAj?$AA?9?$AAN?$AAO@ 0000000180027a40     libucrt:lcidtoname_downlevel.obj
 0002:00007a50       ??_C@_1M@JHGLJMGJ@?$AAa?$AAr?$AA?9?$AAD?$AAZ@ 0000000180027a50     libucrt:lcidtoname_downlevel.obj
 0002:00007a60       ??_C@_1M@JKKFDCNP@?$AAz?$AAh?$AA?9?$AAM?$AAO@ 0000000180027a60     libucrt:lcidtoname_downlevel.obj
 0002:00007a70       ??_C@_1M@GEEFALPE@?$AAd?$AAe?$AA?9?$AAL?$AAI@ 0000000180027a70     libucrt:lcidtoname_downlevel.obj
 0002:00007a80       ??_C@_1M@IGEOFBG@?$AAe?$AAn?$AA?9?$AAN?$AAZ@ 0000000180027a80     libucrt:lcidtoname_downlevel.obj
 0002:00007a90       ??_C@_1M@KDBONEHP@?$AAe?$AAs?$AA?9?$AAC?$AAR@ 0000000180027a90     libucrt:lcidtoname_downlevel.obj
 0002:00007aa0       ??_C@_1M@FHMDOHNN@?$AAf?$AAr?$AA?9?$AAL?$AAU@ 0000000180027aa0     libucrt:lcidtoname_downlevel.obj
 0002:00007ab0       ??_C@_1BG@NFKKMAFG@?$AAb?$AAs?$AA?9?$AAB?$AAA?$AA?9?$AAL?$AAa?$AAt?$AAn@ 0000000180027ab0     libucrt:lcidtoname_downlevel.obj
 0002:00007ac8       ??_C@_1O@IMNBEMCI@?$AAs?$AAm?$AAj?$AA?9?$AAS?$AAE@ 0000000180027ac8     libucrt:lcidtoname_downlevel.obj
 0002:00007ad8       ??_C@_1M@DHHMBNDP@?$AAa?$AAr?$AA?9?$AAM?$AAA@ 0000000180027ad8     libucrt:lcidtoname_downlevel.obj
 0002:00007ae8       ??_C@_1M@BNBLJCGH@?$AAe?$AAn?$AA?9?$AAI?$AAE@ 0000000180027ae8     libucrt:lcidtoname_downlevel.obj
 0002:00007af8       ??_C@_1M@GEPAFMDL@?$AAe?$AAs?$AA?9?$AAP?$AAA@ 0000000180027af8     libucrt:lcidtoname_downlevel.obj
 0002:00007b08       ??_C@_1M@OJONDMDL@?$AAf?$AAr?$AA?9?$AAM?$AAC@ 0000000180027b08     libucrt:lcidtoname_downlevel.obj
 0002:00007b18       ??_C@_1BG@OBCNFJB@?$AAs?$AAr?$AA?9?$AAB?$AAA?$AA?9?$AAL?$AAa?$AAt?$AAn@ 0000000180027b18     libucrt:lcidtoname_downlevel.obj
 0002:00007b30       ??_C@_1O@KEMEEGPO@?$AAs?$AAm?$AAa?$AA?9?$AAN?$AAO@ 0000000180027b30     libucrt:lcidtoname_downlevel.obj
 0002:00007b40       ??_C@_1M@ELMGFODK@?$AAa?$AAr?$AA?9?$AAT?$AAN@ 0000000180027b40     libucrt:lcidtoname_downlevel.obj
 0002:00007b50       ??_C@_1M@BHDLHFAF@?$AAe?$AAn?$AA?9?$AAZ?$AAA@ 0000000180027b50     libucrt:lcidtoname_downlevel.obj
 0002:00007b60       ??_C@_1M@BMGIGLIF@?$AAe?$AAs?$AA?9?$AAD?$AAO@ 0000000180027b60     libucrt:lcidtoname_downlevel.obj
 0002:00007b70       ??_C@_1BG@CMBHIPBE@?$AAs?$AAr?$AA?9?$AAB?$AAA?$AA?9?$AAC?$AAy?$AAr?$AAl@ 0000000180027b70     libucrt:lcidtoname_downlevel.obj
 0002:00007b88       ??_C@_1O@HEDBLHNP@?$AAs?$AAm?$AAa?$AA?9?$AAS?$AAE@ 0000000180027b88     libucrt:lcidtoname_downlevel.obj
 0002:00007b98       ??_C@_1M@DAGCADIM@?$AAa?$AAr?$AA?9?$AAO?$AAM@ 0000000180027b98     libucrt:lcidtoname_downlevel.obj
 0002:00007ba8       ??_C@_1M@FODLMICG@?$AAe?$AAn?$AA?9?$AAJ?$AAM@ 0000000180027ba8     libucrt:lcidtoname_downlevel.obj
 0002:00007bb8       ??_C@_1M@DNMLCIHB@?$AAe?$AAs?$AA?9?$AAV?$AAE@ 0000000180027bb8     libucrt:lcidtoname_downlevel.obj
 0002:00007bc8       ??_C@_1O@EOKHMKJK@?$AAs?$AAm?$AAs?$AA?9?$AAF?$AAI@ 0000000180027bc8     libucrt:lcidtoname_downlevel.obj
 0002:00007bd8       ??_C@_1M@CAFJMKOF@?$AAa?$AAr?$AA?9?$AAY?$AAE@ 0000000180027bd8     libucrt:lcidtoname_downlevel.obj
 0002:00007be8       ??_C@_1M@CBFHIJLI@?$AAe?$AAn?$AA?9?$AAC?$AAB@ 0000000180027be8     libucrt:lcidtoname_downlevel.obj
 0002:00007bf8       ??_C@_1M@BGNFLDN@?$AAe?$AAs?$AA?9?$AAC?$AAO@ 0000000180027bf8     libucrt:lcidtoname_downlevel.obj
 0002:00007c08       ??_C@_1O@JMPHMAMC@?$AAs?$AAm?$AAn?$AA?9?$AAF?$AAI@ 0000000180027c08     libucrt:lcidtoname_downlevel.obj
 0002:00007c18       ??_C@_1M@JLANABKE@?$AAa?$AAr?$AA?9?$AAS?$AAY@ 0000000180027c18     libucrt:lcidtoname_downlevel.obj
 0002:00007c28       ??_C@_1M@HPKGCFGN@?$AAe?$AAn?$AA?9?$AAB?$AAZ@ 0000000180027c28     libucrt:lcidtoname_downlevel.obj
 0002:00007c38       ??_C@_1M@OLJCMLGM@?$AAe?$AAs?$AA?9?$AAP?$AAE@ 0000000180027c38     libucrt:lcidtoname_downlevel.obj
 0002:00007c48       ??_C@_1M@MKKGFKLE@?$AAa?$AAr?$AA?9?$AAJ?$AAO@ 0000000180027c48     libucrt:lcidtoname_downlevel.obj
 0002:00007c58       ??_C@_1M@EKPGLDNI@?$AAe?$AAn?$AA?9?$AAT?$AAT@ 0000000180027c58     libucrt:lcidtoname_downlevel.obj
 0002:00007c68       ??_C@_1M@OONGHFHE@?$AAe?$AAs?$AA?9?$AAA?$AAR@ 0000000180027c68     libucrt:lcidtoname_downlevel.obj
 0002:00007c78       ??_C@_1M@OOJFGBHE@?$AAa?$AAr?$AA?9?$AAL?$AAB@ 0000000180027c78     libucrt:lcidtoname_downlevel.obj
 0002:00007c88       ??_C@_1M@GCEJHNEG@?$AAe?$AAn?$AA?9?$AAZ?$AAW@ 0000000180027c88     libucrt:lcidtoname_downlevel.obj
 0002:00007c98       ??_C@_1M@JNOCAHJI@?$AAe?$AAs?$AA?9?$AAE?$AAC@ 0000000180027c98     libucrt:lcidtoname_downlevel.obj
 0002:00007ca8       ??_C@_1M@JEFHPGGB@?$AAa?$AAr?$AA?9?$AAK?$AAW@ 0000000180027ca8     libucrt:lcidtoname_downlevel.obj
 0002:00007cb8       ??_C@_1M@MLKIBJOJ@?$AAe?$AAn?$AA?9?$AAP?$AAH@ 0000000180027cb8     libucrt:lcidtoname_downlevel.obj
 0002:00007cc8       ??_C@_1M@BDNIPEND@?$AAe?$AAs?$AA?9?$AAC?$AAL@ 0000000180027cc8     libucrt:lcidtoname_downlevel.obj
 0002:00007cd8       ??_C@_1M@MPNMEKBD@?$AAa?$AAr?$AA?9?$AAA?$AAE@ 0000000180027cd8     libucrt:lcidtoname_downlevel.obj
 0002:00007ce8       ??_C@_1M@KBJALCPI@?$AAe?$AAs?$AA?9?$AAU?$AAY@ 0000000180027ce8     libucrt:lcidtoname_downlevel.obj
 0002:00007cf8       ??_C@_1M@LLCCOAGA@?$AAa?$AAr?$AA?9?$AAB?$AAH@ 0000000180027cf8     libucrt:lcidtoname_downlevel.obj
 0002:00007d08       ??_C@_1M@PBFNCDEL@?$AAe?$AAs?$AA?9?$AAP?$AAY@ 0000000180027d08     libucrt:lcidtoname_downlevel.obj
 0002:00007d18       ??_C@_1M@EDGINPNP@?$AAa?$AAr?$AA?9?$AAQ?$AAA@ 0000000180027d18     libucrt:lcidtoname_downlevel.obj
 0002:00007d28       ??_C@_1M@MKDBIIJI@?$AAe?$AAs?$AA?9?$AAB?$AAO@ 0000000180027d28     libucrt:lcidtoname_downlevel.obj
 0002:00007d38       ??_C@_1M@CPKKEBLD@?$AAe?$AAs?$AA?9?$AAS?$AAV@ 0000000180027d38     libucrt:lcidtoname_downlevel.obj
 0002:00007d48       ??_C@_1M@NDBGMMJL@?$AAe?$AAs?$AA?9?$AAH?$AAN@ 0000000180027d48     libucrt:lcidtoname_downlevel.obj
 0002:00007d58       ??_C@_1M@JIJIBHDP@?$AAe?$AAs?$AA?9?$AAN?$AAI@ 0000000180027d58     libucrt:lcidtoname_downlevel.obj
 0002:00007d68       ??_C@_1M@CGFMKEEK@?$AAe?$AAs?$AA?9?$AAP?$AAR@ 0000000180027d68     libucrt:lcidtoname_downlevel.obj
 0002:00007d78       ??_C@_1O@ICJHKIIK@?$AAz?$AAh?$AA?9?$AAC?$AAH?$AAT@ 0000000180027d78     libucrt:lcidtoname_downlevel.obj
 0002:00007d88       ??_C@_15CLNEJCE@?$AAs?$AAr@ 0000000180027d88     libucrt:lcidtoname_downlevel.obj
 0002:00008bd0       ??_C@_1M@KAHEKEIG@?$AAa?$AAf?$AA?9?$AAz?$AAa@ 0000000180028bd0     libucrt:lcidtoname_downlevel.obj
 0002:00008be0       ??_C@_1M@GIECOABL@?$AAa?$AAr?$AA?9?$AAa?$AAe@ 0000000180028be0     libucrt:lcidtoname_downlevel.obj
 0002:00008bf0       ??_C@_1M@BMLMEKGI@?$AAa?$AAr?$AA?9?$AAb?$AAh@ 0000000180028bf0     libucrt:lcidtoname_downlevel.obj
 0002:00008c00       ??_C@_1M@DAPFDGGB@?$AAa?$AAr?$AA?9?$AAd?$AAz@ 0000000180028c00     libucrt:lcidtoname_downlevel.obj
 0002:00008c10       ??_C@_1M@FJNKGKIG@?$AAa?$AAr?$AA?9?$AAe?$AAg@ 0000000180028c10     libucrt:lcidtoname_downlevel.obj
 0002:00008c20       ??_C@_1M@FLGKKCLO@?$AAa?$AAr?$AA?9?$AAi?$AAq@ 0000000180028c20     libucrt:lcidtoname_downlevel.obj
 0002:00008c30       ??_C@_1M@GNDIPALM@?$AAa?$AAr?$AA?9?$AAj?$AAo@ 0000000180028c30     libucrt:lcidtoname_downlevel.obj
 0002:00008c40       ??_C@_1M@DDMJFMGJ@?$AAa?$AAr?$AA?9?$AAk?$AAw@ 0000000180028c40     libucrt:lcidtoname_downlevel.obj
 0002:00008c50       ??_C@_1M@EJALMLHM@?$AAa?$AAr?$AA?9?$AAl?$AAb@ 0000000180028c50     libucrt:lcidtoname_downlevel.obj
 0002:00008c60       ??_C@_1M@MOBDBLOC@?$AAa?$AAr?$AA?9?$AAl?$AAy@ 0000000180028c60     libucrt:lcidtoname_downlevel.obj
 0002:00008c70       ??_C@_1M@JAOCLHDH@?$AAa?$AAr?$AA?9?$AAm?$AAa@ 0000000180028c70     libucrt:lcidtoname_downlevel.obj
 0002:00008c80       ??_C@_1M@JHPMKJIE@?$AAa?$AAr?$AA?9?$AAo?$AAm@ 0000000180028c80     libucrt:lcidtoname_downlevel.obj
 0002:00008c90       ??_C@_1M@OEPGHFNH@?$AAa?$AAr?$AA?9?$AAq?$AAa@ 0000000180028c90     libucrt:lcidtoname_downlevel.obj
 0002:00008ca0       ??_C@_1M@KJDONENM@?$AAa?$AAr?$AA?9?$AAs?$AAa@ 0000000180028ca0     libucrt:lcidtoname_downlevel.obj
 0002:00008cb0       ??_C@_1M@DMJDKLKM@?$AAa?$AAr?$AA?9?$AAs?$AAy@ 0000000180028cb0     libucrt:lcidtoname_downlevel.obj
 0002:00008cc0       ??_C@_1M@OMFIPEDC@?$AAa?$AAr?$AA?9?$AAt?$AAn@ 0000000180028cc0     libucrt:lcidtoname_downlevel.obj
 0002:00008cd0       ??_C@_1M@IHMHGAON@?$AAa?$AAr?$AA?9?$AAy?$AAe@ 0000000180028cd0     libucrt:lcidtoname_downlevel.obj
 0002:00008ce0       ??_C@_1BG@KDCPGJGB@?$AAa?$AAz?$AA?9?$AAa?$AAz?$AA?9?$AAc?$AAy?$AAr?$AAl@ 0000000180028ce0     libucrt:lcidtoname_downlevel.obj
 0002:00008cf8       ??_C@_1BG@IBCKDDOE@?$AAa?$AAz?$AA?9?$AAa?$AAz?$AA?9?$AAl?$AAa?$AAt?$AAn@ 0000000180028cf8     libucrt:lcidtoname_downlevel.obj
 0002:00008d10       ??_C@_1M@EGPFDCPD@?$AAb?$AAe?$AA?9?$AAb?$AAy@ 0000000180028d10     libucrt:lcidtoname_downlevel.obj
 0002:00008d20       ??_C@_1M@PCMGMCGC@?$AAb?$AAg?$AA?9?$AAb?$AAg@ 0000000180028d20     libucrt:lcidtoname_downlevel.obj
 0002:00008d30       ??_C@_1M@BJBMFGOB@?$AAb?$AAn?$AA?9?$AAi?$AAn@ 0000000180028d30     libucrt:lcidtoname_downlevel.obj
 0002:00008d40       ??_C@_1BG@EAKMMACD@?$AAb?$AAs?$AA?9?$AAb?$AAa?$AA?9?$AAl?$AAa?$AAt?$AAn@ 0000000180028d40     libucrt:lcidtoname_downlevel.obj
 0002:00008d58       ??_C@_1M@KGADAODK@?$AAc?$AAa?$AA?9?$AAe?$AAs@ 0000000180028d58     libucrt:lcidtoname_downlevel.obj
 0002:00008d68       ??_C@_1M@COAJPDHI@?$AAc?$AAs?$AA?9?$AAc?$AAz@ 0000000180028d68     libucrt:lcidtoname_downlevel.obj
 0002:00008d78       ??_C@_1M@DHBHFONH@?$AAc?$AAy?$AA?9?$AAg?$AAb@ 0000000180028d78     libucrt:lcidtoname_downlevel.obj
 0002:00008d88       ??_C@_1M@IMGKELGA@?$AAd?$AAa?$AA?9?$AAd?$AAk@ 0000000180028d88     libucrt:lcidtoname_downlevel.obj
 0002:00008d98       ??_C@_1M@NNDGDNGA@?$AAd?$AAe?$AA?9?$AAa?$AAt@ 0000000180028d98     libucrt:lcidtoname_downlevel.obj
 0002:00008da8       ??_C@_1M@IKDBHEEM@?$AAd?$AAe?$AA?9?$AAc?$AAh@ 0000000180028da8     libucrt:lcidtoname_downlevel.obj
 0002:00008db8       ??_C@_1M@GFFOJMCJ@?$AAd?$AAe?$AA?9?$AAd?$AAe@ 0000000180028db8     libucrt:lcidtoname_downlevel.obj
 0002:00008dc8       ??_C@_1M@MDNLKBPM@?$AAd?$AAe?$AA?9?$AAl?$AAi@ 0000000180028dc8     libucrt:lcidtoname_downlevel.obj
 0002:00008dd8       ??_C@_1M@NJBEEJNL@?$AAd?$AAe?$AA?9?$AAl?$AAu@ 0000000180028dd8     libucrt:lcidtoname_downlevel.obj
 0002:00008de8       ??_C@_1O@GNNELBAP@?$AAd?$AAi?$AAv?$AA?9?$AAm?$AAv@ 0000000180028de8     libucrt:lcidtoname_downlevel.obj
 0002:00008df8       ??_C@_1M@EJLEOGAE@?$AAe?$AAl?$AA?9?$AAg?$AAr@ 0000000180028df8     libucrt:lcidtoname_downlevel.obj
 0002:00008e08       ??_C@_1M@GMPONJN@?$AAe?$AAn?$AA?9?$AAa?$AAu@ 0000000180028e08     libucrt:lcidtoname_downlevel.obj
 0002:00008e18       ??_C@_1M@NIDIIPGF@?$AAe?$AAn?$AA?9?$AAb?$AAz@ 0000000180028e18     libucrt:lcidtoname_downlevel.obj
 0002:00008e28       ??_C@_1M@JEHMIMFO@?$AAe?$AAn?$AA?9?$AAc?$AAa@ 0000000180028e28     libucrt:lcidtoname_downlevel.obj
 0002:00008e38       ??_C@_1M@IGMJCDLA@?$AAe?$AAn?$AA?9?$AAc?$AAb@ 0000000180028e38     libucrt:lcidtoname_downlevel.obj
 0002:00008e48       ??_C@_1M@BNFIGBKG@?$AAe?$AAn?$AA?9?$AAg?$AAb@ 0000000180028e48     libucrt:lcidtoname_downlevel.obj
 0002:00008e58       ??_C@_1M@LKIFDIGP@?$AAe?$AAn?$AA?9?$AAi?$AAe@ 0000000180028e58     libucrt:lcidtoname_downlevel.obj
 0002:00008e68       ??_C@_1M@PJKFGCCO@?$AAe?$AAn?$AA?9?$AAj?$AAm@ 0000000180028e68     libucrt:lcidtoname_downlevel.obj
 0002:00008e78       ??_C@_1M@KPPKEPBO@?$AAe?$AAn?$AA?9?$AAn?$AAz@ 0000000180028e78     libucrt:lcidtoname_downlevel.obj
 0002:00008e88       ??_C@_1M@GMDGLDOB@?$AAe?$AAn?$AA?9?$AAp?$AAh@ 0000000180028e88     libucrt:lcidtoname_downlevel.obj
 0002:00008e98       ??_C@_1M@ONGIBJNA@?$AAe?$AAn?$AA?9?$AAt?$AAt@ 0000000180028e98     libucrt:lcidtoname_downlevel.obj
 0002:00008ea8       ??_C@_1M@LLODPCMM@?$AAe?$AAn?$AA?9?$AAu?$AAs@ 0000000180028ea8     libucrt:lcidtoname_downlevel.obj
 0002:00008eb8       ??_C@_1M@LAKFNPAN@?$AAe?$AAn?$AA?9?$AAz?$AAa@ 0000000180028eb8     libucrt:lcidtoname_downlevel.obj
 0002:00008ec8       ??_C@_1M@MFNHNHEO@?$AAe?$AAn?$AA?9?$AAz?$AAw@ 0000000180028ec8     libucrt:lcidtoname_downlevel.obj
 0002:00008ed8       ??_C@_1M@EJEINPHM@?$AAe?$AAs?$AA?9?$AAa?$AAr@ 0000000180028ed8     libucrt:lcidtoname_downlevel.obj
 0002:00008ee8       ??_C@_1M@GNKPCCJA@?$AAe?$AAs?$AA?9?$AAb?$AAo@ 0000000180028ee8     libucrt:lcidtoname_downlevel.obj
 0002:00008ef8       ??_C@_1M@LEEGFONL@?$AAe?$AAs?$AA?9?$AAc?$AAl@ 0000000180028ef8     libucrt:lcidtoname_downlevel.obj
 0002:00008f08       ??_C@_1M@KGPDPBDF@?$AAe?$AAs?$AA?9?$AAc?$AAo@ 0000000180028f08     libucrt:lcidtoname_downlevel.obj
 0002:00008f18       ??_C@_1M@EIAHOHH@?$AAe?$AAs?$AA?9?$AAc?$AAr@ 0000000180028f18     libucrt:lcidtoname_downlevel.obj
 0002:00008f28       ??_C@_1M@LLPGMBIN@?$AAe?$AAs?$AA?9?$AAd?$AAo@ 0000000180028f28     libucrt:lcidtoname_downlevel.obj
 0002:00008f38       ??_C@_1M@DKHMKNJA@?$AAe?$AAs?$AA?9?$AAe?$AAc@ 0000000180028f38     libucrt:lcidtoname_downlevel.obj
 0002:00008f48       ??_C@_1M@GKGFPKAP@?$AAe?$AAs?$AA?9?$AAe?$AAs@ 0000000180028f48     libucrt:lcidtoname_downlevel.obj
 0002:00008f58       ??_C@_1M@LKHKGDLN@?$AAe?$AAs?$AA?9?$AAg?$AAt@ 0000000180028f58     libucrt:lcidtoname_downlevel.obj
 0002:00008f68       ??_C@_1M@HEIIGGJD@?$AAe?$AAs?$AA?9?$AAh?$AAn@ 0000000180028f68     libucrt:lcidtoname_downlevel.obj
 0002:00008f78       ??_C@_1M@FBDHPPGD@?$AAe?$AAs?$AA?9?$AAm?$AAx@ 0000000180028f78     libucrt:lcidtoname_downlevel.obj
 0002:00008f88       ??_C@_1M@DPAGLNDH@?$AAe?$AAs?$AA?9?$AAn?$AAi@ 0000000180028f88     libucrt:lcidtoname_downlevel.obj
 0002:00008f98       ??_C@_1M@MDGOPGDD@?$AAe?$AAs?$AA?9?$AAp?$AAa@ 0000000180028f98     libucrt:lcidtoname_downlevel.obj
 0002:00008fa8       ??_C@_1M@EMAMGBGE@?$AAe?$AAs?$AA?9?$AAp?$AAe@ 0000000180028fa8     libucrt:lcidtoname_downlevel.obj
 0002:00008fb8       ??_C@_1M@IBMCAOEC@?$AAe?$AAs?$AA?9?$AAp?$AAr@ 0000000180028fb8     libucrt:lcidtoname_downlevel.obj
 0002:00008fc8       ??_C@_1M@FGMDIJED@?$AAe?$AAs?$AA?9?$AAp?$AAy@ 0000000180028fc8     libucrt:lcidtoname_downlevel.obj
 0002:00008fd8       ??_C@_1M@IIDEOLLL@?$AAe?$AAs?$AA?9?$AAs?$AAv@ 0000000180028fd8     libucrt:lcidtoname_downlevel.obj
 0002:00008fe8       ??_C@_1M@GAOBIPA@?$AAe?$AAs?$AA?9?$AAu?$AAy@ 0000000180028fe8     libucrt:lcidtoname_downlevel.obj
 0002:00008ff8       ??_C@_1M@JKFFICHJ@?$AAe?$AAs?$AA?9?$AAv?$AAe@ 0000000180028ff8     libucrt:lcidtoname_downlevel.obj
 0002:00009008       ??_C@_1M@PNMLOJDF@?$AAe?$AAt?$AA?9?$AAe?$AAe@ 0000000180029008     libucrt:lcidtoname_downlevel.obj
 0002:00009018       ??_C@_1M@GHHLIKEI@?$AAe?$AAu?$AA?9?$AAe?$AAs@ 0000000180029018     libucrt:lcidtoname_downlevel.obj
 0002:00009028       ??_C@_1M@PBNONODE@?$AAf?$AAa?$AA?9?$AAi?$AAr@ 0000000180029028     libucrt:lcidtoname_downlevel.obj
 0002:00009038       ??_C@_1M@JEEHPMIL@?$AAf?$AAi?$AA?9?$AAf?$AAi@ 0000000180029038     libucrt:lcidtoname_downlevel.obj
 0002:00009048       ??_C@_1M@LMDCNDBA@?$AAf?$AAo?$AA?9?$AAf?$AAo@ 0000000180029048     libucrt:lcidtoname_downlevel.obj
 0002:00009058       ??_C@_1M@JKEOHLDK@?$AAf?$AAr?$AA?9?$AAb?$AAe@ 0000000180029058     libucrt:lcidtoname_downlevel.obj
 0002:00009068       ??_C@_1M@NOHADPMI@?$AAf?$AAr?$AA?9?$AAc?$AAa@ 0000000180029068     libucrt:lcidtoname_downlevel.obj
 0002:00009078       ??_C@_1M@KDHIHAEC@?$AAf?$AAr?$AA?9?$AAc?$AAh@ 0000000180029078     libucrt:lcidtoname_downlevel.obj
 0002:00009088       ??_C@_1M@MMBBFGAK@?$AAf?$AAr?$AA?9?$AAf?$AAr@ 0000000180029088     libucrt:lcidtoname_downlevel.obj
 0002:00009098       ??_C@_1M@PAFNENNF@?$AAf?$AAr?$AA?9?$AAl?$AAu@ 0000000180029098     libucrt:lcidtoname_downlevel.obj
 0002:000090a8       ??_C@_1M@EOHDJGDD@?$AAf?$AAr?$AA?9?$AAm?$AAc@ 00000001800290a8     libucrt:lcidtoname_downlevel.obj
 0002:000090b8       ??_C@_1M@FAPLLOPF@?$AAg?$AAl?$AA?9?$AAe?$AAs@ 00000001800290b8     libucrt:lcidtoname_downlevel.obj
 0002:000090c8       ??_C@_1M@FOPBFLOO@?$AAg?$AAu?$AA?9?$AAi?$AAn@ 00000001800290c8     libucrt:lcidtoname_downlevel.obj
 0002:000090d8       ??_C@_1M@KBMCINPM@?$AAh?$AAe?$AA?9?$AAi?$AAl@ 00000001800290d8     libucrt:lcidtoname_downlevel.obj
 0002:000090e8       ??_C@_1M@BBPHKFPJ@?$AAh?$AAi?$AA?9?$AAi?$AAn@ 00000001800290e8     libucrt:lcidtoname_downlevel.obj
 0002:000090f8       ??_C@_1M@PMBNDPHD@?$AAh?$AAr?$AA?9?$AAb?$AAa@ 00000001800290f8     libucrt:lcidtoname_downlevel.obj
 0002:00009108       ??_C@_1M@BPCKOEGE@?$AAh?$AAr?$AA?9?$AAh?$AAr@ 0000000180029108     libucrt:lcidtoname_downlevel.obj
 0002:00009118       ??_C@_1M@GACBMHKE@?$AAh?$AAu?$AA?9?$AAh?$AAu@ 0000000180029118     libucrt:lcidtoname_downlevel.obj
 0002:00009128       ??_C@_1M@MILPAJJC@?$AAh?$AAy?$AA?9?$AAa?$AAm@ 0000000180029128     libucrt:lcidtoname_downlevel.obj
 0002:00009138       ??_C@_1M@BABBICEC@?$AAi?$AAd?$AA?9?$AAi?$AAd@ 0000000180029138     libucrt:lcidtoname_downlevel.obj
 0002:00009148       ??_C@_1M@BIKNHHPF@?$AAi?$AAs?$AA?9?$AAi?$AAs@ 0000000180029148     libucrt:lcidtoname_downlevel.obj
 0002:00009158       ??_C@_1M@NMPCJPHE@?$AAi?$AAt?$AA?9?$AAc?$AAh@ 0000000180029158     libucrt:lcidtoname_downlevel.obj
 0002:00009168       ??_C@_1M@GHKGFEDF@?$AAi?$AAt?$AA?9?$AAi?$AAt@ 0000000180029168     libucrt:lcidtoname_downlevel.obj
 0002:00009178       ??_C@_1M@NIEJCJJA@?$AAj?$AAa?$AA?9?$AAj?$AAp@ 0000000180029178     libucrt:lcidtoname_downlevel.obj
 0002:00009188       ??_C@_1M@JILFNBIM@?$AAk?$AAa?$AA?9?$AAg?$AAe@ 0000000180029188     libucrt:lcidtoname_downlevel.obj
 0002:00009198       ??_C@_1M@PACPMGPH@?$AAk?$AAk?$AA?9?$AAk?$AAz@ 0000000180029198     libucrt:lcidtoname_downlevel.obj
 0002:000091a8       ??_C@_1M@IELFGMHA@?$AAk?$AAn?$AA?9?$AAi?$AAn@ 00000001800291a8     libucrt:lcidtoname_downlevel.obj
 0002:000091b8       ??_C@_1O@IBBJHCH@?$AAk?$AAo?$AAk?$AA?9?$AAi?$AAn@ 00000001800291b8     libucrt:lcidtoname_downlevel.obj
 0002:000091c8       ??_C@_1M@DMHAEOGC@?$AAk?$AAo?$AA?9?$AAk?$AAr@ 00000001800291c8     libucrt:lcidtoname_downlevel.obj
 0002:000091d8       ??_C@_1M@HBAHBIGA@?$AAk?$AAy?$AA?9?$AAk?$AAg@ 00000001800291d8     libucrt:lcidtoname_downlevel.obj
 0002:000091e8       ??_C@_1M@KPMILCJG@?$AAl?$AAt?$AA?9?$AAl?$AAt@ 00000001800291e8     libucrt:lcidtoname_downlevel.obj
 0002:000091f8       ??_C@_1M@BDEKKCA@?$AAl?$AAv?$AA?9?$AAl?$AAv@ 00000001800291f8     libucrt:lcidtoname_downlevel.obj
 0002:00009208       ??_C@_1M@ELCKCCJJ@?$AAm?$AAi?$AA?9?$AAn?$AAz@ 0000000180029208     libucrt:lcidtoname_downlevel.obj
 0002:00009218       ??_C@_1M@CBOOLAPA@?$AAm?$AAk?$AA?9?$AAm?$AAk@ 0000000180029218     libucrt:lcidtoname_downlevel.obj
 0002:00009228       ??_C@_1M@GPHNBJKN@?$AAm?$AAl?$AA?9?$AAi?$AAn@ 0000000180029228     libucrt:lcidtoname_downlevel.obj
 0002:00009238       ??_C@_1M@PABJILIG@?$AAm?$AAn?$AA?9?$AAm?$AAn@ 0000000180029238     libucrt:lcidtoname_downlevel.obj
 0002:00009248       ??_C@_1M@FGBKKIPG@?$AAm?$AAr?$AA?9?$AAi?$AAn@ 0000000180029248     libucrt:lcidtoname_downlevel.obj
 0002:00009258       ??_C@_1M@NDBPDDAL@?$AAm?$AAs?$AA?9?$AAb?$AAn@ 0000000180029258     libucrt:lcidtoname_downlevel.obj
 0002:00009268       ??_C@_1M@OPIHOOPI@?$AAm?$AAs?$AA?9?$AAm?$AAy@ 0000000180029268     libucrt:lcidtoname_downlevel.obj
 0002:00009278       ??_C@_1M@PPDBCNFM@?$AAm?$AAt?$AA?9?$AAm?$AAt@ 0000000180029278     libucrt:lcidtoname_downlevel.obj
 0002:00009288       ??_C@_1M@KDJDKMDD@?$AAn?$AAb?$AA?9?$AAn?$AAo@ 0000000180029288     libucrt:lcidtoname_downlevel.obj
 0002:00009298       ??_C@_1M@KFCFLMJP@?$AAn?$AAl?$AA?9?$AAb?$AAe@ 0000000180029298     libucrt:lcidtoname_downlevel.obj
 0002:000092a8       ??_C@_1M@KPOPDDGO@?$AAn?$AAl?$AA?9?$AAn?$AAl@ 00000001800292a8     libucrt:lcidtoname_downlevel.obj
 0002:000092b8       ??_C@_1M@LJKPEMLN@?$AAn?$AAn?$AA?9?$AAn?$AAo@ 00000001800292b8     libucrt:lcidtoname_downlevel.obj
 0002:000092c8       ??_C@_1M@BDGHHBFL@?$AAn?$AAs?$AA?9?$AAz?$AAa@ 00000001800292c8     libucrt:lcidtoname_downlevel.obj
 0002:000092d8       ??_C@_1M@IDEHOAP@?$AAp?$AAa?$AA?9?$AAi?$AAn@ 00000001800292d8     libucrt:lcidtoname_downlevel.obj
 0002:000092e8       ??_C@_1M@HDBKGOGH@?$AAp?$AAl?$AA?9?$AAp?$AAl@ 00000001800292e8     libucrt:lcidtoname_downlevel.obj
 0002:000092f8       ??_C@_1M@LJLLCMEH@?$AAp?$AAt?$AA?9?$AAb?$AAr@ 00000001800292f8     libucrt:lcidtoname_downlevel.obj
 0002:00009308       ??_C@_1M@NCMONAAL@?$AAp?$AAt?$AA?9?$AAp?$AAt@ 0000000180029308     libucrt:lcidtoname_downlevel.obj
 0002:00009318       ??_C@_1O@EAKMAJDN@?$AAq?$AAu?$AAz?$AA?9?$AAb?$AAo@ 0000000180029318     libucrt:lcidtoname_downlevel.obj
 0002:00009328       ??_C@_1O@BHHPIGDN@?$AAq?$AAu?$AAz?$AA?9?$AAe?$AAc@ 0000000180029328     libucrt:lcidtoname_downlevel.obj
 0002:00009338       ??_C@_1O@GBAPEKMJ@?$AAq?$AAu?$AAz?$AA?9?$AAp?$AAe@ 0000000180029338     libucrt:lcidtoname_downlevel.obj
 0002:00009348       ??_C@_1M@CLGLEFBO@?$AAr?$AAo?$AA?9?$AAr?$AAo@ 0000000180029348     libucrt:lcidtoname_downlevel.obj
 0002:00009358       ??_C@_1M@CEEDODME@?$AAr?$AAu?$AA?9?$AAr?$AAu@ 0000000180029358     libucrt:lcidtoname_downlevel.obj
 0002:00009368       ??_C@_1M@HPKKKMPP@?$AAs?$AAa?$AA?9?$AAi?$AAn@ 0000000180029368     libucrt:lcidtoname_downlevel.obj
 0002:00009378       ??_C@_1M@BKMAIGOJ@?$AAs?$AAe?$AA?9?$AAf?$AAi@ 0000000180029378     libucrt:lcidtoname_downlevel.obj
 0002:00009388       ??_C@_1M@NDPIFLFI@?$AAs?$AAe?$AA?9?$AAn?$AAo@ 0000000180029388     libucrt:lcidtoname_downlevel.obj
 0002:00009398       ??_C@_1M@DANKKHJ@?$AAs?$AAe?$AA?9?$AAs?$AAe@ 0000000180029398     libucrt:lcidtoname_downlevel.obj
 0002:000093a8       ??_C@_1M@PNBLONPJ@?$AAs?$AAk?$AA?9?$AAs?$AAk@ 00000001800293a8     libucrt:lcidtoname_downlevel.obj
 0002:000093b8       ??_C@_1M@LFMODOAL@?$AAs?$AAl?$AA?9?$AAs?$AAi@ 00000001800293b8     libucrt:lcidtoname_downlevel.obj
 0002:000093c8       ??_C@_1O@DFKOMPG@?$AAs?$AAm?$AAa?$AA?9?$AAn?$AAo@ 00000001800293c8     libucrt:lcidtoname_downlevel.obj
 0002:000093d8       ??_C@_1O@NDKPBNNH@?$AAs?$AAm?$AAa?$AA?9?$AAs?$AAe@ 00000001800293d8     libucrt:lcidtoname_downlevel.obj
 0002:000093e8       ??_C@_1O@PLLKBHAB@?$AAs?$AAm?$AAj?$AA?9?$AAn?$AAo@ 00000001800293e8     libucrt:lcidtoname_downlevel.obj
 0002:000093f8       ??_C@_1O@CLEPOGCA@?$AAs?$AAm?$AAj?$AA?9?$AAs?$AAe@ 00000001800293f8     libucrt:lcidtoname_downlevel.obj
 0002:00009408       ??_C@_1O@DLGJGKMK@?$AAs?$AAm?$AAn?$AA?9?$AAf?$AAi@ 0000000180029408     libucrt:lcidtoname_downlevel.obj
 0002:00009418       ??_C@_1O@OJDJGAJC@?$AAs?$AAm?$AAs?$AA?9?$AAf?$AAi@ 0000000180029418     libucrt:lcidtoname_downlevel.obj
 0002:00009428       ??_C@_1M@BOFOGHPB@?$AAs?$AAq?$AA?9?$AAa?$AAl@ 0000000180029428     libucrt:lcidtoname_downlevel.obj
 0002:00009438       ??_C@_1BG@LJBBIPGB@?$AAs?$AAr?$AA?9?$AAb?$AAa?$AA?9?$AAc?$AAy?$AAr?$AAl@ 0000000180029438     libucrt:lcidtoname_downlevel.obj
 0002:00009450       ??_C@_1BG@JLBENFOE@?$AAs?$AAr?$AA?9?$AAb?$AAa?$AA?9?$AAl?$AAa?$AAt?$AAn@ 0000000180029450     libucrt:lcidtoname_downlevel.obj
 0002:00009468       ??_C@_1BG@KODPNHE@?$AAs?$AAr?$AA?9?$AAs?$AAp?$AA?9?$AAc?$AAy?$AAr?$AAl@ 0000000180029468     libucrt:lcidtoname_downlevel.obj
 0002:00009480       ??_C@_1BG@CIOGKHPB@?$AAs?$AAr?$AA?9?$AAs?$AAp?$AA?9?$AAl?$AAa?$AAt?$AAn@ 0000000180029480     libucrt:lcidtoname_downlevel.obj
 0002:00009498       ??_C@_1M@NGFJLMAC@?$AAs?$AAv?$AA?9?$AAf?$AAi@ 0000000180029498     libucrt:lcidtoname_downlevel.obj
 0002:000094a8       ??_C@_1M@MPJEJAJC@?$AAs?$AAv?$AA?9?$AAs?$AAe@ 00000001800294a8     libucrt:lcidtoname_downlevel.obj
 0002:000094b8       ??_C@_1M@MPNDHLFK@?$AAs?$AAw?$AA?9?$AAk?$AAe@ 00000001800294b8     libucrt:lcidtoname_downlevel.obj
 0002:000094c8       ??_C@_1O@KOHBJJI@?$AAs?$AAy?$AAr?$AA?9?$AAs?$AAy@ 00000001800294c8     libucrt:lcidtoname_downlevel.obj
 0002:000094d8       ??_C@_1M@LDCEFHA@?$AAt?$AAa?$AA?9?$AAi?$AAn@ 00000001800294d8     libucrt:lcidtoname_downlevel.obj
 0002:000094e8       ??_C@_1M@CNJOFAK@?$AAt?$AAe?$AA?9?$AAi?$AAn@ 00000001800294e8     libucrt:lcidtoname_downlevel.obj
 0002:000094f8       ??_C@_1M@GNAECACD@?$AAt?$AAh?$AA?9?$AAt?$AAh@ 00000001800294f8     libucrt:lcidtoname_downlevel.obj
 0002:00009508       ??_C@_1M@CHBIHOJO@?$AAt?$AAn?$AA?9?$AAz?$AAa@ 0000000180029508     libucrt:lcidtoname_downlevel.obj
 0002:00009518       ??_C@_1M@GCCMIGPJ@?$AAt?$AAr?$AA?9?$AAt?$AAr@ 0000000180029518     libucrt:lcidtoname_downlevel.obj
 0002:00009528       ??_C@_1M@CELMCNBK@?$AAt?$AAt?$AA?9?$AAr?$AAu@ 0000000180029528     libucrt:lcidtoname_downlevel.obj
 0002:00009538       ??_C@_1M@KLMCELGA@?$AAu?$AAk?$AA?9?$AAu?$AAa@ 0000000180029538     libucrt:lcidtoname_downlevel.obj
 0002:00009548       ??_C@_1M@EPAJJAJF@?$AAu?$AAr?$AA?9?$AAp?$AAk@ 0000000180029548     libucrt:lcidtoname_downlevel.obj
 0002:00009558       ??_C@_1BG@GEGPMCDJ@?$AAu?$AAz?$AA?9?$AAu?$AAz?$AA?9?$AAc?$AAy?$AAr?$AAl@ 0000000180029558     libucrt:lcidtoname_downlevel.obj
 0002:00009570       ??_C@_1BG@EGGKJILM@?$AAu?$AAz?$AA?9?$AAu?$AAz?$AA?9?$AAl?$AAa?$AAt?$AAn@ 0000000180029570     libucrt:lcidtoname_downlevel.obj
 0002:00009588       ??_C@_1M@GFOCLFF@?$AAv?$AAi?$AA?9?$AAv?$AAn@ 0000000180029588     libucrt:lcidtoname_downlevel.obj
 0002:00009598       ??_C@_1M@CPAMEDFI@?$AAx?$AAh?$AA?9?$AAz?$AAa@ 0000000180029598     libucrt:lcidtoname_downlevel.obj
 0002:000095a8       ??_C@_1O@EBKIFIGN@?$AAz?$AAh?$AA?9?$AAc?$AAh?$AAs@ 00000001800295a8     libucrt:lcidtoname_downlevel.obj
 0002:000095b8       ??_C@_1O@NMHPGANE@?$AAz?$AAh?$AA?9?$AAc?$AAh?$AAt@ 00000001800295b8     libucrt:lcidtoname_downlevel.obj
 0002:000095c8       ??_C@_1M@LPINJOMC@?$AAz?$AAh?$AA?9?$AAc?$AAn@ 00000001800295c8     libucrt:lcidtoname_downlevel.obj
 0002:000095d8       ??_C@_1M@OCJEJODD@?$AAz?$AAh?$AA?9?$AAh?$AAk@ 00000001800295d8     libucrt:lcidtoname_downlevel.obj
 0002:000095e8       ??_C@_1M@DNDLJINH@?$AAz?$AAh?$AA?9?$AAm?$AAo@ 00000001800295e8     libucrt:lcidtoname_downlevel.obj
 0002:000095f8       ??_C@_1M@MBFDNDND@?$AAz?$AAh?$AA?9?$AAs?$AAg@ 00000001800295f8     libucrt:lcidtoname_downlevel.obj
 0002:00009608       ??_C@_1M@IMEPLEPE@?$AAz?$AAh?$AA?9?$AAt?$AAw@ 0000000180029608     libucrt:lcidtoname_downlevel.obj
 0002:00009618       ??_C@_1M@BBGHNHJP@?$AAz?$AAu?$AA?9?$AAz?$AAa@ 0000000180029618     libucrt:lcidtoname_downlevel.obj
 0002:00009650       ?large_power_data@?1??multiply_by_power_of_ten@__crt_strtox@@YA_NAEAUbig_integer@2@I@Z@4QBIB 0000000180029650     libucrt:cfout.obj
 0002:00009f60       ?large_power_indices@?1??multiply_by_power_of_ten@__crt_strtox@@YA_NAEAUbig_integer@2@I@Z@4QBUunpack_index@?1??12@YA_N0I@Z@B 0000000180029f60     libucrt:cfout.obj
 0002:00009ff8       ?small_powers_of_ten@?1??multiply_by_power_of_ten@__crt_strtox@@YA_NAEAUbig_integer@2@I@Z@4QBIB 0000000180029ff8     libucrt:cfout.obj
 0002:0000a01c       ??_C@_01GBGANLPD@0@        000000018002a01c     libucrt:cfout.obj
 0002:0000a020       ??_C@_05DNEBIAHO@1?$CDINF@ 000000018002a020     libucrt:cfout.obj
 0002:0000a028       ??_C@_06IMKFLFPG@1?$CDQNAN@ 000000018002a028     libucrt:cfout.obj
 0002:0000a030       ??_C@_06PGGFOGJG@1?$CDSNAN@ 000000018002a030     libucrt:cfout.obj
 0002:0000a038       ??_C@_05PHHOCPM@1?$CDIND@  000000018002a038     libucrt:cfout.obj
 0002:0000a040       __real@3ff0000000000000    000000018002a040     libucrt:ceil.obj
 0002:0000a2a0       ??_C@_1BA@BALFACEM@?$AAC?$AAO?$AAN?$AAO?$AAU?$AAT?$AA$@ 000000018002a2a0     libucrt:initcon.obj
 0002:0000a2b0       __log10_256_lead           000000018002a2b0     libucrt:log10_256_lead_tail_table.obj
 0002:0000aac0       __log10_256_tail           000000018002aac0     libucrt:log10_256_lead_tail_table.obj
 0002:0000b2d0       __log_F_inv_qword          000000018002b2d0     libucrt:log_f_inv_qword_table.obj
 0002:0000bae0       ??_C@_05HGHHAHAP@log10@    000000018002bae0     libucrt:log_special.obj
 0002:0000bb00       _load_config_used          000000018002bb00     LIBCMT:loadcfg.obj
 0002:0000bd00       ??_R4exception@std@@6B@    000000018002bd00     AccessBridgeMessageQueue.obj
 0002:0000bd28       ??_R3exception@std@@8      000000018002bd28     AccessBridgeMessageQueue.obj
 0002:0000bd40       ??_R2exception@std@@8      000000018002bd40     AccessBridgeMessageQueue.obj
 0002:0000bd50       ??_R1A@?0A@EA@exception@std@@8 000000018002bd50     AccessBridgeMessageQueue.obj
 0002:0000bd78       ??_R4bad_alloc@std@@6B@    000000018002bd78     AccessBridgeMessageQueue.obj
 0002:0000bda0       ??_R3bad_alloc@std@@8      000000018002bda0     AccessBridgeMessageQueue.obj
 0002:0000bdb8       ??_R2bad_alloc@std@@8      000000018002bdb8     AccessBridgeMessageQueue.obj
 0002:0000bdd0       ??_R1A@?0A@EA@bad_alloc@std@@8 000000018002bdd0     AccessBridgeMessageQueue.obj
 0002:0000bdf8       ??_R4type_info@@6B@        000000018002bdf8     LIBCMT:std_type_info_static.obj
 0002:0000be20       ??_R3type_info@@8          000000018002be20     LIBCMT:std_type_info_static.obj
 0002:0000be38       ??_R2type_info@@8          000000018002be38     LIBCMT:std_type_info_static.obj
 0002:0000be48       ??_R1A@?0A@EA@type_info@@8 000000018002be48     LIBCMT:std_type_info_static.obj
 0002:0000be70       ??_R4bad_array_new_length@std@@6B@ 000000018002be70     LIBCMT:throw_bad_alloc.obj
 0002:0000be98       ??_R3bad_array_new_length@std@@8 000000018002be98     LIBCMT:throw_bad_alloc.obj
 0002:0000beb0       ??_R2bad_array_new_length@std@@8 000000018002beb0     LIBCMT:throw_bad_alloc.obj
 0002:0000bed0       ??_R1A@?0A@EA@bad_array_new_length@std@@8 000000018002bed0     LIBCMT:throw_bad_alloc.obj
 0002:0000bef8       ??_R4bad_exception@std@@6B@ 000000018002bef8     libvcruntime:frame.obj
 0002:0000bf20       ??_R3bad_exception@std@@8  000000018002bf20     libvcruntime:frame.obj
 0002:0000bf38       ??_R2bad_exception@std@@8  000000018002bf38     libvcruntime:frame.obj
 0002:0000bf50       ??_R1A@?0A@EA@bad_exception@std@@8 000000018002bf50     libvcruntime:frame.obj
 0002:0000bf74       __volatile_metadata        000000018002bf74     <linker-defined>
 0002:0000c598       __rtc_iaa                  000000018002c598     LIBCMT:initsect.obj
 0002:0000c5a0       __rtc_izz                  000000018002c5a0     LIBCMT:initsect.obj
 0002:0000c5a8       __rtc_taa                  000000018002c5a8     LIBCMT:initsect.obj
 0002:0000c5b0       __rtc_tzz                  000000018002c5b0     LIBCMT:initsect.obj
 0002:0000dc78       _CT??_R0?AVbad_alloc@std@@@8??0bad_alloc@std@@QEAA@AEBV01@@Z24 000000018002dc78     AccessBridgeMessageQueue.obj
 0002:0000dca0       _CT??_R0?AVexception@std@@@8??0exception@std@@QEAA@AEBV01@@Z24 000000018002dca0     AccessBridgeMessageQueue.obj
 0002:0000dcc8       _TI2?AVbad_alloc@std@@     000000018002dcc8     AccessBridgeMessageQueue.obj
 0002:0000dce8       _CTA2?AVbad_alloc@std@@    000000018002dce8     AccessBridgeMessageQueue.obj
 0002:0000dd00       _TI3?AVbad_array_new_length@std@@ 000000018002dd00     LIBCMT:throw_bad_alloc.obj
 0002:0000dd20       _CTA3?AVbad_array_new_length@std@@ 000000018002dd20     LIBCMT:throw_bad_alloc.obj
 0002:0000dd40       _CT??_R0?AVbad_array_new_length@std@@@8??0bad_array_new_length@std@@QEAA@AEBV01@@Z24 000000018002dd40     LIBCMT:throw_bad_alloc.obj
 0002:0000dd68       _TI2?AVbad_exception@std@@ 000000018002dd68     libvcruntime:frame.obj
 0002:0000dd88       _CTA2?AVbad_exception@std@@ 000000018002dd88     libvcruntime:frame.obj
 0002:0000dda0       _CT??_R0?AVbad_exception@std@@@8??0bad_exception@std@@QEAA@AEBV01@@Z24 000000018002dda0     libvcruntime:frame.obj
 0002:0000ec14       __IMPORT_DESCRIPTOR_KERNEL32 000000018002ec14     kernel32:KERNEL32.dll
 0002:0000ec28       __IMPORT_DESCRIPTOR_USER32 000000018002ec28     user32:USER32.dll
 0002:0000ec3c       __NULL_IMPORT_DESCRIPTOR   000000018002ec3c     kernel32:KERNEL32.dll
 0003:00000000       __security_cookie_complement 0000000180030000     LIBCMT:gs_cookie.obj
 0003:00000008       __security_cookie          0000000180030008     LIBCMT:gs_cookie.obj
 0003:00000010       __scrt_native_dllmain_reason 0000000180030010     LIBCMT:utility.obj
 0003:00000018       __isa_available            0000000180030018     LIBCMT:cpu_disp.obj
 0003:0000001c       __isa_enabled              000000018003001c     LIBCMT:cpu_disp.obj
 0003:00000020       __memset_fast_string_threshold 0000000180030020     LIBCMT:cpu_disp.obj
 0003:00000028       __memset_nt_threshold      0000000180030028     LIBCMT:cpu_disp.obj
 0003:00000040       _iob                       0000000180030040     libucrt:_file.obj
 0003:00000150       __abort_behavior           0000000180030150     libucrt:abort.obj
 0003:00000170       __badioinfo                0000000180030170     libucrt:ioinit.obj
 0003:000001c0       __acrt_initial_locale_data 00000001800301c0     libucrt:nlsdata.obj
 0003:00000318       __acrt_initial_locale_pointers 0000000180030318     libucrt:nlsdata.obj
 0003:00000328       __acrt_wide_c_locale_string 0000000180030328     libucrt:nlsdata.obj
 0003:00000330       __acrt_initial_multibyte_data 0000000180030330     libucrt:mbctype.obj
 0003:00000870       __globallocalestatus       0000000180030870     libucrt:glstatus.obj
 0003:00000880       __acrt_lconv_c             0000000180030880     libucrt:localeconv.obj
 0003:00000918       __acrt_lconv_static_decimal 0000000180030918     libucrt:localeconv.obj
 0003:0000091c       __acrt_lconv_static_W_decimal 000000018003091c     libucrt:localeconv.obj
 0003:00000920       _lookuptrailbytes          0000000180030920     libucrt:read.obj
 0003:00000a34       _fltused                   0000000180030a34     LIBCMT:fltused.obj
 0003:00000a40       ??_R0?AVbad_alloc@std@@@8  0000000180030a40     AccessBridgeMessageQueue.obj
 0003:00000a68       ??_R0?AVexception@std@@@8  0000000180030a68     AccessBridgeMessageQueue.obj
 0003:00000a90       ??_R0?AVbad_array_new_length@std@@@8 0000000180030a90     LIBCMT:throw_bad_alloc.obj
 0003:00000ac0       ??_R0?AVbad_exception@std@@@8 0000000180030ac0     libvcruntime:frame.obj
 0003:00000ae8       ??_R0?AVtype_info@@@8      0000000180030ae8     LIBCMT:std_type_info_static.obj
 0003:00000b10       ?_OptionsStorage@?1??__local_stdio_printf_options@@9@4_KA 0000000180030b10     AccessBridgeDebug.obj
 0003:00000b20       ?theFromJavaHelloMsgID@@3IA 0000000180030b20     AccessBridgeMessages.obj
 0003:00000b24       ?theFromWindowsHelloMsgID@@3IA 0000000180030b24     AccessBridgeMessages.obj
 0003:00000b28       ?sendMemoryIPCLock@@3U_RTL_CRITICAL_SECTION@@A 0000000180030b28     WinAccessBridge.obj
 0003:00000b50       ?newJVMs@@3PEAPEADEA       0000000180030b50     WinAccessBridge.obj
 0003:00000b58       ?theWindowsAccessBridge@@3PEAVWinAccessBridge@@EA 0000000180030b58     WinAccessBridge.obj
 0003:00000b60       ?theDialogWindow@@3PEAUHWND__@@EA 0000000180030b60     WinAccessBridge.obj
 0003:00000b68       ?isVMInstanceChainInUse@@3_NA 0000000180030b68     WinAccessBridge.obj
 0003:000010e0       ?__type_info_root_node@@3U__type_info_node@@A 00000001800310e0     LIBCMT:tncleanup.obj
 0003:000010f0       ?_OptionsStorage@?1??__local_stdio_scanf_options@@9@4_KA 00000001800310f0     LIBCMT:default_local_stdio_options.obj
 0003:000010f8       __scrt_current_native_startup_state 00000001800310f8     LIBCMT:utility.obj
 0003:00001100       __scrt_native_startup_lock 0000000180031100     LIBCMT:utility.obj
 0003:00001140       __scrt_debugger_hook_flag  0000000180031140     LIBCMT:utility_desktop.obj
 0003:00001144       __favor                    0000000180031144     LIBCMT:cpu_disp.obj
 0003:00001148       ?__WinRTOutOfMemoryExceptionCallback@@3P6APEAXXZEA 0000000180031148     libvcruntime:ehhelpers.obj
 0003:00001150       ?pArgList@UnDecorator@@0PEAVReplicator@@EA 0000000180031150     libvcruntime:undname.obj
 0003:00001158       ?pZNameList@UnDecorator@@0PEAVReplicator@@EA 0000000180031158     libvcruntime:undname.obj
 0003:00001160       ?pTemplateArgList@UnDecorator@@0PEAVReplicator@@EA 0000000180031160     libvcruntime:undname.obj
 0003:00001168       ?gName@UnDecorator@@0PEBDEB 0000000180031168     libvcruntime:undname.obj
 0003:00001170       ?name@UnDecorator@@0PEBDEB 0000000180031170     libvcruntime:undname.obj
 0003:00001178       ?disableFlags@UnDecorator@@0KA 0000000180031178     libvcruntime:undname.obj
 0003:0000117c       ?fExplicitTemplateParams@UnDecorator@@0_NA 000000018003117c     libvcruntime:undname.obj
 0003:0000117d       ?fGetTemplateArgumentList@UnDecorator@@0_NA 000000018003117d     libvcruntime:undname.obj
 0003:00001180       ?m_pGetParameter@UnDecorator@@0P6APEADJ@ZEA 0000000180031180     libvcruntime:undname.obj
 0003:00001188       ?m_CHPENameOffset@UnDecorator@@0KA 0000000180031188     libvcruntime:undname.obj
 0003:0000118c       ?m_recursionLevel@UnDecorator@@0KA 000000018003118c     libvcruntime:undname.obj
 0003:000012b0       __pPurecall                00000001800312b0     libvcruntime:purevirt_data.obj
 0003:000012b8       _nstream                   00000001800312b8     libucrt:_file.obj
 0003:000012c0       __piob                     00000001800312c0     libucrt:_file.obj
 0003:000012c8       _cflush                    00000001800312c8     libucrt:_file.obj
 0003:000013f8       _environ_table             00000001800313f8     libucrt:environment_initialization.obj
 0003:00001400       _wenviron_table            0000000180031400     libucrt:environment_initialization.obj
 0003:00001408       __dcrt_initial_wide_environment 0000000180031408     libucrt:environment_initialization.obj
 0003:00001410       __dcrt_initial_narrow_environment 0000000180031410     libucrt:environment_initialization.obj
 0003:00001418       __acrt_atexit_table        0000000180031418     libucrt:onexit.obj
 0003:00001430       __acrt_at_quick_exit_table 0000000180031430     libucrt:onexit.obj
 0003:00001600       __pioinfo                  0000000180031600     libucrt:ioinit.obj
 0003:00001a00       _nhandle                   0000000180031a00     libucrt:ioinit.obj
 0003:00001a18       __acrt_stdout_buffer       0000000180031a18     libucrt:_sftbuf.obj
 0003:00001a20       __acrt_stderr_buffer       0000000180031a20     libucrt:_sftbuf.obj
 0003:00001a28       __acrt_locale_changed_data 0000000180031a28     libucrt:wsetlocale.obj
 0003:00001a30       __acrt_current_locale_data 0000000180031a30     libucrt:nlsdata.obj
 0003:00001c78       _mbctype                   0000000180031c78     libucrt:mbctype.obj
 0003:00001c80       _mbcasemap                 0000000180031c80     libucrt:mbctype.obj
 0003:00001c88       __acrt_current_multibyte_data 0000000180031c88     libucrt:mbctype.obj
 0003:00001c98       _pgmptr                    0000000180031c98     libucrt:argv_data.obj
 0003:00001ca0       __argc                     0000000180031ca0     libucrt:argv_data.obj
 0003:00001ca8       __argv                     0000000180031ca8     libucrt:argv_data.obj
 0003:00001cb0       __wargv                    0000000180031cb0     libucrt:argv_data.obj
 0003:00001cb8       _acmdln                    0000000180031cb8     libucrt:argv_data.obj
 0003:00001cc0       _wcmdln                    0000000180031cc0     libucrt:argv_data.obj
 0003:00001cc8       __acrt_heap                0000000180031cc8     libucrt:heap_handle.obj
 0003:00001cfc       __acrt_lconv_static_null   0000000180031cfc     libucrt:localeconv.obj
 0003:00001d00       __acrt_lconv_static_W_null 0000000180031d00     libucrt:localeconv.obj
 0003:00001d04       _commode                   0000000180031d04     libucrt:ncommode.obj
 0003:00001d18       _umaskval                  0000000180031d18     libucrt:umask.obj
 0003:00001d1c       __fma3_is_available        0000000180031d1c     libucrt:fma3_available.obj
 0003:00001d20       __use_fma3_lib             0000000180031d20     libucrt:fma3_available.obj
 0003:00001d24       _fmode                     0000000180031d24     libucrt:txtmode.obj
 0003:00001d28       __scrt_ucrt_dll_is_in_use  0000000180031d28     <common>
 0003:00001d30       __dyn_tls_init_callback    0000000180031d30     <common>

 entry point at        0001:00006b40

 Static symbols

 0000:fffc9000       .debug$S                   0000000180000000     windowsaccessbridge-64.exp
 0000:fffc9000       .debug$S                   0000000180000000     kernel32:KERNEL32.dll
 0000:fffc9000       .debug$S                   0000000180000000     kernel32:KERNEL32.dll
 0000:fffc9000       .debug$S                   0000000180000000     kernel32:KERNEL32.dll
 0000:fffc9000       .debug$S                   0000000180000000     kernel32:KERNEL32.dll
 0000:fffc9000       .debug$S                   0000000180000000     kernel32:KERNEL32.dll
 0000:fffc9000       .debug$S                   0000000180000000     kernel32:KERNEL32.dll
 0000:fffc9000       .debug$S                   0000000180000000     kernel32:KERNEL32.dll
 0000:fffc9000       .debug$S                   0000000180000000     kernel32:KERNEL32.dll
 0000:fffc9000       .debug$S                   0000000180000000     kernel32:KERNEL32.dll
 0000:fffc9000       .debug$S                   0000000180000000     kernel32:KERNEL32.dll
 0000:fffc9000       .debug$S                   0000000180000000     kernel32:KERNEL32.dll
 0000:fffc9000       .debug$S                   0000000180000000     kernel32:KERNEL32.dll
 0000:fffc9000       .debug$S                   0000000180000000     kernel32:KERNEL32.dll
 0000:fffc9000       .debug$S                   0000000180000000     kernel32:KERNEL32.dll
 0000:fffc9000       .debug$S                   0000000180000000     kernel32:KERNEL32.dll
 0000:fffc9000       .debug$S                   0000000180000000     kernel32:KERNEL32.dll
 0000:fffc9000       .debug$S                   0000000180000000     kernel32:KERNEL32.dll
 0000:fffc9000       .debug$S                   0000000180000000     kernel32:KERNEL32.dll
 0000:fffc9000       .debug$S                   0000000180000000     kernel32:KERNEL32.dll
 0000:fffc9000       .debug$S                   0000000180000000     kernel32:KERNEL32.dll
 0000:fffc9000       .debug$S                   0000000180000000     kernel32:KERNEL32.dll
 0000:fffc9000       .debug$S                   0000000180000000     kernel32:KERNEL32.dll
 0000:fffc9000       .debug$S                   0000000180000000     kernel32:KERNEL32.dll
 0000:fffc9000       .debug$S                   0000000180000000     kernel32:KERNEL32.dll
 0000:fffc9000       .debug$S                   0000000180000000     kernel32:KERNEL32.dll
 0000:fffc9000       .debug$S                   0000000180000000     kernel32:KERNEL32.dll
 0000:fffc9000       .debug$S                   0000000180000000     kernel32:KERNEL32.dll
 0000:fffc9000       .debug$S                   0000000180000000     kernel32:KERNEL32.dll
 0000:fffc9000       .debug$S                   0000000180000000     kernel32:KERNEL32.dll
 0000:fffc9000       .debug$S                   0000000180000000     kernel32:KERNEL32.dll
 0000:fffc9000       .debug$S                   0000000180000000     kernel32:KERNEL32.dll
 0000:fffc9000       .debug$S                   0000000180000000     kernel32:KERNEL32.dll
 0000:fffc9000       .debug$S                   0000000180000000     kernel32:KERNEL32.dll
 0000:fffc9000       .debug$S                   0000000180000000     kernel32:KERNEL32.dll
 0000:fffc9000       .debug$S                   0000000180000000     kernel32:KERNEL32.dll
 0000:fffc9000       .debug$S                   0000000180000000     kernel32:KERNEL32.dll
 0000:fffc9000       .debug$S                   0000000180000000     kernel32:KERNEL32.dll
 0000:fffc9000       .debug$S                   0000000180000000     kernel32:KERNEL32.dll
 0000:fffc9000       .debug$S                   0000000180000000     kernel32:KERNEL32.dll
 0000:fffc9000       .debug$S                   0000000180000000     kernel32:KERNEL32.dll
 0000:fffc9000       .debug$S                   0000000180000000     kernel32:KERNEL32.dll
 0000:fffc9000       .debug$S                   0000000180000000     kernel32:KERNEL32.dll
 0000:fffc9000       .debug$S                   0000000180000000     kernel32:KERNEL32.dll
 0000:fffc9000       .debug$S                   0000000180000000     kernel32:KERNEL32.dll
 0000:fffc9000       .debug$S                   0000000180000000     kernel32:KERNEL32.dll
 0000:fffc9000       .debug$S                   0000000180000000     kernel32:KERNEL32.dll
 0000:fffc9000       .debug$S                   0000000180000000     kernel32:KERNEL32.dll
 0000:fffc9000       .debug$S                   0000000180000000     kernel32:KERNEL32.dll
 0000:fffc9000       .debug$S                   0000000180000000     kernel32:KERNEL32.dll
 0000:fffc9000       .debug$S                   0000000180000000     kernel32:KERNEL32.dll
 0000:fffc9000       .debug$S                   0000000180000000     kernel32:KERNEL32.dll
 0000:fffc9000       .debug$S                   0000000180000000     kernel32:KERNEL32.dll
 0000:fffc9000       .debug$S                   0000000180000000     kernel32:KERNEL32.dll
 0000:fffc9000       .debug$S                   0000000180000000     kernel32:KERNEL32.dll
 0000:fffc9000       .debug$S                   0000000180000000     kernel32:KERNEL32.dll
 0000:fffc9000       .debug$S                   0000000180000000     kernel32:KERNEL32.dll
 0000:fffc9000       .debug$S                   0000000180000000     kernel32:KERNEL32.dll
 0000:fffc9000       .debug$S                   0000000180000000     kernel32:KERNEL32.dll
 0000:fffc9000       .debug$S                   0000000180000000     kernel32:KERNEL32.dll
 0000:fffc9000       .debug$S                   0000000180000000     kernel32:KERNEL32.dll
 0000:fffc9000       .debug$S                   0000000180000000     kernel32:KERNEL32.dll
 0000:fffc9000       .debug$S                   0000000180000000     kernel32:KERNEL32.dll
 0000:fffc9000       .debug$S                   0000000180000000     kernel32:KERNEL32.dll
 0000:fffc9000       .debug$S                   0000000180000000     kernel32:KERNEL32.dll
 0000:fffc9000       .debug$S                   0000000180000000     kernel32:KERNEL32.dll
 0000:fffc9000       .debug$S                   0000000180000000     kernel32:KERNEL32.dll
 0000:fffc9000       .debug$S                   0000000180000000     kernel32:KERNEL32.dll
 0000:fffc9000       .debug$S                   0000000180000000     kernel32:KERNEL32.dll
 0000:fffc9000       .debug$S                   0000000180000000     kernel32:KERNEL32.dll
 0000:fffc9000       .debug$S                   0000000180000000     kernel32:KERNEL32.dll
 0000:fffc9000       .debug$S                   0000000180000000     kernel32:KERNEL32.dll
 0000:fffc9000       .debug$S                   0000000180000000     kernel32:KERNEL32.dll
 0000:fffc9000       .debug$S                   0000000180000000     kernel32:KERNEL32.dll
 0000:fffc9000       .debug$S                   0000000180000000     kernel32:KERNEL32.dll
 0000:fffc9000       .debug$S                   0000000180000000     kernel32:KERNEL32.dll
 0000:fffc9000       .debug$S                   0000000180000000     kernel32:KERNEL32.dll
 0000:fffc9000       .debug$S                   0000000180000000     kernel32:KERNEL32.dll
 0000:fffc9000       .debug$S                   0000000180000000     kernel32:KERNEL32.dll
 0000:fffc9000       .debug$S                   0000000180000000     kernel32:KERNEL32.dll
 0000:fffc9000       .debug$S                   0000000180000000     kernel32:KERNEL32.dll
 0000:fffc9000       .debug$S                   0000000180000000     kernel32:KERNEL32.dll
 0000:fffc9000       .debug$S                   0000000180000000     kernel32:KERNEL32.dll
 0000:fffc9000       .debug$S                   0000000180000000     kernel32:KERNEL32.dll
 0000:fffc9000       .debug$S                   0000000180000000     kernel32:KERNEL32.dll
 0000:fffc9000       .debug$S                   0000000180000000     kernel32:KERNEL32.dll
 0000:fffc9000       .debug$S                   0000000180000000     kernel32:KERNEL32.dll
 0000:fffc9000       .debug$S                   0000000180000000     kernel32:KERNEL32.dll
 0000:fffc9000       .debug$S                   0000000180000000     kernel32:KERNEL32.dll
 0000:fffc9000       .debug$S                   0000000180000000     kernel32:KERNEL32.dll
 0000:fffc9000       .debug$S                   0000000180000000     kernel32:KERNEL32.dll
 0000:fffc9000       .debug$S                   0000000180000000     kernel32:KERNEL32.dll
 0000:fffc9000       .debug$S                   0000000180000000     kernel32:KERNEL32.dll
 0000:fffc9000       .debug$S                   0000000180000000     kernel32:KERNEL32.dll
 0000:fffc9000       .debug$S                   0000000180000000     kernel32:KERNEL32.dll
 0000:fffc9000       .debug$S                   0000000180000000     kernel32:KERNEL32.dll
 0000:fffc9000       .debug$S                   0000000180000000     kernel32:KERNEL32.dll
 0000:fffc9000       .debug$S                   0000000180000000     user32:USER32.dll
 0000:fffc9000       .debug$S                   0000000180000000     user32:USER32.dll
 0000:fffc9000       .debug$S                   0000000180000000     user32:USER32.dll
 0000:fffc9000       .debug$S                   0000000180000000     user32:USER32.dll
 0000:fffc9000       .debug$S                   0000000180000000     user32:USER32.dll
 0000:fffc9000       .debug$S                   0000000180000000     user32:USER32.dll
 0000:fffc9000       .debug$S                   0000000180000000     user32:USER32.dll
 0000:fffc9000       .debug$S                   0000000180000000     user32:USER32.dll
 0000:fffc9000       .debug$S                   0000000180000000     user32:USER32.dll
 0000:fffc9000       .debug$S                   0000000180000000     user32:USER32.dll
 0000:fffc9000       .debug$S                   0000000180000000     user32:USER32.dll
 0000:fffc9000       .debug$S                   0000000180000000     user32:USER32.dll
 0000:fffc9000       .debug$S                   0000000180000000     user32:USER32.dll
 0001:00006720       $$000000                   0000000180007720     LIBCMT:amdsecgs.obj
 0001:000067c0       $$000000                   00000001800077c0     LIBCMT:chkstk.obj
 0001:00006820       ?dllmain_crt_dispatch@@YAHQEAUHINSTANCE__@@KQEAX@Z 0000000180007820 f   LIBCMT:dll_dllmain.obj
 0001:00006870       ?dllmain_crt_process_attach@@YAHQEAUHINSTANCE__@@QEAX@Z 0000000180007870 f   LIBCMT:dll_dllmain.obj
 0001:00006988       ?dllmain_crt_process_detach@@YAH_N@Z 0000000180007988 f   LIBCMT:dll_dllmain.obj
 0001:00006a0c       ?dllmain_dispatch@@YAHQEAUHINSTANCE__@@KQEAX@Z 0000000180007a0c f   LIBCMT:dll_dllmain.obj
 0001:00006d40       capture_current_context    0000000180007d40 f   LIBCMT:gs_report.obj
 0001:00006db0       capture_previous_context   0000000180007db0 f   LIBCMT:gs_report.obj
 0001:00007670       $$000000                   0000000180008670     libvcruntime:memcpy.obj
 0001:00007d10       $$000000                   0000000180008d10     libvcruntime:memset.obj
 0001:00008630       $$000000                   0000000180009630     libvcruntime:notify.obj
 0001:00008ea4       ?try_get_function@@YAPEAXW4function_id@?A0x14174aea@@QEBDQEBW4module_id@2@2@Z 0000000180009ea4 f   libvcruntime:winapi_downlevel.obj
 0001:00009290       ??$BuildCatchObjectHelperInternal@V__FrameHandler3@@@@YAHPEAUEHExceptionRecord@@PEAXPEBU_s_HandlerType@@PEBU_s_CatchableType@@@Z 000000018000a290 f   libvcruntime:frame.obj
 0001:00009490       ??$BuildCatchObjectInternal@V__FrameHandler3@@@@YAXPEAUEHExceptionRecord@@PEAXPEBU_s_HandlerType@@PEBU_s_CatchableType@@@Z 000000018000a490 f   libvcruntime:frame.obj
 0001:00009550       ??$CatchIt@V__FrameHandler3@@@@YAXPEAUEHExceptionRecord@@PEA_KPEAU_CONTEXT@@PEAU_xDISPATCHER_CONTEXT@@PEBU_s_FuncInfo@@PEBU_s_HandlerType@@PEBU_s_CatchableType@@PEBU_s_TryBlockMapEntry@@H1EE@Z 000000018000a550 f   libvcruntime:frame.obj
 0001:00009624       ??$FindHandler@V__FrameHandler3@@@@YAXPEAUEHExceptionRecord@@PEA_KPEAU_CONTEXT@@PEAU_xDISPATCHER_CONTEXT@@PEBU_s_FuncInfo@@EH1@Z 000000018000a624 f   libvcruntime:frame.obj
 0001:00009afc       ??$FindHandlerForForeignException@V__FrameHandler3@@@@YAXPEAUEHExceptionRecord@@PEA_KPEAU_CONTEXT@@PEAU_xDISPATCHER_CONTEXT@@PEBU_s_FuncInfo@@HH1@Z 000000018000aafc f   libvcruntime:frame.obj
 0001:0000a2e0       ?ExFilterRethrow@@YAHPEAU_EXCEPTION_POINTERS@@PEAUEHExceptionRecord@@PEAH@Z 000000018000b2e0 f   libvcruntime:frame.obj
 0001:0000a58c       ?IsInExceptionSpec@@YAEPEAUEHExceptionRecord@@PEBU_s_ESTypeList@@@Z 000000018000b58c f   libvcruntime:frame.obj
 0001:0000a67c       ?Is_bad_exception_allowed@@YAEPEBU_s_ESTypeList@@@Z 000000018000b67c f   libvcruntime:frame.obj
 0001:0000a720       $$000000                   000000018000b720     libvcruntime:handlers.obj
 0001:0000a830       $$000000                   000000018000b830     libucrt:strlen.obj
 0001:0000a8f0       $$000000                   000000018000b8f0     libucrt:strncat.obj
 0001:0000aaa0       $$000000                   000000018000baa0     libucrt:strncpy.obj
 0001:0000adbc       ??$?RV<lambda_d854c62834386a3b23916ad6dae2782d>@@AEAV<lambda_303760bc4008a2b3ec4768a30b06a80c>@@V<lambda_4780a7ea4f8cbd2590aec34bd14e2bbf>@@@?$__crt_seh_guarded_call@H@@QEAAH$$QEAV<lambda_d854c62834386a3b23916ad6dae2782d>@@AEAV<lambda_303760bc4008a2b3ec4768a30b06a80c>@@$$QEAV<lambda_4780a7ea4f8cbd2590aec34bd14e2bbf>@@@Z 000000018000bdbc f   libucrt:output.obj
 0001:0000baa8       ??R<lambda_303760bc4008a2b3ec4768a30b06a80c>@@QEBAHXZ 000000018000caa8 f   libucrt:output.obj
 0001:0000da8c       ?_fclose_internal@@YAHQEAU_iobuf@@AEAV__crt_cached_ptd_host@@@Z 000000018000ea8c f   libucrt:fclose.obj
 0001:0000db08       ?_fclose_nolock_internal@@YAHQEAU_iobuf@@AEAV__crt_cached_ptd_host@@@Z 000000018000eb08 f   libucrt:fclose.obj
 0001:0000dc48       ??$common_fsopen@D@@YAPEAU_iobuf@@QEBD0H@Z 000000018000ec48 f   libucrt:fopen.obj
 0001:0000dd10       ??$common_getenv@D@@YAPEADQEBD@Z 000000018000ed10 f   libucrt:getenv.obj
 0001:0000dd70       ??$common_getenv_nolock@D@@YAPEADQEBD@Z 000000018000ed70 f   libucrt:getenv.obj
 0001:0000de10       $$000000                   000000018000ee10     libucrt:strcmp.obj
 0001:0000de90       $$000000                   000000018000ee90     libucrt:strcat.obj
 0001:0000e300       ??$?RV<lambda_d80eeec6fff315bfe5c115232f3240e3>@@AEAV<lambda_6e4b09c48022b2350581041d5f6b0c4c>@@V<lambda_2358e3775559c9db80273638284d5e45>@@@?$__crt_seh_guarded_call@X@@QEAAX$$QEAV<lambda_d80eeec6fff315bfe5c115232f3240e3>@@AEAV<lambda_6e4b09c48022b2350581041d5f6b0c4c>@@$$QEAV<lambda_2358e3775559c9db80273638284d5e45>@@@Z 000000018000f300 f   libucrt:exit.obj
 0001:0000e338       ??R<lambda_6e4b09c48022b2350581041d5f6b0c4c>@@QEBA@XZ 000000018000f338 f   libucrt:exit.obj
 0001:0000e404       ?common_exit@@YAXHW4_crt_exit_cleanup_mode@@W4_crt_exit_return_mode@@@Z 000000018000f404 f   libucrt:exit.obj
 0001:0000e4cc       ?exit_or_terminate_process@@YAXI@Z 000000018000f4cc f   libucrt:exit.obj
 0001:0000e500       ?should_call_terminate_process@@YA_NXZ 000000018000f500 f   libucrt:exit.obj
 0001:0000e524       ?try_cor_exit_process@@YAXI@Z 000000018000f524 f   libucrt:exit.obj
 0001:0000e5c0       ??$parse_command_line@D@@YAXPEADPEAPEAD0PEA_K2@Z 000000018000f5c0 f   libucrt:argv_parsing.obj
 0001:0000e970       ??$common_initialize_environment_nolock@D@@YAHXZ 000000018000f970 f   libucrt:environment_initialization.obj
 0001:0000e9e4       ??$create_environment@D@@YAQEAPEADQEAD@Z 000000018000f9e4 f   libucrt:environment_initialization.obj
 0001:0000eaf4       ??$free_environment@D@@YAXQEAPEAD@Z 000000018000faf4 f   libucrt:environment_initialization.obj
 0001:0000eaf4       ??$free_environment@_W@@YAXQEAPEA_W@Z 000000018000faf4 f   libucrt:environment_initialization.obj
 0001:0000eb38       ??$initialize_environment_by_cloning_nolock@D@@YAHXZ 000000018000fb38 f   libucrt:environment_initialization.obj
 0001:0000ec18       ??$uninitialize_environment_internal@D@@YAXAEAPEAPEAD@Z 000000018000fc18 f   libucrt:environment_initialization.obj
 0001:0000ec34       ??$uninitialize_environment_internal@_W@@YAXAEAPEAPEA_W@Z 000000018000fc34 f   libucrt:environment_initialization.obj
 0001:0000ecd8       ??$?RV<lambda_7777bce6b2f8c936911f934f8298dc43>@@AEAV<lambda_f03950bc5685219e0bcd2087efbe011e>@@V<lambda_3883c3dff614d5e0c5f61bb1ac94921c>@@@?$__crt_seh_guarded_call@H@@QEAAH$$QEAV<lambda_7777bce6b2f8c936911f934f8298dc43>@@AEAV<lambda_f03950bc5685219e0bcd2087efbe011e>@@$$QEAV<lambda_3883c3dff614d5e0c5f61bb1ac94921c>@@@Z 000000018000fcd8 f   libucrt:onexit.obj
 0001:0000ed14       ??R<lambda_f03950bc5685219e0bcd2087efbe011e>@@QEBA@XZ 000000018000fd14 f   libucrt:onexit.obj
 0001:0000eea0       initialize_global_variables 000000018000fea0 f   libucrt:initialization.obj
 0001:0000eeb4       initialize_c               000000018000feb4 f   libucrt:initialization.obj
 0001:0000eed8       initialize_environment     000000018000fed8 f   libucrt:initialization.obj
 0001:0000eed8       initialize_global_state_isolation 000000018000fed8 f   libucrt:initialization.obj
 0001:0000eed8       report_memory_leaks        000000018000fed8 f   libucrt:initialization.obj
 0001:0000eed8       uninitialize_c             000000018000fed8 f   libucrt:initialization.obj
 0001:0000eed8       uninitialize_global_state_isolation 000000018000fed8 f   libucrt:initialization.obj
 0001:0000eedc       uninitialize_environment   000000018000fedc f   libucrt:initialization.obj
 0001:0000eeec       initialize_pointers        000000018000feec f   libucrt:initialization.obj
 0001:0000ef2c       uninitialize_vcruntime     000000018000ff2c f   libucrt:initialization.obj
 0001:0000ef34       uninitialize_allocated_memory 000000018000ff34 f   libucrt:initialization.obj
 0001:0000ef74       uninitialize_allocated_io_buffers 000000018000ff74 f   libucrt:initialization.obj
 0001:0000f140       $$000000                   0000000180010140     libucrt:strncmp.obj
 0001:0000f798       ?try_get_function@@YAPEAXW4function_id@?A0x391cf84c@@QEBDQEBW4module_id@2@2@Z 0000000180010798 f   libucrt:winapi_thunks.obj
 0001:0000fdd4       ??$?RV<lambda_842d9ff0dc9ef11c61343bbaebe7f885>@@AEAV<lambda_c5860995281e5c4ce005b3de8f5874ee>@@V<lambda_d90129c13df834fdcbf8d2b88dafcf2d>@@@?$__crt_seh_guarded_call@X@@QEAAX$$QEAV<lambda_842d9ff0dc9ef11c61343bbaebe7f885>@@AEAV<lambda_c5860995281e5c4ce005b3de8f5874ee>@@$$QEAV<lambda_d90129c13df834fdcbf8d2b88dafcf2d>@@@Z 0000000180010dd4 f   libucrt:fflush.obj
 0001:0000fe70       ??$?RV<lambda_886d6c58226a84441f68b9f2b8217b83>@@AEAV<lambda_ab61a845afdef5b7c387490eaf3616ee>@@V<lambda_f7f22ab5edc0698d5f6905b0d3f44752>@@@?$__crt_seh_guarded_call@X@@QEAAX$$QEAV<lambda_886d6c58226a84441f68b9f2b8217b83>@@AEAV<lambda_ab61a845afdef5b7c387490eaf3616ee>@@$$QEAV<lambda_f7f22ab5edc0698d5f6905b0d3f44752>@@@Z 0000000180010e70 f   libucrt:fflush.obj
 0001:0000ff54       ?common_flush_all@@YAH_N@Z 0000000180010f54 f   libucrt:fflush.obj
 0001:00010160       ?initialize_inherited_file_handles_nolock@@YAXXZ 0000000180011160 f   libucrt:ioinit.obj
 0001:00010250       ?initialize_stdio_handles_nolock@@YAXXZ 0000000180011250 f   libucrt:ioinit.obj
 0001:00010834       ?fp_format_a@@YAHQEBNPEAD_KQEAD2H_NIW4__acrt_rounding_mode@@AEAV__crt_cached_ptd_host@@@Z 0000000180011834 f   libucrt:cvt.obj
 0001:00010bcc       ?fp_format_e@@YAHQEBNQEAD_K12H_NIW4__acrt_rounding_mode@@AEAV__crt_cached_ptd_host@@@Z 0000000180011bcc f   libucrt:cvt.obj
 0001:00010cc8       ?fp_format_e_internal@@YAHQEAD_KH_NIQEAU_strflt@@2AEAV__crt_cached_ptd_host@@@Z 0000000180011cc8 f   libucrt:cvt.obj
 0001:00010eac       ?fp_format_f@@YAHQEBNQEAD_K12HW4__acrt_rounding_mode@@AEAV__crt_cached_ptd_host@@@Z 0000000180011eac f   libucrt:cvt.obj
 0001:00010f84       ?fp_format_f_internal@@YAHQEAD_KHQEAU_strflt@@_NAEAV__crt_cached_ptd_host@@@Z 0000000180011f84 f   libucrt:cvt.obj
 0001:000110dc       ?fp_format_g@@YAHQEBNQEAD_K12H_NIW4__acrt_rounding_mode@@AEAV__crt_cached_ptd_host@@@Z 00000001800120dc f   libucrt:cvt.obj
 0001:00011230       ?should_round_up@@YA_NQEBN_KFW4__acrt_rounding_mode@@@Z 0000000180012230 f   libucrt:cvt.obj
 0001:00011b04       ??$?RV<lambda_0ae27a3a962d80f24befdcbee591983d>@@AEAV<lambda_8d0ee55de4b1038c4002e0adecdf1839>@@V<lambda_dc504788e8f1664fe9b84e20bfb512f2>@@@?$__crt_seh_guarded_call@X@@QEAAX$$QEAV<lambda_0ae27a3a962d80f24befdcbee591983d>@@AEAV<lambda_8d0ee55de4b1038c4002e0adecdf1839>@@$$QEAV<lambda_dc504788e8f1664fe9b84e20bfb512f2>@@@Z 0000000180012b04 f   libucrt:per_thread_data.obj
 0001:00011b44       ??$?RV<lambda_2d41944a1d46af3157314b8a01080d33>@@AEAV<lambda_8f455de75cd7d7f24b4096f044d8b9e6>@@V<lambda_aa500f224e6afead328df44964fe2772>@@@?$__crt_seh_guarded_call@X@@QEAAX$$QEAV<lambda_2d41944a1d46af3157314b8a01080d33>@@AEAV<lambda_8f455de75cd7d7f24b4096f044d8b9e6>@@$$QEAV<lambda_aa500f224e6afead328df44964fe2772>@@@Z 0000000180012b44 f   libucrt:per_thread_data.obj
 0001:00011b84       ??$?RV<lambda_aa87e3671a710a21b5dc78c0bdf72e11>@@AEAV<lambda_92619d2358a28f41a33ba319515a20b9>@@V<lambda_6992ecaafeb10aed2b74cb1fae11a551>@@@?$__crt_seh_guarded_call@X@@QEAAX$$QEAV<lambda_aa87e3671a710a21b5dc78c0bdf72e11>@@AEAV<lambda_92619d2358a28f41a33ba319515a20b9>@@$$QEAV<lambda_6992ecaafeb10aed2b74cb1fae11a551>@@@Z 0000000180012b84 f   libucrt:per_thread_data.obj
 0001:00011bcc       ??$?RV<lambda_f2e299630e499de9f9a165e60fcd3db5>@@AEAV<lambda_2ae9d31cdba2644fcbeaf08da7c24588>@@V<lambda_40d01ff24d0e7b3814fdbdcee8eab3c7>@@@?$__crt_seh_guarded_call@X@@QEAAX$$QEAV<lambda_f2e299630e499de9f9a165e60fcd3db5>@@AEAV<lambda_2ae9d31cdba2644fcbeaf08da7c24588>@@$$QEAV<lambda_40d01ff24d0e7b3814fdbdcee8eab3c7>@@@Z 0000000180012bcc f   libucrt:per_thread_data.obj
 0001:00011c2c       ?construct_ptd_array@@YAXQEAU__acrt_ptd@@@Z 0000000180012c2c f   libucrt:per_thread_data.obj
 0001:00011cfc       ?destroy_fls@@YAXPEAX@Z    0000000180012cfc f   libucrt:per_thread_data.obj
 0001:00011d1c       ?destroy_ptd_array@@YAXQEAU__acrt_ptd@@@Z 0000000180012d1c f   libucrt:per_thread_data.obj
 0001:00011e14       ?replace_current_thread_locale_nolock@@YAXQEAU__acrt_ptd@@QEAU__crt_locale_data@@@Z 0000000180012e14 f   libucrt:per_thread_data.obj
 0001:00012220       ??$?RV<lambda_410d79af7f07d98d83a3f525b3859a53>@@AEAV<lambda_3e16ef9562a7dcce91392c22ab16ea36>@@V<lambda_38119f0e861e05405d8a144b9b982f0a>@@@?$__crt_seh_guarded_call@X@@QEAAX$$QEAV<lambda_410d79af7f07d98d83a3f525b3859a53>@@AEAV<lambda_3e16ef9562a7dcce91392c22ab16ea36>@@$$QEAV<lambda_38119f0e861e05405d8a144b9b982f0a>@@@Z 0000000180013220 f   libucrt:wsetlocale.obj
 0001:000122cc       ??$?RV<lambda_ad8af0d99a0adf03d037d7dffe354bb5>@@AEAV<lambda_c9ba49e555ba839a7b07aa3fbecb7617>@@V<lambda_2f1ebd5d68526518146ae959c9e734c8>@@@?$__crt_seh_guarded_call@H@@QEAAH$$QEAV<lambda_ad8af0d99a0adf03d037d7dffe354bb5>@@AEAV<lambda_c9ba49e555ba839a7b07aa3fbecb7617>@@$$QEAV<lambda_2f1ebd5d68526518146ae959c9e734c8>@@@Z 00000001800132cc f   libucrt:close.obj
 0001:000125e4       ?find_or_allocate_unused_stream_nolock@@YA?AV__crt_stdio_stream@@XZ 00000001800135e4 f   libucrt:stream.obj
 0001:00012d00       ?<lambda_invoker_cdecl>@<lambda_a1ce4c8ae42411fd470c77163914f50e>@@CAHPEBX0@Z 0000000180013d00 f   libucrt:argv_wildcards.obj
 0001:0001301c       ??$common_expand_argv_wildcards@D@@YAHQEAPEADQEAPEAPEAD@Z 000000018001401c f   libucrt:argv_wildcards.obj
 0001:00013260       ??$copy_and_add_argument_to_buffer@D@@YAHQEBD0_KAEAV?$argument_list@D@?A0x5f5c8891@@@Z 0000000180014260 f   libucrt:argv_wildcards.obj
 0001:000133e4       ??$expand_argument_wildcards@D@@YAHQEAD0AEAV?$argument_list@D@?A0x5f5c8891@@@Z 00000001800143e4 f   libucrt:argv_wildcards.obj
 0001:0001397c       ??$?RV<lambda_efdfa57d1f175319df784efa44bb7b81>@@AEAV<lambda_5f0a4c1567f8adc6734073e5d1e1b35c>@@V<lambda_2e8a7d3640ea6ccb4c2413664c2db6fd>@@@?$__crt_seh_guarded_call@X@@QEAAX$$QEAV<lambda_efdfa57d1f175319df784efa44bb7b81>@@AEAV<lambda_5f0a4c1567f8adc6734073e5d1e1b35c>@@$$QEAV<lambda_2e8a7d3640ea6ccb4c2413664c2db6fd>@@@Z 000000018001497c f   libucrt:mbctype.obj
 0001:00013b4c       ?getSystemCP@@YAHH@Z       0000000180014b4c f   libucrt:mbctype.obj
 0001:00013bcc       ?setSBCS@@YAXPEAU__crt_multibyte_data@@@Z 0000000180014bcc f   libucrt:mbctype.obj
 0001:00013c64       ?setSBUpLow@@YAXPEAU__crt_multibyte_data@@@Z 0000000180014c64 f   libucrt:mbctype.obj
 0001:00013e4c       ?setmbcp_internal@@YAHH_NQEAU__acrt_ptd@@QEAPEAU__crt_multibyte_data@@@Z 0000000180014e4c f   libucrt:mbctype.obj
 0001:000140bc       ?update_thread_multibyte_data_internal@@YAPEAU__crt_multibyte_data@@QEAU__acrt_ptd@@QEAPEAU1@@Z 00000001800150bc f   libucrt:mbctype.obj
 0001:000144b0       ?x_ismbbtype_l@@YAHPEAU__crt_locale_pointers@@IHH@Z 00000001800154b0 f   libucrt:ismbbyte.obj
 0001:000147e0       ??$common_set_variable_in_environment_nolock@D@@YAHQEADH@Z 00000001800157e0 f   libucrt:setenv.obj
 0001:00014b38       ??$copy_environment@D@@YAPEAPEADQEAPEAD@Z 0000000180015b38 f   libucrt:setenv.obj
 0001:00014dc4       ??$?RV<lambda_450d765d439847d4c735a33c368b5fc0>@@AEAV<lambda_44731a7d0e6d81c3e6aa82d741081786>@@V<lambda_601a2a7da3b7a96e9554ac7215c4b07c>@@@?$__crt_seh_guarded_call@P6AXH@Z@@QEAAP6AXH@Z$$QEAV<lambda_450d765d439847d4c735a33c368b5fc0>@@AEAV<lambda_44731a7d0e6d81c3e6aa82d741081786>@@$$QEAV<lambda_601a2a7da3b7a96e9554ac7215c4b07c>@@@Z 0000000180015dc4 f   libucrt:signal.obj
 0001:000151e8       ??$?RV<lambda_a37b2b86f63e897a80ea819b0eb08c01>@@AEAV<lambda_38ce7e780aa69e748d6df282ebc68efe>@@V<lambda_99fb1378e971ab6e7edea83e3a7a83a2>@@@?$__crt_seh_guarded_call@H@@QEAAH$$QEAV<lambda_a37b2b86f63e897a80ea819b0eb08c01>@@AEAV<lambda_38ce7e780aa69e748d6df282ebc68efe>@@$$QEAV<lambda_99fb1378e971ab6e7edea83e3a7a83a2>@@@Z 00000001800161e8 f   libucrt:commit.obj
 0001:00015308       ?write_double_translated_ansi_nolock@@YA?AUwrite_result@?A0x17268360@@HQEBDIAEAV__crt_cached_ptd_host@@@Z 0000000180016308 f   libucrt:write.obj
 0001:00015780       ?write_text_ansi_nolock@@YA?AUwrite_result@?A0x17268360@@HQEBDI@Z 0000000180016780 f   libucrt:write.obj
 0001:00015884       ?write_text_utf16le_nolock@@YA?AUwrite_result@?A0x17268360@@HQEBDI@Z 0000000180016884 f   libucrt:write.obj
 0001:000159a0       ?write_text_utf8_nolock@@YA?AUwrite_result@?A0x17268360@@HQEBDI@Z 00000001800169a0 f   libucrt:write.obj
 0001:00016900       ?should_round_up@@YA_NQEBD0HW4__acrt_has_trailing_digits@@W4__acrt_rounding_mode@@@Z 0000000180017900 f   libucrt:_fptostr.obj
 0001:0001820c       memcpy_s                   000000018001920c f   libucrt:cfout.obj
 0001:00018534       ??$write_buffer_nolock@D@@YA_NDV__crt_stdio_stream@@AEAV__crt_cached_ptd_host@@@Z 0000000180019534 f   libucrt:_flsbuf.obj
 0001:0001862c       ?stream_is_at_end_of_file_nolock@@YA_NV__crt_stdio_stream@@@Z 000000018001962c f   libucrt:_flsbuf.obj
 0001:0001894c       ?free_crt_array_internal@@YAXQEAPEBX_K@Z 000000018001994c f   libucrt:inittime.obj
 0001:00018db0       ??$common_sopen_dispatch@D@@YAHQEBDHHHQEAHH@Z 0000000180019db0 f   libucrt:open.obj
 0001:00018e74       ?configure_text_mode@@YAHHUfile_options@?A0xa9d50aae@@HAEAW4__crt_lowio_text_mode@@@Z 0000000180019e74 f   libucrt:open.obj
 0001:000190f4       ?decode_options@@YA?AUfile_options@?A0xa9d50aae@@HHH@Z 000000018001a0f4 f   libucrt:open.obj
 0001:000192fc       ?truncate_ctrl_z_if_present@@YAHH@Z 000000018001a2fc f   libucrt:open.obj
 0001:00019900       ?InternalCompareStringA@@YAHPEAU__crt_locale_pointers@@PEB_WKPEBDH2HH@Z 000000018001a900 f   libucrt:comparestringa.obj
 0001:0001a210       fallbackMethod             000000018001b210 f   libucrt:strpbrk.obj
 0001:0001a5bc       $LN79                      000000018001b5bc     libucrt:strpbrk.obj
 0001:0001a5f8       $LN78                      000000018001b5f8     libucrt:strpbrk.obj
 0001:0001a638       $LN77                      000000018001b638     libucrt:strpbrk.obj
 0001:0001a714       ?__acrt_LCMapStringA_stat@@YAHPEAU__crt_locale_pointers@@PEB_WKPEBDHPEADHHH@Z 000000018001b714 f   libucrt:lcmapstringa.obj
 0001:0001aae0       ?initialize_multibyte@@YAHXZ 000000018001bae0 f   libucrt:multibyte_initializer.obj
 0001:0001ad50       ??$common_lseek@_J@@YA_JH_JHAEAV__crt_cached_ptd_host@@@Z 000000018001bd50 f   libucrt:lseek.obj
 0001:0001ae70       ??$common_lseek_nolock@_J@@YA_JH_JHAEAV__crt_cached_ptd_host@@@Z 000000018001be70 f   libucrt:lseek.obj
 0001:0001b098       ??$translate_text_mode_nolock@_W@@YAHHQEA_W_K@Z 000000018001c098 f   libucrt:read.obj
 0001:0001b258       ?translate_ansi_or_utf8_nolock@@YAHHQEAD_KQEA_W1@Z 000000018001c258 f   libucrt:read.obj
 0001:0001bb70       $$000000                   000000018001cb70     libucrt:log10.obj
 0001:0001cb70       common_control87           000000018001db70 f   libucrt:ieee.obj
 0001:0001ce0c       _call_matherr              000000018001de0c f   libucrt:libm_error.obj
 0001:0001ce74       _exception_enabled         000000018001de74 f   libucrt:libm_error.obj
 0001:0001d110       _log_special_common        000000018001e110 f   libucrt:log_special.obj
 0001:0001d1d0       $$000000                   000000018001e1d0     libucrt:fpsr.obj
 0001:0001d940       $$000000                   000000018001e940     libvcruntime:memcmp.obj
 0001:0001daa0       $$000000                   000000018001eaa0     LIBCMT:guard_dispatch.obj
 0001:0001dac0       $$000000                   000000018001eac0     LIBCMT:guard_xfg_dispatch.obj
 0001:0001dae0       ?fin$0@?0??dllmain_crt_process_attach@@YAHQEAUHINSTANCE__@@QEAX@Z@4HA 000000018001eae0 f   LIBCMT:dll_dllmain.obj
 0001:0001daf7       ?fin$0@?0??dllmain_crt_process_detach@@YAH_N@Z@4HA 000000018001eaf7 f   LIBCMT:dll_dllmain.obj
 0001:0001db10       ?fin$1@?0??dllmain_crt_process_detach@@YAH_N@Z@4HA 000000018001eb10 f   LIBCMT:dll_dllmain.obj
 0001:0001db24       ?filt$0@?0??dllmain_dispatch@@YAHQEAUHINSTANCE__@@KQEAX@Z@4HA 000000018001eb24 f   LIBCMT:dll_dllmain.obj
 0001:0001db5a       __scrt_is_nonwritable_in_current_image$filt$0 000000018001eb5a f   LIBCMT:utility.obj
 0001:0001db72       __DestructExceptionObject$filt$0 000000018001eb72 f   libvcruntime:ehhelpers.obj
 0001:0001dc08       ?filt$0@?0???$_CallSETranslator@V__FrameHandler3@@@@YAHPEAUEHExceptionRecord@@PEA_KPEAU_CONTEXT@@PEAU_xDISPATCHER_CONTEXT@@PEBU_s_FuncInfo@@K1H@Z@4HA 000000018001ec08 f   libvcruntime:risctrnsctrl.obj
 0001:0001dcab       ?filt$0@?0??CxxCallCatchBlock@__FrameHandler3@@SAPEAXPEAU_EXCEPTION_RECORD@@@Z@4HA 000000018001ecab f   libvcruntime:frame.obj
 0001:0001dcd0       ?fin$1@?0??CxxCallCatchBlock@__FrameHandler3@@SAPEAXPEAU_EXCEPTION_RECORD@@@Z@4HA 000000018001ecd0 f   libvcruntime:frame.obj
 0001:0001dd56       ?filt$0@?0??FrameUnwindToState@__FrameHandler3@@SAXPEA_KPEAU_xDISPATCHER_CONTEXT@@PEBU_s_FuncInfo@@H@Z@4HA 000000018001ed56 f   libvcruntime:frame.obj
 0001:0001dd6c       ?fin$1@?0??FrameUnwindToState@__FrameHandler3@@SAXPEA_KPEAU_xDISPATCHER_CONTEXT@@PEBU_s_FuncInfo@@H@Z@4HA 000000018001ed6c f   libvcruntime:frame.obj
 0001:0001dd8f       ?fin$0@?0???$?RV<lambda_842d9ff0dc9ef11c61343bbaebe7f885>@@AEAV<lambda_c5860995281e5c4ce005b3de8f5874ee>@@V<lambda_d90129c13df834fdcbf8d2b88dafcf2d>@@@?$__crt_seh_guarded_call@X@@QEAAX$$QEAV<lambda_842d9ff0dc9ef11c61343bbaebe7f885>@@AEAV<lambda_c5860995281e5c4ce005b3de8f5874ee>@@$$QEAV<lambda_d90129c13df834fdcbf8d2b88dafcf2d>@@@Z@4HA 000000018001ed8f f   libucrt:fflush.obj
 0001:0001dd8f       ?fin$0@?0???$?RV<lambda_d854c62834386a3b23916ad6dae2782d>@@AEAV<lambda_303760bc4008a2b3ec4768a30b06a80c>@@V<lambda_4780a7ea4f8cbd2590aec34bd14e2bbf>@@@?$__crt_seh_guarded_call@H@@QEAAH$$QEAV<lambda_d854c62834386a3b23916ad6dae2782d>@@AEAV<lambda_303760bc4008a2b3ec4768a30b06a80c>@@$$QEAV<lambda_4780a7ea4f8cbd2590aec34bd14e2bbf>@@@Z@4HA 000000018001ed8f f   libucrt:output.obj
 0001:0001ddaa       ?fin$0@?0??_fclose_internal@@YAHQEAU_iobuf@@AEAV__crt_cached_ptd_host@@@Z@4HA 000000018001edaa f   libucrt:fclose.obj
 0001:0001ddc2       ?fin$0@?0???$common_fsopen@D@@YAPEAU_iobuf@@QEBD0H@Z@4HA 000000018001edc2 f   libucrt:fopen.obj
 0001:0001dded       ?fin$0@?0???$common_getenv@D@@YAPEADQEBD@Z@4HA 000000018001eded f   libucrt:getenv.obj
 0001:0001de06       _query_new_handler$fin$0   000000018001ee06 f   libucrt:new_handler.obj
 0001:0001de1c       ?fin$0@?0???$?RV<lambda_0ae27a3a962d80f24befdcbee591983d>@@AEAV<lambda_8d0ee55de4b1038c4002e0adecdf1839>@@V<lambda_dc504788e8f1664fe9b84e20bfb512f2>@@@?$__crt_seh_guarded_call@X@@QEAAX$$QEAV<lambda_0ae27a3a962d80f24befdcbee591983d>@@AEAV<lambda_8d0ee55de4b1038c4002e0adecdf1839>@@$$QEAV<lambda_dc504788e8f1664fe9b84e20bfb512f2>@@@Z@4HA 000000018001ee1c f   libucrt:per_thread_data.obj
 0001:0001de1c       ?fin$0@?0???$?RV<lambda_2d41944a1d46af3157314b8a01080d33>@@AEAV<lambda_8f455de75cd7d7f24b4096f044d8b9e6>@@V<lambda_aa500f224e6afead328df44964fe2772>@@@?$__crt_seh_guarded_call@X@@QEAAX$$QEAV<lambda_2d41944a1d46af3157314b8a01080d33>@@AEAV<lambda_8f455de75cd7d7f24b4096f044d8b9e6>@@$$QEAV<lambda_aa500f224e6afead328df44964fe2772>@@@Z@4HA 000000018001ee1c f   libucrt:per_thread_data.obj
 0001:0001de1c       ?fin$0@?0???$?RV<lambda_aa87e3671a710a21b5dc78c0bdf72e11>@@AEAV<lambda_92619d2358a28f41a33ba319515a20b9>@@V<lambda_6992ecaafeb10aed2b74cb1fae11a551>@@@?$__crt_seh_guarded_call@X@@QEAAX$$QEAV<lambda_aa87e3671a710a21b5dc78c0bdf72e11>@@AEAV<lambda_92619d2358a28f41a33ba319515a20b9>@@$$QEAV<lambda_6992ecaafeb10aed2b74cb1fae11a551>@@@Z@4HA 000000018001ee1c f   libucrt:per_thread_data.obj
 0001:0001de1c       ?fin$0@?0???$?RV<lambda_f2e299630e499de9f9a165e60fcd3db5>@@AEAV<lambda_2ae9d31cdba2644fcbeaf08da7c24588>@@V<lambda_40d01ff24d0e7b3814fdbdcee8eab3c7>@@@?$__crt_seh_guarded_call@X@@QEAAX$$QEAV<lambda_f2e299630e499de9f9a165e60fcd3db5>@@AEAV<lambda_2ae9d31cdba2644fcbeaf08da7c24588>@@$$QEAV<lambda_40d01ff24d0e7b3814fdbdcee8eab3c7>@@@Z@4HA 000000018001ee1c f   libucrt:per_thread_data.obj
 0001:0001de1c       ?fin$0@?0???$?RV<lambda_450d765d439847d4c735a33c368b5fc0>@@AEAV<lambda_44731a7d0e6d81c3e6aa82d741081786>@@V<lambda_601a2a7da3b7a96e9554ac7215c4b07c>@@@?$__crt_seh_guarded_call@P6AXH@Z@@QEAAP6AXH@Z$$QEAV<lambda_450d765d439847d4c735a33c368b5fc0>@@AEAV<lambda_44731a7d0e6d81c3e6aa82d741081786>@@$$QEAV<lambda_601a2a7da3b7a96e9554ac7215c4b07c>@@@Z@4HA 000000018001ee1c f   libucrt:signal.obj
 0001:0001de1c       ?fin$0@?0???$?RV<lambda_d80eeec6fff315bfe5c115232f3240e3>@@AEAV<lambda_6e4b09c48022b2350581041d5f6b0c4c>@@V<lambda_2358e3775559c9db80273638284d5e45>@@@?$__crt_seh_guarded_call@X@@QEAAX$$QEAV<lambda_d80eeec6fff315bfe5c115232f3240e3>@@AEAV<lambda_6e4b09c48022b2350581041d5f6b0c4c>@@$$QEAV<lambda_2358e3775559c9db80273638284d5e45>@@@Z@4HA 000000018001ee1c f   libucrt:exit.obj
 0001:0001de1c       ?fin$0@?0???$?RV<lambda_7777bce6b2f8c936911f934f8298dc43>@@AEAV<lambda_f03950bc5685219e0bcd2087efbe011e>@@V<lambda_3883c3dff614d5e0c5f61bb1ac94921c>@@@?$__crt_seh_guarded_call@H@@QEAAH$$QEAV<lambda_7777bce6b2f8c936911f934f8298dc43>@@AEAV<lambda_f03950bc5685219e0bcd2087efbe011e>@@$$QEAV<lambda_3883c3dff614d5e0c5f61bb1ac94921c>@@@Z@4HA 000000018001ee1c f   libucrt:onexit.obj
 0001:0001de36       ?filt$0@?0???R<lambda_6e4b09c48022b2350581041d5f6b0c4c>@@QEBA@XZ@4HA 000000018001ee36 f   libucrt:exit.obj
 0001:0001de63       _fcloseall$fin$0           000000018001ee63 f   libucrt:closeall.obj
 0001:0001de63       ?fin$0@?0??__acrt_stdio_allocate_stream@@YA?AV__crt_stdio_stream@@XZ@4HA 000000018001ee63 f   libucrt:stream.obj
 0001:0001de7c       ?fin$0@?0???$?RV<lambda_886d6c58226a84441f68b9f2b8217b83>@@AEAV<lambda_ab61a845afdef5b7c387490eaf3616ee>@@V<lambda_f7f22ab5edc0698d5f6905b0d3f44752>@@@?$__crt_seh_guarded_call@X@@QEAAX$$QEAV<lambda_886d6c58226a84441f68b9f2b8217b83>@@AEAV<lambda_ab61a845afdef5b7c387490eaf3616ee>@@$$QEAV<lambda_f7f22ab5edc0698d5f6905b0d3f44752>@@@Z@4HA 000000018001ee7c f   libucrt:fflush.obj
 0001:0001de99       __acrt_initialize_lowio$fin$0 000000018001ee99 f   libucrt:ioinit.obj
 0001:0001de99       __acrt_lowio_ensure_fh_exists$fin$0 000000018001ee99 f   libucrt:osfinfo.obj
 0001:0001de99       _alloc_osfhnd$fin$0        000000018001ee99 f   libucrt:osfinfo.obj
 0001:0001deb2       ?fin$0@?0???$?RV<lambda_410d79af7f07d98d83a3f525b3859a53>@@AEAV<lambda_3e16ef9562a7dcce91392c22ab16ea36>@@V<lambda_38119f0e861e05405d8a144b9b982f0a>@@@?$__crt_seh_guarded_call@X@@QEAAX$$QEAV<lambda_410d79af7f07d98d83a3f525b3859a53>@@AEAV<lambda_3e16ef9562a7dcce91392c22ab16ea36>@@$$QEAV<lambda_38119f0e861e05405d8a144b9b982f0a>@@@Z@4HA 000000018001eeb2 f   libucrt:wsetlocale.obj
 0001:0001decc       ?fin$0@?0???$?RV<lambda_ad8af0d99a0adf03d037d7dffe354bb5>@@AEAV<lambda_c9ba49e555ba839a7b07aa3fbecb7617>@@V<lambda_2f1ebd5d68526518146ae959c9e734c8>@@@?$__crt_seh_guarded_call@H@@QEAAH$$QEAV<lambda_ad8af0d99a0adf03d037d7dffe354bb5>@@AEAV<lambda_c9ba49e555ba839a7b07aa3fbecb7617>@@$$QEAV<lambda_2f1ebd5d68526518146ae959c9e734c8>@@@Z@4HA 000000018001eecc f   libucrt:close.obj
 0001:0001decc       ?fin$0@?0???$?RV<lambda_a37b2b86f63e897a80ea819b0eb08c01>@@AEAV<lambda_38ce7e780aa69e748d6df282ebc68efe>@@V<lambda_99fb1378e971ab6e7edea83e3a7a83a2>@@@?$__crt_seh_guarded_call@H@@QEAAH$$QEAV<lambda_a37b2b86f63e897a80ea819b0eb08c01>@@AEAV<lambda_38ce7e780aa69e748d6df282ebc68efe>@@$$QEAV<lambda_99fb1378e971ab6e7edea83e3a7a83a2>@@@Z@4HA 000000018001eecc f   libucrt:commit.obj
 0001:0001dee6       ?fin$0@?0???$?RV<lambda_efdfa57d1f175319df784efa44bb7b81>@@AEAV<lambda_5f0a4c1567f8adc6734073e5d1e1b35c>@@V<lambda_2e8a7d3640ea6ccb4c2413664c2db6fd>@@@?$__crt_seh_guarded_call@X@@QEAAX$$QEAV<lambda_efdfa57d1f175319df784efa44bb7b81>@@AEAV<lambda_5f0a4c1567f8adc6734073e5d1e1b35c>@@$$QEAV<lambda_2e8a7d3640ea6ccb4c2413664c2db6fd>@@@Z@4HA 000000018001eee6 f   libucrt:mbctype.obj
 0001:0001df00       ?fin$0@?0??update_thread_multibyte_data_internal@@YAPEAU__crt_multibyte_data@@QEAU__acrt_ptd@@QEAPEAU1@@Z@4HA 000000018001ef00 f   libucrt:mbctype.obj
 0001:0001df19       raise$fin$0                000000018001ef19 f   libucrt:signal.obj
 0001:0001df3a       ?fin$0@?0???$common_lseek@_J@@YA_JH_JHAEAV__crt_cached_ptd_host@@@Z@4HA 000000018001ef3a f   libucrt:lseek.obj
 0001:0001df3a       _write_internal$fin$0      000000018001ef3a f   libucrt:write.obj
 0001:0001df51       __acrt_update_thread_locale_data$fin$0 000000018001ef51 f   libucrt:locale_refcounting.obj
 0001:0001df6a       ?fin$0@?0???$common_sopen_dispatch@D@@YAHQEBDHHHQEAHH@Z@4HA 000000018001ef6a f   libucrt:open.obj
 0001:0001dfe2       _ctrlfp$filt$0             000000018001efe2 f   libucrt:fpctrl.obj
 0001:0001dfe2       common_control87$filt$0    000000018001efe2 f   libucrt:ieee.obj
 0001:0001e010       _IsNonwritableInCurrentImage$filt$0 000000018001f010 f   LIBCMT:pesect.obj
 0002:000039e8       GS_ExceptionPointers       00000001800239e8     LIBCMT:gs_report.obj
 0002:00003a50       ?tokenTable@@3QBUStringLiteral@@B 0000000180023a50     libvcruntime:undname.obj
 0002:00003b60       ?nameTable@@3QBUStringLiteral@@B 0000000180023b60     libvcruntime:undname.obj
 0002:00004090       ?rttiTable@@3QBUStringLiteral@@B 0000000180024090     libvcruntime:undname.obj
 0002:000040e0       ?IndirectionName@@3QBUStringLiteral@@B 00000001800240e0     libvcruntime:undname.obj
 0002:00004140       ?PrefixName@@3QBUStringLiteral@@B 0000000180024140     libvcruntime:undname.obj
 0002:00004830       ?ExceptionTemplate@?1??UnwindNestedFrames@__FrameHandler3@@SAXPEA_KPEAUEHExceptionRecord@@PEAU_CONTEXT@@0PEAXPEBU_s_FuncInfo@@HHPEBU_s_HandlerType@@PEAU_xDISPATCHER_CONTEXT@@E@Z@4U_EXCEPTION_RECORD@@B 0000000180024830     libvcruntime:risctrnsctrl.obj
 0002:000048c8       ?module_names@?A0x14174aea@@3QBQEB_WB 00000001800248c8     libvcruntime:winapi_downlevel.obj
 0002:00004988       ?candidate_modules@?1??try_get_FlsAlloc@@YAP6AKP6AXPEAX@Z@ZXZ@4QBW4module_id@?A0x14174aea@@B 0000000180024988     libvcruntime:winapi_downlevel.obj
 0002:000049a0       ?candidate_modules@?1??try_get_FlsFree@@YAP6AHK@ZXZ@4QBW4module_id@?A0x14174aea@@B 00000001800249a0     libvcruntime:winapi_downlevel.obj
 0002:000049b0       ?candidate_modules@?1??try_get_FlsGetValue@@YAP6APEAXK@ZXZ@4QBW4module_id@?A0x14174aea@@B 00000001800249b0     libvcruntime:winapi_downlevel.obj
 0002:000049c8       ?candidate_modules@?1??try_get_FlsSetValue@@YAP6AHKPEAX@ZXZ@4QBW4module_id@?A0x14174aea@@B 00000001800249c8     libvcruntime:winapi_downlevel.obj
 0002:000049e0       ?candidate_modules@?1??try_get_InitializeCriticalSectionEx@@YAP6AHPEAU_RTL_CRITICAL_SECTION@@KK@ZXZ@4QBW4module_id@?A0x14174aea@@B 00000001800249e0     libvcruntime:winapi_downlevel.obj
 0002:00004c28       $cppxdata$?try_cor_exit_process@@YAXI@Z 0000000180024c28     libucrt:exit.obj
 0002:00004c50       $cppxdata$?common_exit@@YAXHW4_crt_exit_cleanup_mode@@W4_crt_exit_return_mode@@@Z 0000000180024c50     libucrt:exit.obj
 0002:00004ca0       $cppxdata$__dcrt_uninitialize_environments_nolock 0000000180024ca0     libucrt:environment_initialization.obj
 0002:00004cc8       $cppxdata$_execute_onexit_table 0000000180024cc8     libucrt:onexit.obj
 0002:00004cf0       __acrt_initializers        0000000180024cf0     libucrt:initialization.obj
 0002:00004df0       ?errtable@@3QBUerrentry@?A0x31fdb9ec@@B 0000000180024df0     libucrt:errno.obj
 0002:00004f60       ?module_names@?A0x391cf84c@@3QBQEB_WB 0000000180024f60     libucrt:winapi_thunks.obj
 0002:000054b8       ?candidate_modules@?1??try_get_AreFileApisANSI@@YAP6AHXZXZ@4QBW4module_id@?A0x391cf84c@@B 00000001800254b8     libucrt:winapi_thunks.obj
 0002:000054d0       ?candidate_modules@?1??try_get_CompareStringEx@@YAP6AHPEB_WK0H0HPEAU_nlsversioninfo@@PEAX_J@ZXZ@4QBW4module_id@?A0x391cf84c@@B 00000001800254d0     libucrt:winapi_thunks.obj
 0002:000054e8       ?candidate_modules@?1??try_get_InitializeCriticalSectionEx@@YAP6AHPEAU_RTL_CRITICAL_SECTION@@KK@ZXZ@4QBW4module_id@?A0x391cf84c@@B 00000001800254e8     libucrt:winapi_thunks.obj
 0002:000054f0       ?candidate_modules@?1??try_get_LCMapStringEx@@YAP6AHPEB_WK0HPEA_WHPEAU_nlsversioninfo@@PEAX_J@ZXZ@4QBW4module_id@?A0x391cf84c@@B 00000001800254f0     libucrt:winapi_thunks.obj
 0002:00005508       ?candidate_modules@?1??try_get_LocaleNameToLCID@@YAP6AKPEB_WK@ZXZ@4QBW4module_id@?A0x391cf84c@@B 0000000180025508     libucrt:winapi_thunks.obj
 0002:00005524       ?candidate_modules@?1??try_get_AppPolicyGetProcessTerminationMethod@@YAP6AJPEAXPEAW4AppPolicyProcessTerminationMethod@@@ZXZ@4QBW4module_id@?A0x391cf84c@@B 0000000180025524     libucrt:winapi_thunks.obj
 0002:00005550       ?strings@?1??fp_format_nan_or_infinity@@YAHW4__acrt_fp_class@@_NPEAD_K1@Z@4QAY03QEBDA 0000000180025550     libucrt:cvt.obj
 0002:00005cc8       ?_mb_locale_names@@3QBQEB_WB 0000000180025cc8     libucrt:mbctype.obj
 0002:00006330       ?LcidToLocaleNameTable@?A0x881e4c05@@3QBULcidToLocaleName@1@B 0000000180026330     libucrt:lcidtoname_downlevel.obj
 0002:00007d90       ?LocaleNameToIndexTable@?A0x881e4c05@@3QBULocaleNameIndex@1@B 0000000180027d90     libucrt:lcidtoname_downlevel.obj
 0002:00009628       $cppxdata$?write_double_translated_ansi_nolock@@YA?AUwrite_result@?A0x17268360@@HQEBDIAEAV__crt_cached_ptd_host@@@Z 0000000180029628     libucrt:write.obj
 0002:0000a050       __real_ninf                000000018002a050     libucrt:log10.obj
 0002:0000a060       __real_inf                 000000018002a060     libucrt:log10.obj
 0002:0000a070       __real_neg_qnan            000000018002a070     libucrt:log10.obj
 0002:0000a080       __real_qnanbit             000000018002a080     libucrt:log10.obj
 0002:0000a090       __int_1023                 000000018002a090     libucrt:log10.obj
 0002:0000a0a0       __mask_001                 000000018002a0a0     libucrt:log10.obj
 0002:0000a0b0       __mask_mant                000000018002a0b0     libucrt:log10.obj
 0002:0000a0c0       __mask_mant_top8           000000018002a0c0     libucrt:log10.obj
 0002:0000a0d0       __mask_mant9               000000018002a0d0     libucrt:log10.obj
 0002:0000a0e0       __real_log10_e             000000018002a0e0     libucrt:log10.obj
 0002:0000a0f0       __real_log10_e_lead        000000018002a0f0     libucrt:log10.obj
 0002:0000a100       __real_log10_e_tail        000000018002a100     libucrt:log10.obj
 0002:0000a110       __real_log10_2_lead        000000018002a110     libucrt:log10.obj
 0002:0000a120       __real_log10_2_tail        000000018002a120     libucrt:log10.obj
 0002:0000a130       __real_two                 000000018002a130     libucrt:log10.obj
 0002:0000a140       __real_one                 000000018002a140     libucrt:log10.obj
 0002:0000a150       __real_half                000000018002a150     libucrt:log10.obj
 0002:0000a160       __mask_100                 000000018002a160     libucrt:log10.obj
 0002:0000a170       __real_1_over_512          000000018002a170     libucrt:log10.obj
 0002:0000a180       __real_1_over_2            000000018002a180     libucrt:log10.obj
 0002:0000a190       __real_1_over_3            000000018002a190     libucrt:log10.obj
 0002:0000a1a0       __real_1_over_4            000000018002a1a0     libucrt:log10.obj
 0002:0000a1b0       __real_1_over_5            000000018002a1b0     libucrt:log10.obj
 0002:0000a1c0       __real_1_over_6            000000018002a1c0     libucrt:log10.obj
 0002:0000a1d0       __real_neg_1023            000000018002a1d0     libucrt:log10.obj
 0002:0000a1e0       __mask_2045                000000018002a1e0     libucrt:log10.obj
 0002:0000a1f0       __real_threshold           000000018002a1f0     libucrt:log10.obj
 0002:0000a200       __real_near_one_lt         000000018002a200     libucrt:log10.obj
 0002:0000a210       __real_near_one_gt         000000018002a210     libucrt:log10.obj
 0002:0000a220       __real_min_norm            000000018002a220     libucrt:log10.obj
 0002:0000a230       __real_notsign             000000018002a230     libucrt:log10.obj
 0002:0000a240       __real_ca1                 000000018002a240     libucrt:log10.obj
 0002:0000a250       __real_ca2                 000000018002a250     libucrt:log10.obj
 0002:0000a260       __real_ca3                 000000018002a260     libucrt:log10.obj
 0002:0000a270       __real_ca4                 000000018002a270     libucrt:log10.obj
 0002:0000a280       __mask_lower               000000018002a280     libucrt:log10.obj
 0002:0000a290       __flag_x_zero              000000018002a290     libucrt:log10.obj
 0002:0000a294       __flag_x_neg               000000018002a294     libucrt:log10.obj
 0002:0000a298       __flag_x_nan               000000018002a298     libucrt:log10.obj
 0002:0000baf0       __real@433fffffffffffff    000000018002baf0     libucrt:fpsr.obj
 0002:0000baf8       __real@c33fffffffffffff    000000018002baf8     libucrt:fpsr.obj
 0002:0000c5b8       $unwind$PrintDebugString   000000018002c5b8     AccessBridgeDebug.obj
 0002:0000c5c0       $unwind$initializeFileLogger 000000018002c5c0     AccessBridgeDebug.obj
 0002:0000c5c0       $unwind$?fp_format_f_internal@@YAHQEAD_KHQEAU_strflt@@_NAEAV__crt_cached_ptd_host@@@Z 000000018002c5c0     libucrt:cvt.obj
 0002:0000c5c0       $unwind$__acrt_DownlevelLocaleNameToLCID 000000018002c5c0     libucrt:lcidtoname_downlevel.obj
 0002:0000c5c0       $unwind$??R<lambda_f03950bc5685219e0bcd2087efbe011e>@@QEBA@XZ 000000018002c5c0     libucrt:onexit.obj
 0002:0000c5c0       $unwind$?write_string_impl@?$output_adapter_common@DV?$stream_output_adapter@D@__crt_stdio_output@@@__crt_stdio_output@@IEBAXQEBDHQEAHAEAV__crt_cached_ptd_host@@@Z 000000018002c5c0     libucrt:output.obj
 0002:0000c5d8       $unwind$finalizeFileLogger 000000018002c5d8     AccessBridgeDebug.obj
 0002:0000c5d8       $unwind$getTimeStamp       000000018002c5d8     AccessBridgeDebug.obj
 0002:0000c5d8       $unwind$?fireCaretUpdate@AccessBridgeEventHandler@@QEAAXJ_J0@Z 000000018002c5d8     AccessBridgeEventHandler.obj
 0002:0000c5d8       $unwind$?fireFocusGained@AccessBridgeEventHandler@@QEAAXJ_J0@Z 000000018002c5d8     AccessBridgeEventHandler.obj
 0002:0000c5d8       $unwind$?fireFocusLost@AccessBridgeEventHandler@@QEAAXJ_J0@Z 000000018002c5d8     AccessBridgeEventHandler.obj
 0002:0000c5d8       $unwind$?fireJavaShutdown@AccessBridgeEventHandler@@QEAAXJ@Z 000000018002c5d8     AccessBridgeEventHandler.obj
 0002:0000c5d8       $unwind$?fireMenuCanceled@AccessBridgeEventHandler@@QEAAXJ_J0@Z 000000018002c5d8     AccessBridgeEventHandler.obj
 0002:0000c5d8       $unwind$?fireMenuDeselected@AccessBridgeEventHandler@@QEAAXJ_J0@Z 000000018002c5d8     AccessBridgeEventHandler.obj
 0002:0000c5d8       $unwind$?fireMenuSelected@AccessBridgeEventHandler@@QEAAXJ_J0@Z 000000018002c5d8     AccessBridgeEventHandler.obj
 0002:0000c5d8       $unwind$?fireMouseClicked@AccessBridgeEventHandler@@QEAAXJ_J0@Z 000000018002c5d8     AccessBridgeEventHandler.obj
 0002:0000c5d8       $unwind$?fireMouseEntered@AccessBridgeEventHandler@@QEAAXJ_J0@Z 000000018002c5d8     AccessBridgeEventHandler.obj
 0002:0000c5d8       $unwind$?fireMouseExited@AccessBridgeEventHandler@@QEAAXJ_J0@Z 000000018002c5d8     AccessBridgeEventHandler.obj
 0002:0000c5d8       $unwind$?fireMousePressed@AccessBridgeEventHandler@@QEAAXJ_J0@Z 000000018002c5d8     AccessBridgeEventHandler.obj
 0002:0000c5d8       $unwind$?fireMouseReleased@AccessBridgeEventHandler@@QEAAXJ_J0@Z 000000018002c5d8     AccessBridgeEventHandler.obj
 0002:0000c5d8       $unwind$?firePopupMenuCanceled@AccessBridgeEventHandler@@QEAAXJ_J0@Z 000000018002c5d8     AccessBridgeEventHandler.obj
 0002:0000c5d8       $unwind$?firePopupMenuWillBecomeInvisible@AccessBridgeEventHandler@@QEAAXJ_J0@Z 000000018002c5d8     AccessBridgeEventHandler.obj
 0002:0000c5d8       $unwind$?firePopupMenuWillBecomeVisible@AccessBridgeEventHandler@@QEAAXJ_J0@Z 000000018002c5d8     AccessBridgeEventHandler.obj
 0002:0000c5d8       $unwind$?firePropertySelectionChange@AccessBridgeEventHandler@@QEAAXJ_J0@Z 000000018002c5d8     AccessBridgeEventHandler.obj
 0002:0000c5d8       $unwind$?firePropertyTextChange@AccessBridgeEventHandler@@QEAAXJ_J0@Z 000000018002c5d8     AccessBridgeEventHandler.obj
 0002:0000c5d8       $unwind$?firePropertyVisibleDataChange@AccessBridgeEventHandler@@QEAAXJ_J0@Z 000000018002c5d8     AccessBridgeEventHandler.obj
 0002:0000c5d8       $unwind$?initBroadcastMessageIDs@@YAHXZ 000000018002c5d8     AccessBridgeMessages.obj
 0002:0000c5d8       $unwind$Windows_run        000000018002c5d8     AccessBridgeWindowsEntryPoints.obj
 0002:0000c5d8       $unwind$addAccessibleSelectionFromContext 000000018002c5d8     AccessBridgeWindowsEntryPoints.obj
 0002:0000c5d8       $unwind$clearAccessibleSelectionFromContext 000000018002c5d8     AccessBridgeWindowsEntryPoints.obj
 0002:0000c5d8       $unwind$getVersionInfo     000000018002c5d8     AccessBridgeWindowsEntryPoints.obj
 0002:0000c5d8       $unwind$releaseJavaObject  000000018002c5d8     AccessBridgeWindowsEntryPoints.obj
 0002:0000c5d8       $unwind$removeAccessibleSelectionFromContext 000000018002c5d8     AccessBridgeWindowsEntryPoints.obj
 0002:0000c5d8       $unwind$selectAllAccessibleSelectionFromContext 000000018002c5d8     AccessBridgeWindowsEntryPoints.obj
 0002:0000c5d8       $unwind$setCaretUpdateFP   000000018002c5d8     AccessBridgeWindowsEntryPoints.obj
 0002:0000c5d8       $unwind$setFocusGainedFP   000000018002c5d8     AccessBridgeWindowsEntryPoints.obj
 0002:0000c5d8       $unwind$setFocusLostFP     000000018002c5d8     AccessBridgeWindowsEntryPoints.obj
 0002:0000c5d8       $unwind$setJavaShutdownFP  000000018002c5d8     AccessBridgeWindowsEntryPoints.obj
 0002:0000c5d8       $unwind$setMenuCanceledFP  000000018002c5d8     AccessBridgeWindowsEntryPoints.obj
 0002:0000c5d8       $unwind$setMenuDeselectedFP 000000018002c5d8     AccessBridgeWindowsEntryPoints.obj
 0002:0000c5d8       $unwind$setMenuSelectedFP  000000018002c5d8     AccessBridgeWindowsEntryPoints.obj
 0002:0000c5d8       $unwind$setMouseClickedFP  000000018002c5d8     AccessBridgeWindowsEntryPoints.obj
 0002:0000c5d8       $unwind$setMouseEnteredFP  000000018002c5d8     AccessBridgeWindowsEntryPoints.obj
 0002:0000c5d8       $unwind$setMouseExitedFP   000000018002c5d8     AccessBridgeWindowsEntryPoints.obj
 0002:0000c5d8       $unwind$setMousePressedFP  000000018002c5d8     AccessBridgeWindowsEntryPoints.obj
 0002:0000c5d8       $unwind$setMouseReleasedFP 000000018002c5d8     AccessBridgeWindowsEntryPoints.obj
 0002:0000c5d8       $unwind$setPopupMenuCanceledFP 000000018002c5d8     AccessBridgeWindowsEntryPoints.obj
 0002:0000c5d8       $unwind$setPopupMenuWillBecomeInvisibleFP 000000018002c5d8     AccessBridgeWindowsEntryPoints.obj
 0002:0000c5d8       $unwind$setPopupMenuWillBecomeVisibleFP 000000018002c5d8     AccessBridgeWindowsEntryPoints.obj
 0002:0000c5d8       $unwind$setPropertyActiveDescendentChangeFP 000000018002c5d8     AccessBridgeWindowsEntryPoints.obj
 0002:0000c5d8       $unwind$setPropertyCaretChangeFP 000000018002c5d8     AccessBridgeWindowsEntryPoints.obj
 0002:0000c5d8       $unwind$setPropertyChangeFP 000000018002c5d8     AccessBridgeWindowsEntryPoints.obj
 0002:0000c5d8       $unwind$setPropertyChildChangeFP 000000018002c5d8     AccessBridgeWindowsEntryPoints.obj
 0002:0000c5d8       $unwind$setPropertyDescriptionChangeFP 000000018002c5d8     AccessBridgeWindowsEntryPoints.obj
 0002:0000c5d8       $unwind$setPropertyNameChangeFP 000000018002c5d8     AccessBridgeWindowsEntryPoints.obj
 0002:0000c5d8       $unwind$setPropertySelectionChangeFP 000000018002c5d8     AccessBridgeWindowsEntryPoints.obj
 0002:0000c5d8       $unwind$setPropertyStateChangeFP 000000018002c5d8     AccessBridgeWindowsEntryPoints.obj
 0002:0000c5d8       $unwind$setPropertyTableModelChangeFP 000000018002c5d8     AccessBridgeWindowsEntryPoints.obj
 0002:0000c5d8       $unwind$setPropertyTextChangeFP 000000018002c5d8     AccessBridgeWindowsEntryPoints.obj
 0002:0000c5d8       $unwind$setPropertyValueChangeFP 000000018002c5d8     AccessBridgeWindowsEntryPoints.obj
 0002:0000c5d8       $unwind$setPropertyVisibleDataChangeFP 000000018002c5d8     AccessBridgeWindowsEntryPoints.obj
 0002:0000c5d8       $unwind$__scrt_initialize_default_local_stdio_options 000000018002c5d8     LIBCMT:default_local_stdio_options.obj
 0002:0000c5d8       $unwind$?dllmain_crt_dispatch@@YAHQEAUHINSTANCE__@@KQEAX@Z 000000018002c5d8     LIBCMT:dll_dllmain.obj
 0002:0000c5d8       $unwind$__report_rangecheckfailure 000000018002c5d8     LIBCMT:gs_report.obj
 0002:0000c5d8       $unwind$__GSHandlerCheck   000000018002c5d8     LIBCMT:gshandler.obj
 0002:0000c5d8       $unwind$__scrt_acquire_startup_lock 000000018002c5d8     LIBCMT:utility.obj
 0002:0000c5d8       $unwind$__scrt_dllmain_after_initialize_c 000000018002c5d8     LIBCMT:utility.obj
 0002:0000c5d8       $unwind$__scrt_dllmain_before_initialize_c 000000018002c5d8     LIBCMT:utility.obj
 0002:0000c5d8       $unwind$__scrt_dllmain_crt_thread_attach 000000018002c5d8     LIBCMT:utility.obj
 0002:0000c5d8       $unwind$__scrt_dllmain_crt_thread_detach 000000018002c5d8     LIBCMT:utility.obj
 0002:0000c5d8       $unwind$__scrt_dllmain_uninitialize_c 000000018002c5d8     LIBCMT:utility.obj
 0002:0000c5d8       $unwind$__scrt_dllmain_uninitialize_critical 000000018002c5d8     LIBCMT:utility.obj
 0002:0000c5d8       $unwind$__std_terminate    000000018002c5d8     libvcruntime:ehhelpers.obj
 0002:0000c5d8       $unwind$?GetCurrentState@__FrameHandler3@@SAHPEA_KPEAU_xDISPATCHER_CONTEXT@@PEBU_s_FuncInfo@@@Z 000000018002c5d8     libvcruntime:ehstate.obj
 0002:0000c5d8       $unwind$__vcrt_initialize  000000018002c5d8     libvcruntime:initialization.obj
 0002:0000c5d8       $unwind$__vcrt_thread_attach 000000018002c5d8     libvcruntime:initialization.obj
 0002:0000c5d8       $unwind$__vcrt_thread_detach 000000018002c5d8     libvcruntime:initialization.obj
 0002:0000c5d8       $unwind$__vcrt_uninitialize 000000018002c5d8     libvcruntime:initialization.obj
 0002:0000c5d8       $unwind$__vcrt_uninitialize_critical 000000018002c5d8     libvcruntime:initialization.obj
 0002:0000c5d8       $unwind$__vcrt_freefls     000000018002c5d8     libvcruntime:per_thread_data.obj
 0002:0000c5d8       $unwind$__vcrt_getptd      000000018002c5d8     libvcruntime:per_thread_data.obj
 0002:0000c5d8       $unwind$__vcrt_initialize_ptd 000000018002c5d8     libvcruntime:per_thread_data.obj
 0002:0000c5d8       $unwind$__vcrt_uninitialize_ptd 000000018002c5d8     libvcruntime:per_thread_data.obj
 0002:0000c5d8       $unwind$_GetImageBase      000000018002c5d8     libvcruntime:risctrnsctrl.obj
 0002:0000c5d8       $unwind$_GetThrowImageBase 000000018002c5d8     libvcruntime:risctrnsctrl.obj
 0002:0000c5d8       $unwind$__dcrt_terminate_console_output 000000018002c5d8     libucrt:initcon.obj
 0002:0000c5d8       $unwind$??$uninitialize_environment_internal@D@@YAXAEAPEAPEAD@Z 000000018002c5d8     libucrt:environment_initialization.obj
 0002:0000c5d8       $unwind$??$uninitialize_environment_internal@_W@@YAXAEAPEAPEA_W@Z 000000018002c5d8     libucrt:environment_initialization.obj
 0002:0000c5d8       $unwind$__dcrt_get_or_create_narrow_environment_nolock 000000018002c5d8     libucrt:environment_initialization.obj
 0002:0000c5d8       $unwind$__acrt_initialize_heap 000000018002c5d8     libucrt:heap_handle.obj
 0002:0000c5d8       $unwind$_msize_base        000000018002c5d8     libucrt:msize.obj
 0002:0000c5d8       $unwind$?initialize_multibyte@@YAHXZ 000000018002c5d8     libucrt:multibyte_initializer.obj
 0002:0000c5d8       $unwind$__acrt_thread_attach 000000018002c5d8     libucrt:initialization.obj
 0002:0000c5d8       $unwind$__acrt_thread_detach 000000018002c5d8     libucrt:initialization.obj
 0002:0000c5d8       $unwind$__acrt_uninitialize 000000018002c5d8     libucrt:initialization.obj
 0002:0000c5d8       $unwind$__acrt_uninitialize_critical 000000018002c5d8     libucrt:initialization.obj
 0002:0000c5d8       $unwind$initialize_c       000000018002c5d8     libucrt:initialization.obj
 0002:0000c5d8       $unwind$uninitialize_allocated_io_buffers 000000018002c5d8     libucrt:initialization.obj
 0002:0000c5d8       $unwind$uninitialize_environment 000000018002c5d8     libucrt:initialization.obj
 0002:0000c5d8       $unwind$__acrt_initialize_ptd 000000018002c5d8     libucrt:per_thread_data.obj
 0002:0000c5d8       $unwind$__acrt_uninitialize_ptd 000000018002c5d8     libucrt:per_thread_data.obj
 0002:0000c5d8       $unwind$__acrt_AreFileApisANSI 000000018002c5d8     libucrt:winapi_thunks.obj
 0002:0000c5d8       $unwind$__acrt_release_locale_ref 000000018002c5d8     libucrt:locale_refcounting.obj
 0002:0000c5d8       $unwind$_isatty            000000018002c5d8     libucrt:isatty.obj
 0002:0000c5d8       $unwind$_get_osfhandle     000000018002c5d8     libucrt:osfinfo.obj
 0002:0000c5d8       $unwind$_get_fmode         000000018002c5d8     libucrt:setmode.obj
 0002:0000c5d8       $unwind$__acrt_initialize_multibyte 000000018002c5d8     libucrt:mbctype.obj
 0002:0000c5d8       $unwind$__acrt_update_thread_multibyte_data 000000018002c5d8     libucrt:mbctype.obj
 0002:0000c5d8       $unwind$__doserrno         000000018002c5d8     libucrt:errno.obj
 0002:0000c5d8       $unwind$_errno             000000018002c5d8     libucrt:errno.obj
 0002:0000c5d8       $unwind$_invoke_watson     000000018002c5d8     libucrt:invalid_parameter.obj
 0002:0000c5d8       $unwind$abort              000000018002c5d8     libucrt:abort.obj
 0002:0000c5d8       $unwind$__acrt_initialize_command_line 000000018002c5d8     libucrt:argv_data.obj
 0002:0000c5d8       $unwind$?should_call_terminate_process@@YA_NXZ 000000018002c5d8     libucrt:exit.obj
 0002:0000c5d8       $unwind$_fileno            000000018002c5d8     libucrt:fileno.obj
 0002:0000c5d8       $unwind$?validate_stream_is_ansi_if_required@?$__acrt_stdio_char_traits@D@@SA_NQEAU_iobuf@@@Z 000000018002c5d8     libucrt:output.obj
 0002:0000c5d8       $unwind$_strnicmp          000000018002c5d8     libucrt:strnicmp.obj
 0002:0000c5d8       $unwind$_statfp            000000018002c5d8     libucrt:fpctrl.obj
 0002:0000c5d8       $unwind$fegetround         000000018002c5d8     libucrt:fegetround.obj
 0002:0000c5d8       $unwind$_set_errno_from_matherr 000000018002c5d8     libucrt:fpexcept.obj
 0002:0000c5e0       $unwind$fprintf            000000018002c5e0     AccessBridgeDebug.obj
 0002:0000c5e0       $unwind$sprintf            000000018002c5e0     AccessBridgeJavaVMInstance.obj
 0002:0000c5ec       $unwind$printf             000000018002c5ec     AccessBridgeDebug.obj
 0002:0000c5f8       $unwind$?firePropertyActiveDescendentChange@AccessBridgeEventHandler@@QEAAXJ_J000@Z 000000018002c5f8     AccessBridgeEventHandler.obj
 0002:0000c5f8       $unwind$?firePropertyCaretChange@AccessBridgeEventHandler@@QEAAXJ_J0HH@Z 000000018002c5f8     AccessBridgeEventHandler.obj
 0002:0000c5f8       $unwind$?firePropertyChildChange@AccessBridgeEventHandler@@QEAAXJ_J000@Z 000000018002c5f8     AccessBridgeEventHandler.obj
 0002:0000c5f8       $unwind$?firePropertyDescriptionChange@AccessBridgeEventHandler@@QEAAXJ_J0PEAG1@Z 000000018002c5f8     AccessBridgeEventHandler.obj
 0002:0000c5f8       $unwind$?firePropertyNameChange@AccessBridgeEventHandler@@QEAAXJ_J0PEAG1@Z 000000018002c5f8     AccessBridgeEventHandler.obj
 0002:0000c5f8       $unwind$?firePropertyStateChange@AccessBridgeEventHandler@@QEAAXJ_J0PEAG1@Z 000000018002c5f8     AccessBridgeEventHandler.obj
 0002:0000c5f8       $unwind$?firePropertyTableModelChange@AccessBridgeEventHandler@@QEAAXJ_J0PEAG1@Z 000000018002c5f8     AccessBridgeEventHandler.obj
 0002:0000c5f8       $unwind$?firePropertyValueChange@AccessBridgeEventHandler@@QEAAXJ_J0PEAG1@Z 000000018002c5f8     AccessBridgeEventHandler.obj
 0002:0000c5f8       $unwind$?processPackage@WinAccessBridge@@QEAAXPEADJ@Z 000000018002c5f8     WinAccessBridge.obj
 0002:0000c5f8       $unwind$?type_case_c_tchar@?$output_processor@DV?$stream_output_adapter@D@__crt_stdio_output@@V?$standard_base@DV?$stream_output_adapter@D@__crt_stdio_output@@@2@@__crt_stdio_output@@AEAA_ND@Z 000000018002c5f8     libucrt:output.obj
 0002:0000c5f8       $unwind$?type_case_c_tchar@?$output_processor@DV?$string_output_adapter@D@__crt_stdio_output@@V?$standard_base@DV?$string_output_adapter@D@__crt_stdio_output@@@2@@__crt_stdio_output@@AEAA_ND@Z 000000018002c5f8     libucrt:output.obj
 0002:0000c5f8       $unwind$?type_case_n@?$output_processor@DV?$stream_output_adapter@D@__crt_stdio_output@@V?$standard_base@DV?$stream_output_adapter@D@__crt_stdio_output@@@2@@__crt_stdio_output@@AEAA_NXZ 000000018002c5f8     libucrt:output.obj
 0002:0000c5f8       $unwind$?type_case_n@?$output_processor@DV?$string_output_adapter@D@__crt_stdio_output@@V?$standard_base@DV?$string_output_adapter@D@__crt_stdio_output@@@2@@__crt_stdio_output@@AEAA_NXZ 000000018002c5f8     libucrt:output.obj
 0002:0000c604       $unwind$??0AccessBridgeJavaVMInstance@@QEAA@PEAUHWND__@@0JPEAV0@@Z 000000018002c604     AccessBridgeJavaVMInstance.obj
 0002:0000c604       $unwind$??1AccessBridgeJavaVMInstance@@QEAA@XZ 000000018002c604     AccessBridgeJavaVMInstance.obj
 0002:0000c604       $unwind$??0bad_alloc@std@@QEAA@AEBV01@@Z 000000018002c604     AccessBridgeMessageQueue.obj
 0002:0000c604       $unwind$??0exception@std@@QEAA@AEBV01@@Z 000000018002c604     AccessBridgeMessageQueue.obj
 0002:0000c604       $unwind$getTopLevelHWND    000000018002c604     AccessBridgeWindowsEntryPoints.obj
 0002:0000c604       $unwind$__raise_securityfailure 000000018002c604     LIBCMT:gs_report.obj
 0002:0000c604       $unwind$??2@YAPEAX_K@Z     000000018002c604     LIBCMT:new_scalar.obj
 0002:0000c604       $unwind$??_Gtype_info@@UEAAPEAXI@Z 000000018002c604     LIBCMT:std_type_info_static.obj
 0002:0000c604       $unwind$??0bad_array_new_length@std@@QEAA@AEBV01@@Z 000000018002c604     LIBCMT:throw_bad_alloc.obj
 0002:0000c604       $unwind$__scrt_initialize_crt 000000018002c604     LIBCMT:utility.obj
 0002:0000c604       $unwind$__scrt_initialize_onexit_tables 000000018002c604     LIBCMT:utility.obj
 0002:0000c604       $unwind$__scrt_release_startup_lock 000000018002c604     LIBCMT:utility.obj
 0002:0000c604       $unwind$__scrt_uninitialize_crt 000000018002c604     LIBCMT:utility.obj
 0002:0000c604       $unwind$_IsExceptionObjectToBeDestroyed 000000018002c604     libvcruntime:ehhelpers.obj
 0002:0000c604       $unwind$?GetUnwindTryBlock@__FrameHandler3@@SAHPEA_KPEAU_xDISPATCHER_CONTEXT@@PEBU_s_FuncInfo@@@Z 000000018002c604     libvcruntime:ehstate.obj
 0002:0000c604       $unwind$?StateFromIp@__FrameHandler3@@SAHPEBU_s_FuncInfo@@PEAU_xDISPATCHER_CONTEXT@@_K@Z 000000018002c604     libvcruntime:ehstate.obj
 0002:0000c604       $unwind$??0bad_exception@std@@QEAA@AEBV01@@Z 000000018002c604     libvcruntime:frame.obj
 0002:0000c604       $unwind$__vcrt_initialize_locks 000000018002c604     libvcruntime:locks.obj
 0002:0000c604       $unwind$__vcrt_uninitialize_locks 000000018002c604     libvcruntime:locks.obj
 0002:0000c604       $unwind$__vcrt_freeptd_for_this_thread 000000018002c604     libvcruntime:per_thread_data.obj
 0002:0000c604       $unwind$?ExecutionInCatch@__FrameHandler3@@SA_NPEAU_xDISPATCHER_CONTEXT@@PEBU_s_FuncInfo@@@Z 000000018002c604     libvcruntime:risctrnsctrl.obj
 0002:0000c604       $unwind$_CreateFrameInfo   000000018002c604     libvcruntime:risctrnsctrl.obj
 0002:0000c604       $unwind$_SetImageBase      000000018002c604     libvcruntime:risctrnsctrl.obj
 0002:0000c604       $unwind$_SetThrowImageBase 000000018002c604     libvcruntime:risctrnsctrl.obj
 0002:0000c604       $unwind$__std_exception_destroy 000000018002c604     libvcruntime:std_exception.obj
 0002:0000c604       $unwind$__std_type_info_destroy_list 000000018002c604     libvcruntime:std_type_info.obj
 0002:0000c604       $unwind$__vcrt_FlsAlloc    000000018002c604     libvcruntime:winapi_downlevel.obj
 0002:0000c604       $unwind$__vcrt_FlsFree     000000018002c604     libvcruntime:winapi_downlevel.obj
 0002:0000c604       $unwind$__vcrt_FlsGetValue 000000018002c604     libvcruntime:winapi_downlevel.obj
 0002:0000c604       $unwind$_calloc_base       000000018002c604     libucrt:calloc_base.obj
 0002:0000c604       $unwind$_malloc_base       000000018002c604     libucrt:malloc_base.obj
 0002:0000c604       $unwind$initialize_pointers 000000018002c604     libucrt:initialization.obj
 0002:0000c604       $unwind$uninitialize_allocated_memory 000000018002c604     libucrt:initialization.obj
 0002:0000c604       $unwind$__acrt_initialize_locks 000000018002c604     libucrt:locks.obj
 0002:0000c604       $unwind$__acrt_uninitialize_locks 000000018002c604     libucrt:locks.obj
 0002:0000c604       $unwind$__acrt_freeptd     000000018002c604     libucrt:per_thread_data.obj
 0002:0000c604       $unwind$__acrt_getptd_head 000000018002c604     libucrt:per_thread_data.obj
 0002:0000c604       $unwind$__acrt_get_process_end_policy 000000018002c604     libucrt:win_policies.obj
 0002:0000c604       $unwind$__acrt_AppPolicyGetProcessTerminationMethodInternal 000000018002c604     libucrt:winapi_thunks.obj
 0002:0000c604       $unwind$__acrt_uninitialize_winapi_thunks 000000018002c604     libucrt:winapi_thunks.obj
 0002:0000c604       $unwind$__acrt_update_locale_info 000000018002c604     libucrt:locale_update.obj
 0002:0000c604       $unwind$__acrt_update_locale_info_explicit 000000018002c604     libucrt:locale_update.obj
 0002:0000c604       $unwind$__acrt_update_multibyte_info 000000018002c604     libucrt:locale_update.obj
 0002:0000c604       $unwind$__acrt_update_multibyte_info_explicit 000000018002c604     libucrt:locale_update.obj
 0002:0000c604       $unwind$__acrt_errno_map_os_error 000000018002c604     libucrt:errno.obj
 0002:0000c604       $unwind$__acrt_errno_map_os_error_ptd 000000018002c604     libucrt:errno.obj
 0002:0000c604       $unwind$__acrt_allocate_buffer_for_argv 000000018002c604     libucrt:argv_parsing.obj
 0002:0000c604       $unwind$?exit_or_terminate_process@@YAXI@Z 000000018002c604     libucrt:exit.obj
 0002:0000c604       $unwind$__acrt_uninitialize_stdio 000000018002c604     libucrt:_file.obj
 0002:0000c604       $unwind$?stream_is_at_end_of_file_nolock@@YA_NV__crt_stdio_stream@@@Z 000000018002c604     libucrt:_flsbuf.obj
 0002:0000c604       $unwind$__acrt_stdio_free_buffer_nolock 000000018002c604     libucrt:_freebuf.obj
 0002:0000c604       $unwind$__acrt_should_use_temporary_buffer 000000018002c604     libucrt:_sftbuf.obj
 0002:0000c604       $unwind$?type_case_s@?$output_processor@DV?$stream_output_adapter@D@__crt_stdio_output@@V?$standard_base@DV?$stream_output_adapter@D@__crt_stdio_output@@@2@@__crt_stdio_output@@AEAA_NXZ 000000018002c604     libucrt:output.obj
 0002:0000c604       $unwind$?type_case_s@?$output_processor@DV?$string_output_adapter@D@__crt_stdio_output@@V?$standard_base@DV?$string_output_adapter@D@__crt_stdio_output@@@2@@__crt_stdio_output@@AEAA_NXZ 000000018002c604     libucrt:output.obj
 0002:0000c604       $unwind$strcpy_s           000000018002c604     libucrt:strcpy_s.obj
 0002:0000c604       $unwind$_clrfp             000000018002c604     libucrt:fpctrl.obj
 0002:0000c604       $unwind$_set_statfp        000000018002c604     libucrt:fpctrl.obj
 0002:0000c604       $unwind$_clearfp           000000018002c604     libucrt:ieee.obj
 0002:0000c604       $unwind$_controlfp_s       000000018002c604     libucrt:contrlfp.obj
 0002:0000c604       $unwind$fegetenv           000000018002c604     libucrt:fegetenv.obj
 0002:0000c604       $unwind$feholdexcept       000000018002c604     libucrt:feholdexcept.obj
 0002:0000c60c       $unwind$?initiateIPC@AccessBridgeJavaVMInstance@@QEAA_JXZ 000000018002c60c     AccessBridgeJavaVMInstance.obj
 0002:0000c624       $unwind$?sendPackage@AccessBridgeJavaVMInstance@@QEAA_JPEADJ@Z 000000018002c624     AccessBridgeJavaVMInstance.obj
 0002:0000c62c       $unwind$?sendMemoryPackage@AccessBridgeJavaVMInstance@@QEAAHPEADJ@Z 000000018002c62c     AccessBridgeJavaVMInstance.obj
 0002:0000c644       $unwind$?findABJavaVMInstanceFromJavaHWND@AccessBridgeJavaVMInstance@@QEAAPEAV1@PEAUHWND__@@@Z 000000018002c644     AccessBridgeJavaVMInstance.obj
 0002:0000c644       $unwind$?findAccessBridgeWindow@AccessBridgeJavaVMInstance@@QEAAPEAUHWND__@@J@Z 000000018002c644     AccessBridgeJavaVMInstance.obj
 0002:0000c644       $unwind$??_Gbad_alloc@std@@UEAAPEAXI@Z 000000018002c644     AccessBridgeMessageQueue.obj
 0002:0000c644       $unwind$??_Gexception@std@@UEAAPEAXI@Z 000000018002c644     AccessBridgeMessageQueue.obj
 0002:0000c644       $unwind$??0WinAccessBridge@@QEAA@PEAUHINSTANCE__@@@Z 000000018002c644     WinAccessBridge.obj
 0002:0000c644       $unwind$??1WinAccessBridge@@QEAA@XZ 000000018002c644     WinAccessBridge.obj
 0002:0000c644       $unwind$?sendMemoryPackage@WinAccessBridge@@QEAAHPEADJPEAUHWND__@@@Z 000000018002c644     WinAccessBridge.obj
 0002:0000c644       $unwind$DllMain            000000018002c644     WinAccessBridge.obj
 0002:0000c644       $unwind$_RTC_Initialize    000000018002c644     LIBCMT:initsect.obj
 0002:0000c644       $unwind$_RTC_Terminate     000000018002c644     LIBCMT:initsect.obj
 0002:0000c644       $unwind$??_Gbad_array_new_length@std@@UEAAPEAXI@Z 000000018002c644     LIBCMT:throw_bad_alloc.obj
 0002:0000c644       $unwind$__C_specific_handler_noexcept 000000018002c644     libvcruntime:chandler_noexcept.obj
 0002:0000c644       $unwind$__FrameUnwindFilter 000000018002c644     libvcruntime:ehhelpers.obj
 0002:0000c644       $unwind$?SetUnwindTryBlock@__FrameHandler3@@SAXPEA_KPEAU_xDISPATCHER_CONTEXT@@PEBU_s_FuncInfo@@H@Z 000000018002c644     libvcruntime:ehstate.obj
 0002:0000c644       $unwind$??_Gbad_exception@std@@UEAAPEAXI@Z 000000018002c644     libvcruntime:frame.obj
 0002:0000c644       $unwind$?ExFilterRethrow@@YAHPEAU_EXCEPTION_POINTERS@@PEAUEHExceptionRecord@@PEAH@Z 000000018002c644     libvcruntime:frame.obj
 0002:0000c644       $unwind$_FindAndUnlinkFrame 000000018002c644     libvcruntime:risctrnsctrl.obj
 0002:0000c644       $unwind$__vcrt_FlsSetValue 000000018002c644     libvcruntime:winapi_downlevel.obj
 0002:0000c644       $unwind$??$common_initialize_environment_nolock@D@@YAHXZ 000000018002c644     libucrt:environment_initialization.obj
 0002:0000c644       $unwind$_callnewh          000000018002c644     libucrt:new_handler.obj
 0002:0000c644       $unwind$_realloc_base      000000018002c644     libucrt:realloc_base.obj
 0002:0000c644       $unwind$?replace_current_thread_locale_nolock@@YAXQEAU__acrt_ptd@@QEAU__crt_locale_data@@@Z 000000018002c644     libucrt:per_thread_data.obj
 0002:0000c644       $unwind$__acrt_execute_uninitializers 000000018002c644     libucrt:shared_initialization.obj
 0002:0000c644       $unwind$__acrt_LocaleNameToLCID 000000018002c644     libucrt:winapi_thunks.obj
 0002:0000c644       $unwind$?free_crt_array_internal@@YAXQEAPEBX_K@Z 000000018002c644     libucrt:inittime.obj
 0002:0000c644       $unwind$_updatetlocinfoEx_nolock 000000018002c644     libucrt:locale_refcounting.obj
 0002:0000c644       $unwind$__acrt_uninitialize_lowio 000000018002c644     libucrt:ioinit.obj
 0002:0000c644       $unwind$?setSBCS@@YAXPEAU__crt_multibyte_data@@@Z 000000018002c644     libucrt:mbctype.obj
 0002:0000c644       $unwind$_initterm_e        000000018002c644     libucrt:initterm.obj
 0002:0000c644       $unwind$__acrt_stdio_allocate_buffer_nolock 000000018002c644     libucrt:_getbuf.obj
 0002:0000c644       $unwind$__acrt_stdio_begin_temporary_buffering_nolock 000000018002c644     libucrt:_sftbuf.obj
 0002:0000c650       $unwind$??0AccessBridgeQueueElement@@QEAA@PEADH@Z 000000018002c650     AccessBridgeMessageQueue.obj
 0002:0000c650       $unwind$_mbsdec_l          000000018002c650     libucrt:mbsdec.obj
 0002:0000c65c       $unwind$?add@AccessBridgeMessageQueue@@QEAA?AW4QueueReturns@@PEAVAccessBridgeQueueElement@@@Z 000000018002c65c     AccessBridgeMessageQueue.obj
 0002:0000c65c       $unwind$?remove@AccessBridgeMessageQueue@@QEAA?AW4QueueReturns@@PEAPEAVAccessBridgeQueueElement@@@Z 000000018002c65c     AccessBridgeMessageQueue.obj
 0002:0000c65c       $unwind$isSameObject       000000018002c65c     AccessBridgeWindowsEntryPoints.obj
 0002:0000c65c       $unwind$?JavaVMDestroyed@WinAccessBridge@@QEAAXPEAUHWND__@@@Z 000000018002c65c     WinAccessBridge.obj
 0002:0000c65c       $unwind$?preProcessPackage@WinAccessBridge@@QEAAXPEADJ@Z 000000018002c65c     WinAccessBridge.obj
 0002:0000c65c       $unwind$?queuePackage@WinAccessBridge@@QEAAHPEADJ@Z 000000018002c65c     WinAccessBridge.obj
 0002:0000c65c       $unwind$AccessBridgeDialogProc 000000018002c65c     WinAccessBridge.obj
 0002:0000c65c       $unwind$_DllMainCRTStartup 000000018002c65c     LIBCMT:dll_dllmain.obj
 0002:0000c65c       $unwind$__vcrt_getptd_noexit 000000018002c65c     libvcruntime:per_thread_data.obj
 0002:0000c65c       $unwind$?FrameUnwindToEmptyState@__FrameHandler3@@SAXPEA_KPEAU_xDISPATCHER_CONTEXT@@PEBU_s_FuncInfo@@@Z 000000018002c65c     libvcruntime:risctrnsctrl.obj
 0002:0000c65c       $unwind$__vcrt_InitializeCriticalSectionEx 000000018002c65c     libvcruntime:winapi_downlevel.obj
 0002:0000c65c       $unwind$??$common_getenv_nolock@D@@YAPEADQEBD@Z 000000018002c65c     libucrt:getenv.obj
 0002:0000c65c       $unwind$memcpy_s           000000018002c65c     libucrt:cfout.obj
 0002:0000c65c       $unwind$__acrt_getptd      000000018002c65c     libucrt:per_thread_data.obj
 0002:0000c65c       $unwind$__acrt_getptd_noexit 000000018002c65c     libucrt:per_thread_data.obj
 0002:0000c65c       $unwind$__acrt_getptd_noexit_explicit 000000018002c65c     libucrt:per_thread_data.obj
 0002:0000c65c       $unwind$__acrt_execute_initializers 000000018002c65c     libucrt:shared_initialization.obj
 0002:0000c65c       $unwind$__acrt_InitializeCriticalSectionEx 000000018002c65c     libucrt:winapi_thunks.obj
 0002:0000c65c       $unwind$_close_nolock_internal 000000018002c65c     libucrt:close.obj
 0002:0000c65c       $unwind$?value@?$dual_state_global@P6AXPEB_W00I_K@Z@__crt_state_management@@QEAAAEAP6AXPEB_W00I_K@ZAEAV__crt_cached_ptd_host@@@Z 000000018002c65c     libucrt:invalid_parameter.obj
 0002:0000c65c       $unwind$__acrt_stdio_flush_and_write_narrow_nolock 000000018002c65c     libucrt:_flsbuf.obj
 0002:0000c65c       $unwind$??$__acrt_stdio_parse_mode@D@@YA?AU__acrt_stdio_stream_mode@@QEBD@Z 000000018002c65c     libucrt:openfile.obj
 0002:0000c65c       $unwind$?update_locale_slow@__crt_cached_ptd_host@@AEAAXXZ 000000018002c65c     libucrt:output.obj
 0002:0000c65c       $unwind$strncpy_s          000000018002c65c     libucrt:strncpy_s.obj
 0002:0000c65c       $unwind$??0_LocaleUpdate@@QEAA@QEAU__crt_locale_pointers@@@Z 000000018002c65c     libucrt:wcsnicol.obj
 0002:0000c65c       $unwind$_exception_enabled 000000018002c65c     libucrt:libm_error.obj
 0002:0000c66c       $unwind$doAccessibleActions 000000018002c66c     AccessBridgeWindowsEntryPoints.obj
 0002:0000c66c       $unwind$getAccessibleContextAt 000000018002c66c     AccessBridgeWindowsEntryPoints.obj
 0002:0000c66c       $unwind$getAccessibleHyperlink 000000018002c66c     AccessBridgeWindowsEntryPoints.obj
 0002:0000c66c       $unwind$getAccessibleHypertextExt 000000018002c66c     AccessBridgeWindowsEntryPoints.obj
 0002:0000c66c       $unwind$getAccessibleTableCellInfo 000000018002c66c     AccessBridgeWindowsEntryPoints.obj
 0002:0000c66c       $unwind$getAccessibleTableColumnSelections 000000018002c66c     AccessBridgeWindowsEntryPoints.obj
 0002:0000c66c       $unwind$getAccessibleTableIndex 000000018002c66c     AccessBridgeWindowsEntryPoints.obj
 0002:0000c66c       $unwind$getAccessibleTableRowSelections 000000018002c66c     AccessBridgeWindowsEntryPoints.obj
 0002:0000c66c       $unwind$getAccessibleTextAttributes 000000018002c66c     AccessBridgeWindowsEntryPoints.obj
 0002:0000c66c       $unwind$getAccessibleTextInfo 000000018002c66c     AccessBridgeWindowsEntryPoints.obj
 0002:0000c66c       $unwind$getAccessibleTextItems 000000018002c66c     AccessBridgeWindowsEntryPoints.obj
 0002:0000c66c       $unwind$getAccessibleTextLineBounds 000000018002c66c     AccessBridgeWindowsEntryPoints.obj
 0002:0000c66c       $unwind$getAccessibleTextRect 000000018002c66c     AccessBridgeWindowsEntryPoints.obj
 0002:0000c66c       $unwind$getCaretLocation   000000018002c66c     AccessBridgeWindowsEntryPoints.obj
 0002:0000c66c       $unwind$getCurrentAccessibleValueFromContext 000000018002c66c     AccessBridgeWindowsEntryPoints.obj
 0002:0000c66c       $unwind$getMaximumAccessibleValueFromContext 000000018002c66c     AccessBridgeWindowsEntryPoints.obj
 0002:0000c66c       $unwind$getMinimumAccessibleValueFromContext 000000018002c66c     AccessBridgeWindowsEntryPoints.obj
 0002:0000c66c       $unwind$getVirtualAccessibleName 000000018002c66c     AccessBridgeWindowsEntryPoints.obj
 0002:0000c66c       $unwind$getVisibleChildren 000000018002c66c     AccessBridgeWindowsEntryPoints.obj
 0002:0000c66c       $unwind$selectTextRange    000000018002c66c     AccessBridgeWindowsEntryPoints.obj
 0002:0000c66c       $unwind$_sopen_s           000000018002c66c     libucrt:open.obj
 0002:0000c66c       $unwind$_invalid_parameter_noinfo 000000018002c66c     libucrt:invalid_parameter.obj
 0002:0000c66c       $unwind$?state_case_size@?$output_processor@DV?$stream_output_adapter@D@__crt_stdio_output@@V?$standard_base@DV?$stream_output_adapter@D@__crt_stdio_output@@@2@@__crt_stdio_output@@AEAA_NXZ 000000018002c66c     libucrt:output.obj
 0002:0000c66c       $unwind$?state_case_size@?$output_processor@DV?$string_output_adapter@D@__crt_stdio_output@@V?$standard_base@DV?$string_output_adapter@D@__crt_stdio_output@@@2@@__crt_stdio_output@@AEAA_NXZ 000000018002c66c     libucrt:output.obj
 0002:0000c66c       $unwind$_log10_special     000000018002c66c     libucrt:log_special.obj
 0002:0000c674       $unwind$getAccessibleTextRange 000000018002c674     AccessBridgeWindowsEntryPoints.obj
 0002:0000c674       $unwind$getTextAttributesInRange 000000018002c674     AccessBridgeWindowsEntryPoints.obj
 0002:0000c674       $unwind$?__scrt_throw_std_bad_alloc@@YAXXZ 000000018002c674     LIBCMT:throw_bad_alloc.obj
 0002:0000c674       $unwind$?__scrt_throw_std_bad_array_new_length@@YAXXZ 000000018002c674     LIBCMT:throw_bad_alloc.obj
 0002:0000c674       $unwind$_raise_exc         000000018002c674     libucrt:fpexcept.obj
 0002:0000c67c       $unwind$?initWindow@WinAccessBridge@@QEAAHXZ 000000018002c67c     WinAccessBridge.obj
 0002:0000c684       $unwind$?rendezvousWithNewJavaDLL@WinAccessBridge@@QEAA_JPEAUHWND__@@J@Z 000000018002c684     WinAccessBridge.obj
 0002:0000c694       $unwind$?sendPackage@WinAccessBridge@@QEAAXPEADJPEAUHWND__@@@Z 000000018002c694     WinAccessBridge.obj
 0002:0000c69c       $unwind$?receiveAQueuedPackage@WinAccessBridge@@QEAAHXZ 000000018002c69c     WinAccessBridge.obj
 0002:0000c69c       $unwind$?get_raw_ptd_noexit@__crt_cached_ptd_host@@QEAAPEAU__acrt_ptd@@XZ 000000018002c69c     libucrt:invalid_parameter.obj
 0002:0000c6ac       $unwind$?getHWNDFromAccessibleContext@WinAccessBridge@@QEAAPEAUHWND__@@J_J@Z 000000018002c6ac     WinAccessBridge.obj
 0002:0000c6ac       $unwind$?releaseJavaObject@WinAccessBridge@@QEAAXJ_J@Z 000000018002c6ac     WinAccessBridge.obj
 0002:0000c6ac       $unwind$?requestFocus@WinAccessBridge@@QEAAHJ_J@Z 000000018002c6ac     WinAccessBridge.obj
 0002:0000c6c0       $unwind$?getAccessibleTextSelectionInfo@WinAccessBridge@@QEAAHJ_JPEAUAccessibleTextSelectionInfoTag@@@Z 000000018002c6c0     WinAccessBridge.obj
 0002:0000c6c0       $unwind$?getVersionInfo@WinAccessBridge@@QEAAHJPEAUAccessBridgeVersionInfoTag@@@Z 000000018002c6c0     WinAccessBridge.obj
 0002:0000c6d8       $unwind$?isJavaWindow@WinAccessBridge@@QEAAHPEAUHWND__@@@Z 000000018002c6d8     WinAccessBridge.obj
 0002:0000c6ec       $unwind$?getAccessibleContextFromHWND@WinAccessBridge@@QEAAHPEAUHWND__@@PEAJPEA_J@Z 000000018002c6ec     WinAccessBridge.obj
 0002:0000c704       $unwind$?activateAccessibleHyperlink@WinAccessBridge@@QEAAHJ_J0@Z 000000018002c704     WinAccessBridge.obj
 0002:0000c704       $unwind$?isSameObject@WinAccessBridge@@QEAAHJ_J0@Z 000000018002c704     WinAccessBridge.obj
 0002:0000c71c       $unwind$?getVirtualAccessibleName@WinAccessBridge@@QEAAHJ_JPEAGH@Z 000000018002c71c     WinAccessBridge.obj
 0002:0000c71c       $unwind$?setTextContents@WinAccessBridge@@QEAAHJ_JPEBG@Z 000000018002c71c     WinAccessBridge.obj
 0002:0000c734       $unwind$?getParentWithRole@WinAccessBridge@@QEAA_JJ_JPEBG@Z 000000018002c734     WinAccessBridge.obj
 0002:0000c734       $unwind$?getParentWithRoleElseRoot@WinAccessBridge@@QEAA_JJ_JPEBG@Z 000000018002c734     WinAccessBridge.obj
 0002:0000c74c       $unwind$?getAccessibleParentFromContext@WinAccessBridge@@QEAA_JJ_J@Z 000000018002c74c     WinAccessBridge.obj
 0002:0000c74c       $unwind$?getActiveDescendent@WinAccessBridge@@QEAA_JJ_J@Z 000000018002c74c     WinAccessBridge.obj
 0002:0000c74c       $unwind$?getObjectDepth@WinAccessBridge@@QEAAHJ_J@Z 000000018002c74c     WinAccessBridge.obj
 0002:0000c74c       $unwind$?getTopLevelObject@WinAccessBridge@@QEAA_JJ_J@Z 000000018002c74c     WinAccessBridge.obj
 0002:0000c74c       $unwind$?getVisibleChildrenCount@WinAccessBridge@@QEAAHJ_J@Z 000000018002c74c     WinAccessBridge.obj
 0002:0000c760       $unwind$?getAccessibleContextAt@WinAccessBridge@@QEAAHJ_JJJPEA_J@Z 000000018002c760     WinAccessBridge.obj
 0002:0000c774       $unwind$?getAccessibleContextWithFocus@WinAccessBridge@@QEAAHPEAUHWND__@@PEAJPEA_J@Z 000000018002c774     WinAccessBridge.obj
 0002:0000c774       $unwind$?getAccessibleTableColumn@WinAccessBridge@@QEAAJJ_JJ@Z 000000018002c774     WinAccessBridge.obj
 0002:0000c774       $unwind$?getAccessibleTableRow@WinAccessBridge@@QEAAJJ_JJ@Z 000000018002c774     WinAccessBridge.obj
 0002:0000c78c       $unwind$?getAccessibleContextInfo@WinAccessBridge@@QEAAHJ_JPEAUAccessibleContextInfoTag@@@Z 000000018002c78c     WinAccessBridge.obj
 0002:0000c7a4       $unwind$?getAccessibleChildFromContext@WinAccessBridge@@QEAA_JJ_JJ@Z 000000018002c7a4     WinAccessBridge.obj
 0002:0000c7b8       $unwind$?getAccessibleTableColumnHeader@WinAccessBridge@@QEAAHJ_JPEAUAccessibleTableInfoTag@@@Z 000000018002c7b8     WinAccessBridge.obj
 0002:0000c7b8       $unwind$?getAccessibleTableInfo@WinAccessBridge@@QEAAHJ_JPEAUAccessibleTableInfoTag@@@Z 000000018002c7b8     WinAccessBridge.obj
 0002:0000c7b8       $unwind$?getAccessibleTableRowHeader@WinAccessBridge@@QEAAHJ_JPEAUAccessibleTableInfoTag@@@Z 000000018002c7b8     WinAccessBridge.obj
 0002:0000c7d0       $unwind$?getAccessibleTableCellInfo@WinAccessBridge@@QEAAHJ_JJJPEAUAccessibleTableCellInfoTag@@@Z 000000018002c7d0     WinAccessBridge.obj
 0002:0000c7ec       $unwind$?getAccessibleTableColumnDescription@WinAccessBridge@@QEAA_JJ_JJ@Z 000000018002c7ec     WinAccessBridge.obj
 0002:0000c7ec       $unwind$?getAccessibleTableRowDescription@WinAccessBridge@@QEAA_JJ_JJ@Z 000000018002c7ec     WinAccessBridge.obj
 0002:0000c7ec       $unwind$?getAccessibleTextLineBounds@WinAccessBridge@@QEAAHJ_JJPEAJ1@Z 000000018002c7ec     WinAccessBridge.obj
 0002:0000c804       $unwind$?getAccessibleHyperlinkCount@WinAccessBridge@@QEAAJJ_J@Z 000000018002c804     WinAccessBridge.obj
 0002:0000c804       $unwind$?getAccessibleTableColumnSelectionCount@WinAccessBridge@@QEAAJJ_J@Z 000000018002c804     WinAccessBridge.obj
 0002:0000c804       $unwind$?getAccessibleTableRowSelectionCount@WinAccessBridge@@QEAAJJ_J@Z 000000018002c804     WinAccessBridge.obj
 0002:0000c804       $unwind$?setCaretPosition@WinAccessBridge@@QEAAHJ_JH@Z 000000018002c804     WinAccessBridge.obj
 0002:0000c818       $unwind$?getAccessibleHypertextLinkIndex@WinAccessBridge@@QEAAJJ_JJ@Z 000000018002c818     WinAccessBridge.obj
 0002:0000c818       $unwind$?isAccessibleTableColumnSelected@WinAccessBridge@@QEAAHJ_JJ@Z 000000018002c818     WinAccessBridge.obj
 0002:0000c818       $unwind$?isAccessibleTableRowSelected@WinAccessBridge@@QEAAHJ_JJ@Z 000000018002c818     WinAccessBridge.obj
 0002:0000c830       $unwind$?getAccessibleTableColumnSelections@WinAccessBridge@@QEAAHJ_JJPEAJ@Z 000000018002c830     WinAccessBridge.obj
 0002:0000c830       $unwind$?getAccessibleTableRowSelections@WinAccessBridge@@QEAAHJ_JJPEAJ@Z 000000018002c830     WinAccessBridge.obj
 0002:0000c84c       $unwind$?getAccessibleTableIndex@WinAccessBridge@@QEAAJJ_JJJ@Z 000000018002c84c     WinAccessBridge.obj
 0002:0000c864       $unwind$?getAccessibleRelationSet@WinAccessBridge@@QEAAHJ_JPEAUAccessibleRelationSetInfoTag@@@Z 000000018002c864     WinAccessBridge.obj
 0002:0000c87c       $unwind$?getAccessibleHypertext@WinAccessBridge@@QEAAHJ_JPEAUAccessibleHypertextInfoTag@@@Z 000000018002c87c     WinAccessBridge.obj
 0002:0000c894       $unwind$?getAccessibleHypertextExt@WinAccessBridge@@QEAAHJ_JJPEAUAccessibleHypertextInfoTag@@@Z 000000018002c894     WinAccessBridge.obj
 0002:0000c8b0       $unwind$?getAccessibleHyperlink@WinAccessBridge@@QEAAHJ_JJPEAUAccessibleHyperlinkInfoTag@@@Z 000000018002c8b0     WinAccessBridge.obj
 0002:0000c8cc       $unwind$?getAccessibleKeyBindings@WinAccessBridge@@QEAAHJ_JPEAUAccessibleKeyBindingsTag@@@Z 000000018002c8cc     WinAccessBridge.obj
 0002:0000c8e8       $unwind$?getAccessibleIcons@WinAccessBridge@@QEAAHJ_JPEAUAccessibleIconsTag@@@Z 000000018002c8e8     WinAccessBridge.obj
 0002:0000c900       $unwind$?getAccessibleActions@WinAccessBridge@@QEAAHJ_JPEAUAccessibleActionsTag@@@Z 000000018002c900     WinAccessBridge.obj
 0002:0000c918       $unwind$?doAccessibleActions@WinAccessBridge@@QEAAHJ_JPEAUAccessibleActionsToDoTag@@PEAJ@Z 000000018002c918     WinAccessBridge.obj
 0002:0000c934       $unwind$?getAccessibleTextInfo@WinAccessBridge@@QEAAHJ_JPEAUAccessibleTextInfoTag@@JJ@Z 000000018002c934     WinAccessBridge.obj
 0002:0000c934       $unwind$?getAccessibleTextRect@WinAccessBridge@@QEAAHJ_JPEAUAccessibleTextRectInfoTag@@J@Z 000000018002c934     WinAccessBridge.obj
 0002:0000c934       $unwind$?getCaretLocation@WinAccessBridge@@QEAAHJ_JPEAUAccessibleTextRectInfoTag@@J@Z 000000018002c934     WinAccessBridge.obj
 0002:0000c948       $unwind$?getAccessibleTextItems@WinAccessBridge@@QEAAHJ_JPEAUAccessibleTextItemsInfoTag@@J@Z 000000018002c948     WinAccessBridge.obj
 0002:0000c960       $unwind$?getAccessibleTextAttributes@WinAccessBridge@@QEAAHJ_JJPEAUAccessibleTextAttributesInfoTag@@@Z 000000018002c960     WinAccessBridge.obj
 0002:0000c978       $unwind$?getAccessibleTextRange@WinAccessBridge@@QEAAHJ_JJJPEAGF@Z 000000018002c978     WinAccessBridge.obj
 0002:0000c990       $unwind$?getCurrentAccessibleValueFromContext@WinAccessBridge@@QEAAHJ_JPEAGF@Z 000000018002c990     WinAccessBridge.obj
 0002:0000c990       $unwind$?getMaximumAccessibleValueFromContext@WinAccessBridge@@QEAAHJ_JPEAGF@Z 000000018002c990     WinAccessBridge.obj
 0002:0000c990       $unwind$?getMinimumAccessibleValueFromContext@WinAccessBridge@@QEAAHJ_JPEAGF@Z 000000018002c990     WinAccessBridge.obj
 0002:0000c9a8       $unwind$?addAccessibleSelectionFromContext@WinAccessBridge@@QEAAXJ_JH@Z 000000018002c9a8     WinAccessBridge.obj
 0002:0000c9a8       $unwind$?getAccessibleSelectionCountFromContext@WinAccessBridge@@QEAAHJ_J@Z 000000018002c9a8     WinAccessBridge.obj
 0002:0000c9a8       $unwind$?removeAccessibleSelectionFromContext@WinAccessBridge@@QEAAXJ_JH@Z 000000018002c9a8     WinAccessBridge.obj
 0002:0000c9b8       $unwind$?clearAccessibleSelectionFromContext@WinAccessBridge@@QEAAXJ_J@Z 000000018002c9b8     WinAccessBridge.obj
 0002:0000c9b8       $unwind$?selectAllAccessibleSelectionFromContext@WinAccessBridge@@QEAAXJ_J@Z 000000018002c9b8     WinAccessBridge.obj
 0002:0000c9c8       $unwind$?getAccessibleSelectionFromContext@WinAccessBridge@@QEAA_JJ_JH@Z 000000018002c9c8     WinAccessBridge.obj
 0002:0000c9d8       $unwind$?isAccessibleChildSelectedFromContext@WinAccessBridge@@QEAAHJ_JH@Z 000000018002c9d8     WinAccessBridge.obj
 0002:0000c9ec       $unwind$?addAccessibilityEventNotification@WinAccessBridge@@QEAAX_J@Z 000000018002c9ec     WinAccessBridge.obj
 0002:0000c9ec       $unwind$?addJavaEventNotification@WinAccessBridge@@QEAAX_J@Z 000000018002c9ec     WinAccessBridge.obj
 0002:0000c9ec       $unwind$?removeAccessibilityEventNotification@WinAccessBridge@@QEAAX_J@Z 000000018002c9ec     WinAccessBridge.obj
 0002:0000c9ec       $unwind$?removeJavaEventNotification@WinAccessBridge@@QEAAX_J@Z 000000018002c9ec     WinAccessBridge.obj
 0002:0000ca00       $unwind$?selectTextRange@WinAccessBridge@@QEAAHJ_JHH@Z 000000018002ca00     WinAccessBridge.obj
 0002:0000ca14       $unwind$?getTextAttributesInRange@WinAccessBridge@@QEAAHJ_JHHPEAUAccessibleTextAttributesInfoTag@@PEAF@Z 000000018002ca14     WinAccessBridge.obj
 0002:0000ca34       $unwind$?getVisibleChildren@WinAccessBridge@@QEAAHJ_JHPEAUVisibleChildenInfoTag@@@Z 000000018002ca34     WinAccessBridge.obj
 0002:0000ca4c       $unwind$__GSHandlerCheckCommon 000000018002ca4c     LIBCMT:gshandler.obj
 0002:0000ca58       $xdatasym                  000000018002ca58     LIBCMT:amdsecgs.obj
 0002:0000ca60       $xdatasym                  000000018002ca60     LIBCMT:chkstk.obj
 0002:0000ca68       $unwind$?dllmain_crt_process_attach@@YAHQEAUHINSTANCE__@@QEAX@Z 000000018002ca68     LIBCMT:dll_dllmain.obj
 0002:0000caa4       $unwind$?fin$0@?0??dllmain_crt_process_attach@@YAHQEAUHINSTANCE__@@QEAX@Z@4HA 000000018002caa4     LIBCMT:dll_dllmain.obj
 0002:0000caa4       $unwind$?fin$0@?0??dllmain_crt_process_detach@@YAH_N@Z@4HA 000000018002caa4     LIBCMT:dll_dllmain.obj
 0002:0000caa4       $unwind$?fin$1@?0??dllmain_crt_process_detach@@YAH_N@Z@4HA 000000018002caa4     LIBCMT:dll_dllmain.obj
 0002:0000caa4       $unwind$_IsNonwritableInCurrentImage$filt$0 000000018002caa4     LIBCMT:pesect.obj
 0002:0000caa4       $unwind$?filt$0@?0??CxxCallCatchBlock@__FrameHandler3@@SAPEAXPEAU_EXCEPTION_RECORD@@@Z@4HA 000000018002caa4     libvcruntime:frame.obj
 0002:0000caa4       $unwind$?filt$0@?0??FrameUnwindToState@__FrameHandler3@@SAXPEA_KPEAU_xDISPATCHER_CONTEXT@@PEBU_s_FuncInfo@@H@Z@4HA 000000018002caa4     libvcruntime:frame.obj
 0002:0000caa4       $unwind$?fin$1@?0??FrameUnwindToState@__FrameHandler3@@SAXPEA_KPEAU_xDISPATCHER_CONTEXT@@PEBU_s_FuncInfo@@H@Z@4HA 000000018002caa4     libvcruntime:frame.obj
 0002:0000caa4       $unwind$?fin$0@?0???$common_getenv@D@@YAPEADQEBD@Z@4HA 000000018002caa4     libucrt:getenv.obj
 0002:0000caa4       $unwind$_query_new_handler$fin$0 000000018002caa4     libucrt:new_handler.obj
 0002:0000caa4       $unwind$?fin$0@?0???$?RV<lambda_0ae27a3a962d80f24befdcbee591983d>@@AEAV<lambda_8d0ee55de4b1038c4002e0adecdf1839>@@V<lambda_dc504788e8f1664fe9b84e20bfb512f2>@@@?$__crt_seh_guarded_call@X@@QEAAX$$QEAV<lambda_0ae27a3a962d80f24befdcbee591983d>@@AEAV<lambda_8d0ee55de4b1038c4002e0adecdf1839>@@$$QEAV<lambda_dc504788e8f1664fe9b84e20bfb512f2>@@@Z@4HA 000000018002caa4     libucrt:per_thread_data.obj
 0002:0000caa4       $unwind$?fin$0@?0???$?RV<lambda_2d41944a1d46af3157314b8a01080d33>@@AEAV<lambda_8f455de75cd7d7f24b4096f044d8b9e6>@@V<lambda_aa500f224e6afead328df44964fe2772>@@@?$__crt_seh_guarded_call@X@@QEAAX$$QEAV<lambda_2d41944a1d46af3157314b8a01080d33>@@AEAV<lambda_8f455de75cd7d7f24b4096f044d8b9e6>@@$$QEAV<lambda_aa500f224e6afead328df44964fe2772>@@@Z@4HA 000000018002caa4     libucrt:per_thread_data.obj
 0002:0000caa4       $unwind$?fin$0@?0???$?RV<lambda_aa87e3671a710a21b5dc78c0bdf72e11>@@AEAV<lambda_92619d2358a28f41a33ba319515a20b9>@@V<lambda_6992ecaafeb10aed2b74cb1fae11a551>@@@?$__crt_seh_guarded_call@X@@QEAAX$$QEAV<lambda_aa87e3671a710a21b5dc78c0bdf72e11>@@AEAV<lambda_92619d2358a28f41a33ba319515a20b9>@@$$QEAV<lambda_6992ecaafeb10aed2b74cb1fae11a551>@@@Z@4HA 000000018002caa4     libucrt:per_thread_data.obj
 0002:0000caa4       $unwind$?fin$0@?0???$?RV<lambda_f2e299630e499de9f9a165e60fcd3db5>@@AEAV<lambda_2ae9d31cdba2644fcbeaf08da7c24588>@@V<lambda_40d01ff24d0e7b3814fdbdcee8eab3c7>@@@?$__crt_seh_guarded_call@X@@QEAAX$$QEAV<lambda_f2e299630e499de9f9a165e60fcd3db5>@@AEAV<lambda_2ae9d31cdba2644fcbeaf08da7c24588>@@$$QEAV<lambda_40d01ff24d0e7b3814fdbdcee8eab3c7>@@@Z@4HA 000000018002caa4     libucrt:per_thread_data.obj
 0002:0000caa4       $unwind$__acrt_update_thread_locale_data$fin$0 000000018002caa4     libucrt:locale_refcounting.obj
 0002:0000caa4       $unwind$?fin$0@?0???$?RV<lambda_410d79af7f07d98d83a3f525b3859a53>@@AEAV<lambda_3e16ef9562a7dcce91392c22ab16ea36>@@V<lambda_38119f0e861e05405d8a144b9b982f0a>@@@?$__crt_seh_guarded_call@X@@QEAAX$$QEAV<lambda_410d79af7f07d98d83a3f525b3859a53>@@AEAV<lambda_3e16ef9562a7dcce91392c22ab16ea36>@@$$QEAV<lambda_38119f0e861e05405d8a144b9b982f0a>@@@Z@4HA 000000018002caa4     libucrt:wsetlocale.obj
 0002:0000caa4       $unwind$?fin$0@?0???$?RV<lambda_ad8af0d99a0adf03d037d7dffe354bb5>@@AEAV<lambda_c9ba49e555ba839a7b07aa3fbecb7617>@@V<lambda_2f1ebd5d68526518146ae959c9e734c8>@@@?$__crt_seh_guarded_call@H@@QEAAH$$QEAV<lambda_ad8af0d99a0adf03d037d7dffe354bb5>@@AEAV<lambda_c9ba49e555ba839a7b07aa3fbecb7617>@@$$QEAV<lambda_2f1ebd5d68526518146ae959c9e734c8>@@@Z@4HA 000000018002caa4     libucrt:close.obj
 0002:0000caa4       $unwind$?fin$0@?0???$?RV<lambda_a37b2b86f63e897a80ea819b0eb08c01>@@AEAV<lambda_38ce7e780aa69e748d6df282ebc68efe>@@V<lambda_99fb1378e971ab6e7edea83e3a7a83a2>@@@?$__crt_seh_guarded_call@H@@QEAAH$$QEAV<lambda_a37b2b86f63e897a80ea819b0eb08c01>@@AEAV<lambda_38ce7e780aa69e748d6df282ebc68efe>@@$$QEAV<lambda_99fb1378e971ab6e7edea83e3a7a83a2>@@@Z@4HA 000000018002caa4     libucrt:commit.obj
 0002:0000caa4       $unwind$__acrt_initialize_lowio$fin$0 000000018002caa4     libucrt:ioinit.obj
 0002:0000caa4       $unwind$__acrt_lowio_ensure_fh_exists$fin$0 000000018002caa4     libucrt:osfinfo.obj
 0002:0000caa4       $unwind$_alloc_osfhnd$fin$0 000000018002caa4     libucrt:osfinfo.obj
 0002:0000caa4       $unwind$?fin$0@?0???$?RV<lambda_efdfa57d1f175319df784efa44bb7b81>@@AEAV<lambda_5f0a4c1567f8adc6734073e5d1e1b35c>@@V<lambda_2e8a7d3640ea6ccb4c2413664c2db6fd>@@@?$__crt_seh_guarded_call@X@@QEAAX$$QEAV<lambda_efdfa57d1f175319df784efa44bb7b81>@@AEAV<lambda_5f0a4c1567f8adc6734073e5d1e1b35c>@@$$QEAV<lambda_2e8a7d3640ea6ccb4c2413664c2db6fd>@@@Z@4HA 000000018002caa4     libucrt:mbctype.obj
 0002:0000caa4       $unwind$?fin$0@?0??update_thread_multibyte_data_internal@@YAPEAU__crt_multibyte_data@@QEAU__acrt_ptd@@QEAPEAU1@@Z@4HA 000000018002caa4     libucrt:mbctype.obj
 0002:0000caa4       $unwind$?fin$0@?0???$?RV<lambda_450d765d439847d4c735a33c368b5fc0>@@AEAV<lambda_44731a7d0e6d81c3e6aa82d741081786>@@V<lambda_601a2a7da3b7a96e9554ac7215c4b07c>@@@?$__crt_seh_guarded_call@P6AXH@Z@@QEAAP6AXH@Z$$QEAV<lambda_450d765d439847d4c735a33c368b5fc0>@@AEAV<lambda_44731a7d0e6d81c3e6aa82d741081786>@@$$QEAV<lambda_601a2a7da3b7a96e9554ac7215c4b07c>@@@Z@4HA 000000018002caa4     libucrt:signal.obj
 0002:0000caa4       $unwind$raise$fin$0        000000018002caa4     libucrt:signal.obj
 0002:0000caa4       $unwind$?filt$0@?0???R<lambda_6e4b09c48022b2350581041d5f6b0c4c>@@QEBA@XZ@4HA 000000018002caa4     libucrt:exit.obj
 0002:0000caa4       $unwind$?fin$0@?0???$?RV<lambda_d80eeec6fff315bfe5c115232f3240e3>@@AEAV<lambda_6e4b09c48022b2350581041d5f6b0c4c>@@V<lambda_2358e3775559c9db80273638284d5e45>@@@?$__crt_seh_guarded_call@X@@QEAAX$$QEAV<lambda_d80eeec6fff315bfe5c115232f3240e3>@@AEAV<lambda_6e4b09c48022b2350581041d5f6b0c4c>@@$$QEAV<lambda_2358e3775559c9db80273638284d5e45>@@@Z@4HA 000000018002caa4     libucrt:exit.obj
 0002:0000caa4       $unwind$?fin$0@?0???$?RV<lambda_7777bce6b2f8c936911f934f8298dc43>@@AEAV<lambda_f03950bc5685219e0bcd2087efbe011e>@@V<lambda_3883c3dff614d5e0c5f61bb1ac94921c>@@@?$__crt_seh_guarded_call@H@@QEAAH$$QEAV<lambda_7777bce6b2f8c936911f934f8298dc43>@@AEAV<lambda_f03950bc5685219e0bcd2087efbe011e>@@$$QEAV<lambda_3883c3dff614d5e0c5f61bb1ac94921c>@@@Z@4HA 000000018002caa4     libucrt:onexit.obj
 0002:0000caa4       $unwind$_fcloseall$fin$0   000000018002caa4     libucrt:closeall.obj
 0002:0000caa4       $unwind$?fin$0@?0???$?RV<lambda_842d9ff0dc9ef11c61343bbaebe7f885>@@AEAV<lambda_c5860995281e5c4ce005b3de8f5874ee>@@V<lambda_d90129c13df834fdcbf8d2b88dafcf2d>@@@?$__crt_seh_guarded_call@X@@QEAAX$$QEAV<lambda_842d9ff0dc9ef11c61343bbaebe7f885>@@AEAV<lambda_c5860995281e5c4ce005b3de8f5874ee>@@$$QEAV<lambda_d90129c13df834fdcbf8d2b88dafcf2d>@@@Z@4HA 000000018002caa4     libucrt:fflush.obj
 0002:0000caa4       $unwind$?fin$0@?0???$?RV<lambda_886d6c58226a84441f68b9f2b8217b83>@@AEAV<lambda_ab61a845afdef5b7c387490eaf3616ee>@@V<lambda_f7f22ab5edc0698d5f6905b0d3f44752>@@@?$__crt_seh_guarded_call@X@@QEAAX$$QEAV<lambda_886d6c58226a84441f68b9f2b8217b83>@@AEAV<lambda_ab61a845afdef5b7c387490eaf3616ee>@@$$QEAV<lambda_f7f22ab5edc0698d5f6905b0d3f44752>@@@Z@4HA 000000018002caa4     libucrt:fflush.obj
 0002:0000caa4       $unwind$?fin$0@?0???$common_fsopen@D@@YAPEAU_iobuf@@QEBD0H@Z@4HA 000000018002caa4     libucrt:fopen.obj
 0002:0000caa4       $unwind$?fin$0@?0???$?RV<lambda_d854c62834386a3b23916ad6dae2782d>@@AEAV<lambda_303760bc4008a2b3ec4768a30b06a80c>@@V<lambda_4780a7ea4f8cbd2590aec34bd14e2bbf>@@@?$__crt_seh_guarded_call@H@@QEAAH$$QEAV<lambda_d854c62834386a3b23916ad6dae2782d>@@AEAV<lambda_303760bc4008a2b3ec4768a30b06a80c>@@$$QEAV<lambda_4780a7ea4f8cbd2590aec34bd14e2bbf>@@@Z@4HA 000000018002caa4     libucrt:output.obj
 0002:0000caa4       $unwind$?fin$0@?0??__acrt_stdio_allocate_stream@@YA?AV__crt_stdio_stream@@XZ@4HA 000000018002caa4     libucrt:stream.obj
 0002:0000caa4       $unwind$_ctrlfp$filt$0     000000018002caa4     libucrt:fpctrl.obj
 0002:0000caa4       $unwind$common_control87$filt$0 000000018002caa4     libucrt:ieee.obj
 0002:0000caac       $unwind$?dllmain_crt_process_detach@@YAH_N@Z 000000018002caac     LIBCMT:dll_dllmain.obj
 0002:0000cb00       $unwind$?dllmain_dispatch@@YAHQEAUHINSTANCE__@@KQEAX@Z 000000018002cb00     LIBCMT:dll_dllmain.obj
 0002:0000cb28       $unwind$?filt$0@?0??dllmain_dispatch@@YAHQEAUHINSTANCE__@@KQEAX@Z@4HA 000000018002cb28     LIBCMT:dll_dllmain.obj
 0002:0000cb28       $unwind$?fin$0@?0???$common_lseek@_J@@YA_JH_JHAEAV__crt_cached_ptd_host@@@Z@4HA 000000018002cb28     libucrt:lseek.obj
 0002:0000cb28       $unwind$_write_internal$fin$0 000000018002cb28     libucrt:write.obj
 0002:0000cb28       $unwind$?fin$0@?0??_fclose_internal@@YAHQEAU_iobuf@@AEAV__crt_cached_ptd_host@@@Z@4HA 000000018002cb28     libucrt:fclose.obj
 0002:0000cb30       $unwind$__report_securityfailure 000000018002cb30     LIBCMT:gs_report.obj
 0002:0000cb38       $unwind$__report_gsfailure 000000018002cb38     LIBCMT:gs_report.obj
 0002:0000cb40       $unwind$capture_current_context 000000018002cb40     LIBCMT:gs_report.obj
 0002:0000cb4c       $unwind$capture_previous_context 000000018002cb4c     LIBCMT:gs_report.obj
 0002:0000cb58       $unwind$__security_init_cookie 000000018002cb58     LIBCMT:gs_support.obj
 0002:0000cb64       $unwind$__scrt_is_nonwritable_in_current_image 000000018002cb64     LIBCMT:utility.obj
 0002:0000cb84       $unwind$__scrt_is_nonwritable_in_current_image$filt$0 000000018002cb84     LIBCMT:utility.obj
 0002:0000cb8c       $unwind$__scrt_dllmain_exception_filter 000000018002cb8c     LIBCMT:utility.obj
 0002:0000cb8c       $unwind$?GetHandlerSearchState@__FrameHandler3@@SAHPEA_KPEAU_xDISPATCHER_CONTEXT@@PEBU_s_FuncInfo@@@Z 000000018002cb8c     libvcruntime:frame.obj
 0002:0000cb8c       $unwind$?Is_bad_exception_allowed@@YAEPEBU_s_ESTypeList@@@Z 000000018002cb8c     libvcruntime:frame.obj
 0002:0000cb8c       $unwind$?CatchTryBlock@__FrameHandler3@@SAPEBU_s_TryBlockMapEntry@@PEBU_s_FuncInfo@@H@Z 000000018002cb8c     libvcruntime:risctrnsctrl.obj
 0002:0000cb8c       $unwind$?should_round_up@@YA_NQEBD0HW4__acrt_has_trailing_digits@@W4__acrt_rounding_mode@@@Z 000000018002cb8c     libucrt:_fptostr.obj
 0002:0000cb8c       $unwind$_recalloc_base     000000018002cb8c     libucrt:recalloc.obj
 0002:0000cb8c       $unwind$__acrt_free_locale 000000018002cb8c     libucrt:locale_refcounting.obj
 0002:0000cb8c       $unwind$__acrt_lowio_create_handle_array 000000018002cb8c     libucrt:osfinfo.obj
 0002:0000cb8c       $unwind$_seh_filter_exe    000000018002cb8c     libucrt:exception_filter.obj
 0002:0000cb8c       $unwind$__acrt_stdio_flush_nolock 000000018002cb8c     libucrt:fflush.obj
 0002:0000cb8c       $unwind$??$ensure_buffer_is_big_enough@D@formatting_buffer@__crt_stdio_output@@QEAA_N_KAEAV__crt_cached_ptd_host@@@Z 000000018002cb8c     libucrt:output.obj
 0002:0000cba0       $unwind$__scrt_fastfail    000000018002cba0     LIBCMT:utility_desktop.obj
 0002:0000cbb0       $unwind$__isa_available_init 000000018002cbb0     LIBCMT:cpu_disp.obj
 0002:0000cbc0       $xdatasym                  000000018002cbc0     LIBCMT:guard_dispatch.obj
 0002:0000cbc8       $xdatasym                  000000018002cbc8     LIBCMT:guard_xfg_dispatch.obj
 0002:0000cbd0       $xdatasym                  000000018002cbd0     libvcruntime:memcpy.obj
 0002:0000cbe0       $xdatasym                  000000018002cbe0     libvcruntime:memset.obj
 0002:0000cbf0       $unwind$__std_exception_copy 000000018002cbf0     libvcruntime:std_exception.obj
 0002:0000cbf0       $unwind$_free_osfhnd       000000018002cbf0     libucrt:osfinfo.obj
 0002:0000cc04       $unwind$_CxxThrowException 000000018002cc04     libvcruntime:throw.obj
 0002:0000cc14       $unwind$__C_specific_handler 000000018002cc14     libvcruntime:riscchandler.obj
 0002:0000cc14       $unwind$?GetRangeOfTrysToCheck@__FrameHandler3@@SA?AU?$pair@Viterator@TryBlockMap@__FrameHandler3@@V123@@std@@AEAVTryBlockMap@1@HPEAU_xDISPATCHER_CONTEXT@@PEBU_s_FuncInfo@@H@Z 000000018002cc14     libvcruntime:risctrnsctrl.obj
 0002:0000cc30       $unwind$__DestructExceptionObject 000000018002cc30     libvcruntime:ehhelpers.obj
 0002:0000cc50       $unwind$__DestructExceptionObject$filt$0 000000018002cc50     libvcruntime:ehhelpers.obj
 0002:0000cc50       $unwind$?fin$1@?0??CxxCallCatchBlock@__FrameHandler3@@SAPEAXPEAU_EXCEPTION_RECORD@@@Z@4HA 000000018002cc50     libvcruntime:frame.obj
 0002:0000cc60       $xdatasym                  000000018002cc60     libvcruntime:notify.obj
 0002:0000cc6c       $unwind$?GetEstablisherFrame@__FrameHandler3@@SAPEA_KPEA_KPEAU_xDISPATCHER_CONTEXT@@PEBU_s_FuncInfo@@0@Z 000000018002cc6c     libvcruntime:risctrnsctrl.obj
 0002:0000cc84       $unwind$?UnwindNestedFrames@__FrameHandler3@@SAXPEA_KPEAUEHExceptionRecord@@PEAU_CONTEXT@@0PEAXPEBU_s_FuncInfo@@HHPEBU_s_HandlerType@@PEAU_xDISPATCHER_CONTEXT@@E@Z 000000018002cc84     libvcruntime:risctrnsctrl.obj
 0002:0000cc98       $unwind$__CxxFrameHandler3 000000018002cc98     libvcruntime:risctrnsctrl.obj
 0002:0000ccac       $unwind$??$_CallSETranslator@V__FrameHandler3@@@@YAHPEAUEHExceptionRecord@@PEA_KPEAU_CONTEXT@@PEAU_xDISPATCHER_CONTEXT@@PEBU_s_FuncInfo@@K1H@Z 000000018002ccac     libvcruntime:risctrnsctrl.obj
 0002:0000cccc       $unwind$?filt$0@?0???$_CallSETranslator@V__FrameHandler3@@@@YAHPEAUEHExceptionRecord@@PEA_KPEAU_CONTEXT@@PEAU_xDISPATCHER_CONTEXT@@PEBU_s_FuncInfo@@K1H@Z@4HA 000000018002cccc     libvcruntime:risctrnsctrl.obj
 0002:0000ccd8       $unwind$?try_get_function@@YAPEAXW4function_id@?A0x14174aea@@QEBDQEBW4module_id@2@2@Z 000000018002ccd8     libvcruntime:winapi_downlevel.obj
 0002:0000ccd8       $unwind$?try_get_function@@YAPEAXW4function_id@?A0x391cf84c@@QEBDQEBW4module_id@2@2@Z 000000018002ccd8     libucrt:winapi_thunks.obj
 0002:0000ccd8       $unwind$??$parse_command_line@D@@YAXPEADPEAPEAD0PEA_K2@Z 000000018002ccd8     libucrt:argv_parsing.obj
 0002:0000ccf4       $unwind$?FrameUnwindToState@__FrameHandler3@@SAXPEA_KPEAU_xDISPATCHER_CONTEXT@@PEBU_s_FuncInfo@@H@Z 000000018002ccf4     libvcruntime:frame.obj
 0002:0000cd40       $unwind$?CxxCallCatchBlock@__FrameHandler3@@SAPEAXPEAU_EXCEPTION_RECORD@@@Z 000000018002cd40     libvcruntime:frame.obj
 0002:0000cd7c       $unwind$?IsInExceptionSpec@@YAEPEAUEHExceptionRecord@@PEBU_s_ESTypeList@@@Z 000000018002cd7c     libvcruntime:frame.obj
 0002:0000cd98       $unwind$__GSHandlerCheck_EH 000000018002cd98     LIBCMT:gshandlereh.obj
 0002:0000cd98       $unwind$??$TypeMatchHelper@V__FrameHandler3@@@@YAHPEBU_s_HandlerType@@PEBU_s_CatchableType@@PEBU_s_ThrowInfo@@@Z 000000018002cd98     libvcruntime:frame.obj
 0002:0000cd98       $unwind$?initialize_stdio_handles_nolock@@YAXXZ 000000018002cd98     libucrt:ioinit.obj
 0002:0000cd98       $unwind$__acrt_lowio_set_os_handle 000000018002cd98     libucrt:osfinfo.obj
 0002:0000cd98       $unwind$__acrt_initialize_stdio 000000018002cd98     libucrt:_file.obj
 0002:0000cdb0       $unwind$??$BuildCatchObjectHelperInternal@V__FrameHandler3@@@@YAHPEAUEHExceptionRecord@@PEAXPEBU_s_HandlerType@@PEBU_s_CatchableType@@@Z 000000018002cdb0     libvcruntime:frame.obj
 0002:0000cdf0       $unwind$??$BuildCatchObjectInternal@V__FrameHandler3@@@@YAXPEAUEHExceptionRecord@@PEAXPEBU_s_HandlerType@@PEBU_s_CatchableType@@@Z 000000018002cdf0     libvcruntime:frame.obj
 0002:0000ce1c       $unwind$??$__InternalCxxFrameHandler@V__FrameHandler3@@@@YA?AW4_EXCEPTION_DISPOSITION@@PEAUEHExceptionRecord@@PEA_KPEAU_CONTEXT@@PEAU_xDISPATCHER_CONTEXT@@PEBU_s_FuncInfo@@H1E@Z 000000018002ce1c     libvcruntime:frame.obj
 0002:0000ce1c       $unwind$?fp_format_e@@YAHQEBNQEAD_K12H_NIW4__acrt_rounding_mode@@AEAV__crt_cached_ptd_host@@@Z 000000018002ce1c     libucrt:cvt.obj
 0002:0000ce34       $unwind$??$FindHandler@V__FrameHandler3@@@@YAXPEAUEHExceptionRecord@@PEA_KPEAU_CONTEXT@@PEAU_xDISPATCHER_CONTEXT@@PEBU_s_FuncInfo@@EH1@Z 000000018002ce34     libvcruntime:frame.obj
 0002:0000ce54       $unwind$??$CatchIt@V__FrameHandler3@@@@YAXPEAUEHExceptionRecord@@PEA_KPEAU_CONTEXT@@PEAU_xDISPATCHER_CONTEXT@@PEBU_s_FuncInfo@@PEBU_s_HandlerType@@PEBU_s_CatchableType@@PEBU_s_TryBlockMapEntry@@H1EE@Z 000000018002ce54     libvcruntime:frame.obj
 0002:0000ce6c       $unwind$??$FindHandlerForForeignException@V__FrameHandler3@@@@YAXPEAUEHExceptionRecord@@PEA_KPEAU_CONTEXT@@PEAU_xDISPATCHER_CONTEXT@@PEBU_s_FuncInfo@@HH1@Z 000000018002ce6c     libvcruntime:frame.obj
 0002:0000ce88       $xdatasym                  000000018002ce88     libvcruntime:handlers.obj
 0002:0000cea8       $xdatasym                  000000018002cea8     libucrt:strlen.obj
 0002:0000ceb0       $xdatasym                  000000018002ceb0     libucrt:strncat.obj
 0002:0000ceb8       $xdatasym                  000000018002ceb8     libucrt:strncpy.obj
 0002:0000cebc       $unwind$__stdio_common_vfprintf 000000018002cebc     libucrt:output.obj
 0002:0000cecc       $unwind$__stdio_common_vsprintf 000000018002cecc     libucrt:output.obj
 0002:0000ceec       $unwind$?get_raw_ptd@__crt_cached_ptd_host@@QEAAPEAU__acrt_ptd@@XZ 000000018002ceec     libucrt:output.obj
 0002:0000cef4       $chain$0$?get_raw_ptd@__crt_cached_ptd_host@@QEAAPEAU__acrt_ptd@@XZ 000000018002cef4     libucrt:output.obj
 0002:0000cf08       $chain$1$?get_raw_ptd@__crt_cached_ptd_host@@QEAAPEAU__acrt_ptd@@XZ 000000018002cf08     libucrt:output.obj
 0002:0000cf18       $unwind$??$create_environment@D@@YAQEAPEADQEAD@Z 000000018002cf18     libucrt:environment_initialization.obj
 0002:0000cf18       $unwind$_mbtowc_internal   000000018002cf18     libucrt:mbtowc.obj
 0002:0000cf18       $unwind$??$__acrt_convert_wcs_mbs_cp@D_WV<lambda_7c9dea7b4ca7285d2cdb541a38da6275>@@U__crt_win32_buffer_internal_dynamic_resizing@@@@YAHQEBDAEAV?$__crt_win32_buffer@_WU__crt_win32_buffer_internal_dynamic_resizing@@@@AEBV<lambda_7c9dea7b4ca7285d2cdb541a38da6275>@@I@Z 000000018002cf18     libucrt:argv_wildcards.obj
 0002:0000cf18       $unwind$??$type_case_integer@$07@?$output_processor@DV?$stream_output_adapter@D@__crt_stdio_output@@V?$standard_base@DV?$stream_output_adapter@D@__crt_stdio_output@@@2@@__crt_stdio_output@@AEAA_N_N@Z 000000018002cf18     libucrt:output.obj
 0002:0000cf18       $unwind$??$type_case_integer@$07@?$output_processor@DV?$string_output_adapter@D@__crt_stdio_output@@V?$standard_base@DV?$string_output_adapter@D@__crt_stdio_output@@@2@@__crt_stdio_output@@AEAA_N_N@Z 000000018002cf18     libucrt:output.obj
 0002:0000cf18       $unwind$??$type_case_integer@$09@?$output_processor@DV?$stream_output_adapter@D@__crt_stdio_output@@V?$standard_base@DV?$stream_output_adapter@D@__crt_stdio_output@@@2@@__crt_stdio_output@@AEAA_N_N@Z 000000018002cf18     libucrt:output.obj
 0002:0000cf18       $unwind$??$type_case_integer@$09@?$output_processor@DV?$string_output_adapter@D@__crt_stdio_output@@V?$standard_base@DV?$string_output_adapter@D@__crt_stdio_output@@@2@@__crt_stdio_output@@AEAA_N_N@Z 000000018002cf18     libucrt:output.obj
 0002:0000cf18       $unwind$??$type_case_integer@$0BA@@?$output_processor@DV?$stream_output_adapter@D@__crt_stdio_output@@V?$standard_base@DV?$stream_output_adapter@D@__crt_stdio_output@@@2@@__crt_stdio_output@@AEAA_N_N@Z 000000018002cf18     libucrt:output.obj
 0002:0000cf18       $unwind$??$type_case_integer@$0BA@@?$output_processor@DV?$string_output_adapter@D@__crt_stdio_output@@V?$standard_base@DV?$string_output_adapter@D@__crt_stdio_output@@@2@@__crt_stdio_output@@AEAA_N_N@Z 000000018002cf18     libucrt:output.obj
 0002:0000cf18       $unwind$?process@?$output_processor@DV?$stream_output_adapter@D@__crt_stdio_output@@V?$standard_base@DV?$stream_output_adapter@D@__crt_stdio_output@@@2@@__crt_stdio_output@@QEAAHXZ 000000018002cf18     libucrt:output.obj
 0002:0000cf18       $unwind$?process@?$output_processor@DV?$string_output_adapter@D@__crt_stdio_output@@V?$standard_base@DV?$string_output_adapter@D@__crt_stdio_output@@@2@@__crt_stdio_output@@QEAAHXZ 000000018002cf18     libucrt:output.obj
 0002:0000cf30       $unwind$?parse_int_from_format_string@?$output_processor@DV?$stream_output_adapter@D@__crt_stdio_output@@V?$standard_base@DV?$stream_output_adapter@D@__crt_stdio_output@@@2@@__crt_stdio_output@@AEAA_NQEAH@Z 000000018002cf30     libucrt:output.obj
 0002:0000cf30       $unwind$?parse_int_from_format_string@?$output_processor@DV?$string_output_adapter@D@__crt_stdio_output@@V?$standard_base@DV?$string_output_adapter@D@__crt_stdio_output@@@2@@__crt_stdio_output@@AEAA_NQEAH@Z 000000018002cf30     libucrt:output.obj
 0002:0000cf44       $unwind$?state_case_type@?$output_processor@DV?$stream_output_adapter@D@__crt_stdio_output@@V?$standard_base@DV?$stream_output_adapter@D@__crt_stdio_output@@@2@@__crt_stdio_output@@AEAA_NXZ 000000018002cf44     libucrt:output.obj
 0002:0000cf64       $unwind$?type_case_a@?$output_processor@DV?$stream_output_adapter@D@__crt_stdio_output@@V?$standard_base@DV?$stream_output_adapter@D@__crt_stdio_output@@@2@@__crt_stdio_output@@AEAA_NXZ 000000018002cf64     libucrt:output.obj
 0002:0000cf64       $unwind$?type_case_a@?$output_processor@DV?$string_output_adapter@D@__crt_stdio_output@@V?$standard_base@DV?$string_output_adapter@D@__crt_stdio_output@@@2@@__crt_stdio_output@@AEAA_NXZ 000000018002cf64     libucrt:output.obj
 0002:0000cf78       $unwind$??R<lambda_303760bc4008a2b3ec4768a30b06a80c>@@QEBAHXZ 000000018002cf78     libucrt:output.obj
 0002:0000cf9c       $unwind$?write_string@?$string_output_adapter@D@__crt_stdio_output@@QEBAXQEBDHQEAHAEAV__crt_cached_ptd_host@@@Z 000000018002cf9c     libucrt:output.obj
 0002:0000cfb4       $unwind$?state_case_type@?$output_processor@DV?$string_output_adapter@D@__crt_stdio_output@@V?$standard_base@DV?$string_output_adapter@D@__crt_stdio_output@@@2@@__crt_stdio_output@@AEAA_NXZ 000000018002cfb4     libucrt:output.obj
 0002:0000cfd8       $unwind$??$?RV<lambda_d854c62834386a3b23916ad6dae2782d>@@AEAV<lambda_303760bc4008a2b3ec4768a30b06a80c>@@V<lambda_4780a7ea4f8cbd2590aec34bd14e2bbf>@@@?$__crt_seh_guarded_call@H@@QEAAH$$QEAV<lambda_d854c62834386a3b23916ad6dae2782d>@@AEAV<lambda_303760bc4008a2b3ec4768a30b06a80c>@@$$QEAV<lambda_4780a7ea4f8cbd2590aec34bd14e2bbf>@@@Z 000000018002cfd8     libucrt:output.obj
 0002:0000cffc       $unwind$??$copy_and_add_argument_to_buffer@D@@YAHQEBD0_KAEAV?$argument_list@D@?A0x5f5c8891@@@Z 000000018002cffc     libucrt:argv_wildcards.obj
 0002:0000cffc       $unwind$??$parse_integer@KV?$c_string_character_source@D@__crt_strtox@@$0A@@__crt_strtox@@YAKAEAV__crt_cached_ptd_host@@V?$c_string_character_source@D@0@H_N@Z 000000018002cffc     libucrt:output.obj
 0002:0000d018       $unwind$strrchr            000000018002d018     libvcruntime:strrchr.obj
 0002:0000d018       $unwind$??$type_case_integer_parse_into_buffer@I$09@?$output_processor@DV?$stream_output_adapter@D@__crt_stdio_output@@V?$standard_base@DV?$stream_output_adapter@D@__crt_stdio_output@@@2@@__crt_stdio_output@@AEAAXI_N@Z 000000018002d018     libucrt:output.obj
 0002:0000d018       $unwind$??$type_case_integer_parse_into_buffer@I$09@?$output_processor@DV?$string_output_adapter@D@__crt_stdio_output@@V?$standard_base@DV?$string_output_adapter@D@__crt_stdio_output@@@2@@__crt_stdio_output@@AEAAXI_N@Z 000000018002d018     libucrt:output.obj
 0002:0000d018       $unwind$??$type_case_integer_parse_into_buffer@_K$09@?$output_processor@DV?$stream_output_adapter@D@__crt_stdio_output@@V?$standard_base@DV?$stream_output_adapter@D@__crt_stdio_output@@@2@@__crt_stdio_output@@AEAAX_K_N@Z 000000018002d018     libucrt:output.obj
 0002:0000d018       $unwind$??$type_case_integer_parse_into_buffer@_K$09@?$output_processor@DV?$string_output_adapter@D@__crt_stdio_output@@V?$standard_base@DV?$string_output_adapter@D@__crt_stdio_output@@@2@@__crt_stdio_output@@AEAAX_K_N@Z 000000018002d018     libucrt:output.obj
 0002:0000d020       $unwind$_chsize_nolock     000000018002d020     libucrt:chsize.obj
 0002:0000d020       $unwind$_close_nolock      000000018002d020     libucrt:close.obj
 0002:0000d020       $unwind$_lseeki64          000000018002d020     libucrt:lseek.obj
 0002:0000d020       $unwind$_lseeki64_nolock   000000018002d020     libucrt:lseek.obj
 0002:0000d020       $unwind$_write             000000018002d020     libucrt:write.obj
 0002:0000d020       $unwind$fclose             000000018002d020     libucrt:fclose.obj
 0002:0000d020       $unwind$_fflush_nolock     000000018002d020     libucrt:fflush.obj
 0002:0000d030       $unwind$?_fclose_nolock_internal@@YAHQEAU_iobuf@@AEAV__crt_cached_ptd_host@@@Z 000000018002d030     libucrt:fclose.obj
 0002:0000d040       $unwind$?_fclose_internal@@YAHQEAU_iobuf@@AEAV__crt_cached_ptd_host@@@Z 000000018002d040     libucrt:fclose.obj
 0002:0000d064       $unwind$??$common_fsopen@D@@YAPEAU_iobuf@@QEBD0H@Z 000000018002d064     libucrt:fopen.obj
 0002:0000d08c       $unwind$??$common_getenv@D@@YAPEADQEBD@Z 000000018002d08c     libucrt:getenv.obj
 0002:0000d0b0       $xdatasym                  000000018002d0b0     libucrt:strcmp.obj
 0002:0000d0b8       $xdatasym                  000000018002d0b8     libucrt:strcat.obj
 0002:0000d0c0       $unwind$__acrt_initialize_winapi_thunks 000000018002d0c0     libucrt:winapi_thunks.obj
 0002:0000d0c0       $unwind$wcsncpy            000000018002d0c0     libucrt:wcsncpy.obj
 0002:0000d0c8       $unwind$_query_new_handler 000000018002d0c8     libucrt:new_handler.obj
 0002:0000d0e8       $unwind$??$free_environment@D@@YAXQEAPEAD@Z 000000018002d0e8     libucrt:environment_initialization.obj
 0002:0000d0e8       $unwind$??$free_environment@_W@@YAXQEAPEA_W@Z 000000018002d0e8     libucrt:environment_initialization.obj
 0002:0000d0e8       $unwind$_initterm          000000018002d0e8     libucrt:initterm.obj
 0002:0000d0f4       $unwind$?try_cor_exit_process@@YAXI@Z 000000018002d0f4     libucrt:exit.obj
 0002:0000d108       $ip2state$?try_cor_exit_process@@YAXI@Z 000000018002d108     libucrt:exit.obj
 0002:0000d110       $unwind$?common_exit@@YAXHW4_crt_exit_cleanup_mode@@W4_crt_exit_return_mode@@@Z 000000018002d110     libucrt:exit.obj
 0002:0000d124       $stateUnwindMap$__dcrt_uninitialize_environments_nolock 000000018002d124     libucrt:environment_initialization.obj
 0002:0000d124       $stateUnwindMap$?common_exit@@YAXHW4_crt_exit_cleanup_mode@@W4_crt_exit_return_mode@@@Z 000000018002d124     libucrt:exit.obj
 0002:0000d124       $stateUnwindMap$_execute_onexit_table 000000018002d124     libucrt:onexit.obj
 0002:0000d130       $ip2state$?common_exit@@YAXHW4_crt_exit_cleanup_mode@@W4_crt_exit_return_mode@@@Z 000000018002d130     libucrt:exit.obj
 0002:0000d138       $unwind$??R<lambda_6e4b09c48022b2350581041d5f6b0c4c>@@QEBA@XZ 000000018002d138     libucrt:exit.obj
 0002:0000d158       $unwind$??$?RV<lambda_d80eeec6fff315bfe5c115232f3240e3>@@AEAV<lambda_6e4b09c48022b2350581041d5f6b0c4c>@@V<lambda_2358e3775559c9db80273638284d5e45>@@@?$__crt_seh_guarded_call@X@@QEAAX$$QEAV<lambda_d80eeec6fff315bfe5c115232f3240e3>@@AEAV<lambda_6e4b09c48022b2350581041d5f6b0c4c>@@$$QEAV<lambda_2358e3775559c9db80273638284d5e45>@@@Z 000000018002d158     libucrt:exit.obj
 0002:0000d17c       $unwind$_configure_narrow_argv 000000018002d17c     libucrt:argv_parsing.obj
 0002:0000d190       $unwind$__dcrt_uninitialize_environments_nolock 000000018002d190     libucrt:environment_initialization.obj
 0002:0000d1a0       $unwind$??$initialize_environment_by_cloning_nolock@D@@YAHXZ 000000018002d1a0     libucrt:environment_initialization.obj
 0002:0000d1b4       $unwind$_execute_onexit_table 000000018002d1b4     libucrt:onexit.obj
 0002:0000d1c8       $ip2state$_execute_onexit_table 000000018002d1c8     libucrt:onexit.obj
 0002:0000d1d0       $unwind$??$?RV<lambda_7777bce6b2f8c936911f934f8298dc43>@@AEAV<lambda_f03950bc5685219e0bcd2087efbe011e>@@V<lambda_3883c3dff614d5e0c5f61bb1ac94921c>@@@?$__crt_seh_guarded_call@H@@QEAAH$$QEAV<lambda_7777bce6b2f8c936911f934f8298dc43>@@AEAV<lambda_f03950bc5685219e0bcd2087efbe011e>@@$$QEAV<lambda_3883c3dff614d5e0c5f61bb1ac94921c>@@@Z 000000018002d1d0     libucrt:onexit.obj
 0002:0000d1f4       $unwind$terminate          000000018002d1f4     libucrt:terminate.obj
 0002:0000d218       $xdatasym                  000000018002d218     libucrt:strncmp.obj
 0002:0000d21c       $unwind$__acrt_call_reportfault 000000018002d21c     libucrt:invalid_parameter.obj
 0002:0000d23c       $unwind$__acrt_fp_strflt_to_string 000000018002d23c     libucrt:_fptostr.obj
 0002:0000d23c       $unwind$??$common_lseek_nolock@_J@@YA_JH_JHAEAV__crt_cached_ptd_host@@@Z 000000018002d23c     libucrt:lseek.obj
 0002:0000d23c       $unwind$_invalid_parameter_internal 000000018002d23c     libucrt:invalid_parameter.obj
 0002:0000d250       $unwind$_invalid_parameter 000000018002d250     libucrt:invalid_parameter.obj
 0002:0000d25c       $unwind$_free_base         000000018002d25c     libucrt:free_base.obj
 0002:0000d25c       $unwind$?destroy_fls@@YAXPEAX@Z 000000018002d25c     libucrt:per_thread_data.obj
 0002:0000d25c       $unwind$__acrt_locale_free_numeric 000000018002d25c     libucrt:initnum.obj
 0002:0000d25c       $unwind$__acrt_locale_free_lc_time_if_unreferenced 000000018002d25c     libucrt:locale_refcounting.obj
 0002:0000d264       $unwind$?fp_format_f@@YAHQEBNQEAD_K12HW4__acrt_rounding_mode@@AEAV__crt_cached_ptd_host@@@Z 000000018002d264     libucrt:cvt.obj
 0002:0000d264       $unwind$__acrt_CompareStringEx 000000018002d264     libucrt:winapi_thunks.obj
 0002:0000d264       $unwind$__acrt_LCMapStringEx 000000018002d264     libucrt:winapi_thunks.obj
 0002:0000d278       $unwind$_fcloseall         000000018002d278     libucrt:closeall.obj
 0002:0000d29c       $unwind$?common_flush_all@@YAH_N@Z 000000018002d29c     libucrt:fflush.obj
 0002:0000d2a4       $unwind$??$?RV<lambda_842d9ff0dc9ef11c61343bbaebe7f885>@@AEAV<lambda_c5860995281e5c4ce005b3de8f5874ee>@@V<lambda_d90129c13df834fdcbf8d2b88dafcf2d>@@@?$__crt_seh_guarded_call@X@@QEAAX$$QEAV<lambda_842d9ff0dc9ef11c61343bbaebe7f885>@@AEAV<lambda_c5860995281e5c4ce005b3de8f5874ee>@@$$QEAV<lambda_d90129c13df834fdcbf8d2b88dafcf2d>@@@Z 000000018002d2a4     libucrt:fflush.obj
 0002:0000d2c8       $unwind$??$?RV<lambda_886d6c58226a84441f68b9f2b8217b83>@@AEAV<lambda_ab61a845afdef5b7c387490eaf3616ee>@@V<lambda_f7f22ab5edc0698d5f6905b0d3f44752>@@@?$__crt_seh_guarded_call@X@@QEAAX$$QEAV<lambda_886d6c58226a84441f68b9f2b8217b83>@@AEAV<lambda_ab61a845afdef5b7c387490eaf3616ee>@@$$QEAV<lambda_f7f22ab5edc0698d5f6905b0d3f44752>@@@Z 000000018002d2c8     libucrt:fflush.obj
 0002:0000d2f0       $unwind$__acrt_initialize_lowio 000000018002d2f0     libucrt:ioinit.obj
 0002:0000d310       $unwind$?initialize_inherited_file_handles_nolock@@YAXXZ 000000018002d310     libucrt:ioinit.obj
 0002:0000d32c       $unwind$__acrt_fp_format   000000018002d32c     libucrt:cvt.obj
 0002:0000d33c       $unwind$?fp_format_e_internal@@YAHQEAD_KH_NIQEAU_strflt@@2AEAV__crt_cached_ptd_host@@@Z 000000018002d33c     libucrt:cvt.obj
 0002:0000d358       $unwind$?should_round_up@@YA_NQEBN_KFW4__acrt_rounding_mode@@@Z 000000018002d358     libucrt:cvt.obj
 0002:0000d358       $unwind$_chsize_nolock_internal 000000018002d358     libucrt:chsize.obj
 0002:0000d374       $unwind$?fp_format_a@@YAHQEBNPEAD_KQEAD2H_NIW4__acrt_rounding_mode@@AEAV__crt_cached_ptd_host@@@Z 000000018002d374     libucrt:cvt.obj
 0002:0000d390       $unwind$?fp_format_g@@YAHQEBNQEAD_K12H_NIW4__acrt_rounding_mode@@AEAV__crt_cached_ptd_host@@@Z 000000018002d390     libucrt:cvt.obj
 0002:0000d3a8       $unwind$_wctomb_internal   000000018002d3a8     libucrt:wctomb.obj
 0002:0000d3bc       $unwind$__acrt_stdio_end_temporary_buffering_nolock 000000018002d3bc     libucrt:_sftbuf.obj
 0002:0000d3c4       $unwind$?construct_ptd_array@@YAXQEAU__acrt_ptd@@@Z 000000018002d3c4     libucrt:per_thread_data.obj
 0002:0000d3cc       $unwind$?destroy_ptd_array@@YAXQEAU__acrt_ptd@@@Z 000000018002d3cc     libucrt:per_thread_data.obj
 0002:0000d3d4       $unwind$??$?RV<lambda_0ae27a3a962d80f24befdcbee591983d>@@AEAV<lambda_8d0ee55de4b1038c4002e0adecdf1839>@@V<lambda_dc504788e8f1664fe9b84e20bfb512f2>@@@?$__crt_seh_guarded_call@X@@QEAAX$$QEAV<lambda_0ae27a3a962d80f24befdcbee591983d>@@AEAV<lambda_8d0ee55de4b1038c4002e0adecdf1839>@@$$QEAV<lambda_dc504788e8f1664fe9b84e20bfb512f2>@@@Z 000000018002d3d4     libucrt:per_thread_data.obj
 0002:0000d3f8       $unwind$??$?RV<lambda_aa87e3671a710a21b5dc78c0bdf72e11>@@AEAV<lambda_92619d2358a28f41a33ba319515a20b9>@@V<lambda_6992ecaafeb10aed2b74cb1fae11a551>@@@?$__crt_seh_guarded_call@X@@QEAAX$$QEAV<lambda_aa87e3671a710a21b5dc78c0bdf72e11>@@AEAV<lambda_92619d2358a28f41a33ba319515a20b9>@@$$QEAV<lambda_6992ecaafeb10aed2b74cb1fae11a551>@@@Z 000000018002d3f8     libucrt:per_thread_data.obj
 0002:0000d41c       $unwind$??$?RV<lambda_f2e299630e499de9f9a165e60fcd3db5>@@AEAV<lambda_2ae9d31cdba2644fcbeaf08da7c24588>@@V<lambda_40d01ff24d0e7b3814fdbdcee8eab3c7>@@@?$__crt_seh_guarded_call@X@@QEAAX$$QEAV<lambda_f2e299630e499de9f9a165e60fcd3db5>@@AEAV<lambda_2ae9d31cdba2644fcbeaf08da7c24588>@@$$QEAV<lambda_40d01ff24d0e7b3814fdbdcee8eab3c7>@@@Z 000000018002d41c     libucrt:per_thread_data.obj
 0002:0000d440       $unwind$??$?RV<lambda_2d41944a1d46af3157314b8a01080d33>@@AEAV<lambda_8f455de75cd7d7f24b4096f044d8b9e6>@@V<lambda_aa500f224e6afead328df44964fe2772>@@@?$__crt_seh_guarded_call@X@@QEAAX$$QEAV<lambda_2d41944a1d46af3157314b8a01080d33>@@AEAV<lambda_8f455de75cd7d7f24b4096f044d8b9e6>@@$$QEAV<lambda_aa500f224e6afead328df44964fe2772>@@@Z 000000018002d440     libucrt:per_thread_data.obj
 0002:0000d464       $unwind$__acrt_uninitialize_locale 000000018002d464     libucrt:wsetlocale.obj
 0002:0000d464       $unwind$__acrt_get_sigabrt_handler 000000018002d464     libucrt:signal.obj
 0002:0000d46c       $unwind$??$?RV<lambda_410d79af7f07d98d83a3f525b3859a53>@@AEAV<lambda_3e16ef9562a7dcce91392c22ab16ea36>@@V<lambda_38119f0e861e05405d8a144b9b982f0a>@@@?$__crt_seh_guarded_call@X@@QEAAX$$QEAV<lambda_410d79af7f07d98d83a3f525b3859a53>@@AEAV<lambda_3e16ef9562a7dcce91392c22ab16ea36>@@$$QEAV<lambda_38119f0e861e05405d8a144b9b982f0a>@@@Z 000000018002d46c     libucrt:wsetlocale.obj
 0002:0000d494       $unwind$_close_internal    000000018002d494     libucrt:close.obj
 0002:0000d49c       $unwind$??$?RV<lambda_ad8af0d99a0adf03d037d7dffe354bb5>@@AEAV<lambda_c9ba49e555ba839a7b07aa3fbecb7617>@@V<lambda_2f1ebd5d68526518146ae959c9e734c8>@@@?$__crt_seh_guarded_call@H@@QEAAH$$QEAV<lambda_ad8af0d99a0adf03d037d7dffe354bb5>@@AEAV<lambda_c9ba49e555ba839a7b07aa3fbecb7617>@@$$QEAV<lambda_2f1ebd5d68526518146ae959c9e734c8>@@@Z 000000018002d49c     libucrt:close.obj
 0002:0000d4c0       $unwind$?__acrt_stdio_allocate_stream@@YA?AV__crt_stdio_stream@@XZ 000000018002d4c0     libucrt:stream.obj
 0002:0000d4e0       $unwind$?find_or_allocate_unused_stream_nolock@@YA?AV__crt_stdio_stream@@XZ 000000018002d4e0     libucrt:stream.obj
 0002:0000d4f4       $unwind$_openfile          000000018002d4f4     libucrt:openfile.obj
 0002:0000d508       $unwind$_strnicoll_l       000000018002d508     libucrt:strnicol.obj
 0002:0000d51c       $unwind$??$common_expand_argv_wildcards@D@@YAHQEAPEADQEAPEAPEAD@Z 000000018002d51c     libucrt:argv_wildcards.obj
 0002:0000d534       $unwind$__dcrt_get_narrow_environment_from_os 000000018002d534     libucrt:get_environment_from_os.obj
 0002:0000d534       $unwind$??$__acrt_convert_wcs_mbs_cp@_WDV<lambda_d8593a27d1aa8c02be35c86a17d324c4>@@U__crt_win32_buffer_internal_dynamic_resizing@@@@YAHQEB_WAEAV?$__crt_win32_buffer@DU__crt_win32_buffer_internal_dynamic_resizing@@@@AEBV<lambda_d8593a27d1aa8c02be35c86a17d324c4>@@I@Z 000000018002d534     libucrt:argv_wildcards.obj
 0002:0000d54c       $unwind$??$expand_argument_wildcards@D@@YAHQEAD0AEAV?$argument_list@D@?A0x5f5c8891@@@Z 000000018002d54c     libucrt:argv_wildcards.obj
 0002:0000d56c       $unwind$__acrt_GetModuleFileNameA 000000018002d56c     libucrt:getmodulefilenamea.obj
 0002:0000d588       $unwind$__dcrt_write_console 000000018002d588     libucrt:initcon.obj
 0002:0000d588       $unwind$??$__acrt_convert_wcs_mbs_cp@_WDV<lambda_f788ae46380686e8b737efdd8c720d07>@@U__crt_win32_buffer_no_resizing@@@@YAHQEB_WAEAV?$__crt_win32_buffer@DU__crt_win32_buffer_no_resizing@@@@AEBV<lambda_f788ae46380686e8b737efdd8c720d07>@@I@Z 000000018002d588     libucrt:getmodulefilenamea.obj
 0002:0000d59c       $unwind$_setmbcp_nolock    000000018002d59c     libucrt:mbctype.obj
 0002:0000d5bc       $unwind$__dcrt_lowio_ensure_console_output_initialized 000000018002d5bc     libucrt:initcon.obj
 0002:0000d5bc       $unwind$?__mbrtowc_utf8@__crt_mbstring@@YA_KPEA_WPEBD_KPEAU_Mbstatet@@AEAV__crt_cached_ptd_host@@@Z 000000018002d5bc     libucrt:mbrtowc.obj
 0002:0000d5bc       $unwind$?getSystemCP@@YAHH@Z 000000018002d5bc     libucrt:mbctype.obj
 0002:0000d5c4       $unwind$?update_thread_multibyte_data_internal@@YAPEAU__crt_multibyte_data@@QEAU__acrt_ptd@@QEAPEAU1@@Z 000000018002d5c4     libucrt:mbctype.obj
 0002:0000d5ec       $unwind$?setmbcp_internal@@YAHH_NQEAU__acrt_ptd@@QEAPEAU__crt_multibyte_data@@@Z 000000018002d5ec     libucrt:mbctype.obj
 0002:0000d604       $unwind$?setSBUpLow@@YAXPEAU__crt_multibyte_data@@@Z 000000018002d604     libucrt:mbctype.obj
 0002:0000d620       $unwind$??$?RV<lambda_efdfa57d1f175319df784efa44bb7b81>@@AEAV<lambda_5f0a4c1567f8adc6734073e5d1e1b35c>@@V<lambda_2e8a7d3640ea6ccb4c2413664c2db6fd>@@@?$__crt_seh_guarded_call@X@@QEAAX$$QEAV<lambda_efdfa57d1f175319df784efa44bb7b81>@@AEAV<lambda_5f0a4c1567f8adc6734073e5d1e1b35c>@@$$QEAV<lambda_2e8a7d3640ea6ccb4c2413664c2db6fd>@@@Z 000000018002d620     libucrt:mbctype.obj
 0002:0000d644       $unwind$?x_ismbbtype_l@@YAHPEAU__crt_locale_pointers@@IHH@Z 000000018002d644     libucrt:ismbbyte.obj
 0002:0000d644       $unwind$_strnicmp_l        000000018002d644     libucrt:strnicmp.obj
 0002:0000d654       $unwind$__acrt_WideCharToMultiByte 000000018002d654     libucrt:widechartomultibyte.obj
 0002:0000d660       $unwind$??$common_set_variable_in_environment_nolock@D@@YAHQEADH@Z 000000018002d660     libucrt:setenv.obj
 0002:0000d678       $unwind$??$copy_environment@D@@YAPEAPEADQEAPEAD@Z 000000018002d678     libucrt:setenv.obj
 0002:0000d68c       $unwind$raise              000000018002d68c     libucrt:signal.obj
 0002:0000d6cc       $unwind$??$?RV<lambda_450d765d439847d4c735a33c368b5fc0>@@AEAV<lambda_44731a7d0e6d81c3e6aa82d741081786>@@V<lambda_601a2a7da3b7a96e9554ac7215c4b07c>@@@?$__crt_seh_guarded_call@P6AXH@Z@@QEAAP6AXH@Z$$QEAV<lambda_450d765d439847d4c735a33c368b5fc0>@@AEAV<lambda_44731a7d0e6d81c3e6aa82d741081786>@@$$QEAV<lambda_601a2a7da3b7a96e9554ac7215c4b07c>@@@Z 000000018002d6cc     libucrt:signal.obj
 0002:0000d6f0       $unwind$_commit            000000018002d6f0     libucrt:commit.obj
 0002:0000d6f8       $unwind$??$?RV<lambda_a37b2b86f63e897a80ea819b0eb08c01>@@AEAV<lambda_38ce7e780aa69e748d6df282ebc68efe>@@V<lambda_99fb1378e971ab6e7edea83e3a7a83a2>@@@?$__crt_seh_guarded_call@H@@QEAAH$$QEAV<lambda_a37b2b86f63e897a80ea819b0eb08c01>@@AEAV<lambda_38ce7e780aa69e748d6df282ebc68efe>@@$$QEAV<lambda_99fb1378e971ab6e7edea83e3a7a83a2>@@@Z 000000018002d6f8     libucrt:commit.obj
 0002:0000d71c       $unwind$_write_nolock      000000018002d71c     libucrt:write.obj
 0002:0000d734       $unwind$_write_internal    000000018002d734     libucrt:write.obj
 0002:0000d760       $unwind$?write_double_translated_ansi_nolock@@YA?AUwrite_result@?A0x17268360@@HQEBDIAEAV__crt_cached_ptd_host@@@Z 000000018002d760     libucrt:write.obj
 0002:0000d788       $ip2state$?write_double_translated_ansi_nolock@@YA?AUwrite_result@?A0x17268360@@HQEBDIAEAV__crt_cached_ptd_host@@@Z 000000018002d788     libucrt:write.obj
 0002:0000d790       $unwind$?write_text_ansi_nolock@@YA?AUwrite_result@?A0x17268360@@HQEBDI@Z 000000018002d790     libucrt:write.obj
 0002:0000d790       $unwind$?write_text_utf16le_nolock@@YA?AUwrite_result@?A0x17268360@@HQEBDI@Z 000000018002d790     libucrt:write.obj
 0002:0000d7b0       $unwind$?write_text_utf8_nolock@@YA?AUwrite_result@?A0x17268360@@HQEBDI@Z 000000018002d7b0     libucrt:write.obj
 0002:0000d7d4       $unwind$_alloc_osfhnd      000000018002d7d4     libucrt:osfinfo.obj
 0002:0000d804       $unwind$__acrt_lowio_destroy_handle_array 000000018002d804     libucrt:osfinfo.obj
 0002:0000d814       $unwind$__acrt_lowio_ensure_fh_exists 000000018002d814     libucrt:osfinfo.obj
 0002:0000d840       $unwind$__acrt_update_thread_locale_data 000000018002d840     libucrt:locale_refcounting.obj
 0002:0000d864       $unwind$__acrt_fltout      000000018002d864     libucrt:cfout.obj
 0002:0000d884       $unwind$?divide@__crt_strtox@@YA_KAEAUbig_integer@1@AEBU21@@Z 000000018002d884     libucrt:cfout.obj
 0002:0000d89c       $chain$0$?divide@__crt_strtox@@YA_KAEAUbig_integer@1@AEBU21@@Z 000000018002d89c     libucrt:cfout.obj
 0002:0000d8b0       $chain$1$?divide@__crt_strtox@@YA_KAEAUbig_integer@1@AEBU21@@Z 000000018002d8b0     libucrt:cfout.obj
 0002:0000d8c0       $unwind$?__mbsrtowcs_utf8@__crt_mbstring@@YA_KPEA_WPEAPEBD_KPEAU_Mbstatet@@AEAV__crt_cached_ptd_host@@@Z 000000018002d8c0     libucrt:mbrtowc.obj
 0002:0000d8d8       $unwind$??$write_buffer_nolock@D@@YA_NDV__crt_stdio_stream@@AEAV__crt_cached_ptd_host@@@Z 000000018002d8d8     libucrt:_flsbuf.obj
 0002:0000d8ec       $unwind$__acrt_locale_free_monetary 000000018002d8ec     libucrt:initmon.obj
 0002:0000d8f4       $unwind$__acrt_locale_free_time 000000018002d8f4     libucrt:inittime.obj
 0002:0000d904       $unwind$__acrt_GetStringTypeA 000000018002d904     libucrt:getstringtypea.obj
 0002:0000d92c       $unwind$_sopen_nolock      000000018002d92c     libucrt:open.obj
 0002:0000d948       $unwind$_wsopen_nolock     000000018002d948     libucrt:open.obj
 0002:0000d968       $unwind$??$common_sopen_dispatch@D@@YAHQEBDHHHQEAHH@Z 000000018002d968     libucrt:open.obj
 0002:0000d98c       $unwind$?fin$0@?0???$common_sopen_dispatch@D@@YAHQEBDHHHQEAHH@Z@4HA 000000018002d98c     libucrt:open.obj
 0002:0000d994       $unwind$?decode_options@@YA?AUfile_options@?A0xa9d50aae@@HHH@Z 000000018002d994     libucrt:open.obj
 0002:0000d9a8       $unwind$?truncate_ctrl_z_if_present@@YAHH@Z 000000018002d9a8     libucrt:open.obj
 0002:0000d9b8       $unwind$?configure_text_mode@@YAHHUfile_options@?A0xa9d50aae@@HAEAW4__crt_lowio_text_mode@@@Z 000000018002d9b8     libucrt:open.obj
 0002:0000d9d0       $unwind$__acrt_CompareStringA 000000018002d9d0     libucrt:comparestringa.obj
 0002:0000d9e0       $unwind$?InternalCompareStringA@@YAHPEAU__crt_locale_pointers@@PEB_WKPEBDH2HH@Z 000000018002d9e0     libucrt:comparestringa.obj
 0002:0000da04       $unwind$qsort              000000018002da04     libucrt:qsort.obj
 0002:0000da1c       $chain$4$qsort             000000018002da1c     libucrt:qsort.obj
 0002:0000da40       $chain$5$qsort             000000018002da40     libucrt:qsort.obj
 0002:0000da50       $unwind$strpbrk            000000018002da50     libucrt:strpbrk.obj
 0002:0000da60       $unwind$fallbackMethod     000000018002da60     libucrt:strpbrk.obj
 0002:0000da70       $unwind$__acrt_LCMapStringA 000000018002da70     libucrt:lcmapstringa.obj
 0002:0000da80       $unwind$?__acrt_LCMapStringA_stat@@YAHPEAU__crt_locale_pointers@@PEB_WKPEBDHPEADHHH@Z 000000018002da80     libucrt:lcmapstringa.obj
 0002:0000daa8       $unwind$__acrt_SetEnvironmentVariableA 000000018002daa8     libucrt:setenvironmentvariablea.obj
 0002:0000dac4       $unwind$??$common_lseek@_J@@YA_JH_JHAEAV__crt_cached_ptd_host@@@Z 000000018002dac4     libucrt:lseek.obj
 0002:0000daf0       $unwind$_putwch_nolock     000000018002daf0     libucrt:putwch.obj
 0002:0000daf8       $unwind$_read_nolock       000000018002daf8     libucrt:read.obj
 0002:0000db10       $unwind$?translate_ansi_or_utf8_nolock@@YAHHQEAD_KQEA_W1@Z 000000018002db10     libucrt:read.obj
 0002:0000db28       $unwind$??$translate_text_mode_nolock@_W@@YAHHQEA_W_K@Z 000000018002db28     libucrt:read.obj
 0002:0000db40       $unwind$fesetenv           000000018002db40     libucrt:fesetenv.obj
 0002:0000db50       $xdatasym                  000000018002db50     libucrt:log10.obj
 0002:0000db5c       $unwind$__acrt_fenv_get_control 000000018002db5c     libucrt:_fenvutils.obj
 0002:0000db64       $unwind$__acrt_fenv_set_control 000000018002db64     libucrt:_fenvutils.obj
 0002:0000db74       $unwind$?__mbrtoc32_utf8@__crt_mbstring@@YA_KPEA_UPEBD_KPEAU_Mbstatet@@AEAV__crt_cached_ptd_host@@@Z 000000018002db74     libucrt:mbrtoc32.obj
 0002:0000db90       $unwind$_setmode_nolock    000000018002db90     libucrt:setmode.obj
 0002:0000dba0       $unwind$common_control87   000000018002dba0     libucrt:ieee.obj
 0002:0000dbcc       $unwind$_call_matherr      000000018002dbcc     libucrt:libm_error.obj
 0002:0000dbd4       $unwind$_handle_error      000000018002dbd4     libucrt:libm_error.obj
 0002:0000dbf4       $unwind$__acrt_initialize_fma3 000000018002dbf4     libucrt:fma3_available.obj
 0002:0000dbfc       $unwind$_log_special_common 000000018002dbfc     libucrt:log_special.obj
 0002:0000dc08       $xdatasym                  000000018002dc08     libucrt:fpsr.obj
 0002:0000dc10       $unwind$_raise_exc_ex      000000018002dc10     libucrt:fpexcept.obj
 0002:0000dc24       $unwind$_ctrlfp            000000018002dc24     libucrt:fpctrl.obj
 0002:0000dc4c       $unwind$_IsNonwritableInCurrentImage 000000018002dc4c     LIBCMT:pesect.obj
 0002:0000dc70       $xdatasym                  000000018002dc70     libvcruntime:memcmp.obj
 0002:0000ddd0       .edata                     000000018002ddd0     windowsaccessbridge-64.exp
 0002:0000ddf8       rgpv                       000000018002ddf8     windowsaccessbridge-64.exp
 0002:0000df8c       rgszName                   000000018002df8c     windowsaccessbridge-64.exp
 0002:0000e120       rgwOrd                     000000018002e120     windowsaccessbridge-64.exp
 0002:0000e1ea       szName                     000000018002e1ea     windowsaccessbridge-64.exp
 0002:0000e205       $N00001                    000000018002e205     windowsaccessbridge-64.exp
 0002:0000e227       $N00002                    000000018002e227     windowsaccessbridge-64.exp
 0002:0000e240       $N00003                    000000018002e240     windowsaccessbridge-64.exp
 0002:0000e265       $N00004                    000000018002e265     windowsaccessbridge-64.exp
 0002:0000e281       $N00005                    000000018002e281     windowsaccessbridge-64.exp
 0002:0000e28d       $N00006                    000000018002e28d     windowsaccessbridge-64.exp
 0002:0000e2a9       $N00007                    000000018002e2a9     windowsaccessbridge-64.exp
 0002:0000e2cb       $N00008                    000000018002e2cb     windowsaccessbridge-64.exp
 0002:0000e2ef       $N00009                    000000018002e2ef     windowsaccessbridge-64.exp
 0002:0000e303       $N00010                    000000018002e303     windowsaccessbridge-64.exp
 0002:0000e318       $N00011                    000000018002e318     windowsaccessbridge-64.exp
 0002:0000e336       $N00012                    000000018002e336     windowsaccessbridge-64.exp
 0002:0000e34d       $N00013                    000000018002e34d     windowsaccessbridge-64.exp
 0002:0000e36a       $N00014                    000000018002e36a     windowsaccessbridge-64.exp
 0002:0000e383       $N00015                    000000018002e383     windowsaccessbridge-64.exp
 0002:0000e3a1       $N00016                    000000018002e3a1     windowsaccessbridge-64.exp
 0002:0000e3b8       $N00017                    000000018002e3b8     windowsaccessbridge-64.exp
 0002:0000e3d4       $N00018                    000000018002e3d4     windowsaccessbridge-64.exp
 0002:0000e3eb       $N00019                    000000018002e3eb     windowsaccessbridge-64.exp
 0002:0000e405       $N00020                    000000018002e405     windowsaccessbridge-64.exp
 0002:0000e425       $N00021                    000000018002e425     windowsaccessbridge-64.exp
 0002:0000e438       $N00022                    000000018002e438     windowsaccessbridge-64.exp
 0002:0000e451       $N00023                    000000018002e451     windowsaccessbridge-64.exp
 0002:0000e470       $N00024                    000000018002e470     windowsaccessbridge-64.exp
 0002:0000e489       $N00025                    000000018002e489     windowsaccessbridge-64.exp
 0002:0000e4b0       $N00026                    000000018002e4b0     windowsaccessbridge-64.exp
 0002:0000e4d2       $N00027                    000000018002e4d2     windowsaccessbridge-64.exp
 0002:0000e4ed       $N00028                    000000018002e4ed     windowsaccessbridge-64.exp
 0002:0000e506       $N00029                    000000018002e506     windowsaccessbridge-64.exp
 0002:0000e52a       $N00030                    000000018002e52a     windowsaccessbridge-64.exp
 0002:0000e549       $N00031                    000000018002e549     windowsaccessbridge-64.exp
 0002:0000e570       $N00032                    000000018002e570     windowsaccessbridge-64.exp
 0002:0000e593       $N00033                    000000018002e593     windowsaccessbridge-64.exp
 0002:0000e5ab       $N00034                    000000018002e5ab     windowsaccessbridge-64.exp
 0002:0000e5c2       $N00035                    000000018002e5c2     windowsaccessbridge-64.exp
 0002:0000e5d8       $N00036                    000000018002e5d8     windowsaccessbridge-64.exp
 0002:0000e5f9       $N00037                    000000018002e5f9     windowsaccessbridge-64.exp
 0002:0000e615       $N00038                    000000018002e615     windowsaccessbridge-64.exp
 0002:0000e639       $N00039                    000000018002e639     windowsaccessbridge-64.exp
 0002:0000e659       $N00040                    000000018002e659     windowsaccessbridge-64.exp
 0002:0000e675       $N00041                    000000018002e675     windowsaccessbridge-64.exp
 0002:0000e68b       $N00042                    000000018002e68b     windowsaccessbridge-64.exp
 0002:0000e6a2       $N00043                    000000018002e6a2     windowsaccessbridge-64.exp
 0002:0000e6be       $N00044                    000000018002e6be     windowsaccessbridge-64.exp
 0002:0000e6d5       $N00045                    000000018002e6d5     windowsaccessbridge-64.exp
 0002:0000e6eb       $N00046                    000000018002e6eb     windowsaccessbridge-64.exp
 0002:0000e70a       $N00047                    000000018002e70a     windowsaccessbridge-64.exp
 0002:0000e71e       $N00048                    000000018002e71e     windowsaccessbridge-64.exp
 0002:0000e72f       $N00049                    000000018002e72f     windowsaccessbridge-64.exp
 0002:0000e754       $N00050                    000000018002e754     windowsaccessbridge-64.exp
 0002:0000e765       $N00051                    000000018002e765     windowsaccessbridge-64.exp
 0002:0000e782       $N00052                    000000018002e782     windowsaccessbridge-64.exp
 0002:0000e7a7       $N00053                    000000018002e7a7     windowsaccessbridge-64.exp
 0002:0000e7cc       $N00054                    000000018002e7cc     windowsaccessbridge-64.exp
 0002:0000e7db       $N00055                    000000018002e7db     windowsaccessbridge-64.exp
 0002:0000e7ed       $N00056                    000000018002e7ed     windowsaccessbridge-64.exp
 0002:0000e807       $N00057                    000000018002e807     windowsaccessbridge-64.exp
 0002:0000e820       $N00058                    000000018002e820     windowsaccessbridge-64.exp
 0002:0000e832       $N00059                    000000018002e832     windowsaccessbridge-64.exp
 0002:0000e841       $N00060                    000000018002e841     windowsaccessbridge-64.exp
 0002:0000e85a       $N00061                    000000018002e85a     windowsaccessbridge-64.exp
 0002:0000e86d       $N00062                    000000018002e86d     windowsaccessbridge-64.exp
 0002:0000e885       $N00063                    000000018002e885     windowsaccessbridge-64.exp
 0002:0000e8aa       $N00064                    000000018002e8aa     windowsaccessbridge-64.exp
 0002:0000e8ca       $N00065                    000000018002e8ca     windowsaccessbridge-64.exp
 0002:0000e8e7       $N00066                    000000018002e8e7     windowsaccessbridge-64.exp
 0002:0000e8f4       $N00067                    000000018002e8f4     windowsaccessbridge-64.exp
 0002:0000e901       $N00068                    000000018002e901     windowsaccessbridge-64.exp
 0002:0000e913       $N00069                    000000018002e913     windowsaccessbridge-64.exp
 0002:0000e938       $N00070                    000000018002e938     windowsaccessbridge-64.exp
 0002:0000e945       $N00071                    000000018002e945     windowsaccessbridge-64.exp
 0002:0000e96d       $N00072                    000000018002e96d     windowsaccessbridge-64.exp
 0002:0000e97d       $N00073                    000000018002e97d     windowsaccessbridge-64.exp
 0002:0000e98e       $N00074                    000000018002e98e     windowsaccessbridge-64.exp
 0002:0000e99f       $N00075                    000000018002e99f     windowsaccessbridge-64.exp
 0002:0000e9b0       $N00076                    000000018002e9b0     windowsaccessbridge-64.exp
 0002:0000e9bf       $N00077                    000000018002e9bf     windowsaccessbridge-64.exp
 0002:0000e9d1       $N00078                    000000018002e9d1     windowsaccessbridge-64.exp
 0002:0000e9e3       $N00079                    000000018002e9e3     windowsaccessbridge-64.exp
 0002:0000e9f7       $N00080                    000000018002e9f7     windowsaccessbridge-64.exp
 0002:0000ea09       $N00081                    000000018002ea09     windowsaccessbridge-64.exp
 0002:0000ea1b       $N00082                    000000018002ea1b     windowsaccessbridge-64.exp
 0002:0000ea2d       $N00083                    000000018002ea2d     windowsaccessbridge-64.exp
 0002:0000ea3e       $N00084                    000000018002ea3e     windowsaccessbridge-64.exp
 0002:0000ea50       $N00085                    000000018002ea50     windowsaccessbridge-64.exp
 0002:0000ea63       $N00086                    000000018002ea63     windowsaccessbridge-64.exp
 0002:0000ea7a       $N00087                    000000018002ea7a     windowsaccessbridge-64.exp
 0002:0000ea9c       $N00088                    000000018002ea9c     windowsaccessbridge-64.exp
 0002:0000eabc       $N00089                    000000018002eabc     windowsaccessbridge-64.exp
 0002:0000eae0       $N00090                    000000018002eae0     windowsaccessbridge-64.exp
 0002:0000eaf9       $N00091                    000000018002eaf9     windowsaccessbridge-64.exp
 0002:0000eb0d       $N00092                    000000018002eb0d     windowsaccessbridge-64.exp
 0002:0000eb26       $N00093                    000000018002eb26     windowsaccessbridge-64.exp
 0002:0000eb45       $N00094                    000000018002eb45     windowsaccessbridge-64.exp
 0002:0000eb5d       $N00095                    000000018002eb5d     windowsaccessbridge-64.exp
 0002:0000eb7a       $N00096                    000000018002eb7a     windowsaccessbridge-64.exp
 0002:0000eb93       $N00097                    000000018002eb93     windowsaccessbridge-64.exp
 0002:0000ebb1       $N00098                    000000018002ebb1     windowsaccessbridge-64.exp
 0002:0000ebc9       $N00099                    000000018002ebc9     windowsaccessbridge-64.exp
 0002:0000ebe2       $N00100                    000000018002ebe2     windowsaccessbridge-64.exp
 0002:0000ec01       $N00101                    000000018002ec01     windowsaccessbridge-64.exp
 0002:0000effc       .idata$6                   000000018002effc     kernel32:KERNEL32.dll
 0002:0000f0b8       .idata$6                   000000018002f0b8     user32:USER32.dll
 0003:00000030       ?__vcrt_flsindex@@3KA      0000000180030030     libvcruntime:per_thread_data.obj
 0003:00000160       ?errno_no_memory@@3HA      0000000180030160     libucrt:errno.obj
 0003:00000164       ?doserrno_no_memory@@3KA   0000000180030164     libucrt:errno.obj
 0003:000001b8       ?__acrt_flsindex@@3KA      00000001800301b8     libucrt:per_thread_data.obj
 0003:00000560       _mbctypes                  0000000180030560     libucrt:mbctype.obj
 0003:00000670       _mbcasemaps                0000000180030670     libucrt:mbctype.obj
 0003:00000770       ?__rgctypeflag@@3PADA      0000000180030770     libucrt:mbctype.obj
 0003:00000780       ?__rgcode_page_info@@3PAUcode_page_info@@A 0000000180030780     libucrt:mbctype.obj
 0003:00000a20       ?__dcrt_lowio_console_output_handle@@3PEAXEA 0000000180030a20     libucrt:initcon.obj
 0003:00000a28       ?dazSupported@?1??common_control87@@9@9 0000000180030a28     libucrt:ieee.obj
 0003:00000a30       ?dazSupported@?1??_ctrlfp@@9@9 0000000180030a30     libucrt:fpctrl.obj
 0003:00000b18       logFP                      0000000180030b18     AccessBridgeDebug.obj
 0003:00000b6c       ?__proc_attached@@3HA      0000000180030b6c     LIBCMT:dll_dllmain.obj
 0003:00000b70       GS_ExceptionRecord         0000000180030b70     LIBCMT:gs_report.obj
 0003:00000c10       GS_ContextRecord           0000000180030c10     LIBCMT:gs_report.obj
 0003:00001108       ?is_initialized_as_dll@@3_NA 0000000180031108     LIBCMT:utility.obj
 0003:00001109       ?module_local_atexit_table_initialized@@3_NA 0000000180031109     LIBCMT:utility.obj
 0003:00001110       ?module_local_atexit_table@@3U_onexit_table_t@@A 0000000180031110     LIBCMT:utility.obj
 0003:00001128       ?module_local_at_quick_exit_table@@3U_onexit_table_t@@A 0000000180031128     LIBCMT:utility.obj
 0003:00001190       ?heap@@3V_HeapManager@@A   0000000180031190     libvcruntime:undname.obj
 0003:000011c0       ?__vcrt_startup_thread_ptd@@3U__vcrt_ptd@@A 00000001800311c0     libvcruntime:per_thread_data.obj
 0003:00001240       __vcrt_lock_table          0000000180031240     libvcruntime:locks.obj
 0003:00001268       __vcrt_locks_initialized   0000000180031268     libvcruntime:locks.obj
 0003:00001270       ?module_handles@@3PAPEAUHINSTANCE__@@A 0000000180031270     libvcruntime:winapi_downlevel.obj
 0003:00001288       ?function_pointers@@3PAPEAXA 0000000180031288     libvcruntime:winapi_downlevel.obj
 0003:000012d0       ?__acrt_new_handler@@3V?$dual_state_global@P6AH_K@Z@__crt_state_management@@A 00000001800312d0     libucrt:new_handler.obj
 0003:000012d8       ?c_termination_complete@@3JA 00000001800312d8     libucrt:exit.obj
 0003:000012e0       ?thread_local_exit_callback_func@@3P6AXPEAXK0@ZEA 00000001800312e0     libucrt:exit.obj
 0003:000012e8       ?c_exit_complete@?1???R<lambda_6e4b09c48022b2350581041d5f6b0c4c>@@QEBA@XZ@4_NA 00000001800312e8     libucrt:exit.obj
 0003:000012f0       ?program_name@?1???$common_configure_argv@D@@YAHW4_crt_argv_mode@@@Z@4PADA 00000001800312f0     libucrt:argv_parsing.obj
 0003:00001448       ?__acrt_invalid_parameter_handler@@3V?$dual_state_global@P6AXPEB_W00I_K@Z@__crt_state_management@@A 0000000180031448     libucrt:invalid_parameter.obj
 0003:00001450       ?module_handles@@3PAPEAUHINSTANCE__@@A 0000000180031450     libucrt:winapi_thunks.obj
 0003:00001500       ?encoded_function_pointers@@3PAPEAXA 0000000180031500     libucrt:winapi_thunks.obj
 0003:00001a08       ?internal_state@?1??_mbtowc_internal@@9@4U_Mbstatet@@A 0000000180031a08     libucrt:mbtowc.obj
 0003:00001a10       ?enable_percent_n@@3_KA    0000000180031a10     libucrt:printf_count_output.obj
 0003:00001a40       ?__acrt_lock_table@@3PAU_RTL_CRITICAL_SECTION@@A 0000000180031a40     libucrt:locks.obj
 0003:00001c70       ?__acrt_locks_initialized@@3IA 0000000180031c70     libucrt:locks.obj
 0003:00001c90       ?fSystemSet@@3HA           0000000180031c90     libucrt:mbctype.obj
 0003:00001c94       ?initialized@?1??__acrt_initialize_multibyte@@9@4_NA 0000000180031c94     libucrt:mbctype.obj
 0003:00001cd0       ?ctrlc_action@@3V?$dual_state_global@P6AXH@Z@__crt_state_management@@A 0000000180031cd0     libucrt:signal.obj
 0003:00001cd8       ?ctrlbreak_action@@3V?$dual_state_global@P6AXH@Z@__crt_state_management@@A 0000000180031cd8     libucrt:signal.obj
 0003:00001ce0       ?abort_action@@3V?$dual_state_global@P6AXH@Z@__crt_state_management@@A 0000000180031ce0     libucrt:signal.obj
 0003:00001ce8       ?term_action@@3V?$dual_state_global@P6AXH@Z@__crt_state_management@@A 0000000180031ce8     libucrt:signal.obj
 0003:00001cf0       ?user_matherr@@3V?$dual_state_global@P6AHPEAU_exception@@@Z@__crt_state_management@@A 0000000180031cf0     libucrt:matherr.obj
 0003:00001cf8       ?__acrt_global_new_mode@@3V?$dual_state_global@J@__crt_state_management@@A 0000000180031cf8     libucrt:new_mode.obj
 0003:00001d08       ?__acrt_app_type@@3W4_crt_app_type@@A 0000000180031d08     libucrt:report_runtime_error.obj
 0003:00001d10       ?internal_pst@?1??__mbrtoc32_utf8@__crt_mbstring@@YA_KPEA_UPEBD_KPEAU_Mbstatet@@AEAV__crt_cached_ptd_host@@@Z@4U3@A 0000000180031d10     libucrt:mbrtoc32.obj
 0005:00000000       MoveSmall                  0000000180034000     libvcruntime:memcpy.obj
 0005:00000040       MoveSmallYmm               0000000180034040     libvcruntime:memcpy.obj
 0005:00000064       MoveSmallYmmNT             0000000180034064     libvcruntime:memcpy.obj
 0005:00000088       MoveSmallXmm               0000000180034088     libvcruntime:memcpy.obj
 0005:000000b0       SetSmall                   00000001800340b0     libvcruntime:memset.obj
 0005:000000f0       SetSmallYmm                00000001800340f0     libvcruntime:memset.obj
 0005:00000114       SetSmallYmmNT              0000000180034114     libvcruntime:memset.obj
 0005:00000138       SetSmallXmm                0000000180034138     libvcruntime:memset.obj
 0006:00000120       $R000000                   0000000180035120     windowsaccessbridge-64.dll.res
 0006:00000338       $R000218                   0000000180035338     windowsaccessbridge-64.dll.res
 0006:000003c8       $R0002A8                   00000001800353c8     windowsaccessbridge-64.dll.res
